 metaphlan2_support

 Timestamp is 5c76226b (Wed Feb 27 12:38:51 2019)

 Preferred load address is 10000000

 Start         Length     Name                   Class
 0001:00000000 00003c78H .text$di                CODE
 0001:00003c80 0000e00eH .text$mn                CODE
 0001:00011c90 00003324H .text$x                 CODE
 0001:00014fc0 00000c7bH .text$yd                CODE
 0002:00000000 00000744H .idata$5                DATA
 0002:00000744 00000004H .CRT$XCA                DATA
 0002:00000748 000002a0H .CRT$XCU                DATA
 0002:000009e8 00000004H .CRT$XCZ                DATA
 0002:000009ec 00000004H .CRT$XIA                DATA
 0002:000009f0 00000004H .CRT$XIAA               DATA
 0002:000009f4 00000004H .CRT$XIC                DATA
 0002:000009f8 00000004H .CRT$XIZ                DATA
 0002:00000a00 00002448H .rdata                  DATA
 0002:00002e48 00000078H .rdata$debug            DATA
 0002:00002ec0 000010c0H .rdata$r                DATA
 0002:00003f80 000002e0H .rdata$sxdata           DATA
 0002:00004260 00000004H .rtc$IAA                DATA
 0002:00004264 00000004H .rtc$IZZ                DATA
 0002:00004268 00000004H .rtc$TAA                DATA
 0002:0000426c 00000004H .rtc$TZZ                DATA
 0002:00004270 00003a34H .xdata$x                DATA
 0002:00007cb0 0000005bH .edata                  DATA
 0002:00007d0c 00000104H .idata$2                DATA
 0002:00007e10 00000014H .idata$3                DATA
 0002:00007e24 00000744H .idata$4                DATA
 0002:00008568 00005f78H .idata$6                DATA
 0003:00000000 00000094H .data                   DATA
 0003:00000098 000008dcH .data$r                 DATA
 0003:00000978 000007bcH .bss                    DATA
 0004:00000000 00000058H .rsrc$01                DATA
 0004:00000060 00000180H .rsrc$02                DATA

  Address         Publics by Value              Rva+Base       Lib:Object

 0000:00000000       ___guard_flags             00000000     <absolute>
 0000:00000000       ___guard_fids_count        00000000     <absolute>
 0000:00000000       __except_list              00000000     <absolute>
 0000:00000000       ___guard_fids_table        00000000     <absolute>
 0000:000000b8       ___safe_se_handler_count   000000b8     <absolute>
 0000:00009876       __fltused                  00009876     <absolute>
 0000:00009876       __ldused                   00009876     <absolute>
 0000:00000000       ___ImageBase               10000000     <linker-defined>
 0001:00003c80       ??$_Allocate@D@std@@YAPADIPAD@Z 10004c80 f i Metaphlan2LogParser.obj
 0001:00003cb0       ??$addressof@D@std@@YAPADAAD@Z 10004cb0 f i Metaphlan2LogParser.obj
 0001:00003cc0       ??$atomic@H@?$QAtomicOpsBySize@$03@@CAPAJPAH@Z 10004cc0 f i Metaphlan2LogParser.obj
 0001:00003cd0       ??$construct@PADAAPAD@?$_Wrap_alloc@V?$allocator@D@std@@@std@@QAEXPAPADAAPAD@Z 10004cd0 f i Metaphlan2LogParser.obj
 0001:00003cf0       ??$construct@PADAAPAD@?$allocator@D@std@@QAEXPAPADAAPAD@Z 10004cf0 f i Metaphlan2LogParser.obj
 0001:00003d10       ??$construct@PADAAPAD@?$allocator_traits@V?$allocator@D@std@@@std@@SAXAAV?$allocator@D@1@PAPADAAPAD@Z 10004d10 f i Metaphlan2LogParser.obj
 0001:00003d30       ??$deref@H@?$QAtomicOpsBySize@$03@@SA_NAAH@Z 10004d30 f i Metaphlan2LogParser.obj
 0001:00003d50       ??$destroy@PAD@?$_Wrap_alloc@V?$allocator@D@std@@@std@@QAEXPAPAD@Z 10004d50 f i Metaphlan2LogParser.obj
 0001:00003d60       ??$destroy@PAD@?$allocator@D@std@@QAEXPAPAD@Z 10004d60 f i Metaphlan2LogParser.obj
 0001:00003d70       ??$destroy@PAD@?$allocator_traits@V?$allocator@D@std@@@std@@SAXAAV?$allocator@D@1@PAPAD@Z 10004d70 f i Metaphlan2LogParser.obj
 0001:00003d80       ??$forward@AAPAD@std@@YAAAPADAAPAD@Z 10004d80 f i Metaphlan2LogParser.obj
 0001:00003d90       ??$load@H@?$QGenericAtomicOps@U?$QAtomicOpsBySize@$03@@@@SAHABH@Z 10004d90 f i Metaphlan2LogParser.obj
 0001:00003da0       ??$ref@H@?$QAtomicOpsBySize@$03@@SA_NAAH@Z 10004da0 f i Metaphlan2LogParser.obj
 0001:00003dc0       ??0?$QForeachContainer@$$CBVQStringList@@@@QAE@ABVQStringList@@@Z 10004dc0 f i Metaphlan2LogParser.obj
 0001:00003e00       ??0?$QList@VQString@@@@QAE@ABV0@@Z 10004e00 f i Metaphlan2LogParser.obj
 0001:00003ec0       ??0?$QList@VQString@@@@QAE@XZ 10004ec0 f i Metaphlan2LogParser.obj
 0001:00003ed0       ??0?$_String_alloc@$0A@U?$_String_base_types@DV?$allocator@D@std@@@std@@@std@@QAE@ABV?$allocator@D@1@@Z 10004ed0 f i Metaphlan2LogParser.obj
 0001:00003ef0       ??0?$_String_val@U?$_Simple_types@D@std@@@std@@QAE@XZ 10004ef0 f i Metaphlan2LogParser.obj
 0001:00003f10       ??0?$_Wrap_alloc@V?$allocator@D@std@@@std@@QAE@XZ 10004f10 f i Metaphlan2LogParser.obj
 0001:00003f20       ??0?$allocator@D@std@@QAE@XZ 10004f20 f i Metaphlan2LogParser.obj
 0001:00003f30       ??0?$basic_string@DU?$char_traits@D@std@@V?$allocator@D@2@@std@@QAE@PBD@Z 10004f30 f i Metaphlan2LogParser.obj
 0001:00003f90       ??0QStringList@@QAE@ABV0@@Z 10004f90 f i Metaphlan2LogParser.obj
 0001:00003fb0       ??0QStringList@@QAE@XZ     10004fb0 f i Metaphlan2LogParser.obj
 0001:00003fc0       ??0_Generic_error_category@std@@QAE@XZ 10004fc0 f i Metaphlan2LogParser.obj
 0001:00003fd0       ??0_Ignore@std@@QAE@XZ     10004fd0 f i Metaphlan2LogParser.obj
 0001:00003fe0       ??0_Iostream_error_category@std@@QAE@XZ 10004fe0 f i Metaphlan2LogParser.obj
 0001:00003ff0       ??0_System_error_category@std@@QAE@XZ 10004ff0 f i Metaphlan2LogParser.obj
 0001:00004000       ??0const_iterator@?$QList@VQString@@@@QAE@PAUNode@1@@Z 10005000 f i Metaphlan2LogParser.obj
 0001:00004010       ??0error_category@std@@QAE@XZ 10005010 f i Metaphlan2LogParser.obj
 0001:00004020       ??0error_condition@std@@QAE@HABVerror_category@1@@Z 10005020 f i Metaphlan2LogParser.obj
 0001:00004040       ??1?$QForeachContainer@$$CBVQStringList@@@@QAE@XZ 10005040 f i Metaphlan2LogParser.obj
 0001:00004050       ??1?$QList@VQString@@@@QAE@XZ 10005050 f i Metaphlan2LogParser.obj
 0001:000040b0       ??1?$basic_string@DU?$char_traits@D@std@@V?$allocator@D@2@@std@@QAE@XZ 100050b0 f i Metaphlan2LogParser.obj
 0001:000040e0       ??1QStringList@@QAE@XZ     100050e0 f i Metaphlan2LogParser.obj
 0001:000040f0       ??1_Generic_error_category@std@@UAE@XZ 100050f0 f i Metaphlan2LogParser.obj
 0001:00004100       ??1_Iostream_error_category@std@@UAE@XZ 10005100 f i Metaphlan2LogParser.obj
 0001:00004110       ??1_System_error_category@std@@UAE@XZ 10005110 f i Metaphlan2LogParser.obj
 0001:00004120       ??1error_category@std@@UAE@XZ 10005120 f i Metaphlan2LogParser.obj
 0001:00004130       ??2@YAPAXIPAX@Z            10005130 f i Metaphlan2LogParser.obj
 0001:00004140       ??3@YAXPAX0@Z              10005140 f i Metaphlan2LogParser.obj
 0001:00004150       ??6QStringList@@QAEAAV0@ABVQString@@@Z 10005150 f i Metaphlan2LogParser.obj
 0001:00004170       ??8error_category@std@@QBE_NABV01@@Z 10005170 f i Metaphlan2LogParser.obj
 0001:00004180       ??8error_condition@std@@QBE_NABV01@@Z 10005180 f i Metaphlan2LogParser.obj
 0001:000041a0       ??9const_iterator@?$QList@VQString@@@@QBE_NABV01@@Z 100051a0 f i Metaphlan2LogParser.obj
 0001:000041c0       ??Dconst_iterator@?$QList@VQString@@@@QBEABVQString@@XZ 100051c0 f i Metaphlan2LogParser.obj
 0001:000041d0       ??Econst_iterator@?$QList@VQString@@@@QAEAAV01@XZ 100051d0 f i Metaphlan2LogParser.obj
 0001:000041e0       ??_GQString@@QAEPAXI@Z     100051e0 f i Metaphlan2LogParser.obj
 0001:00004210       ??_G_Generic_error_category@std@@UAEPAXI@Z 10005210 f i Metaphlan2LogParser.obj
 0001:00004210       ??_E_Generic_error_category@std@@UAEPAXI@Z 10005210 f i Metaphlan2LogParser.obj
 0001:00004240       ??_G_Iostream_error_category@std@@UAEPAXI@Z 10005240 f i Metaphlan2LogParser.obj
 0001:00004240       ??_E_Iostream_error_category@std@@UAEPAXI@Z 10005240 f i Metaphlan2LogParser.obj
 0001:00004270       ??_G_System_error_category@std@@UAEPAXI@Z 10005270 f i Metaphlan2LogParser.obj
 0001:00004270       ??_E_System_error_category@std@@UAEPAXI@Z 10005270 f i Metaphlan2LogParser.obj
 0001:000042a0       ??_Eerror_category@std@@UAEPAXI@Z 100052a0 f i Metaphlan2LogParser.obj
 0001:000042a0       ??_Gerror_category@std@@UAEPAXI@Z 100052a0 f i Metaphlan2LogParser.obj
 0001:000042d0       ?_Copy@?$basic_string@DU?$char_traits@D@std@@V?$allocator@D@2@@std@@QAEXII@Z 100052d0 f i Metaphlan2LogParser.obj
 0001:00004420       ?_Eos@?$basic_string@DU?$char_traits@D@std@@V?$allocator@D@2@@std@@QAEXI@Z 10005420 f i Metaphlan2LogParser.obj
 0001:00004450       ?_Getal@?$_String_alloc@$0A@U?$_String_base_types@DV?$allocator@D@std@@@std@@@std@@QBE?AU?$_Wrap_alloc@V?$allocator@D@std@@@2@XZ 10005450 f i Metaphlan2LogParser.obj
 0001:00004460       ?_Grow@?$basic_string@DU?$char_traits@D@std@@V?$allocator@D@2@@std@@QAE_NI_N@Z 10005460 f i Metaphlan2LogParser.obj
 0001:00004510       ?_Inside@?$basic_string@DU?$char_traits@D@std@@V?$allocator@D@2@@std@@QAE_NPBD@Z 10005510 f i Metaphlan2LogParser.obj
 0001:00004550       ?_Myptr@?$_String_val@U?$_Simple_types@D@std@@@std@@QAEPADXZ 10005550 f i Metaphlan2LogParser.obj
 0001:00004560       ?_Myptr@?$_String_val@U?$_Simple_types@D@std@@@std@@QBEPBDXZ 10005560 f i Metaphlan2LogParser.obj
 0001:00004570       ?_Tidy@?$basic_string@DU?$char_traits@D@std@@V?$allocator@D@2@@std@@QAEX_NI@Z 10005570 f i Metaphlan2LogParser.obj
 0001:000045c0       ?_Xlen@?$basic_string@DU?$char_traits@D@std@@V?$allocator@D@2@@std@@QBEXXZ 100055c0 f i Metaphlan2LogParser.obj
 0001:000045d0       ?_Xran@?$basic_string@DU?$char_traits@D@std@@V?$allocator@D@2@@std@@QBEXXZ 100055d0 f i Metaphlan2LogParser.obj
 0001:000045e0       ?allocate@?$_Wrap_alloc@V?$allocator@D@std@@@std@@QAEPADI@Z 100055e0 f i Metaphlan2LogParser.obj
 0001:00004610       ?allocate@?$allocator@D@std@@QAEPADI@Z 10005610 f i Metaphlan2LogParser.obj
 0001:00004640       ?append@?$QList@VQString@@@@QAEXABVQString@@@Z 10005640 f i Metaphlan2LogParser.obj
 0001:00004730       ?assign@?$basic_string@DU?$char_traits@D@std@@V?$allocator@D@2@@std@@QAEAAV12@ABV12@II@Z 10005730 f i Metaphlan2LogParser.obj
 0001:00004850       ?assign@?$basic_string@DU?$char_traits@D@std@@V?$allocator@D@2@@std@@QAEAAV12@PBD@Z 10005850 f i Metaphlan2LogParser.obj
 0001:00004890       ?assign@?$basic_string@DU?$char_traits@D@std@@V?$allocator@D@2@@std@@QAEAAV12@PBDI@Z 10005890 f i Metaphlan2LogParser.obj
 0001:00004990       ?assign@?$char_traits@D@std@@SAXAADABD@Z 10005990 f i Metaphlan2LogParser.obj
 0001:000049a0       ?begin@?$QList@VQString@@@@QBE?AVconst_iterator@1@XZ 100059a0 f i Metaphlan2LogParser.obj
 0001:000049c0       ?category@error_code@std@@QBEABVerror_category@2@XZ 100059c0 f i Metaphlan2LogParser.obj
 0001:000049d0       ?category@error_condition@std@@QBEABVerror_category@2@XZ 100059d0 f i Metaphlan2LogParser.obj
 0001:000049e0       ?copy@?$char_traits@D@std@@SAPADPADPBDI@Z 100059e0 f i Metaphlan2LogParser.obj
 0001:00004a00       ?dealloc@?$QList@VQString@@@@AAEXPAUData@QListData@@@Z 10005a00 f i Metaphlan2LogParser.obj
 0001:00004a40       ?deallocate@?$_Wrap_alloc@V?$allocator@D@std@@@std@@QAEXPADI@Z 10005a40 f i Metaphlan2LogParser.obj
 0001:00004a60       ?deallocate@?$allocator@D@std@@QAEXPADI@Z 10005a60 f i Metaphlan2LogParser.obj
 0001:00004a80       ?default_error_condition@_System_error_category@std@@UBE?AVerror_condition@2@H@Z 10005a80 f i Metaphlan2LogParser.obj
 0001:00004ac0       ?default_error_condition@error_category@std@@UBE?AVerror_condition@2@H@Z 10005ac0 f i Metaphlan2LogParser.obj
 0001:00004ae0       ?deref@?$QBasicAtomicInteger@H@@QAE_NXZ 10005ae0 f i Metaphlan2LogParser.obj
 0001:00004af0       ?deref@RefCount@QtPrivate@@QAE_NXZ 10005af0 f i Metaphlan2LogParser.obj
 0001:00004b10       ?detach_helper_grow@?$QList@VQString@@@@AAEPAUNode@1@HH@Z 10005b10 f i Metaphlan2LogParser.obj
 0001:00004c90       ?end@?$QList@VQString@@@@QBE?AVconst_iterator@1@XZ 10005c90 f i Metaphlan2LogParser.obj
 0001:00004cb0       ?equivalent@error_category@std@@UBE_NABVerror_code@2@H@Z 10005cb0 f i Metaphlan2LogParser.obj
 0001:00004cd0       ?equivalent@error_category@std@@UBE_NHABVerror_condition@2@@Z 10005cd0 f i Metaphlan2LogParser.obj
 0001:00004d10       ?erase@?$basic_string@DU?$char_traits@D@std@@V?$allocator@D@2@@std@@QAEAAV12@I@Z 10005d10 f i Metaphlan2LogParser.obj
 0001:00004d50       ?erase@?$basic_string@DU?$char_traits@D@std@@V?$allocator@D@2@@std@@QAEAAV12@II@Z 10005d50 f i Metaphlan2LogParser.obj
 0001:00004df0       ?generic_category@std@@YAABVerror_category@1@XZ 10005df0 f i Metaphlan2LogParser.obj
 0001:00004e00       ?initWellKnownErrors@Metaphlan2LogParser@U2@@CA?AVQStringList@@XZ 10005e00 f   Metaphlan2LogParser.obj
 0001:00004e90       ?isError@Metaphlan2LogParser@U2@@EBE_NABVQString@@@Z 10005e90 f   Metaphlan2LogParser.obj
 0001:00005000       ?isShared@RefCount@QtPrivate@@QBE_NXZ 10006000 f i Metaphlan2LogParser.obj
 0001:00005020       ?length@?$char_traits@D@std@@SAIPBD@Z 10006020 f i Metaphlan2LogParser.obj
 0001:00005040       ?load@?$QBasicAtomicInteger@H@@QBEHXZ 10006040 f i Metaphlan2LogParser.obj
 0001:00005050       ?max_size@?$_Wrap_alloc@V?$allocator@D@std@@@std@@QBEIXZ 10006050 f i Metaphlan2LogParser.obj
 0001:00005060       ?max_size@?$allocator@D@std@@QBEIXZ 10006060 f i Metaphlan2LogParser.obj
 0001:00005070       ?max_size@?$allocator_traits@V?$allocator@D@std@@@std@@SAIABV?$allocator@D@2@@Z 10006070 f i Metaphlan2LogParser.obj
 0001:00005080       ?max_size@?$basic_string@DU?$char_traits@D@std@@V?$allocator@D@2@@std@@QBEIXZ 10006080 f i Metaphlan2LogParser.obj
 0001:00005090       ?message@_Generic_error_category@std@@UBE?AV?$basic_string@DU?$char_traits@D@std@@V?$allocator@D@2@@2@H@Z 10006090 f i Metaphlan2LogParser.obj
 0001:00005110       ?message@_Iostream_error_category@std@@UBE?AV?$basic_string@DU?$char_traits@D@std@@V?$allocator@D@2@@2@H@Z 10006110 f i Metaphlan2LogParser.obj
 0001:00005160       ?message@_System_error_category@std@@UBE?AV?$basic_string@DU?$char_traits@D@std@@V?$allocator@D@2@@2@H@Z 10006160 f i Metaphlan2LogParser.obj
 0001:000051e0       ?move@?$char_traits@D@std@@SAPADPADPBDI@Z 100061e0 f i Metaphlan2LogParser.obj
 0001:00005200       ?name@_Generic_error_category@std@@UBEPBDXZ 10006200 f i Metaphlan2LogParser.obj
 0001:00005210       ?name@_Iostream_error_category@std@@UBEPBDXZ 10006210 f i Metaphlan2LogParser.obj
 0001:00005220       ?name@_System_error_category@std@@UBEPBDXZ 10006220 f i Metaphlan2LogParser.obj
 0001:00005230       ?node_construct@?$QList@VQString@@@@AAEXPAUNode@1@ABVQString@@@Z 10006230 f i Metaphlan2LogParser.obj
 0001:00005280       ?node_copy@?$QList@VQString@@@@AAEXPAUNode@1@00@Z 10006280 f i Metaphlan2LogParser.obj
 0001:00005320       ?node_destruct@?$QList@VQString@@@@AAEXPAUNode@1@0@Z 10006320 f i Metaphlan2LogParser.obj
 0001:00005350       ?node_destruct@?$QList@VQString@@@@AAEXPAUNode@1@@Z 10006350 f i Metaphlan2LogParser.obj
 0001:00005360       ?ref@?$QBasicAtomicInteger@H@@QAE_NXZ 10006360 f i Metaphlan2LogParser.obj
 0001:00005380       ?ref@RefCount@QtPrivate@@QAE_NXZ 10006380 f i Metaphlan2LogParser.obj
 0001:000053a0       ?size@?$basic_string@DU?$char_traits@D@std@@V?$allocator@D@2@@std@@QBEIXZ 100063a0 f i Metaphlan2LogParser.obj
 0001:000053b0       ?system_category@std@@YAABVerror_category@1@XZ 100063b0 f i Metaphlan2LogParser.obj
 0001:000053c0       ?t@Node@?$QList@VQString@@@@QAEAAVQString@@XZ 100063c0 f i Metaphlan2LogParser.obj
 0001:000053d0       ?value@error_code@std@@QBEHXZ 100063d0 f i Metaphlan2LogParser.obj
 0001:000053e0       ?value@error_condition@std@@QBEHXZ 100063e0 f i Metaphlan2LogParser.obj
 0001:000053f0       _hypot                     100063f0 f i Metaphlan2LogParser.obj
 0001:00005420       ??0?$PrompterBase@VMetaphlan2Prompter@LocalWorkflow@U2@@@U2@@QAE@PAVActor@Workflow@1@_N@Z 10006420 f i Metaphlan2Prompter.obj
 0001:00005450       ??0?$QForeachContainer@V?$QList@PAVPort@Workflow@U2@@@@@@QAE@ABV?$QList@PAVPort@Workflow@U2@@@@@Z 10006450 f i Metaphlan2Prompter.obj
 0001:00005490       ??0?$QList@PAVPort@Workflow@U2@@@@QAE@ABV0@@Z 10006490 f i Metaphlan2Prompter.obj
 0001:00005550       ??0Metaphlan2Prompter@LocalWorkflow@U2@@QAE@PAVActor@Workflow@2@@Z 10006550 f   Metaphlan2Prompter.obj
 0001:00005580       ??0QLatin1Char@@QAE@D@Z    10006580 f i Metaphlan2Prompter.obj
 0001:00005590       ??0const_iterator@?$QList@PAVPort@Workflow@U2@@@@QAE@PAUNode@1@@Z 10006590 f i Metaphlan2Prompter.obj
 0001:000055a0       ??1?$PrompterBase@VMetaphlan2Prompter@LocalWorkflow@U2@@@U2@@UAE@XZ 100065a0 f i Metaphlan2Prompter.obj
 0001:000055b0       ??1?$QForeachContainer@V?$QList@PAVPort@Workflow@U2@@@@@@QAE@XZ 100065b0 f i Metaphlan2Prompter.obj
 0001:000055e0       ??1?$QList@PAVPort@Workflow@U2@@@@QAE@XZ 100065e0 f i Metaphlan2Prompter.obj
 0001:00005610       ??1Metaphlan2Prompter@LocalWorkflow@U2@@UAE@XZ 10006610 f i Metaphlan2Prompter.obj
 0001:00005620       ??9const_iterator@?$QList@PAVPort@Workflow@U2@@@@QBE_NABV01@@Z 10006620 f i Metaphlan2Prompter.obj
 0001:00005640       ??Dconst_iterator@?$QList@PAVPort@Workflow@U2@@@@QBEABQAVPort@Workflow@U2@@XZ 10006640 f i Metaphlan2Prompter.obj
 0001:00005650       ??Econst_iterator@?$QList@PAVPort@Workflow@U2@@@@QAEAAV01@XZ 10006650 f i Metaphlan2Prompter.obj
 0001:00005656       ??_E?$PrompterBase@VMetaphlan2Prompter@LocalWorkflow@U2@@@U2@@WM@AEPAXI@Z 10006656 f i Metaphlan2Prompter.obj
 0001:0000565e       ??_EMetaphlan2Prompter@LocalWorkflow@U2@@WM@AEPAXI@Z 1000665e f i Metaphlan2Prompter.obj
 0001:00005670       ??_G?$PrompterBase@VMetaphlan2Prompter@LocalWorkflow@U2@@@U2@@UAEPAXI@Z 10006670 f i Metaphlan2Prompter.obj
 0001:00005670       ??_E?$PrompterBase@VMetaphlan2Prompter@LocalWorkflow@U2@@@U2@@UAEPAXI@Z 10006670 f i Metaphlan2Prompter.obj
 0001:000056a0       ??_GMetaphlan2Prompter@LocalWorkflow@U2@@UAEPAXI@Z 100066a0 f i Metaphlan2Prompter.obj
 0001:000056a0       ??_EMetaphlan2Prompter@LocalWorkflow@U2@@UAEPAXI@Z 100066a0 f i Metaphlan2Prompter.obj
 0001:000056d0       ?begin@?$QList@PAVPort@Workflow@U2@@@@QBE?AVconst_iterator@1@XZ 100066d0 f i Metaphlan2Prompter.obj
 0001:000056f0       ?composeRichDoc@Metaphlan2Prompter@LocalWorkflow@U2@@EAE?AVQString@@XZ 100066f0 f   Metaphlan2Prompter.obj
 0001:00005880       ?createDescription@?$PrompterBase@VMetaphlan2Prompter@LocalWorkflow@U2@@@U2@@UAEPAVActorDocument@Workflow@2@PAVActor@42@@Z 10006880 f i Metaphlan2Prompter.obj
 0001:00005b20       ?dealloc@?$QList@PAVPort@Workflow@U2@@@@AAEXPAUData@QListData@@@Z 10006b20 f i Metaphlan2Prompter.obj
 0001:00005b40       ?end@?$QList@PAVPort@Workflow@U2@@@@QBE?AVconst_iterator@1@XZ 10006b40 f i Metaphlan2Prompter.obj
 0001:00005b60       ?node_copy@?$QList@PAVPort@Workflow@U2@@@@AAEXPAUNode@1@00@Z 10006b60 f i Metaphlan2Prompter.obj
 0001:00005b90       ?node_destruct@?$QList@PAVPort@Workflow@U2@@@@AAEXPAUNode@1@0@Z 10006b90 f i Metaphlan2Prompter.obj
 0001:00005ba0       ?t@Node@?$QList@PAVPort@Workflow@U2@@@@QAEAAPAVPort@Workflow@U2@@XZ 10006ba0 f i Metaphlan2Prompter.obj
 0001:00005bb0       ?tr@Metaphlan2Prompter@LocalWorkflow@U2@@SA?AVQString@@PBD0H@Z 10006bb0 f i Metaphlan2Prompter.obj
 0001:00005be0       ??0Metaphlan2Support@U2@@QAE@ABVQString@@0@Z 10006be0 f   Metaphlan2Support.obj
 0001:00005d80       ??1Metaphlan2Support@U2@@UAE@XZ 10006d80 f i Metaphlan2Support.obj
 0001:00005d90       ??_GMetaphlan2Support@U2@@UAEPAXI@Z 10006d90 f i Metaphlan2Support.obj
 0001:00005d90       ??_EMetaphlan2Support@U2@@UAEPAXI@Z 10006d90 f i Metaphlan2Support.obj
 0001:00005dc0       ?performAdditionalChecks@Metaphlan2Support@U2@@UAEXABVQString@@@Z 10006dc0 f   Metaphlan2Support.obj
 0001:00005f70       ?tr@Metaphlan2Support@U2@@SA?AVQString@@PBD0H@Z 10006f70 f i Metaphlan2Support.obj
 0001:00005fa0       ??0MetaphlanSupportPlugin@U2@@QAE@XZ 10006fa0 f   Metaphlan2SupportPlugin.obj
 0001:00006090       ??1MetaphlanSupportPlugin@U2@@UAE@XZ 10007090 f   Metaphlan2SupportPlugin.obj
 0001:00006100       ??_EMetaphlanSupportPlugin@U2@@UAEPAXI@Z 10007100 f i Metaphlan2SupportPlugin.obj
 0001:00006100       ??_GMetaphlanSupportPlugin@U2@@UAEPAXI@Z 10007100 f i Metaphlan2SupportPlugin.obj
 0001:00006180       _ugene_plugin_init         10007180 f   Metaphlan2SupportPlugin.obj
 0001:000061a0       ??0?$QFlags@W4Filter@QDir@@@@QAE@W4Filter@QDir@@@Z 100071a0 f i Metaphlan2Task.obj
 0001:000061b0       ??0?$QFlags@W4SortFlag@QDir@@@@QAE@W4SortFlag@QDir@@@Z 100071b0 f i Metaphlan2Task.obj
 0001:000061c0       ??0?$QFlags@W4TaskFlag@U2@@@@QAE@VQFlag@@@Z 100071c0 f i Metaphlan2Task.obj
 0001:000061d0       ??0?$QFlags@W4TaskFlag@U2@@@@QAE@W4TaskFlag@U2@@@Z 100071d0 f i Metaphlan2Task.obj
 0001:000061e0       ??0?$QList@PAVTask@U2@@@@QAE@$$QAV0@@Z 100071e0 f i Metaphlan2Task.obj
 0001:00006200       ??0?$QList@PAVTask@U2@@@@QAE@XZ 10007200 f i Metaphlan2Task.obj
 0001:00006210       ??0Metaphlan2ClassifyTask@U2@@QAE@ABUMetaphlan2TaskSettings@1@@Z 10007210 f   Metaphlan2Task.obj
 0001:00006480       ??0Metaphlan2LogParser@U2@@QAE@XZ 10007480 f i Metaphlan2Task.obj
 0001:000064a0       ??0Metaphlan2TaskSettings@U2@@QAE@ABU01@@Z 100074a0 f i Metaphlan2Task.obj
 0001:000065b0       ??0Metaphlan2TaskSettings@U2@@QAE@XZ 100075b0 f   Metaphlan2Task.obj
 0001:00006690       ??0QFlag@@QAE@H@Z          10007690 f i Metaphlan2Task.obj
 0001:000066a0       ??0iterator@?$QList@VQString@@@@QAE@PAUNode@1@@Z 100076a0 f i Metaphlan2Task.obj
 0001:000066b0       ??1?$QList@PAVTask@U2@@@@QAE@XZ 100076b0 f i Metaphlan2Task.obj
 0001:000066e0       ??1Metaphlan2ClassifyTask@U2@@UAE@XZ 100076e0 f i Metaphlan2Task.obj
 0001:00006740       ??1Metaphlan2LogParser@U2@@UAE@XZ 10007740 f i Metaphlan2Task.obj
 0001:00006750       ??1Metaphlan2TaskSettings@U2@@QAE@XZ 10007750 f i Metaphlan2Task.obj
 0001:00006820       ??6?$QList@PAVTask@U2@@@@QAEAAV0@ABQAVTask@U2@@@Z 10007820 f i Metaphlan2Task.obj
 0001:00006840       ??BQFlag@@QBEHXZ           10007840 f i Metaphlan2Task.obj
 0001:00006850       ??Diterator@?$QList@VQString@@@@QBEAAVQString@@XZ 10007850 f i Metaphlan2Task.obj
 0001:00006860       ??U?$QFlags@W4TaskFlag@U2@@@@QBE?AV0@W4TaskFlag@U2@@@Z 10007860 f i Metaphlan2Task.obj
 0001:00006880       ??_ECalculateSequencesNumberTask@U2@@UAEPAXI@Z 10007880 f i Metaphlan2Task.obj
 0001:00006880       ??_GCalculateSequencesNumberTask@U2@@UAEPAXI@Z 10007880 f i Metaphlan2Task.obj
 0001:000068b0       ??_EExternalToolRunTask@U2@@UAEPAXI@Z 100078b0 f i Metaphlan2Task.obj
 0001:000068b0       ??_GExternalToolRunTask@U2@@UAEPAXI@Z 100078b0 f i Metaphlan2Task.obj
 0001:000068e0       ??_GMetaphlan2ClassifyTask@U2@@UAEPAXI@Z 100078e0 f i Metaphlan2Task.obj
 0001:000068e0       ??_EMetaphlan2ClassifyTask@U2@@UAEPAXI@Z 100078e0 f i Metaphlan2Task.obj
 0001:00006950       ??_GMetaphlan2LogParser@U2@@UAEPAXI@Z 10007950 f i Metaphlan2Task.obj
 0001:00006950       ??_EMetaphlan2LogParser@U2@@UAEPAXI@Z 10007950 f i Metaphlan2Task.obj
 0001:00006980       ?append@?$QList@PAVTask@U2@@@@QAEXABQAVTask@U2@@@Z 10007980 f i Metaphlan2Task.obj
 0001:00006a10       ?begin@?$QList@VQString@@@@QAE?AViterator@1@XZ 10007a10 f i Metaphlan2Task.obj
 0001:00006a50       ?dealloc@?$QList@PAVTask@U2@@@@AAEXPAUData@QListData@@@Z 10007a50 f i Metaphlan2Task.obj
 0001:00006a70       ?detach@?$QList@VQString@@@@QAEXXZ 10007a70 f i Metaphlan2Task.obj
 0001:00006a90       ?detach_helper@?$QList@VQString@@@@AAEXH@Z 10007a90 f i Metaphlan2Task.obj
 0001:00006b80       ?detach_helper@?$QList@VQString@@@@AAEXXZ 10007b80 f i Metaphlan2Task.obj
 0001:00006b90       ?detach_helper_grow@?$QList@PAVTask@U2@@@@AAEPAUNode@1@HH@Z 10007b90 f i Metaphlan2Task.obj
 0001:00006ca0       ?detectFormat@Metaphlan2ClassifyTask@U2@@AAE?AVQString@@ABVGUrl@2@@Z 10007ca0 f   Metaphlan2Task.obj
 0001:00006dd0       ?detectInputFormats@Metaphlan2ClassifyTask@U2@@AAE?AVQString@@XZ 10007dd0 f   Metaphlan2Task.obj
 0001:00006f10       ?first@?$QList@VQString@@@@QAEAAVQString@@XZ 10007f10 f i Metaphlan2Task.obj
 0001:00006f40       ?getArguments@Metaphlan2ClassifyTask@U2@@AAE?AVQStringList@@XZ 10007f40 f   Metaphlan2Task.obj
 0001:00007810       ?getBowtie2OutputUrl@Metaphlan2ClassifyTask@U2@@QBEABVQString@@XZ 10008810 f   Metaphlan2Task.obj
 0001:00007820       ?getOutputUrl@Metaphlan2ClassifyTask@U2@@QBEABVQString@@XZ 10008820 f   Metaphlan2Task.obj
 0001:00007830       ?isEmpty@?$QList@VQString@@@@QBE_NXZ 10008830 f i Metaphlan2Task.obj
 0001:00007840       ?node_construct@?$QList@PAVTask@U2@@@@AAEXPAUNode@1@ABQAVTask@U2@@@Z 10008840 f i Metaphlan2Task.obj
 0001:00007860       ?node_copy@?$QList@PAVTask@U2@@@@AAEXPAUNode@1@00@Z 10008860 f i Metaphlan2Task.obj
 0001:00007890       ?node_destruct@?$QList@PAVTask@U2@@@@AAEXPAUNode@1@0@Z 10008890 f i Metaphlan2Task.obj
 0001:000078a0       ?node_destruct@?$QList@PAVTask@U2@@@@AAEXPAUNode@1@@Z 100088a0 f i Metaphlan2Task.obj
 0001:000078b0       ?onSubTaskFinished@Metaphlan2ClassifyTask@U2@@EAE?AV?$QList@PAVTask@U2@@@@PAVTask@2@@Z 100088b0 f   Metaphlan2Task.obj
 0001:000079a0       ?prepare@Metaphlan2ClassifyTask@U2@@EAEXXZ 100089a0 f   Metaphlan2Task.obj
 0001:00007a50       ?prepareClassifyTask@Metaphlan2ClassifyTask@U2@@AAEXXZ 10008a50 f   Metaphlan2Task.obj
 0001:00007c10       ?qt_noop@@YAXXZ            10008c10 f i Metaphlan2Task.obj
 0001:00007c20       ?size@?$QList@VQString@@@@QBEHXZ 10008c20 f i Metaphlan2Task.obj
 0001:00007c30       ?tr@Metaphlan2ClassifyTask@U2@@SA?AVQString@@PBD0H@Z 10008c30 f i Metaphlan2Task.obj
 0001:00007c60       ??$getAttributeValueWithoutScript@VQString@@@Attribute@U2@@QBE?AVQString@@XZ 10008c60 f i Metaphlan2Validator.obj
 0001:00007c80       ??$qMetaTypeId@VQString@@@@YAHXZ 10008c80 f i Metaphlan2Validator.obj
 0001:00007c90       ??$qvariant_cast@VQString@@@@YA?AVQString@@ABVQVariant@@@Z 10008c90 f i Metaphlan2Validator.obj
 0001:00007cb0       ??$value@VQString@@@QVariant@@QBE?AVQString@@XZ 10008cb0 f i Metaphlan2Validator.obj
 0001:00007cd0       ??6?$QList@VWorkflowNotification@U2@@@@QAEAAV0@ABVWorkflowNotification@U2@@@Z 10008cd0 f i Metaphlan2Validator.obj
 0001:00007cf0       ??_GWorkflowNotification@U2@@QAEPAXI@Z 10008cf0 f i Metaphlan2Validator.obj
 0001:00007d20       ?append@?$QList@VWorkflowNotification@U2@@@@QAEXABVWorkflowNotification@U2@@@Z 10008d20 f i Metaphlan2Validator.obj
 0001:00007e00       ?dealloc@?$QList@VWorkflowNotification@U2@@@@AAEXPAUData@QListData@@@Z 10008e00 f i Metaphlan2Validator.obj
 0001:00007e60       ?detach_helper_grow@?$QList@VWorkflowNotification@U2@@@@AAEPAUNode@1@HH@Z 10008e60 f i Metaphlan2Validator.obj
 0001:00007fb0       ?invoke@?$MetaTypeInvoker@U?$QVariantValueHelper@VQString@@@QtPrivate@@ABVQVariant@@VQString@@@QtPrivate@@SA?AVQString@@ABVQVariant@@@Z 10008fb0 f i Metaphlan2Validator.obj
 0001:00007fd0       ?metaType@?$QVariantValueHelper@VQString@@@QtPrivate@@SA?AVQString@@ABVQVariant@@@Z 10008fd0 f i Metaphlan2Validator.obj
 0001:00008090       ?node_construct@?$QList@VWorkflowNotification@U2@@@@AAEXPAUNode@1@ABVWorkflowNotification@U2@@@Z 10009090 f i Metaphlan2Validator.obj
 0001:00008110       ?node_copy@?$QList@VWorkflowNotification@U2@@@@AAEXPAUNode@1@00@Z 10009110 f i Metaphlan2Validator.obj
 0001:000081e0       ?node_destruct@?$QList@VWorkflowNotification@U2@@@@AAEXPAUNode@1@0@Z 100091e0 f i Metaphlan2Validator.obj
 0001:00008220       ?node_destruct@?$QList@VWorkflowNotification@U2@@@@AAEXPAUNode@1@@Z 10009220 f i Metaphlan2Validator.obj
 0001:00008250       ?qt_metatype_id@?$QMetaTypeId2@VQString@@@@SAHXZ 10009250 f i Metaphlan2Validator.obj
 0001:00008260       ?tr@Metaphlan2Validator@Workflow@U2@@SA?AVQString@@PBD0H@Z 10009260 f i Metaphlan2Validator.obj
 0001:00008290       ?validate@Metaphlan2Validator@Workflow@U2@@UBE_NPBVActor@23@AAV?$QList@VWorkflowNotification@U2@@@@ABV?$QMap@VQString@@V1@@@@Z 10009290 f   Metaphlan2Validator.obj
 0001:000082b0       ?validateDatabase@Metaphlan2Validator@Workflow@U2@@ABE_NPBVActor@23@AAV?$QList@VWorkflowNotification@U2@@@@@Z 100092b0 f   Metaphlan2Validator.obj
 0001:00008580       ??$getAttributeValue@H@Attribute@U2@@QBEHPAVWorkflowContext@Workflow@1@@Z 10009580 f i Metaphlan2Worker.obj
 0001:00008950       ??$getAttributeValue@VQString@@@Attribute@U2@@QBE?AVQString@@PAVWorkflowContext@Workflow@1@@Z 10009950 f i Metaphlan2Worker.obj
 0001:00008ce0       ??$getAttributeValueWithoutScript@H@Attribute@U2@@QBEHXZ 10009ce0 f i Metaphlan2Worker.obj
 0001:00008d20       ??$getValue@H@BaseWorker@LocalWorkflow@U2@@IBEHABVQString@@@Z 10009d20 f i Metaphlan2Worker.obj
 0001:00008d50       ??$getValue@VQString@@@BaseWorker@LocalWorkflow@U2@@IBE?AVQString@@ABV3@@Z 10009d50 f i Metaphlan2Worker.obj
 0001:00008e60       ??$qMapLessThanKey@VDescriptor@U2@@@@YA_NABVDescriptor@U2@@0@Z 10009e60 f i Metaphlan2Worker.obj
 0001:00008e80       ??$qMapLessThanKey@VQString@@@@YA_NABVQString@@0@Z 10009e80 f i Metaphlan2Worker.obj
 0001:00008e90       ??$qMetaTypeId@H@@YAHXZ    10009e90 f i Metaphlan2Worker.obj
 0001:00008ea0       ??$qobject_cast@PAVMetaphlan2ClassifyTask@U2@@@@YAPAVMetaphlan2ClassifyTask@U2@@PAVQObject@@@Z 10009ea0 f i Metaphlan2Worker.obj
 0001:00008ec0       ??$qvariant_cast@H@@YAHABVQVariant@@@Z 10009ec0 f i Metaphlan2Worker.obj
 0001:00008f00       ??$value@H@QVariant@@QBEHXZ 10009f00 f i Metaphlan2Worker.obj
 0001:00008f40       ??0?$QForeachContainer@V?$QList@VDescriptor@U2@@@@@@QAE@ABV?$QList@VDescriptor@U2@@@@@Z 10009f40 f i Metaphlan2Worker.obj
 0001:00008f80       ??0?$QHash@VQString@@UQHashDummyValue@@@@QAE@XZ 10009f80 f i Metaphlan2Worker.obj
 0001:00008f90       ??0?$QList@VDescriptor@U2@@@@QAE@$$QAV0@@Z 10009f90 f i Metaphlan2Worker.obj
 0001:00008fb0       ??0?$QList@VDescriptor@U2@@@@QAE@ABV0@@Z 10009fb0 f i Metaphlan2Worker.obj
 0001:00009070       ??0?$QList@VDescriptor@U2@@@@QAE@XZ 1000a070 f i Metaphlan2Worker.obj
 0001:00009080       ??0?$QMap@VQString@@VQScriptValue@@@@QAE@XZ 1000a080 f i Metaphlan2Worker.obj
 0001:00009090       ??0?$QSet@VQString@@@@QAE@XZ 1000a090 f i Metaphlan2Worker.obj
 0001:000090a0       ??0Metaphlan2Worker@LocalWorkflow@U2@@QAE@PAVActor@Workflow@2@@Z 1000a0a0 f   Metaphlan2Worker.obj
 0001:000090e0       ??0const_iterator@?$QList@VDescriptor@U2@@@@QAE@PAUNode@1@@Z 1000a0e0 f i Metaphlan2Worker.obj
 0001:000090f0       ??0const_iterator@?$QMap@VDescriptor@U2@@VQVariant@@@@QAE@PBU?$QMapNode@VDescriptor@U2@@VQVariant@@@@@Z 1000a0f0 f i Metaphlan2Worker.obj
 0001:00009100       ??0iterator@?$QMap@VQString@@VQScriptValue@@@@QAE@PAU?$QMapNode@VQString@@VQScriptValue@@@@@Z 1000a100 f i Metaphlan2Worker.obj
 0001:00009110       ??0iterator@?$QMap@VQString@@VQVariant@@@@QAE@PAU?$QMapNode@VQString@@VQVariant@@@@@Z 1000a110 f i Metaphlan2Worker.obj
 0001:00009120       ??1?$QForeachContainer@V?$QList@VDescriptor@U2@@@@@@QAE@XZ 1000a120 f i Metaphlan2Worker.obj
 0001:00009150       ??1?$QHash@VQString@@UQHashDummyValue@@@@QAE@XZ 1000a150 f i Metaphlan2Worker.obj
 0001:00009180       ??1?$QHashNode@VQString@@UQHashDummyValue@@@@QAE@XZ 1000a180 f i Metaphlan2Worker.obj
 0001:00009190       ??1?$QList@PAVExternalToolListener@U2@@@@QAE@XZ 1000a190 f i Metaphlan2Worker.obj
 0001:000091c0       ??1?$QList@VDescriptor@U2@@@@QAE@XZ 1000a1c0 f i Metaphlan2Worker.obj
 0001:000091f0       ??1?$QMap@VQString@@VQScriptValue@@@@QAE@XZ 1000a1f0 f i Metaphlan2Worker.obj
 0001:00009240       ??1?$QMap@VQString@@VQVariant@@@@QAE@XZ 1000a240 f i Metaphlan2Worker.obj
 0001:00009290       ??1?$QSet@VQString@@@@QAE@XZ 1000a290 f i Metaphlan2Worker.obj
 0001:000092c0       ??1Metaphlan2Worker@LocalWorkflow@U2@@UAE@XZ 1000a2c0 f i Metaphlan2Worker.obj
 0001:000092d0       ??8const_iterator@?$QMap@VDescriptor@U2@@VQVariant@@@@QBE_NABV01@@Z 1000a2d0 f i Metaphlan2Worker.obj
 0001:000092f0       ??9const_iterator@?$QList@VDescriptor@U2@@@@QBE_NABV01@@Z 1000a2f0 f i Metaphlan2Worker.obj
 0001:00009310       ??9const_iterator@?$QMap@VDescriptor@U2@@VQVariant@@@@QBE_NABV01@@Z 1000a310 f i Metaphlan2Worker.obj
 0001:00009330       ??A?$QMap@VQString@@VQScriptValue@@@@QAEAAVQScriptValue@@ABVQString@@@Z 1000a330 f i Metaphlan2Worker.obj
 0001:00009400       ??A?$QMap@VQString@@VQVariant@@@@QAEAAVQVariant@@ABVQString@@@Z 1000a400 f i Metaphlan2Worker.obj
 0001:000094d0       ??Dconst_iterator@?$QList@VDescriptor@U2@@@@QBEABVDescriptor@U2@@XZ 1000a4d0 f i Metaphlan2Worker.obj
 0001:000094e0       ??Diterator@?$QMap@VQString@@VQScriptValue@@@@QBEAAVQScriptValue@@XZ 1000a4e0 f i Metaphlan2Worker.obj
 0001:000094f0       ??Diterator@?$QMap@VQString@@VQVariant@@@@QBEAAVQVariant@@XZ 1000a4f0 f i Metaphlan2Worker.obj
 0001:00009500       ??Econst_iterator@?$QList@VDescriptor@U2@@@@QAEAAV01@XZ 1000a500 f i Metaphlan2Worker.obj
 0001:00009510       ??Econst_iterator@?$QMap@VDescriptor@U2@@VQVariant@@@@QAEAAV01@XZ 1000a510 f i Metaphlan2Worker.obj
 0001:00009521       ??_EMetaphlan2Worker@LocalWorkflow@U2@@W7AEPAXI@Z 1000a521 f i Metaphlan2Worker.obj
 0001:00009529       ??_EMetaphlan2Worker@LocalWorkflow@U2@@WBA@AEPAXI@Z 1000a529 f i Metaphlan2Worker.obj
 0001:00009540       ??_G?$QHashNode@VQString@@UQHashDummyValue@@@@QAEPAXI@Z 1000a540 f i Metaphlan2Worker.obj
 0001:00009570       ??_EDescriptor@U2@@UAEPAXI@Z 1000a570 f i Metaphlan2Worker.obj
 0001:00009570       ??_GDescriptor@U2@@UAEPAXI@Z 1000a570 f i Metaphlan2Worker.obj
 0001:000095a0       ??_EFailTask@U2@@UAEPAXI@Z 1000a5a0 f i Metaphlan2Worker.obj
 0001:000095a0       ??_GFailTask@U2@@UAEPAXI@Z 1000a5a0 f i Metaphlan2Worker.obj
 0001:000095d0       ??_EMetaphlan2Worker@LocalWorkflow@U2@@UAEPAXI@Z 1000a5d0 f i Metaphlan2Worker.obj
 0001:000095d0       ??_GMetaphlan2Worker@LocalWorkflow@U2@@UAEPAXI@Z 1000a5d0 f i Metaphlan2Worker.obj
 0001:00009600       ??_GQScriptValue@@QAEPAXI@Z 1000a600 f i Metaphlan2Worker.obj
 0001:00009630       ??_GQVariant@@QAEPAXI@Z    1000a630 f i Metaphlan2Worker.obj
 0001:00009660       ??_GTaskSignalMapper@U2@@UAEPAXI@Z 1000a660 f i Metaphlan2Worker.obj
 0001:00009660       ??_ETaskSignalMapper@U2@@UAEPAXI@Z 1000a660 f i Metaphlan2Worker.obj
 0001:00009690       ?addOutputToDashboard@Metaphlan2Worker@LocalWorkflow@U2@@ABEXABVQString@@0@Z 1000a690 f   Metaphlan2Worker.obj
 0001:00009780       ?append@?$QList@VDescriptor@U2@@@@QAEXABVDescriptor@U2@@@Z 1000a780 f i Metaphlan2Worker.obj
 0001:00009870       ?begin@?$QList@VDescriptor@U2@@@@QBE?AVconst_iterator@1@XZ 1000a870 f i Metaphlan2Worker.obj
 0001:00009890       ?begin@?$QMap@VDescriptor@U2@@VQVariant@@@@QBE?AVconst_iterator@1@XZ 1000a890 f i Metaphlan2Worker.obj
 0001:000098b0       ?begin@?$QMapData@VDescriptor@U2@@VQVariant@@@@QAEPAU?$QMapNode@VDescriptor@U2@@VQVariant@@@@XZ 1000a8b0 f i Metaphlan2Worker.obj
 0001:000098c0       ?cleanup@Metaphlan2Worker@LocalWorkflow@U2@@UAEXXZ 1000a8c0 f   Metaphlan2Worker.obj
 0001:000098d0       ?concrete@?$QHash@VQString@@UQHashDummyValue@@@@CAPAU?$QHashNode@VQString@@UQHashDummyValue@@@@PAUNode@QHashData@@@Z 1000a8d0 f i Metaphlan2Worker.obj
 0001:000098e0       ?copy@?$QMapNode@VQString@@VQScriptValue@@@@QBEPAU1@PAU?$QMapData@VQString@@VQScriptValue@@@@@Z 1000a8e0 f i Metaphlan2Worker.obj
 0001:00009970       ?copy@?$QMapNode@VQString@@VQVariant@@@@QBEPAU1@PAU?$QMapData@VQString@@VQVariant@@@@@Z 1000a970 f i Metaphlan2Worker.obj
 0001:00009a00       ?create@?$QMapData@VQString@@VQScriptValue@@@@SAPAU1@XZ 1000aa00 f i Metaphlan2Worker.obj
 0001:00009a10       ?create@?$QMapData@VQString@@VQVariant@@@@SAPAU1@XZ 1000aa10 f i Metaphlan2Worker.obj
 0001:00009a20       ?createDirectory@Metaphlan2Worker@LocalWorkflow@U2@@ABEXAAVQString@@@Z 1000aa20 f   Metaphlan2Worker.obj
 0001:00009b20       ?createNode@?$QMapData@VQString@@VQScriptValue@@@@QAEPAU?$QMapNode@VQString@@VQScriptValue@@@@ABVQString@@ABVQScriptValue@@PAU2@_N@Z 1000ab20 f i Metaphlan2Worker.obj
 0001:00009be0       ?createNode@?$QMapData@VQString@@VQVariant@@@@QAEPAU?$QMapNode@VQString@@VQVariant@@@@ABVQString@@ABVQVariant@@PAU2@_N@Z 1000abe0 f i Metaphlan2Worker.obj
 0001:00009ca0       ?createOutputToolDirectory@Metaphlan2Worker@LocalWorkflow@U2@@ABE?AVQString@@ABV4@ABVMessage@Workflow@3@_NW4Output@123@@Z 1000aca0 f   Metaphlan2Worker.obj
 0001:00009ef0       ?dataFinished@Metaphlan2Worker@LocalWorkflow@U2@@ABE_NXZ 1000aef0 f   Metaphlan2Worker.obj
 0001:00009f00       ?dealloc@?$QList@PAVExternalToolListener@U2@@@@AAEXPAUData@QListData@@@Z 1000af00 f i Metaphlan2Worker.obj
 0001:00009f20       ?dealloc@?$QList@VDescriptor@U2@@@@AAEXPAUData@QListData@@@Z 1000af20 f i Metaphlan2Worker.obj
 0001:00009f70       ?deleteNode2@?$QHash@VQString@@UQHashDummyValue@@@@CAXPAUNode@QHashData@@@Z 1000af70 f i Metaphlan2Worker.obj
 0001:00009f80       ?destroy@?$QMapData@VQString@@VQScriptValue@@@@QAEXXZ 1000af80 f i Metaphlan2Worker.obj
 0001:00009fb0       ?destroy@?$QMapData@VQString@@VQVariant@@@@QAEXXZ 1000afb0 f i Metaphlan2Worker.obj
 0001:00009fe0       ?destroySubTree@?$QMapNode@VQString@@VQScriptValue@@@@QAEXXZ 1000afe0 f i Metaphlan2Worker.obj
 0001:0000a020       ?destroySubTree@?$QMapNode@VQString@@VQVariant@@@@QAEXXZ 1000b020 f i Metaphlan2Worker.obj
 0001:0000a060       ?detach@?$QMap@VQString@@VQScriptValue@@@@QAEXXZ 1000b060 f i Metaphlan2Worker.obj
 0001:0000a080       ?detach@?$QMap@VQString@@VQVariant@@@@QAEXXZ 1000b080 f i Metaphlan2Worker.obj
 0001:0000a0a0       ?detach_helper@?$QList@VDescriptor@U2@@@@AAEXH@Z 1000b0a0 f i Metaphlan2Worker.obj
 0001:0000a170       ?detach_helper@?$QMap@VQString@@VQScriptValue@@@@AAEXXZ 1000b170 f i Metaphlan2Worker.obj
 0001:0000a1f0       ?detach_helper@?$QMap@VQString@@VQVariant@@@@AAEXXZ 1000b1f0 f i Metaphlan2Worker.obj
 0001:0000a270       ?detach_helper_grow@?$QList@VDescriptor@U2@@@@AAEPAUNode@1@HH@Z 1000b270 f i Metaphlan2Worker.obj
 0001:0000a3c0       ?end@?$QList@VDescriptor@U2@@@@QBE?AVconst_iterator@1@XZ 1000b3c0 f i Metaphlan2Worker.obj
 0001:0000a3e0       ?end@?$QMap@VDescriptor@U2@@VQVariant@@@@QBE?AVconst_iterator@1@XZ 1000b3e0 f i Metaphlan2Worker.obj
 0001:0000a400       ?end@?$QMapData@VDescriptor@U2@@VQVariant@@@@QAEPAU?$QMapNode@VDescriptor@U2@@VQVariant@@@@XZ 1000b400 f i Metaphlan2Worker.obj
 0001:0000a410       ?end@?$QMapData@VQString@@VQScriptValue@@@@QAEPAU?$QMapNode@VQString@@VQScriptValue@@@@XZ 1000b410 f i Metaphlan2Worker.obj
 0001:0000a420       ?end@?$QMapData@VQString@@VQVariant@@@@QAEPAU?$QMapNode@VQString@@VQVariant@@@@XZ 1000b420 f i Metaphlan2Worker.obj
 0001:0000a430       ?findNode@?$QMapData@VDescriptor@U2@@VQVariant@@@@QBEPAU?$QMapNode@VDescriptor@U2@@VQVariant@@@@ABVDescriptor@U2@@@Z 1000b430 f i Metaphlan2Worker.obj
 0001:0000a470       ?findNode@?$QMapData@VQString@@PAVIntegralBus@Workflow@U2@@@@QBEPAU?$QMapNode@VQString@@PAVIntegralBus@Workflow@U2@@@@ABVQString@@@Z 1000b470 f i Metaphlan2Worker.obj
 0001:0000a4b0       ?findNode@?$QMapData@VQString@@VQScriptValue@@@@QBEPAU?$QMapNode@VQString@@VQScriptValue@@@@ABVQString@@@Z 1000b4b0 f i Metaphlan2Worker.obj
 0001:0000a4f0       ?findNode@?$QMapData@VQString@@VQVariant@@@@QBEPAU?$QMapNode@VQString@@VQVariant@@@@ABVQString@@@Z 1000b4f0 f i Metaphlan2Worker.obj
 0001:0000a530       ?freeData@?$QHash@VQString@@UQHashDummyValue@@@@AAEXPAUQHashData@@@Z 1000b530 f i Metaphlan2Worker.obj
 0001:0000a550       ?getDefaultOutputDir@Metaphlan2Worker@LocalWorkflow@U2@@ABE?AVQString@@XZ 1000b550 f   Metaphlan2Worker.obj
 0001:0000a6b0       ?getSettings@Metaphlan2Worker@LocalWorkflow@U2@@AAE?AUMetaphlan2TaskSettings@3@AAVU2OpStatus@3@@Z 1000b6b0 f   Metaphlan2Worker.obj
 0001:0000b010       ?init@Metaphlan2Worker@LocalWorkflow@U2@@UAEXXZ 1000c010 f   Metaphlan2Worker.obj
 0001:0000b1d0       ?insert@?$QMap@VQString@@VQScriptValue@@@@QAE?AViterator@1@ABVQString@@ABVQScriptValue@@@Z 1000c1d0 f i Metaphlan2Worker.obj
 0001:0000b290       ?insert@?$QMap@VQString@@VQVariant@@@@QAE?AViterator@1@ABVQString@@ABVQVariant@@@Z 1000c290 f i Metaphlan2Worker.obj
 0001:0000b350       ?invoke@?$MetaTypeInvoker@U?$QVariantValueHelper@H@QtPrivate@@ABVQVariant@@H@QtPrivate@@SAHABVQVariant@@@Z 1000c350 f i Metaphlan2Worker.obj
 0001:0000b390       ?isReadyToRun@Metaphlan2Worker@LocalWorkflow@U2@@ABE_NXZ 1000c390 f   Metaphlan2Worker.obj
 0001:0000b3b0       ?key@const_iterator@?$QMap@VDescriptor@U2@@VQVariant@@@@QBEABVDescriptor@U2@@XZ 1000c3b0 f i Metaphlan2Worker.obj
 0001:0000b3c0       ?leftNode@?$QMapNode@VDescriptor@U2@@VQVariant@@@@QBEPAU1@XZ 1000c3c0 f i Metaphlan2Worker.obj
 0001:0000b3d0       ?leftNode@?$QMapNode@VQString@@PAVIntegralBus@Workflow@U2@@@@QBEPAU1@XZ 1000c3d0 f i Metaphlan2Worker.obj
 0001:0000b3e0       ?leftNode@?$QMapNode@VQString@@VQScriptValue@@@@QBEPAU1@XZ 1000c3e0 f i Metaphlan2Worker.obj
 0001:0000b3f0       ?leftNode@?$QMapNode@VQString@@VQVariant@@@@QBEPAU1@XZ 1000c3f0 f i Metaphlan2Worker.obj
 0001:0000b400       ?lowerBound@?$QMapNode@VDescriptor@U2@@VQVariant@@@@QAEPAU1@ABVDescriptor@U2@@@Z 1000c400 f i Metaphlan2Worker.obj
 0001:0000b440       ?lowerBound@?$QMapNode@VQString@@PAVIntegralBus@Workflow@U2@@@@QAEPAU1@ABVQString@@@Z 1000c440 f i Metaphlan2Worker.obj
 0001:0000b480       ?lowerBound@?$QMapNode@VQString@@VQScriptValue@@@@QAEPAU1@ABVQString@@@Z 1000c480 f i Metaphlan2Worker.obj
 0001:0000b4c0       ?lowerBound@?$QMapNode@VQString@@VQVariant@@@@QAEPAU1@ABVQString@@@Z 1000c4c0 f i Metaphlan2Worker.obj
 0001:0000b500       ?metaType@?$QVariantValueHelper@H@QtPrivate@@SAHABVQVariant@@@Z 1000c500 f i Metaphlan2Worker.obj
 0001:0000b540       ?nextNode@?$QMapNode@VDescriptor@U2@@VQVariant@@@@QBEPBU1@XZ 1000c540 f i Metaphlan2Worker.obj
 0001:0000b550       ?node_construct@?$QList@VDescriptor@U2@@@@AAEXPAUNode@1@ABVDescriptor@U2@@@Z 1000c550 f i Metaphlan2Worker.obj
 0001:0000b5e0       ?node_copy@?$QList@VDescriptor@U2@@@@AAEXPAUNode@1@00@Z 1000c5e0 f i Metaphlan2Worker.obj
 0001:0000b6b0       ?node_destruct@?$QList@PAVExternalToolListener@U2@@@@AAEXPAUNode@1@0@Z 1000c6b0 f i Metaphlan2Worker.obj
 0001:0000b6c0       ?node_destruct@?$QList@VDescriptor@U2@@@@AAEXPAUNode@1@0@Z 1000c6c0 f i Metaphlan2Worker.obj
 0001:0000b6f0       ?node_destruct@?$QList@VDescriptor@U2@@@@AAEXPAUNode@1@@Z 1000c6f0 f i Metaphlan2Worker.obj
 0001:0000b710       ?qt_metatype_id@?$QMetaTypeId2@H@@SAHXZ 1000c710 f i Metaphlan2Worker.obj
 0001:0000b720       ?reserve@?$QList@VDescriptor@U2@@@@QAEXH@Z 1000c720 f i Metaphlan2Worker.obj
 0001:0000b750       ?rightNode@?$QMapNode@VDescriptor@U2@@VQVariant@@@@QBEPAU1@XZ 1000c750 f i Metaphlan2Worker.obj
 0001:0000b760       ?rightNode@?$QMapNode@VQString@@PAVIntegralBus@Workflow@U2@@@@QBEPAU1@XZ 1000c760 f i Metaphlan2Worker.obj
 0001:0000b770       ?rightNode@?$QMapNode@VQString@@VQScriptValue@@@@QBEPAU1@XZ 1000c770 f i Metaphlan2Worker.obj
 0001:0000b780       ?rightNode@?$QMapNode@VQString@@VQVariant@@@@QBEPAU1@XZ 1000c780 f i Metaphlan2Worker.obj
 0001:0000b790       ?root@?$QMapData@VDescriptor@U2@@VQVariant@@@@QBEPAU?$QMapNode@VDescriptor@U2@@VQVariant@@@@XZ 1000c790 f i Metaphlan2Worker.obj
 0001:0000b7a0       ?root@?$QMapData@VQString@@PAVIntegralBus@Workflow@U2@@@@QBEPAU?$QMapNode@VQString@@PAVIntegralBus@Workflow@U2@@@@XZ 1000c7a0 f i Metaphlan2Worker.obj
 0001:0000b7b0       ?root@?$QMapData@VQString@@VQScriptValue@@@@QBEPAU?$QMapNode@VQString@@VQScriptValue@@@@XZ 1000c7b0 f i Metaphlan2Worker.obj
 0001:0000b7c0       ?root@?$QMapData@VQString@@VQVariant@@@@QBEPAU?$QMapNode@VQString@@VQVariant@@@@XZ 1000c7c0 f i Metaphlan2Worker.obj
 0001:0000b7d0       ?size@?$QMap@VDescriptor@U2@@VQVariant@@@@QBEHXZ 1000c7d0 f i Metaphlan2Worker.obj
 0001:0000b7e0       ?sl_taskFinished@Metaphlan2Worker@LocalWorkflow@U2@@AAEXPAVTask@3@@Z 1000c7e0 f   Metaphlan2Worker.obj
 0001:0000b8d0       ?t@Node@?$QList@VDescriptor@U2@@@@QAEAAVDescriptor@U2@@XZ 1000c8d0 f i Metaphlan2Worker.obj
 0001:0000b8e0       ?tick@Metaphlan2Worker@LocalWorkflow@U2@@UAEPAVTask@3@XZ 1000c8e0 f   Metaphlan2Worker.obj
 0001:0000bae0       ?tr@Metaphlan2Worker@LocalWorkflow@U2@@SA?AVQString@@PBD0H@Z 1000cae0 f i Metaphlan2Worker.obj
 0001:0000bb10       ?uniqueKeys@?$QMap@VDescriptor@U2@@VQVariant@@@@QBE?AV?$QList@VDescriptor@U2@@@@XZ 1000cb10 f i Metaphlan2Worker.obj
 0001:0000bc10       ?value@?$QMap@VDescriptor@U2@@VQVariant@@@@QBE?BVQVariant@@ABVDescriptor@U2@@ABV2@@Z 1000cc10 f i Metaphlan2Worker.obj
 0001:0000bc70       ?value@?$QMap@VQString@@PAVIntegralBus@Workflow@U2@@@@QBEQAVIntegralBus@Workflow@U2@@ABVQString@@ABQAV234@@Z 1000cc70 f i Metaphlan2Worker.obj
 0001:0000bcc0       ??$_Move@AAPAVDataType@U2@@@std@@YA$$QAPAVDataType@U2@@AAPAV12@@Z 1000ccc0 f i Metaphlan2WorkerFactory.obj
 0001:0000bcd0       ??$qSwap@PAVDataType@U2@@@@YAXAAPAVDataType@U2@@0@Z 1000ccd0 f i Metaphlan2WorkerFactory.obj
 0001:0000bcf0       ??$swap@PAVDataType@U2@@@std@@YAXAAPAVDataType@U2@@0@Z 1000ccf0 f i Metaphlan2WorkerFactory.obj
 0001:0000bd10       ??0?$QExplicitlySharedDataPointer@VDataType@U2@@@@QAE@ABV0@@Z 1000cd10 f i Metaphlan2WorkerFactory.obj
 0001:0000bd30       ??0?$QExplicitlySharedDataPointer@VDataType@U2@@@@QAE@PAVDataType@U2@@@Z 1000cd30 f i Metaphlan2WorkerFactory.obj
 0001:0000bd50       ??0?$QExplicitlySharedDataPointer@VDataType@U2@@@@QAE@XZ 1000cd50 f i Metaphlan2WorkerFactory.obj
 0001:0000bd60       ??0?$QFlags@W4Flag@Attribute@U2@@@@QAE@VQFlag@@@Z 1000cd60 f i Metaphlan2WorkerFactory.obj
 0001:0000bd70       ??0?$QFlags@W4Flag@Attribute@U2@@@@QAE@W4Flag@Attribute@U2@@@Z 1000cd70 f i Metaphlan2WorkerFactory.obj
 0001:0000bd80       ??0?$QList@PAVAttribute@U2@@@@QAE@XZ 1000cd80 f i Metaphlan2WorkerFactory.obj
 0001:0000bd90       ??0?$QList@PAVPortDescriptor@Workflow@U2@@@@QAE@XZ 1000cd90 f i Metaphlan2WorkerFactory.obj
 0001:0000bda0       ??0?$QList@U?$QPair@VQString@@V1@@@@@QAE@XZ 1000cda0 f i Metaphlan2WorkerFactory.obj
 0001:0000bdb0       ??0?$QList@VQVariant@@@@QAE@XZ 1000cdb0 f i Metaphlan2WorkerFactory.obj
 0001:0000bdc0       ??0?$QMap@VDescriptor@U2@@V?$QExplicitlySharedDataPointer@VDataType@U2@@@@@@QAE@XZ 1000cdc0 f i Metaphlan2WorkerFactory.obj
 0001:0000bdd0       ??0?$QMap@VQString@@PAVPropertyDelegate@U2@@@@QAE@XZ 1000cdd0 f i Metaphlan2WorkerFactory.obj
 0001:0000bde0       ??0?$QMap@VQString@@VQVariant@@@@QAE@XZ 1000cde0 f i Metaphlan2WorkerFactory.obj
 0001:0000bdf0       ??0?$QPair@VQString@@V1@@@QAE@ABU0@@Z 1000cdf0 f i Metaphlan2WorkerFactory.obj
 0001:0000be50       ??0?$QPair@VQString@@V1@@@QAE@ABVQString@@0@Z 1000ce50 f i Metaphlan2WorkerFactory.obj
 0001:0000beb0       ??0Metaphlan2Validator@Workflow@U2@@QAE@XZ 1000ceb0 f i Metaphlan2WorkerFactory.obj
 0001:0000bec0       ??0Metaphlan2WorkerFactory@LocalWorkflow@U2@@QAE@XZ 1000cec0 f   Metaphlan2WorkerFactory.obj
 0001:0000bee0       ??0iterator@?$QMap@VDescriptor@U2@@V?$QExplicitlySharedDataPointer@VDataType@U2@@@@@@QAE@PAU?$QMapNode@VDescriptor@U2@@V?$QExplicitlySharedDataPointer@VDataType@U2@@@@@@@Z 1000cee0 f i Metaphlan2WorkerFactory.obj
 0001:0000bef0       ??0iterator@?$QMap@VQString@@PAVPropertyDelegate@U2@@@@QAE@PAU?$QMapNode@VQString@@PAVPropertyDelegate@U2@@@@@Z 1000cef0 f i Metaphlan2WorkerFactory.obj
 0001:0000bf00       ??1?$QExplicitlySharedDataPointer@VDataType@U2@@@@QAE@XZ 1000cf00 f i Metaphlan2WorkerFactory.obj
 0001:0000bf20       ??1?$QList@PAVAttribute@U2@@@@QAE@XZ 1000cf20 f i Metaphlan2WorkerFactory.obj
 0001:0000bf50       ??1?$QList@PAVPortDescriptor@Workflow@U2@@@@QAE@XZ 1000cf50 f i Metaphlan2WorkerFactory.obj
 0001:0000bf80       ??1?$QList@U?$QPair@VQString@@V1@@@@@QAE@XZ 1000cf80 f i Metaphlan2WorkerFactory.obj
 0001:0000bfd0       ??1?$QList@VQVariant@@@@QAE@XZ 1000cfd0 f i Metaphlan2WorkerFactory.obj
 0001:0000c000       ??1?$QMap@VDescriptor@U2@@V?$QExplicitlySharedDataPointer@VDataType@U2@@@@@@QAE@XZ 1000d000 f i Metaphlan2WorkerFactory.obj
 0001:0000c050       ??1?$QMap@VQString@@PAVPropertyDelegate@U2@@@@QAE@XZ 1000d050 f i Metaphlan2WorkerFactory.obj
 0001:0000c0c0       ??1?$QPair@VQString@@V1@@@QAE@XZ 1000d0c0 f i Metaphlan2WorkerFactory.obj
 0001:0000c120       ??1Metaphlan2Validator@Workflow@U2@@UAE@XZ 1000d120 f i Metaphlan2WorkerFactory.obj
 0001:0000c130       ??1Metaphlan2WorkerFactory@LocalWorkflow@U2@@UAE@XZ 1000d130 f i Metaphlan2WorkerFactory.obj
 0001:0000c140       ??4?$QExplicitlySharedDataPointer@VDataType@U2@@@@QAEAAV0@$$QAV0@@Z 1000d140 f i Metaphlan2WorkerFactory.obj
 0001:0000c160       ??4?$QExplicitlySharedDataPointer@VDataType@U2@@@@QAEAAV0@ABV0@@Z 1000d160 f i Metaphlan2WorkerFactory.obj
 0001:0000c1b0       ??6?$QList@PAVAttribute@U2@@@@QAEAAV0@ABQAVAttribute@U2@@@Z 1000d1b0 f i Metaphlan2WorkerFactory.obj
 0001:0000c1d0       ??6?$QList@PAVPortDescriptor@Workflow@U2@@@@QAEAAV0@ABQAVPortDescriptor@Workflow@U2@@@Z 1000d1d0 f i Metaphlan2WorkerFactory.obj
 0001:0000c1f0       ??6?$QList@U?$QPair@VQString@@V1@@@@@QAEAAV0@ABU?$QPair@VQString@@V1@@@@Z 1000d1f0 f i Metaphlan2WorkerFactory.obj
 0001:0000c210       ??6?$QList@VQVariant@@@@QAEAAV0@ABVQVariant@@@Z 1000d210 f i Metaphlan2WorkerFactory.obj
 0001:0000c230       ??A?$QMap@VDescriptor@U2@@V?$QExplicitlySharedDataPointer@VDataType@U2@@@@@@QAEAAV?$QExplicitlySharedDataPointer@VDataType@U2@@@@ABVDescriptor@U2@@@Z 1000d230 f i Metaphlan2WorkerFactory.obj
 0001:0000c2f0       ??A?$QMap@VQString@@PAVPropertyDelegate@U2@@@@QAEAAPAVPropertyDelegate@U2@@ABVQString@@@Z 1000d2f0 f i Metaphlan2WorkerFactory.obj
 0001:0000c370       ??Diterator@?$QMap@VDescriptor@U2@@V?$QExplicitlySharedDataPointer@VDataType@U2@@@@@@QBEAAV?$QExplicitlySharedDataPointer@VDataType@U2@@@@XZ 1000d370 f i Metaphlan2WorkerFactory.obj
 0001:0000c380       ??Diterator@?$QMap@VQString@@PAVPropertyDelegate@U2@@@@QBEAAPAVPropertyDelegate@U2@@XZ 1000d380 f i Metaphlan2WorkerFactory.obj
 0001:0000c390       ??H@YA?BVQString@@ABV0@PBD@Z 1000d390 f i Metaphlan2WorkerFactory.obj
 0001:0000c430       ??U?$QFlags@W4Flag@Attribute@U2@@@@QBE?AV0@W4Flag@Attribute@U2@@@Z 1000d430 f i Metaphlan2WorkerFactory.obj
 0001:0000c450       ??U@YA?AV?$QFlags@W4Flag@Attribute@U2@@@@W4Flag@Attribute@U2@@0@Z 1000d450 f i Metaphlan2WorkerFactory.obj
 0001:0000c460       ??_EMetaphlan2WorkerFactory@LocalWorkflow@U2@@W7AEPAXI@Z 1000d460 f i Metaphlan2WorkerFactory.obj
 0001:0000c470       ??_G?$QExplicitlySharedDataPointer@VDataType@U2@@@@QAEPAXI@Z 1000d470 f i Metaphlan2WorkerFactory.obj
 0001:0000c4b0       ??_G?$QPair@VQString@@V1@@@QAEPAXI@Z 1000d4b0 f i Metaphlan2WorkerFactory.obj
 0001:0000c520       ??_EAttribute@U2@@UAEPAXI@Z 1000d520 f i Metaphlan2WorkerFactory.obj
 0001:0000c520       ??_GAttribute@U2@@UAEPAXI@Z 1000d520 f i Metaphlan2WorkerFactory.obj
 0001:0000c550       ??_EComboBoxDelegate@U2@@UAEPAXI@Z 1000d550 f i Metaphlan2WorkerFactory.obj
 0001:0000c550       ??_GComboBoxDelegate@U2@@UAEPAXI@Z 1000d550 f i Metaphlan2WorkerFactory.obj
 0001:0000c580       ??_GDatabaseDelegate@LocalWorkflow@U2@@UAEPAXI@Z 1000d580 f i Metaphlan2WorkerFactory.obj
 0001:0000c580       ??_EDatabaseDelegate@LocalWorkflow@U2@@UAEPAXI@Z 1000d580 f i Metaphlan2WorkerFactory.obj
 0001:0000c5b0       ??_EDelegateEditor@U2@@UAEPAXI@Z 1000d5b0 f i Metaphlan2WorkerFactory.obj
 0001:0000c5b0       ??_GDelegateEditor@U2@@UAEPAXI@Z 1000d5b0 f i Metaphlan2WorkerFactory.obj
 0001:0000c5e0       ??_EIntegralBusActorPrototype@Workflow@U2@@UAEPAXI@Z 1000d5e0 f i Metaphlan2WorkerFactory.obj
 0001:0000c5e0       ??_GIntegralBusActorPrototype@Workflow@U2@@UAEPAXI@Z 1000d5e0 f i Metaphlan2WorkerFactory.obj
 0001:0000c610       ??_EMapDataType@U2@@UAEPAXI@Z 1000d610 f i Metaphlan2WorkerFactory.obj
 0001:0000c610       ??_GMapDataType@U2@@UAEPAXI@Z 1000d610 f i Metaphlan2WorkerFactory.obj
 0001:0000c640       ??_GMetaphlan2Validator@Workflow@U2@@UAEPAXI@Z 1000d640 f i Metaphlan2WorkerFactory.obj
 0001:0000c640       ??_EMetaphlan2Validator@Workflow@U2@@UAEPAXI@Z 1000d640 f i Metaphlan2WorkerFactory.obj
 0001:0000c670       ??_EMetaphlan2WorkerFactory@LocalWorkflow@U2@@UAEPAXI@Z 1000d670 f i Metaphlan2WorkerFactory.obj
 0001:0000c670       ??_GMetaphlan2WorkerFactory@LocalWorkflow@U2@@UAEPAXI@Z 1000d670 f i Metaphlan2WorkerFactory.obj
 0001:0000c6a0       ??_EPairedReadsPortValidator@Workflow@U2@@UAEPAXI@Z 1000d6a0 f i Metaphlan2WorkerFactory.obj
 0001:0000c6a0       ??_GPairedReadsPortValidator@Workflow@U2@@UAEPAXI@Z 1000d6a0 f i Metaphlan2WorkerFactory.obj
 0001:0000c6d0       ??_EPortDescriptor@Workflow@U2@@UAEPAXI@Z 1000d6d0 f i Metaphlan2WorkerFactory.obj
 0001:0000c6d0       ??_GPortDescriptor@Workflow@U2@@UAEPAXI@Z 1000d6d0 f i Metaphlan2WorkerFactory.obj
 0001:0000c700       ??_ESlotRelationDescriptor@U2@@UAEPAXI@Z 1000d700 f i Metaphlan2WorkerFactory.obj
 0001:0000c700       ??_GSlotRelationDescriptor@U2@@UAEPAXI@Z 1000d700 f i Metaphlan2WorkerFactory.obj
 0001:0000c730       ??_ESpinBoxDelegate@U2@@UAEPAXI@Z 1000d730 f i Metaphlan2WorkerFactory.obj
 0001:0000c730       ??_GSpinBoxDelegate@U2@@UAEPAXI@Z 1000d730 f i Metaphlan2WorkerFactory.obj
 0001:0000c760       ??_GURLDelegate@U2@@UAEPAXI@Z 1000d760 f i Metaphlan2WorkerFactory.obj
 0001:0000c760       ??_EURLDelegate@U2@@UAEPAXI@Z 1000d760 f i Metaphlan2WorkerFactory.obj
 0001:0000c790       ??_GVisibilityRelation@U2@@UAEPAXI@Z 1000d790 f i Metaphlan2WorkerFactory.obj
 0001:0000c790       ??_EVisibilityRelation@U2@@UAEPAXI@Z 1000d790 f i Metaphlan2WorkerFactory.obj
 0001:0000c7c0       ?append@?$QList@PAVAttribute@U2@@@@QAEXABQAVAttribute@U2@@@Z 1000d7c0 f i Metaphlan2WorkerFactory.obj
 0001:0000c850       ?append@?$QList@PAVPortDescriptor@Workflow@U2@@@@QAEXABQAVPortDescriptor@Workflow@U2@@@Z 1000d850 f i Metaphlan2WorkerFactory.obj
 0001:0000c8e0       ?append@?$QList@U?$QPair@VQString@@V1@@@@@QAEXABU?$QPair@VQString@@V1@@@@Z 1000d8e0 f i Metaphlan2WorkerFactory.obj
 0001:0000c970       ?append@?$QList@VQVariant@@@@QAEXABVQVariant@@@Z 1000d970 f i Metaphlan2WorkerFactory.obj
 0001:0000ca50       ?cleanup@Metaphlan2WorkerFactory@LocalWorkflow@U2@@SAXXZ 1000da50 f   Metaphlan2WorkerFactory.obj
 0001:0000caa0       ?copy@?$QMapNode@VDescriptor@U2@@V?$QExplicitlySharedDataPointer@VDataType@U2@@@@@@QBEPAU1@PAU?$QMapData@VDescriptor@U2@@V?$QExplicitlySharedDataPointer@VDataType@U2@@@@@@@Z 1000daa0 f i Metaphlan2WorkerFactory.obj
 0001:0000cb30       ?copy@?$QMapNode@VQString@@PAVPropertyDelegate@U2@@@@QBEPAU1@PAU?$QMapData@VQString@@PAVPropertyDelegate@U2@@@@@Z 1000db30 f i Metaphlan2WorkerFactory.obj
 0001:0000cbc0       ?create@?$QMapData@VDescriptor@U2@@V?$QExplicitlySharedDataPointer@VDataType@U2@@@@@@SAPAU1@XZ 1000dbc0 f i Metaphlan2WorkerFactory.obj
 0001:0000cbd0       ?create@?$QMapData@VQString@@PAVPropertyDelegate@U2@@@@SAPAU1@XZ 1000dbd0 f i Metaphlan2WorkerFactory.obj
 0001:0000cbe0       ?createNode@?$QMapData@VDescriptor@U2@@V?$QExplicitlySharedDataPointer@VDataType@U2@@@@@@QAEPAU?$QMapNode@VDescriptor@U2@@V?$QExplicitlySharedDataPointer@VDataType@U2@@@@@@ABVDescriptor@U2@@ABV?$QExplicitlySharedDataPointer@VDataType@U2@@@@PAU2@_N@Z 1000dbe0 f i Metaphlan2WorkerFactory.obj
 0001:0000cca0       ?createNode@?$QMapData@VQString@@PAVPropertyDelegate@U2@@@@QAEPAU?$QMapNode@VQString@@PAVPropertyDelegate@U2@@@@ABVQString@@ABQAVPropertyDelegate@U2@@PAU2@_N@Z 1000dca0 f i Metaphlan2WorkerFactory.obj
 0001:0000cd40       ?createWorker@Metaphlan2WorkerFactory@LocalWorkflow@U2@@UAEPAVWorker@Workflow@3@PAVActor@53@@Z 1000dd40 f   Metaphlan2WorkerFactory.obj
 0001:0000cdb0       ?dealloc@?$QList@PAVAttribute@U2@@@@AAEXPAUData@QListData@@@Z 1000ddb0 f i Metaphlan2WorkerFactory.obj
 0001:0000cdd0       ?dealloc@?$QList@PAVPortDescriptor@Workflow@U2@@@@AAEXPAUData@QListData@@@Z 1000ddd0 f i Metaphlan2WorkerFactory.obj
 0001:0000cdf0       ?dealloc@?$QList@U?$QPair@VQString@@V1@@@@@AAEXPAUData@QListData@@@Z 1000ddf0 f i Metaphlan2WorkerFactory.obj
 0001:0000ce20       ?dealloc@?$QList@VQVariant@@@@AAEXPAUData@QListData@@@Z 1000de20 f i Metaphlan2WorkerFactory.obj
 0001:0000ce80       ?destroy@?$QMapData@VDescriptor@U2@@V?$QExplicitlySharedDataPointer@VDataType@U2@@@@@@QAEXXZ 1000de80 f i Metaphlan2WorkerFactory.obj
 0001:0000ceb0       ?destroy@?$QMapData@VQString@@PAVPropertyDelegate@U2@@@@QAEXXZ 1000deb0 f i Metaphlan2WorkerFactory.obj
 0001:0000cf00       ?destroySubTree@?$QMapNode@VDescriptor@U2@@V?$QExplicitlySharedDataPointer@VDataType@U2@@@@@@QAEXXZ 1000df00 f i Metaphlan2WorkerFactory.obj
 0001:0000cf50       ?destroySubTree@?$QMapNode@VQString@@PAVPropertyDelegate@U2@@@@QAEXXZ 1000df50 f i Metaphlan2WorkerFactory.obj
 0001:0000cf80       ?detach@?$QMap@VDescriptor@U2@@V?$QExplicitlySharedDataPointer@VDataType@U2@@@@@@QAEXXZ 1000df80 f i Metaphlan2WorkerFactory.obj
 0001:0000cfa0       ?detach@?$QMap@VQString@@PAVPropertyDelegate@U2@@@@QAEXXZ 1000dfa0 f i Metaphlan2WorkerFactory.obj
 0001:0000cfc0       ?detach_helper@?$QMap@VDescriptor@U2@@V?$QExplicitlySharedDataPointer@VDataType@U2@@@@@@AAEXXZ 1000dfc0 f i Metaphlan2WorkerFactory.obj
 0001:0000d040       ?detach_helper@?$QMap@VQString@@PAVPropertyDelegate@U2@@@@AAEXXZ 1000e040 f i Metaphlan2WorkerFactory.obj
 0001:0000d0f0       ?detach_helper_grow@?$QList@PAVAttribute@U2@@@@AAEPAUNode@1@HH@Z 1000e0f0 f i Metaphlan2WorkerFactory.obj
 0001:0000d200       ?detach_helper_grow@?$QList@PAVPortDescriptor@Workflow@U2@@@@AAEPAUNode@1@HH@Z 1000e200 f i Metaphlan2WorkerFactory.obj
 0001:0000d310       ?detach_helper_grow@?$QList@U?$QPair@VQString@@V1@@@@@AAEPAUNode@1@HH@Z 1000e310 f i Metaphlan2WorkerFactory.obj
 0001:0000d480       ?detach_helper_grow@?$QList@VQVariant@@@@AAEPAUNode@1@HH@Z 1000e480 f i Metaphlan2WorkerFactory.obj
 0001:0000d5d0       ?end@?$QMapData@VDescriptor@U2@@V?$QExplicitlySharedDataPointer@VDataType@U2@@@@@@QAEPAU?$QMapNode@VDescriptor@U2@@V?$QExplicitlySharedDataPointer@VDataType@U2@@@@@@XZ 1000e5d0 f i Metaphlan2WorkerFactory.obj
 0001:0000d5e0       ?end@?$QMapData@VQString@@PAVPropertyDelegate@U2@@@@QAEPAU?$QMapNode@VQString@@PAVPropertyDelegate@U2@@@@XZ 1000e5e0 f i Metaphlan2WorkerFactory.obj
 0001:0000d5f0       ?findNode@?$QMapData@VDescriptor@U2@@V?$QExplicitlySharedDataPointer@VDataType@U2@@@@@@QBEPAU?$QMapNode@VDescriptor@U2@@V?$QExplicitlySharedDataPointer@VDataType@U2@@@@@@ABVDescriptor@U2@@@Z 1000e5f0 f i Metaphlan2WorkerFactory.obj
 0001:0000d630       ?findNode@?$QMapData@VQString@@PAVPropertyDelegate@U2@@@@QBEPAU?$QMapNode@VQString@@PAVPropertyDelegate@U2@@@@ABVQString@@@Z 1000e630 f i Metaphlan2WorkerFactory.obj
 0001:0000d670       ?init@Metaphlan2WorkerFactory@LocalWorkflow@U2@@SAXXZ 1000e670 f   Metaphlan2WorkerFactory.obj
 0001:0000f7e0       ?insert@?$QMap@VDescriptor@U2@@V?$QExplicitlySharedDataPointer@VDataType@U2@@@@@@QAE?AViterator@1@ABVDescriptor@U2@@ABV?$QExplicitlySharedDataPointer@VDataType@U2@@@@@Z 100107e0 f i Metaphlan2WorkerFactory.obj
 0001:0000f8e0       ?insert@?$QMap@VQString@@PAVPropertyDelegate@U2@@@@QAE?AViterator@1@ABVQString@@ABQAVPropertyDelegate@U2@@@Z 100108e0 f i Metaphlan2WorkerFactory.obj
 0001:0000f9a0       ?leftNode@?$QMapNode@VDescriptor@U2@@V?$QExplicitlySharedDataPointer@VDataType@U2@@@@@@QBEPAU1@XZ 100109a0 f i Metaphlan2WorkerFactory.obj
 0001:0000f9b0       ?leftNode@?$QMapNode@VQString@@PAVPropertyDelegate@U2@@@@QBEPAU1@XZ 100109b0 f i Metaphlan2WorkerFactory.obj
 0001:0000f9c0       ?lowerBound@?$QMapNode@VDescriptor@U2@@V?$QExplicitlySharedDataPointer@VDataType@U2@@@@@@QAEPAU1@ABVDescriptor@U2@@@Z 100109c0 f i Metaphlan2WorkerFactory.obj
 0001:0000fa00       ?lowerBound@?$QMapNode@VQString@@PAVPropertyDelegate@U2@@@@QAEPAU1@ABVQString@@@Z 10010a00 f i Metaphlan2WorkerFactory.obj
 0001:0000fa40       ?max@?$numeric_limits@H@std@@SAHXZ 10010a40 f i Metaphlan2WorkerFactory.obj
 0001:0000fa50       ?node_construct@?$QList@PAVAttribute@U2@@@@AAEXPAUNode@1@ABQAVAttribute@U2@@@Z 10010a50 f i Metaphlan2WorkerFactory.obj
 0001:0000fa70       ?node_construct@?$QList@PAVPortDescriptor@Workflow@U2@@@@AAEXPAUNode@1@ABQAVPortDescriptor@Workflow@U2@@@Z 10010a70 f i Metaphlan2WorkerFactory.obj
 0001:0000fa90       ?node_construct@?$QList@U?$QPair@VQString@@V1@@@@@AAEXPAUNode@1@ABU?$QPair@VQString@@V1@@@@Z 10010a90 f i Metaphlan2WorkerFactory.obj
 0001:0000fb20       ?node_construct@?$QList@VQVariant@@@@AAEXPAUNode@1@ABVQVariant@@@Z 10010b20 f i Metaphlan2WorkerFactory.obj
 0001:0000fba0       ?node_copy@?$QList@PAVAttribute@U2@@@@AAEXPAUNode@1@00@Z 10010ba0 f i Metaphlan2WorkerFactory.obj
 0001:0000fbd0       ?node_copy@?$QList@PAVPortDescriptor@Workflow@U2@@@@AAEXPAUNode@1@00@Z 10010bd0 f i Metaphlan2WorkerFactory.obj
 0001:0000fc00       ?node_copy@?$QList@U?$QPair@VQString@@V1@@@@@AAEXPAUNode@1@00@Z 10010c00 f i Metaphlan2WorkerFactory.obj
 0001:0000fd00       ?node_copy@?$QList@VQVariant@@@@AAEXPAUNode@1@00@Z 10010d00 f i Metaphlan2WorkerFactory.obj
 0001:0000fdd0       ?node_destruct@?$QList@PAVAttribute@U2@@@@AAEXPAUNode@1@0@Z 10010dd0 f i Metaphlan2WorkerFactory.obj
 0001:0000fde0       ?node_destruct@?$QList@PAVAttribute@U2@@@@AAEXPAUNode@1@@Z 10010de0 f i Metaphlan2WorkerFactory.obj
 0001:0000fdf0       ?node_destruct@?$QList@PAVPortDescriptor@Workflow@U2@@@@AAEXPAUNode@1@0@Z 10010df0 f i Metaphlan2WorkerFactory.obj
 0001:0000fe00       ?node_destruct@?$QList@PAVPortDescriptor@Workflow@U2@@@@AAEXPAUNode@1@@Z 10010e00 f i Metaphlan2WorkerFactory.obj
 0001:0000fe10       ?node_destruct@?$QList@U?$QPair@VQString@@V1@@@@@AAEXPAUNode@1@0@Z 10010e10 f i Metaphlan2WorkerFactory.obj
 0001:0000fe90       ?node_destruct@?$QList@U?$QPair@VQString@@V1@@@@@AAEXPAUNode@1@@Z 10010e90 f i Metaphlan2WorkerFactory.obj
 0001:0000ff00       ?node_destruct@?$QList@VQVariant@@@@AAEXPAUNode@1@0@Z 10010f00 f i Metaphlan2WorkerFactory.obj
 0001:0000ff40       ?node_destruct@?$QList@VQVariant@@@@AAEXPAUNode@1@@Z 10010f40 f i Metaphlan2WorkerFactory.obj
 0001:0000ff70       ?rightNode@?$QMapNode@VDescriptor@U2@@V?$QExplicitlySharedDataPointer@VDataType@U2@@@@@@QBEPAU1@XZ 10010f70 f i Metaphlan2WorkerFactory.obj
 0001:0000ff80       ?rightNode@?$QMapNode@VQString@@PAVPropertyDelegate@U2@@@@QBEPAU1@XZ 10010f80 f i Metaphlan2WorkerFactory.obj
 0001:0000ff90       ?root@?$QMapData@VDescriptor@U2@@V?$QExplicitlySharedDataPointer@VDataType@U2@@@@@@QBEPAU?$QMapNode@VDescriptor@U2@@V?$QExplicitlySharedDataPointer@VDataType@U2@@@@@@XZ 10010f90 f i Metaphlan2WorkerFactory.obj
 0001:0000ffa0       ?root@?$QMapData@VQString@@PAVPropertyDelegate@U2@@@@QBEPAU?$QMapNode@VQString@@PAVPropertyDelegate@U2@@@@XZ 10010fa0 f i Metaphlan2WorkerFactory.obj
 0001:0000ffb0       ?tr@Metaphlan2WorkerFactory@LocalWorkflow@U2@@SA?AVQString@@PBD0H@Z 10010fb0 f i Metaphlan2WorkerFactory.obj
 0001:0000ffe0       ??C?$QScopedPointer@VQObjectData@@U?$QScopedPointerDeleter@VQObjectData@@@@@@QBEPAVQObjectData@@XZ 10010fe0 f i moc_Metaphlan2Prompter.obj
 0001:0000fff0       ?metaObject@Metaphlan2Prompter@LocalWorkflow@U2@@UBEPBUQMetaObject@@XZ 10010ff0 f   moc_Metaphlan2Prompter.obj
 0001:00010010       ?qt_metacall@Metaphlan2Prompter@LocalWorkflow@U2@@UAEHW4Call@QMetaObject@@HPAPAX@Z 10011010 f   moc_Metaphlan2Prompter.obj
 0001:00010020       ?qt_metacast@Metaphlan2Prompter@LocalWorkflow@U2@@UAEPAXPBD@Z 10011020 f   moc_Metaphlan2Prompter.obj
 0001:00010080       ?qt_static_metacall@Metaphlan2Prompter@LocalWorkflow@U2@@CAXPAVQObject@@W4Call@QMetaObject@@HPAPAX@Z 10011080 f   moc_Metaphlan2Prompter.obj
 0001:00010090       ?metaObject@Metaphlan2Support@U2@@UBEPBUQMetaObject@@XZ 10011090 f   moc_Metaphlan2Support.obj
 0001:000100b0       ?qt_metacall@Metaphlan2Support@U2@@UAEHW4Call@QMetaObject@@HPAPAX@Z 100110b0 f   moc_Metaphlan2Support.obj
 0001:000100c0       ?qt_metacast@Metaphlan2Support@U2@@UAEPAXPBD@Z 100110c0 f   moc_Metaphlan2Support.obj
 0001:00010120       ?qt_static_metacall@Metaphlan2Support@U2@@CAXPAVQObject@@W4Call@QMetaObject@@HPAPAX@Z 10011120 f   moc_Metaphlan2Support.obj
 0001:00010130       ?metaObject@MetaphlanSupportPlugin@U2@@UBEPBUQMetaObject@@XZ 10011130 f   moc_Metaphlan2SupportPlugin.obj
 0001:00010150       ?qt_metacall@MetaphlanSupportPlugin@U2@@UAEHW4Call@QMetaObject@@HPAPAX@Z 10011150 f   moc_Metaphlan2SupportPlugin.obj
 0001:00010160       ?qt_metacast@MetaphlanSupportPlugin@U2@@UAEPAXPBD@Z 10011160 f   moc_Metaphlan2SupportPlugin.obj
 0001:000101c0       ?qt_static_metacall@MetaphlanSupportPlugin@U2@@CAXPAVQObject@@W4Call@QMetaObject@@HPAPAX@Z 100111c0 f   moc_Metaphlan2SupportPlugin.obj
 0001:000101d0       ?metaObject@Metaphlan2ClassifyTask@U2@@UBEPBUQMetaObject@@XZ 100111d0 f   moc_Metaphlan2Task.obj
 0001:000101f0       ?qt_metacall@Metaphlan2ClassifyTask@U2@@UAEHW4Call@QMetaObject@@HPAPAX@Z 100111f0 f   moc_Metaphlan2Task.obj
 0001:00010200       ?qt_metacast@Metaphlan2ClassifyTask@U2@@UAEPAXPBD@Z 10011200 f   moc_Metaphlan2Task.obj
 0001:00010260       ?qt_static_metacall@Metaphlan2ClassifyTask@U2@@CAXPAVQObject@@W4Call@QMetaObject@@HPAPAX@Z 10011260 f   moc_Metaphlan2Task.obj
 0001:00010270       ??$acquireMemoryFence@H@?$QGenericAtomicOps@U?$QAtomicOpsBySize@$03@@@@SAXABH@Z 10011270 f i moc_Metaphlan2Worker.obj
 0001:00010280       ??$loadAcquire@H@?$QGenericAtomicOps@U?$QAtomicOpsBySize@$03@@@@SAHABH@Z 10011280 f i moc_Metaphlan2Worker.obj
 0001:00010290       ??$orderedMemoryFence@H@?$QGenericAtomicOps@U?$QAtomicOpsBySize@$03@@@@SAXABH@Z 10011290 f i moc_Metaphlan2Worker.obj
 0001:000102a0       ??$qMetaTypeId@PAVTask@U2@@@@YAHXZ 100112a0 f i moc_Metaphlan2Worker.obj
 0001:000102b0       ??$qRegisterMetaType@PAVTask@U2@@@@YAHXZ 100112b0 f i moc_Metaphlan2Worker.obj
 0001:000102c0       ??$qRegisterNormalizedMetaType@PAVTask@U2@@@@YAHABVQByteArray@@PAPAVTask@U2@@W4DefinedType@?$MetaTypeDefinedHelper@PAVTask@U2@@$00@QtPrivate@@@Z 100112c0 f i moc_Metaphlan2Worker.obj
 0001:00010320       ??$releaseMemoryFence@H@?$QGenericAtomicOps@U?$QAtomicOpsBySize@$03@@@@SAXABH@Z 10011320 f i moc_Metaphlan2Worker.obj
 0001:00010330       ??$storeRelease@HH@?$QGenericAtomicOps@U?$QAtomicOpsBySize@$03@@@@SAXAAHH@Z 10011330 f i moc_Metaphlan2Worker.obj
 0001:00010340       ??0?$QFlags@W4TypeFlag@QMetaType@@@@QAE@VQFlag@@@Z 10011340 f i moc_Metaphlan2Worker.obj
 0001:00010350       ??_5?$QFlags@W4TypeFlag@QMetaType@@@@QAEAAV0@W4TypeFlag@QMetaType@@@Z 10011350 f i moc_Metaphlan2Worker.obj
 0001:00010360       ?Construct@?$QMetaTypeFunctionHelper@PAVTask@U2@@$00@QtMetaTypePrivate@@SAPAXPAXPBX@Z 10011360 f i moc_Metaphlan2Worker.obj
 0001:00010390       ?Create@?$QMetaTypeFunctionHelper@PAVTask@U2@@$00@QtMetaTypePrivate@@SAPAXPBX@Z 10011390 f i moc_Metaphlan2Worker.obj
 0001:000103d0       ?Delete@?$QMetaTypeFunctionHelper@PAVTask@U2@@$00@QtMetaTypePrivate@@SAXPAX@Z 100113d0 f i moc_Metaphlan2Worker.obj
 0001:000103e0       ?Destruct@?$QMetaTypeFunctionHelper@PAVTask@U2@@$00@QtMetaTypePrivate@@SAXPAX@Z 100113e0 f i moc_Metaphlan2Worker.obj
 0001:000103f0       ?loadAcquire@?$QBasicAtomicInteger@H@@QBEHXZ 100113f0 f i moc_Metaphlan2Worker.obj
 0001:00010400       ?metaObject@Metaphlan2Worker@LocalWorkflow@U2@@UBEPBUQMetaObject@@XZ 10011400 f   moc_Metaphlan2Worker.obj
 0001:00010420       ?qt_metacall@Metaphlan2Worker@LocalWorkflow@U2@@UAEHW4Call@QMetaObject@@HPAPAX@Z 10011420 f   moc_Metaphlan2Worker.obj
 0001:00010480       ?qt_metacast@Metaphlan2Worker@LocalWorkflow@U2@@UAEPAXPBD@Z 10011480 f   moc_Metaphlan2Worker.obj
 0001:000104e0       ?qt_metatype_id@?$QMetaTypeId2@PAVTask@U2@@@@SAHXZ 100114e0 f i moc_Metaphlan2Worker.obj
 0001:000104f0       ?qt_metatype_id@?$QMetaTypeIdHelper@PAVTask@U2@@$00@QtPrivate@@SAHXZ 100114f0 f i moc_Metaphlan2Worker.obj
 0001:00010500       ?qt_metatype_id@?$QMetaTypeIdQObject@PAVTask@U2@@$00@@SAHXZ 10011500 f i moc_Metaphlan2Worker.obj
 0001:000105e0       ?qt_static_metacall@Metaphlan2Worker@LocalWorkflow@U2@@CAXPAVQObject@@W4Call@QMetaObject@@HPAPAX@Z 100115e0 f   moc_Metaphlan2Worker.obj
 0001:00010640       ?registerConverter@?$AssociativeContainerConverterHelper@PAVTask@U2@@$0A@@QtPrivate@@SA_NH@Z 10011640 f i moc_Metaphlan2Worker.obj
 0001:00010650       ?registerConverter@?$IsPair@PAVTask@U2@@@QtPrivate@@SA_NH@Z 10011650 f i moc_Metaphlan2Worker.obj
 0001:00010660       ?registerConverter@?$MetaTypeSmartPointerHelper@PAVTask@U2@@X@QtPrivate@@SA_NH@Z 10011660 f i moc_Metaphlan2Worker.obj
 0001:00010670       ?registerConverter@?$SequentialContainerConverterHelper@PAVTask@U2@@$0A@@QtPrivate@@SA_NH@Z 10011670 f i moc_Metaphlan2Worker.obj
 0001:00010680       ?storeRelease@?$QBasicAtomicInteger@H@@QAEXH@Z 10011680 f i moc_Metaphlan2Worker.obj
 0001:00010690       ?value@?$MetaObjectForType@PAVTask@U2@@$00@QtPrivate@@SAPBUQMetaObject@@XZ 10011690 f i moc_Metaphlan2Worker.obj
 0001:00010696       ?getBaseFileNameWithSuffixes@NgsReadsClassificationUtils@U2@@SA?AVQString@@ABV3@ABVQStringList@@0_N@Z 10011696 f   ngs_reads_classification:ngs_reads_classification.dll
 0001:0001069c       ??0DatabaseDelegate@LocalWorkflow@U2@@QAE@ABVQString@@0ABV?$QList@U?$QPair@VQString@@V1@@@@@0_N@Z 1001169c f   ngs_reads_classification:ngs_reads_classification.dll
 0001:000106a2       ??1DatabaseDelegate@LocalWorkflow@U2@@UAE@XZ 100116a2 f   ngs_reads_classification:ngs_reads_classification.dll
 0001:000106a8       ?update@DatabaseDelegate@LocalWorkflow@U2@@UAEXXZ 100116a8 f   ngs_reads_classification:ngs_reads_classification.dll
 0001:000106ae       ??0Logger@U2@@QAE@ABVQString@@@Z 100116ae f   U2Core:U2Core.dll
 0001:000106b4       ??1Logger@U2@@UAE@XZ       100116b4 f   U2Core:U2Core.dll
 0001:000106ba       ??0ExternalTool@U2@@QAE@VQString@@0@Z 100116ba f   U2Core:U2Core.dll
 0001:000106c0       ??1ExternalTool@U2@@UAE@XZ 100116c0 f   U2Core:U2Core.dll
 0001:000106c6       ?getAdditionalParameters@ExternalTool@U2@@UAEXABVQString@@@Z 100116c6 f   U2Core:U2Core.dll
 0001:000106cc       ?getAdditionalPaths@ExternalTool@U2@@UBE?AVQStringList@@XZ 100116cc f   U2Core:U2Core.dll
 0001:000106d2       ?getToolRunnerAdditionalOptions@ExternalTool@U2@@UAE?BVQStringList@@XZ 100116d2 f   U2Core:U2Core.dll
 0001:000106d8       ?getExternalToolRegistry@AppContext@U2@@SAPAVExternalToolRegistry@2@XZ 100116d8 f   U2Core:U2Core.dll
 0001:000106de       ?registerEntry@ExternalToolRegistry@U2@@QAE_NPAVExternalTool@2@@Z 100116de f   U2Core:U2Core.dll
 0001:000106e4       ?unregisterEntry@ExternalToolRegistry@U2@@QAEXABVQString@@@Z 100116e4 f   U2Core:U2Core.dll
 0001:000106ea       ??0Plugin@U2@@QAE@ABVQString@@0_NW4PluginState@1@@Z 100116ea f   U2Core:U2Core.dll
 0001:000106f0       ??1Plugin@U2@@UAE@XZ       100116f0 f   U2Core:U2Core.dll
 0001:000106f6       ??1GCounter@U2@@UAE@XZ     100116f6 f   U2Core:U2Core.dll
 0001:000106fc       ??0GReportableCounter@U2@@QAE@ABVQString@@0N@Z 100116fc f   U2Core:U2Core.dll
 0001:00010702       ??1SimpleEventCounter@U2@@UAE@XZ 10011702 f   U2Core:U2Core.dll
 0001:00010708       ??0GUrl@U2@@QAE@ABVQString@@@Z 10011708 f   U2Core:U2Core.dll
 0001:0001070e       ??1GUrl@U2@@QAE@XZ         1001170e f   U2Core:U2Core.dll
 0001:00010714       ?detectFormat@DocumentUtils@U2@@SA?AW4Detection@12@ABVGUrl@2@AAVQString@@@Z 10011714 f   U2Core:U2Core.dll
 0001:0001071a       ?addSubTask@Task@U2@@QAEXPAV12@@Z 1001171a f   U2Core:U2Core.dll
 0001:00010720       ?hasError@Task@U2@@QBE_NXZ 10011720 f   U2Core:U2Core.dll
 0001:00010726       ?setError@Task@U2@@QAEXABVQString@@@Z 10011726 f   U2Core:U2Core.dll
 0001:0001072c       ??0ExternalToolRunTask@U2@@QAE@ABVQString@@ABVQStringList@@PAVExternalToolLogParser@1@010_N@Z 1001172c f   U2Core:U2Core.dll
 0001:00010732       ??1ExternalToolRunTask@U2@@UAE@XZ 10011732 f   U2Core:U2Core.dll
 0001:00010738       ??0ExternalToolSupportTask@U2@@QAE@ABVQString@@V?$QFlags@W4TaskFlag@U2@@@@@Z 10011738 f   U2Core:U2Core.dll
 0001:0001073e       ??1ExternalToolSupportTask@U2@@UAE@XZ 1001173e f   U2Core:U2Core.dll
 0001:00010744       ??0ExternalToolLogParser@U2@@QAE@XZ 10011744 f   U2Core:U2Core.dll
 0001:0001074a       ??1ExternalToolLogParser@U2@@UAE@XZ 1001174a f   U2Core:U2Core.dll
 0001:00010750       ?cleanup@Task@U2@@UAEXXZ   10011750 f   U2Core:U2Core.dll
 0001:00010756       ?generateReport@Task@U2@@UBE?AVQString@@XZ 10011756 f   U2Core:U2Core.dll
 0001:0001075c       ?getNumParallelSubtasks@Task@U2@@UBEHXZ 1001175c f   U2Core:U2Core.dll
 0001:00010762       ?getParentTask@Task@U2@@UBEPAV12@XZ 10011762 f   U2Core:U2Core.dll
 0001:00010768       ?getProgress@ExternalToolLogParser@U2@@UAEHXZ 10011768 f   U2Core:U2Core.dll
 0001:0001076e       ?getSubtaskWithErrors@Task@U2@@UBEPAV12@XZ 1001176e f   U2Core:U2Core.dll
 0001:00010774       ?getTaskId@Task@U2@@UBE_JXZ 10011774 f   U2Core:U2Core.dll
 0001:0001077a       ?getTopLevelParentTask@Task@U2@@UAEPAV12@XZ 1001177a f   U2Core:U2Core.dll
 0001:00010780       ?getWarnings@Task@U2@@UBE?AVQStringList@@XZ 10011780 f   U2Core:U2Core.dll
 0001:00010786       ?hasSubtasksWithErrors@Task@U2@@UBE_NXZ 10011786 f   U2Core:U2Core.dll
 0001:0001078c       ?hasWarning@Task@U2@@UBE_NXZ 1001178c f   U2Core:U2Core.dll
 0001:00010792       ?isNotificationReport@Task@U2@@UBE_NXZ 10011792 f   U2Core:U2Core.dll
 0001:00010798       ?isReportingEnabled@Task@U2@@UBE_NXZ 10011798 f   U2Core:U2Core.dll
 0001:0001079e       ?isReportingSupported@Task@U2@@UBE_NXZ 1001179e f   U2Core:U2Core.dll
 0001:000107a4       ?isTopLevelTask@Task@U2@@UBE_NXZ 100117a4 f   U2Core:U2Core.dll
 0001:000107aa       ?metaObject@ExternalToolLogParser@U2@@UBEPBUQMetaObject@@XZ 100117aa f   U2Core:U2Core.dll
 0001:000107b0       ?metaObject@ExternalToolRunTask@U2@@UBEPBUQMetaObject@@XZ 100117b0 f   U2Core:U2Core.dll
 0001:000107b6       ?metaObject@Task@U2@@UBEPBUQMetaObject@@XZ 100117b6 f   U2Core:U2Core.dll
 0001:000107bc       ?onSubTaskFinished@Task@U2@@MAE?AV?$QList@PAVTask@U2@@@@PAV12@@Z 100117bc f   U2Core:U2Core.dll
 0001:000107c2       ?parseErrOutput@ExternalToolLogParser@U2@@UAEXABVQString@@@Z 100117c2 f   U2Core:U2Core.dll
 0001:000107c8       ?parseOutput@ExternalToolLogParser@U2@@UAEXABVQString@@@Z 100117c8 f   U2Core:U2Core.dll
 0001:000107ce       ?prepare@Task@U2@@UAEXXZ   100117ce f   U2Core:U2Core.dll
 0001:000107d4       ?processErrLine@ExternalToolLogParser@U2@@MAEXABVQString@@@Z 100117d4 f   U2Core:U2Core.dll
 0001:000107da       ?processLine@ExternalToolLogParser@U2@@MAEXABVQString@@@Z 100117da f   U2Core:U2Core.dll
 0001:000107e0       ?propagateSubtaskError@Task@U2@@UAE_NXZ 100117e0 f   U2Core:U2Core.dll
 0001:000107e6       ?qt_metacall@ExternalToolLogParser@U2@@UAEHW4Call@QMetaObject@@HPAPAX@Z 100117e6 f   U2Core:U2Core.dll
 0001:000107ec       ?qt_metacall@ExternalToolRunTask@U2@@UAEHW4Call@QMetaObject@@HPAPAX@Z 100117ec f   U2Core:U2Core.dll
 0001:000107f2       ?qt_metacall@Task@U2@@UAEHW4Call@QMetaObject@@HPAPAX@Z 100117f2 f   U2Core:U2Core.dll
 0001:000107f8       ?qt_metacast@ExternalToolLogParser@U2@@UAEPAXPBD@Z 100117f8 f   U2Core:U2Core.dll
 0001:000107fe       ?qt_metacast@ExternalToolRunTask@U2@@UAEPAXPBD@Z 100117fe f   U2Core:U2Core.dll
 0001:00010804       ?qt_metacast@Task@U2@@UAEPAXPBD@Z 10011804 f   U2Core:U2Core.dll
 0001:0001080a       ?report@Task@U2@@UAE?AW4ReportResult@12@XZ 1001180a f   U2Core:U2Core.dll
 0001:00010810       ?run@ExternalToolRunTask@U2@@UAEXXZ 10011810 f   U2Core:U2Core.dll
 0001:00010816       ?run@Task@U2@@UAEXXZ       10011816 f   U2Core:U2Core.dll
 0001:0001081c       ?setCollectChildrensWarningsFlag@Task@U2@@UAEX_N@Z 1001181c f   U2Core:U2Core.dll
 0001:00010822       ?setLastError@ExternalToolLogParser@U2@@MAEXABVQString@@@Z 10011822 f   U2Core:U2Core.dll
 0001:00010828       ?setListenerForHelper@ExternalToolSupportTask@U2@@MAEXPAVExternalToolRunTaskHelper@2@H@Z 10011828 f   U2Core:U2Core.dll
 0001:0001082e       ?setListenerForTask@ExternalToolSupportTask@U2@@MAEXPAVExternalToolRunTask@2@H@Z 1001182e f   U2Core:U2Core.dll
 0001:00010834       ?setNoAutoDelete@Task@U2@@UAEX_N@Z 10011834 f   U2Core:U2Core.dll
 0001:0001083a       ?setNotificationReport@Task@U2@@UAEX_N@Z 1001183a f   U2Core:U2Core.dll
 0001:00010840       ?setReportingEnabled@Task@U2@@UAEX_N@Z 10011840 f   U2Core:U2Core.dll
 0001:00010846       ?setReportingSupported@Task@U2@@UAEX_N@Z 10011846 f   U2Core:U2Core.dll
 0001:0001084c       ?getAppSettings@AppContext@U2@@SAPAVAppSettings@2@XZ 1001184c f   U2Core:U2Core.dll
 0001:00010852       ?error@Logger@U2@@QAEXABVQString@@@Z 10011852 f   U2Core:U2Core.dll
 0001:00010858       ??0TaskStateInfo@U2@@QAE@XZ 10011858 f   U2Core:U2Core.dll
 0001:0001085e       ?getError@TaskStateInfo@U2@@UBE?AVQString@@XZ 1001185e f   U2Core:U2Core.dll
 0001:00010864       ?setError@TaskStateInfo@U2@@UAEXABVQString@@@Z 10011864 f   U2Core:U2Core.dll
 0001:0001086a       ??1TaskStateInfo@U2@@UAE@XZ 1001186a f   U2Core:U2Core.dll
 0001:00010870       ??0FailTask@U2@@QAE@ABVQString@@@Z 10011870 f   U2Core:U2Core.dll
 0001:00010876       ??1FailTask@U2@@UAE@XZ     10011876 f   U2Core:U2Core.dll
 0001:0001087c       ?getWorkingDir@FileAndDirectoryUtils@U2@@SA?AVQString@@ABV3@H00@Z 1001187c f   U2Core:U2Core.dll
 0001:00010882       ?rollFileName@GUrlUtils@U2@@SA?AVQString@@ABV3@0ABV?$QSet@VQString@@@@@Z 10011882 f   U2Core:U2Core.dll
 0001:00010888       ??0TaskSignalMapper@U2@@QAE@PAVTask@1@@Z 10011888 f   U2Core:U2Core.dll
 0001:0001088e       ?getError@U2OpStatusImpl@U2@@UBE?AVQString@@XZ 1001188e f   U2Core:U2Core.dll
 0001:00010894       ??0U2OpStatus2Log@U2@@QAE@W4LogLevel@1@@Z 10011894 f   U2Core:U2Core.dll
 0001:0001089a       ??1U2OpStatus2Log@U2@@UAE@XZ 1001189a f   U2Core:U2Core.dll
 0001:000108a0       ?createCurrentProcessTemporarySubDir@UserAppsSettings@U2@@QBE?AVQString@@AAVU2OpStatus@2@ABV3@@Z 100118a0 f   U2Core:U2Core.dll
 0001:000108a6       ?addListeners@ExternalToolSupportTask@U2@@QAEXABV?$QList@PAVExternalToolListener@U2@@@@@Z 100118a6 f   U2Core:U2Core.dll
 0001:000108ac       ?runScript@ScriptTask@U2@@SA?AVQScriptValue@@PAVQScriptEngine@@ABV?$QMap@VQString@@VQScriptValue@@@@ABVQString@@AAVTaskStateInfo@2@@Z 100118ac f   U2Core:U2Core.dll
 0001:000108b2       ?metaObject@FailTask@U2@@UBEPBUQMetaObject@@XZ 100118b2 f   U2Core:U2Core.dll
 0001:000108b8       ?metaObject@TaskSignalMapper@U2@@UBEPBUQMetaObject@@XZ 100118b8 f   U2Core:U2Core.dll
 0001:000108be       ?qt_metacall@FailTask@U2@@UAEHW4Call@QMetaObject@@HPAPAX@Z 100118be f   U2Core:U2Core.dll
 0001:000108c4       ?qt_metacall@TaskSignalMapper@U2@@UAEHW4Call@QMetaObject@@HPAPAX@Z 100118c4 f   U2Core:U2Core.dll
 0001:000108ca       ?qt_metacast@FailTask@U2@@UAEPAXPBD@Z 100118ca f   U2Core:U2Core.dll
 0001:000108d0       ?qt_metacast@TaskSignalMapper@U2@@UAEPAXPBD@Z 100118d0 f   U2Core:U2Core.dll
 0001:000108d6       ?getDataPathRegistry@AppContext@U2@@SAPAVU2DataPathRegistry@2@XZ 100118d6 f   U2Core:U2Core.dll
 0001:000108dc       ?isValid@U2DataPath@U2@@QBE_NXZ 100118dc f   U2Core:U2Core.dll
 0001:000108e2       ?getPathByName@U2DataPath@U2@@QBE?AVQString@@ABV3@@Z 100118e2 f   U2Core:U2Core.dll
 0001:000108e8       ?getDataPathByName@U2DataPathRegistry@U2@@QAEPAVU2DataPath@2@ABVQString@@@Z 100118e8 f   U2Core:U2Core.dll
 0001:000108ee       ?qt_metacast@ExternalTool@U2@@UAEPAXPBD@Z 100118ee f   U2Core:U2Core.dll
 0001:000108f4       ?qt_metacall@ExternalTool@U2@@UAEHW4Call@QMetaObject@@HPAPAX@Z 100118f4 f   U2Core:U2Core.dll
 0001:000108fa       ?qt_metacast@Plugin@U2@@UAEPAXPBD@Z 100118fa f   U2Core:U2Core.dll
 0001:00010900       ?qt_metacall@Plugin@U2@@UAEHW4Call@QMetaObject@@HPAPAX@Z 10011900 f   U2Core:U2Core.dll
 0001:00010906       ??0CalculateSequencesNumberTask@U2@@QAE@ABVQString@@@Z 10011906 f   U2Formats:U2Formats.dll
 0001:0001090c       ?getSequencesNumber@CalculateSequencesNumberTask@U2@@QBEHXZ 1001190c f   U2Formats:U2Formats.dll
 0001:00010912       ??1CalculateSequencesNumberTask@U2@@UAE@XZ 10011912 f   U2Formats:U2Formats.dll
 0001:00010918       ?run@CalculateSequencesNumberTask@U2@@EAEXXZ 10011918 f   U2Formats:U2Formats.dll
 0001:0001091e       ?prepareDocumentsFileFilter@DialogUtils@U2@@SA?AVQString@@ABV3@_NABVQStringList@@@Z 1001191e f   U2Gui:U2Gui.dll
 0001:00010924       ?getInputPorts@Actor@Workflow@U2@@QBE?AV?$QList@PAVPort@Workflow@U2@@@@XZ 10011924 f   U2Lang:U2Lang.dll
 0001:0001092a       ?getOutputPorts@Actor@Workflow@U2@@QBE?AV?$QList@PAVPort@Workflow@U2@@@@XZ 1001192a f   U2Lang:U2Lang.dll
 0001:00010930       ??0PrompterBaseImpl@U2@@QAE@PAVActor@Workflow@1@@Z 10011930 f   U2Lang:U2Lang.dll
 0001:00010936       ?getURL@PrompterBaseImpl@U2@@QAE?AVQString@@ABV3@PA_N00@Z 10011936 f   U2Lang:U2Lang.dll
 0001:0001093c       ?getProducersOrUnset@PrompterBaseImpl@U2@@QAE?AVQString@@ABV3@0@Z 1001193c f   U2Lang:U2Lang.dll
 0001:00010942       ?getHyperlink@PrompterBaseImpl@U2@@SA?AVQString@@ABV3@0@Z 10011942 f   U2Lang:U2Lang.dll
 0001:00010948       ??1PrompterBaseImpl@U2@@UAE@XZ 10011948 f   U2Lang:U2Lang.dll
 0001:0001094e       ?metaObject@PrompterBaseImpl@U2@@UBEPBUQMetaObject@@XZ 1001194e f   U2Lang:U2Lang.dll
 0001:00010954       ?qt_metacall@PrompterBaseImpl@U2@@UAEHW4Call@QMetaObject@@HPAPAX@Z 10011954 f   U2Lang:U2Lang.dll
 0001:0001095a       ?qt_metacast@PrompterBaseImpl@U2@@UAEPAXPBD@Z 1001195a f   U2Lang:U2Lang.dll
 0001:00010960       ?sl_actorModified@PrompterBaseImpl@U2@@MAEXXZ 10011960 f   U2Lang:U2Lang.dll
 0001:00010966       ?update@PrompterBaseImpl@U2@@UAEXABV?$QMap@VQString@@VQVariant@@@@@Z 10011966 f   U2Lang:U2Lang.dll
 0001:0001096c       ??0WorkflowNotification@U2@@QAE@ABVQString@@00@Z 1001196c f   U2Lang:U2Lang.dll
 0001:00010972       ??1WorkflowNotification@U2@@QAE@XZ 10011972 f   U2Lang:U2Lang.dll
 0001:00010978       ??0WorkflowNotification@U2@@QAE@ABV01@@Z 10011978 f   U2Lang:U2Lang.dll
 0001:0001097e       ?getId@Actor@Workflow@U2@@QBE?AVQString@@XZ 1001197e f   U2Lang:U2Lang.dll
 0001:00010984       ??1Descriptor@U2@@UAE@XZ   10011984 f   U2Lang:U2Lang.dll
 0001:0001098a       ?getId@Descriptor@U2@@QBE?AVQString@@XZ 1001198a f   U2Lang:U2Lang.dll
 0001:00010990       ??0Descriptor@U2@@QAE@ABV01@@Z 10011990 f   U2Lang:U2Lang.dll
 0001:00010996       ?getFileUrl@MessageMetadata@U2@@QBEABVQString@@XZ 10011996 f   U2Lang:U2Lang.dll
 0001:0001099c       ??1MessageMetadata@U2@@QAE@XZ 1001199c f   U2Lang:U2Lang.dll
 0001:000109a2       ?get@MessageMetadataStorage@U2@@QBE?AVMessageMetadata@2@H@Z 100119a2 f   U2Lang:U2Lang.dll
 0001:000109a8       ?getMonitor@WorkflowContext@Workflow@U2@@QAEPAVWorkflowMonitor@23@XZ 100119a8 f   U2Lang:U2Lang.dll
 0001:000109ae       ?workingDir@WorkflowContext@Workflow@U2@@QBE?AVQString@@XZ 100119ae f   U2Lang:U2Lang.dll
 0001:000109b4       ?absolutePath@WorkflowContext@Workflow@U2@@QBE?AVQString@@ABV4@@Z 100119b4 f   U2Lang:U2Lang.dll
 0001:000109ba       ?getMetadataStorage@WorkflowContext@Workflow@U2@@QAEAAVMessageMetadataStorage@3@XZ 100119ba f   U2Lang:U2Lang.dll
 0001:000109c0       ?initEngine@WorkflowScriptLibrary@U2@@SAXPAVWorkflowScriptEngine@2@@Z 100119c0 f   U2Lang:U2Lang.dll
 0001:000109c6       ??0WorkflowScriptEngine@U2@@QAE@PAVWorkflowContext@Workflow@1@@Z 100119c6 f   U2Lang:U2Lang.dll
 0001:000109cc       ??1WorkflowScriptEngine@U2@@UAE@XZ 100119cc f   U2Lang:U2Lang.dll
 0001:000109d2       ?isEmpty@AttributeScript@U2@@QBE_NXZ 100119d2 f   U2Lang:U2Lang.dll
 0001:000109d8       ?getScriptText@AttributeScript@U2@@QBEABVQString@@XZ 100119d8 f   U2Lang:U2Lang.dll
 0001:000109de       ?getScriptVars@AttributeScript@U2@@QBEABV?$QMap@VDescriptor@U2@@VQVariant@@@@XZ 100119de f   U2Lang:U2Lang.dll
 0001:000109e4       ?getData@Message@Workflow@U2@@QBE?AVQVariant@@XZ 100119e4 f   U2Lang:U2Lang.dll
 0001:000109ea       ?getMetadataId@Message@Workflow@U2@@QBEHXZ 100119ea f   U2Lang:U2Lang.dll
 0001:000109f0       ??1Message@Workflow@U2@@QAE@XZ 100119f0 f   U2Lang:U2Lang.dll
 0001:000109f6       ?addOutputFile@WorkflowMonitor@Workflow@U2@@QAEXABVQString@@0_N@Z 100119f6 f   U2Lang:U2Lang.dll
 0001:000109fc       ?isOutUrlAttribute@RFSUtils@U2@@SA_NPAVAttribute@2@PAVActor@Workflow@2@AA_N@Z 100119fc f   U2Lang:U2Lang.dll
 0001:00010a02       ?getExternalToolPath@WorkflowUtils@U2@@SA?AVQString@@ABV3@@Z 10011a02 f   U2Lang:U2Lang.dll
 0001:00010a08       ??0BaseWorker@LocalWorkflow@U2@@QAE@PAVActor@Workflow@2@_N@Z 10011a08 f   U2Lang:U2Lang.dll
 0001:00010a0e       ??1BaseWorker@LocalWorkflow@U2@@UAE@XZ 10011a0e f   U2Lang:U2Lang.dll
 0001:00010a14       ?createLogListeners@BaseWorker@LocalWorkflow@U2@@QAE?AV?$QList@PAVExternalToolListener@U2@@@@H@Z 10011a14 f   U2Lang:U2Lang.dll
 0001:00010a1a       ?addCommunication@BaseWorker@LocalWorkflow@U2@@UAE_NABVQString@@PAVCommunicationChannel@Workflow@3@@Z 10011a1a f   U2Lang:U2Lang.dll
 0001:00010a20       ?canTaskBeCanceled@BaseWorker@LocalWorkflow@U2@@MBE_NPAVTask@3@@Z 10011a20 f   U2Lang:U2Lang.dll
 0001:00010a26       ?getActorId@BaseWorker@LocalWorkflow@U2@@UBE?AVQString@@XZ 10011a26 f   U2Lang:U2Lang.dll
 0001:00010a2c       ?getCommunication@BaseWorker@LocalWorkflow@U2@@UAEPAVCommunicationChannel@Workflow@3@ABVQString@@@Z 10011a2c f   U2Lang:U2Lang.dll
 0001:00010a32       ?getMessageAndSetupScriptValues@BaseWorker@LocalWorkflow@U2@@UAE?AVMessage@Workflow@3@PAVCommunicationChannel@53@@Z 10011a32 f   U2Lang:U2Lang.dll
 0001:00010a38       ?getOutputFiles@BaseWorker@LocalWorkflow@U2@@UAE?AVQStringList@@XZ 10011a38 f   U2Lang:U2Lang.dll
 0001:00010a3e       ?isDone@BaseWorker@LocalWorkflow@U2@@UBE_NXZ 10011a3e f   U2Lang:U2Lang.dll
 0001:00010a44       ?isReady@BaseWorker@LocalWorkflow@U2@@UBE_NXZ 10011a44 f   U2Lang:U2Lang.dll
 0001:00010a4a       ?setDone@BaseWorker@LocalWorkflow@U2@@UAEXXZ 10011a4a f   U2Lang:U2Lang.dll
 0001:00010a50       ??0Descriptor@U2@@QAE@ABVQString@@00@Z 10011a50 f   U2Lang:U2Lang.dll
 0001:00010a56       ??0Descriptor@U2@@QAE@ABVQString@@@Z 10011a56 f   U2Lang:U2Lang.dll
 0001:00010a5c       ??0VisibilityRelation@U2@@QAE@ABVQString@@ABV?$QList@VQVariant@@@@_N@Z 10011a5c f   U2Lang:U2Lang.dll
 0001:00010a62       ??1VisibilityRelation@U2@@UAE@XZ 10011a62 f   U2Lang:U2Lang.dll
 0001:00010a68       ??0MapDataType@U2@@QAE@ABVDescriptor@1@ABV?$QMap@VDescriptor@U2@@V?$QExplicitlySharedDataPointer@VDataType@U2@@@@@@@Z 10011a68 f   U2Lang:U2Lang.dll
 0001:00010a6e       ??1MapDataType@U2@@UAE@XZ  10011a6e f   U2Lang:U2Lang.dll
 0001:00010a74       ??0SlotRelationDescriptor@U2@@QAE@ABVQString@@0ABV?$QList@VQVariant@@@@@Z 10011a74 f   U2Lang:U2Lang.dll
 0001:00010a7a       ??1SlotRelationDescriptor@U2@@UAE@XZ 10011a7a f   U2Lang:U2Lang.dll
 0001:00010a80       ??0Attribute@U2@@QAE@ABVDescriptor@1@V?$QExplicitlySharedDataPointer@VDataType@U2@@@@V?$QFlags@W4Flag@Attribute@U2@@@@ABVQVariant@@@Z 10011a80 f   U2Lang:U2Lang.dll
 0001:00010a86       ??0Attribute@U2@@QAE@ABVDescriptor@1@V?$QExplicitlySharedDataPointer@VDataType@U2@@@@_NABVQVariant@@@Z 10011a86 f   U2Lang:U2Lang.dll
 0001:00010a8c       ??1Attribute@U2@@UAE@XZ    10011a8c f   U2Lang:U2Lang.dll
 0001:00010a92       ?addRelation@Attribute@U2@@QAEXPBVAttributeRelation@2@@Z 10011a92 f   U2Lang:U2Lang.dll
 0001:00010a98       ?addSlotRelation@Attribute@U2@@QAEXPAVSlotRelationDescriptor@2@@Z 10011a98 f   U2Lang:U2Lang.dll
 0001:00010a9e       ??0DelegateTags@U2@@QAE@PAVQObject@@@Z 10011a9e f   U2Lang:U2Lang.dll
 0001:00010aa4       ?set@DelegateTags@U2@@QAEXABVQString@@ABVQVariant@@@Z 10011aa4 f   U2Lang:U2Lang.dll
 0001:00010aaa       ??1DelegateTags@U2@@UAE@XZ 10011aaa f   U2Lang:U2Lang.dll
 0001:00010ab0       ??0PortDescriptor@Workflow@U2@@QAE@ABVDescriptor@2@V?$QExplicitlySharedDataPointer@VDataType@U2@@@@_N2I@Z 10011ab0 f   U2Lang:U2Lang.dll
 0001:00010ab6       ??1PortDescriptor@Workflow@U2@@UAE@XZ 10011ab6 f   U2Lang:U2Lang.dll
 0001:00010abc       ??0ActorPrototype@Workflow@U2@@QAE@ABVDescriptor@2@ABV?$QList@PAVPortDescriptor@Workflow@U2@@@@ABV?$QList@PAVAttribute@U2@@@@@Z 10011abc f   U2Lang:U2Lang.dll
 0001:00010ac2       ??1ActorPrototype@Workflow@U2@@UAE@XZ 10011ac2 f   U2Lang:U2Lang.dll
 0001:00010ac8       ?setEditor@ActorPrototype@Workflow@U2@@QAEXPAVConfigurationEditor@3@@Z 10011ac8 f   U2Lang:U2Lang.dll
 0001:00010ace       ?setValidator@ActorPrototype@Workflow@U2@@QAEXPAVConfigurationValidator@3@@Z 10011ace f   U2Lang:U2Lang.dll
 0001:00010ad4       ?setPrompter@ActorPrototype@Workflow@U2@@QAEXPAVPrompter@23@@Z 10011ad4 f   U2Lang:U2Lang.dll
 0001:00010ada       ?setPortValidator@ActorPrototype@Workflow@U2@@QAEXABVQString@@PAVConfigurationValidator@3@@Z 10011ada f   U2Lang:U2Lang.dll
 0001:00010ae0       ?addExternalTool@ActorPrototype@Workflow@U2@@QAEXABVQString@@0@Z 10011ae0 f   U2Lang:U2Lang.dll
 0001:00010ae6       ??0DomainFactory@Workflow@U2@@QAE@ABVQString@@@Z 10011ae6 f   U2Lang:U2Lang.dll
 0001:00010aec       ??1DomainFactory@Workflow@U2@@UAE@XZ 10011aec f   U2Lang:U2Lang.dll
 0001:00010af2       ?registerProto@ActorPrototypeRegistry@Workflow@U2@@QAEXABVDescriptor@3@PAVActorPrototype@23@@Z 10011af2 f   U2Lang:U2Lang.dll
 0001:00010af8       ?unregisterProto@ActorPrototypeRegistry@Workflow@U2@@QAEPAVActorPrototype@23@ABVQString@@@Z 10011af8 f   U2Lang:U2Lang.dll
 0001:00010afe       ?STRING_TYPE@BaseTypes@U2@@SA?AV?$QExplicitlySharedDataPointer@VDataType@U2@@@@XZ 10011afe f   U2Lang:U2Lang.dll
 0001:00010b04       ?NUM_TYPE@BaseTypes@U2@@SA?AV?$QExplicitlySharedDataPointer@VDataType@U2@@@@XZ 10011b04 f   U2Lang:U2Lang.dll
 0001:00010b0a       ??0PairedReadsPortValidator@Workflow@U2@@QAE@ABVQString@@0@Z 10011b0a f   U2Lang:U2Lang.dll
 0001:00010b10       ??1PairedReadsPortValidator@Workflow@U2@@UAE@XZ 10011b10 f   U2Lang:U2Lang.dll
 0001:00010b16       ?getInstance@WorkflowEnv@Workflow@U2@@KAPAV123@XZ 10011b16 f   U2Lang:U2Lang.dll
 0001:00010b1c       ?clone@Attribute@U2@@UAEPAV12@XZ 10011b1c f   U2Lang:U2Lang.dll
 0001:00010b22       ?clone@SlotRelationDescriptor@U2@@UBEPAV12@XZ 10011b22 f   U2Lang:U2Lang.dll
 0001:00010b28       ?clone@VisibilityRelation@U2@@UBEPAV12@XZ 10011b28 f   U2Lang:U2Lang.dll
 0001:00010b2e       ?createConnection@DomainFactory@Workflow@U2@@UAEPAVCommunicationChannel@23@PAVLink@23@@Z 10011b2e f   U2Lang:U2Lang.dll
 0001:00010b34       ?createInstance@ActorPrototype@Workflow@U2@@UAEPAVActor@23@ABVQString@@PAVAttributeScript@3@ABV?$QMap@VQString@@VQVariant@@@@@Z 10011b34 f   U2Lang:U2Lang.dll
 0001:00010b3a       ?createPort@IntegralBusActorPrototype@Workflow@U2@@UAEPAVPort@23@ABVPortDescriptor@23@PAVActor@23@@Z 10011b3a f   U2Lang:U2Lang.dll
 0001:00010b40       ?createScheduler@DomainFactory@Workflow@U2@@UAEPAVScheduler@23@PAVSchema@23@@Z 10011b40 f   U2Lang:U2Lang.dll
 0001:00010b46       ?destroy@DomainFactory@Workflow@U2@@UAEXPAVScheduler@23@PAVSchema@23@@Z 10011b46 f   U2Lang:U2Lang.dll
 0001:00010b4c       ?getAffectResult@VisibilityRelation@U2@@UBE?AVQVariant@@ABV3@0PAVDelegateTags@2@1@Z 10011b4c f   U2Lang:U2Lang.dll
 0001:00010b52       ?getAllDescriptors@MapDataType@U2@@UBE?AV?$QList@VDescriptor@U2@@@@XZ 10011b52 f   U2Lang:U2Lang.dll
 0001:00010b58       ?getAllEntries@?$IdRegistry@VDomainFactory@Workflow@U2@@@U2@@UBE?AV?$QList@PAVDomainFactory@Workflow@U2@@@@XZ 10011b58 f   U2Lang:U2Lang.dll
 0001:00010b5e       ?getAllIds@?$IdRegistry@VDomainFactory@Workflow@U2@@@U2@@UBE?AV?$QList@VQString@@@@XZ 10011b5e f   U2Lang:U2Lang.dll
 0001:00010b64       ?getAttributePureValue@Attribute@U2@@UBEABVQVariant@@XZ 10011b64 f   U2Lang:U2Lang.dll
 0001:00010b6a       ?getById@?$IdRegistry@VDomainFactory@Workflow@U2@@@U2@@UAEPAVDomainFactory@Workflow@2@ABVQString@@@Z 10011b6a f   U2Lang:U2Lang.dll
 0001:00010b70       ?getDatatypeByDescriptor@MapDataType@U2@@UBE?AV?$QExplicitlySharedDataPointer@VDataType@U2@@@@ABVDescriptor@2@@Z 10011b70 f   U2Lang:U2Lang.dll
 0001:00010b76       ?getDatatypesMap@MapDataType@U2@@UBE?AV?$QMap@VDescriptor@U2@@V?$QExplicitlySharedDataPointer@VDataType@U2@@@@@@XZ 10011b76 f   U2Lang:U2Lang.dll
 0001:00010b7c       ?getDefaultPureValue@Attribute@U2@@UBEABVQVariant@@XZ 10011b7c f   U2Lang:U2Lang.dll
 0001:00010b82       ?getGroup@Attribute@U2@@UAE?AW4AttributeGroup@2@XZ 10011b82 f   U2Lang:U2Lang.dll
 0001:00010b88       ?getItems@PropertyDelegate@U2@@UBEXAAV?$QMap@VQString@@VQVariant@@@@@Z 10011b88 f   U2Lang:U2Lang.dll
 0001:00010b8e       ?getType@PortDescriptor@Workflow@U2@@UBE?AV?$QExplicitlySharedDataPointer@VDataType@U2@@@@XZ 10011b8e f   U2Lang:U2Lang.dll
 0001:00010b94       ?getType@VisibilityRelation@U2@@UBE?AW4RelationType@2@XZ 10011b94 f   U2Lang:U2Lang.dll
 0001:00010b9a       ?getWidget@ConfigurationEditor@U2@@UAEPAVQWidget@@XZ 10011b9a f   U2Lang:U2Lang.dll
 0001:00010ba0       ?isAcceptableDrop@ActorPrototype@Workflow@U2@@UBE_NPBVQMimeData@@PAV?$QMap@VQString@@VQVariant@@@@@Z 10011ba0 f   U2Lang:U2Lang.dll
 0001:00010ba6       ?isDefaultValue@Attribute@U2@@UBE_NXZ 10011ba6 f   U2Lang:U2Lang.dll
 0001:00010bac       ?isEmpty@Attribute@U2@@UBE_NXZ 10011bac f   U2Lang:U2Lang.dll
 0001:00010bb2       ?isEmpty@ConfigurationEditor@U2@@UBE_NXZ 10011bb2 f   U2Lang:U2Lang.dll
 0001:00010bb8       ?isSlotEnabled@SlotRelationDescriptor@U2@@UBE_NABVQVariant@@@Z 10011bb8 f   U2Lang:U2Lang.dll
 0001:00010bbe       ?kind@MapDataType@U2@@UBE?AW4Kind@DataType@2@XZ 10011bbe f   U2Lang:U2Lang.dll
 0001:00010bc4       ?registerEntry@?$IdRegistry@VDomainFactory@Workflow@U2@@@U2@@UAE_NPAVDomainFactory@Workflow@2@@Z 10011bc4 f   U2Lang:U2Lang.dll
 0001:00010bca       ?setAttributeValue@Attribute@U2@@UAEXABVQVariant@@@Z 10011bca f   U2Lang:U2Lang.dll
 0001:00010bd0       ?setVisibleSlot@PortDescriptor@Workflow@U2@@UAEXABVQString@@_N@Z 10011bd0 f   U2Lang:U2Lang.dll
 0001:00010bd6       ?type@PropertyDelegate@U2@@UBE?AW4Type@12@XZ 10011bd6 f   U2Lang:U2Lang.dll
 0001:00010bdc       ?unregisterEntry@?$IdRegistry@VDomainFactory@Workflow@U2@@@U2@@UAEPAVDomainFactory@Workflow@2@ABVQString@@@Z 10011bdc f   U2Lang:U2Lang.dll
 0001:00010be2       ?update@PropertyDelegate@U2@@UAEXXZ 10011be2 f   U2Lang:U2Lang.dll
 0001:00010be8       ?updateActorIds@Attribute@U2@@UAEXABV?$QMap@VQString@@V1@@@@Z 10011be8 f   U2Lang:U2Lang.dll
 0001:00010bee       ?updateDelegateTags@AttributeRelation@U2@@UBEXABVQVariant@@PAVDelegateTags@2@@Z 10011bee f   U2Lang:U2Lang.dll
 0001:00010bf4       ?validate@ActorValidator@Workflow@U2@@UBE_NPBVConfiguration@3@AAV?$QList@VWorkflowNotification@U2@@@@@Z 10011bf4 f   U2Lang:U2Lang.dll
 0001:00010bfa       ?validate@Attribute@U2@@UAE_NAAV?$QList@VWorkflowNotification@U2@@@@@Z 10011bfa f   U2Lang:U2Lang.dll
 0001:00010c00       ?validate@PairedReadsPortValidator@Workflow@U2@@UBE_NPBVIntegralBusPort@23@AAV?$QList@VWorkflowNotification@U2@@@@@Z 10011c00 f   U2Lang:U2Lang.dll
 0001:00010c06       ?validate@PortValidator@Workflow@U2@@UBE_NPBVConfiguration@3@AAV?$QList@VWorkflowNotification@U2@@@@@Z 10011c06 f   U2Lang:U2Lang.dll
 0001:00010c0c       ?valueChangingRelation@VisibilityRelation@U2@@UBE_NXZ 10011c0c f   U2Lang:U2Lang.dll
 0001:00010c12       ?qt_metacast@BaseWorker@LocalWorkflow@U2@@UAEPAXPBD@Z 10011c12 f   U2Lang:U2Lang.dll
 0001:00010c18       ?qt_metacall@BaseWorker@LocalWorkflow@U2@@UAEHW4Call@QMetaObject@@HPAPAX@Z 10011c18 f   U2Lang:U2Lang.dll
 0001:00010c1e       ??0DelegateEditor@U2@@QAE@ABV?$QMap@VQString@@PAVPropertyDelegate@U2@@@@@Z 10011c1e f   U2Designer:U2Designer.dll
 0001:00010c24       ??1DelegateEditor@U2@@UAE@XZ 10011c24 f   U2Designer:U2Designer.dll
 0001:00010c2a       ??0URLDelegate@U2@@QAE@ABVDelegateTags@1@ABVQString@@_N22PAVQObject@@2@Z 10011c2a f   U2Designer:U2Designer.dll
 0001:00010c30       ??1URLDelegate@U2@@UAE@XZ  10011c30 f   U2Designer:U2Designer.dll
 0001:00010c36       ??0SpinBoxDelegate@U2@@QAE@ABV?$QMap@VQString@@VQVariant@@@@PAVQObject@@@Z 10011c36 f   U2Designer:U2Designer.dll
 0001:00010c3c       ??1SpinBoxDelegate@U2@@UAE@XZ 10011c3c f   U2Designer:U2Designer.dll
 0001:00010c42       ??0ComboBoxDelegate@U2@@QAE@ABV?$QMap@VQString@@VQVariant@@@@PAVQObject@@@Z 10011c42 f   U2Designer:U2Designer.dll
 0001:00010c48       ??1ComboBoxDelegate@U2@@UAE@XZ 10011c48 f   U2Designer:U2Designer.dll
 0001:00010c4e       ?addDelegate@DelegateEditor@U2@@UAEXPAVPropertyDelegate@2@ABVQString@@@Z 10011c4e f   U2Designer:U2Designer.dll
 0001:00010c54       ?clone@ComboBoxDelegate@U2@@UAEPAVPropertyDelegate@2@XZ 10011c54 f   U2Designer:U2Designer.dll
 0001:00010c5a       ?clone@DelegateEditor@U2@@UAEPAVConfigurationEditor@2@XZ 10011c5a f   U2Designer:U2Designer.dll
 0001:00010c60       ?clone@SpinBoxDelegate@U2@@UAEPAVPropertyDelegate@2@XZ 10011c60 f   U2Designer:U2Designer.dll
 0001:00010c66       ?clone@URLDelegate@U2@@UAEPAVPropertyDelegate@2@XZ 10011c66 f   U2Designer:U2Designer.dll
 0001:00010c6c       ?commit@DelegateEditor@U2@@UAEXXZ 10011c6c f   U2Designer:U2Designer.dll
 0001:00010c72       ?createEditor@ComboBoxDelegate@U2@@UBEPAVQWidget@@PAV3@ABVQStyleOptionViewItem@@ABVQModelIndex@@@Z 10011c72 f   U2Designer:U2Designer.dll
 0001:00010c78       ?createEditor@SpinBoxDelegate@U2@@UBEPAVQWidget@@PAV3@ABVQStyleOptionViewItem@@ABVQModelIndex@@@Z 10011c78 f   U2Designer:U2Designer.dll
 0001:00010c7e       ?createEditor@URLDelegate@U2@@UBEPAVQWidget@@PAV3@ABVQStyleOptionViewItem@@ABVQModelIndex@@@Z 10011c7e f   U2Designer:U2Designer.dll
 0001:00010c84       ?createWizardWidget@ComboBoxDelegate@U2@@UBEPAVPropertyWidget@2@AAVU2OpStatus@2@PAVQWidget@@@Z 10011c84 f   U2Designer:U2Designer.dll
 0001:00010c8a       ?createWizardWidget@SpinBoxDelegate@U2@@UBEPAVPropertyWidget@2@AAVU2OpStatus@2@PAVQWidget@@@Z 10011c8a f   U2Designer:U2Designer.dll
 0001:00010c90       ?createWizardWidget@URLDelegate@U2@@UBEPAVPropertyWidget@2@AAVU2OpStatus@2@PAVQWidget@@@Z 10011c90 f   U2Designer:U2Designer.dll
 0001:00010c96       ?getDelegate@DelegateEditor@U2@@UAEPAVPropertyDelegate@2@ABVQString@@@Z 10011c96 f   U2Designer:U2Designer.dll
 0001:00010c9c       ?getDisplayValue@ComboBoxDelegate@U2@@UBE?AVQVariant@@ABV3@@Z 10011c9c f   U2Designer:U2Designer.dll
 0001:00010ca2       ?getDisplayValue@SpinBoxDelegate@U2@@UBE?AVQVariant@@ABV3@@Z 10011ca2 f   U2Designer:U2Designer.dll
 0001:00010ca8       ?getDisplayValue@URLDelegate@U2@@UBE?AVQVariant@@ABV3@@Z 10011ca8 f   U2Designer:U2Designer.dll
 0001:00010cae       ?getItems@ComboBoxDelegate@U2@@UBEXAAV?$QMap@VQString@@VQVariant@@@@@Z 10011cae f   U2Designer:U2Designer.dll
 0001:00010cb4       ?getItems@SpinBoxDelegate@U2@@UBEXAAV?$QMap@VQString@@VQVariant@@@@@Z 10011cb4 f   U2Designer:U2Designer.dll
 0001:00010cba       ?metaObject@ComboBoxDelegate@U2@@UBEPBUQMetaObject@@XZ 10011cba f   U2Designer:U2Designer.dll
 0001:00010cc0       ?metaObject@DelegateEditor@U2@@UBEPBUQMetaObject@@XZ 10011cc0 f   U2Designer:U2Designer.dll
 0001:00010cc6       ?metaObject@SpinBoxDelegate@U2@@UBEPBUQMetaObject@@XZ 10011cc6 f   U2Designer:U2Designer.dll
 0001:00010ccc       ?metaObject@URLDelegate@U2@@UBEPBUQMetaObject@@XZ 10011ccc f   U2Designer:U2Designer.dll
 0001:00010cd2       ?qt_metacall@ComboBoxDelegate@U2@@UAEHW4Call@QMetaObject@@HPAPAX@Z 10011cd2 f   U2Designer:U2Designer.dll
 0001:00010cd8       ?qt_metacall@DelegateEditor@U2@@UAEHW4Call@QMetaObject@@HPAPAX@Z 10011cd8 f   U2Designer:U2Designer.dll
 0001:00010cde       ?qt_metacall@SpinBoxDelegate@U2@@UAEHW4Call@QMetaObject@@HPAPAX@Z 10011cde f   U2Designer:U2Designer.dll
 0001:00010ce4       ?qt_metacall@URLDelegate@U2@@UAEHW4Call@QMetaObject@@HPAPAX@Z 10011ce4 f   U2Designer:U2Designer.dll
 0001:00010cea       ?qt_metacast@ComboBoxDelegate@U2@@UAEPAXPBD@Z 10011cea f   U2Designer:U2Designer.dll
 0001:00010cf0       ?qt_metacast@DelegateEditor@U2@@UAEPAXPBD@Z 10011cf0 f   U2Designer:U2Designer.dll
 0001:00010cf6       ?qt_metacast@SpinBoxDelegate@U2@@UAEPAXPBD@Z 10011cf6 f   U2Designer:U2Designer.dll
 0001:00010cfc       ?qt_metacast@URLDelegate@U2@@UAEPAXPBD@Z 10011cfc f   U2Designer:U2Designer.dll
 0001:00010d02       ?removeDelegate@DelegateEditor@U2@@UAEPAVPropertyDelegate@2@ABVQString@@@Z 10011d02 f   U2Designer:U2Designer.dll
 0001:00010d08       ?setEditorData@ComboBoxDelegate@U2@@UBEXPAVQWidget@@ABVQModelIndex@@@Z 10011d08 f   U2Designer:U2Designer.dll
 0001:00010d0e       ?setEditorData@SpinBoxDelegate@U2@@UBEXPAVQWidget@@ABVQModelIndex@@@Z 10011d0e f   U2Designer:U2Designer.dll
 0001:00010d14       ?setEditorData@URLDelegate@U2@@UBEXPAVQWidget@@ABVQModelIndex@@@Z 10011d14 f   U2Designer:U2Designer.dll
 0001:00010d1a       ?setModelData@ComboBoxDelegate@U2@@UBEXPAVQWidget@@PAVQAbstractItemModel@@ABVQModelIndex@@@Z 10011d1a f   U2Designer:U2Designer.dll
 0001:00010d20       ?setModelData@SpinBoxDelegate@U2@@UBEXPAVQWidget@@PAVQAbstractItemModel@@ABVQModelIndex@@@Z 10011d20 f   U2Designer:U2Designer.dll
 0001:00010d26       ?setModelData@URLDelegate@U2@@UBEXPAVQWidget@@PAVQAbstractItemModel@@ABVQModelIndex@@@Z 10011d26 f   U2Designer:U2Designer.dll
 0001:00010d2c       ?type@URLDelegate@U2@@UBE?AW4Type@PropertyDelegate@2@XZ 10011d2c f   U2Designer:U2Designer.dll
 0001:00010d32       ?updateDelegate@DelegateEditor@U2@@UAEXABVQString@@@Z 10011d32 f   U2Designer:U2Designer.dll
 0001:00010d38       ?updateDelegates@DelegateEditor@U2@@UAEXXZ 10011d38 f   U2Designer:U2Designer.dll
 0001:00010d3e       ?destroyEditor@QAbstractItemDelegate@@UBEXPAVQWidget@@ABVQModelIndex@@@Z 10011d3e f   Qt5Widgets:Qt5Widgets.dll
 0001:00010d44       ?drawCheck@QItemDelegate@@MBEXPAVQPainter@@ABVQStyleOptionViewItem@@ABVQRect@@W4CheckState@Qt@@@Z 10011d44 f   Qt5Widgets:Qt5Widgets.dll
 0001:00010d4a       ?drawDecoration@QItemDelegate@@MBEXPAVQPainter@@ABVQStyleOptionViewItem@@ABVQRect@@ABVQPixmap@@@Z 10011d4a f   Qt5Widgets:Qt5Widgets.dll
 0001:00010d50       ?drawDisplay@QItemDelegate@@MBEXPAVQPainter@@ABVQStyleOptionViewItem@@ABVQRect@@ABVQString@@@Z 10011d50 f   Qt5Widgets:Qt5Widgets.dll
 0001:00010d56       ?drawFocus@QItemDelegate@@MBEXPAVQPainter@@ABVQStyleOptionViewItem@@ABVQRect@@@Z 10011d56 f   Qt5Widgets:Qt5Widgets.dll
 0001:00010d5c       ?editorEvent@QItemDelegate@@MAE_NPAVQEvent@@PAVQAbstractItemModel@@ABVQStyleOptionViewItem@@ABVQModelIndex@@@Z 10011d5c f   Qt5Widgets:Qt5Widgets.dll
 0001:00010d62       ?eventFilter@QItemDelegate@@MAE_NPAVQObject@@PAVQEvent@@@Z 10011d62 f   Qt5Widgets:Qt5Widgets.dll
 0001:00010d68       ?helpEvent@QAbstractItemDelegate@@UAE_NPAVQHelpEvent@@PAVQAbstractItemView@@ABVQStyleOptionViewItem@@ABVQModelIndex@@@Z 10011d68 f   Qt5Widgets:Qt5Widgets.dll
 0001:00010d6e       ?paint@QItemDelegate@@UBEXPAVQPainter@@ABVQStyleOptionViewItem@@ABVQModelIndex@@@Z 10011d6e f   Qt5Widgets:Qt5Widgets.dll
 0001:00010d74       ?paintingRoles@QAbstractItemDelegate@@UBE?AV?$QVector@H@@XZ 10011d74 f   Qt5Widgets:Qt5Widgets.dll
 0001:00010d7a       ?sizeHint@QItemDelegate@@UBE?AVQSize@@ABVQStyleOptionViewItem@@ABVQModelIndex@@@Z 10011d7a f   Qt5Widgets:Qt5Widgets.dll
 0001:00010d80       ?updateEditorGeometry@QItemDelegate@@UBEXPAVQWidget@@ABVQStyleOptionViewItem@@ABVQModelIndex@@@Z 10011d80 f   Qt5Widgets:Qt5Widgets.dll
 0001:00010d86       ?clear@QTextDocument@@UAEXXZ 10011d86 f   Qt5Gui:Qt5Gui.dll
 0001:00010d8c       ?createObject@QTextDocument@@MAEPAVQTextObject@@ABVQTextFormat@@@Z 10011d8c f   Qt5Gui:Qt5Gui.dll
 0001:00010d92       ?loadResource@QTextDocument@@MAE?AVQVariant@@HABVQUrl@@@Z 10011d92 f   Qt5Gui:Qt5Gui.dll
 0001:00010d98       ??0QScriptValue@@QAE@XZ    10011d98 f   Qt5Script:Qt5Script.dll
 0001:00010d9e       ??1QScriptValue@@QAE@XZ    10011d9e f   Qt5Script:Qt5Script.dll
 0001:00010da4       ??0QScriptValue@@QAE@ABV0@@Z 10011da4 f   Qt5Script:Qt5Script.dll
 0001:00010daa       ??4QScriptValue@@QAEAAV0@ABV0@@Z 10011daa f   Qt5Script:Qt5Script.dll
 0001:00010db0       ?isNumber@QScriptValue@@QBE_NXZ 10011db0 f   Qt5Script:Qt5Script.dll
 0001:00010db6       ?isString@QScriptValue@@QBE_NXZ 10011db6 f   Qt5Script:Qt5Script.dll
 0001:00010dbc       ?toString@QScriptValue@@QBE?AVQString@@XZ 10011dbc f   Qt5Script:Qt5Script.dll
 0001:00010dc2       ?toInt32@QScriptValue@@QBEHXZ 10011dc2 f   Qt5Script:Qt5Script.dll
 0001:00010dc8       ??1QScriptEngine@@UAE@XZ   10011dc8 f   Qt5Script:Qt5Script.dll
 0001:00010dce       ?newVariant@QScriptEngine@@QAE?AVQScriptValue@@ABVQVariant@@@Z 10011dce f   Qt5Script:Qt5Script.dll
 0001:00010dd4       ??0QString@@QAE@ABV0@@Z    10011dd4 f   Qt5Core:Qt5Core.dll
 0001:00010dda       ??1QString@@QAE@XZ         10011dda f   Qt5Core:Qt5Core.dll
 0001:00010de0       ?indexOf@QString@@QBEHABV1@HW4CaseSensitivity@Qt@@@Z 10011de0 f   Qt5Core:Qt5Core.dll
 0001:00010de6       ?fromAscii_helper@QString@@CAPAU?$QTypedArrayData@G@@PBDH@Z 10011de6 f   Qt5Core:Qt5Core.dll
 0001:00010dec       ?detach@QListData@@QAEPAUData@1@H@Z 10011dec f   Qt5Core:Qt5Core.dll
 0001:00010df2       ?detach_grow@QListData@@QAEPAUData@1@PAHH@Z 10011df2 f   Qt5Core:Qt5Core.dll
 0001:00010df8       ?dispose@QListData@@SAXPAUData@1@@Z 10011df8 f   Qt5Core:Qt5Core.dll
 0001:00010dfe       ?append@QListData@@QAEPAPAXXZ 10011dfe f   Qt5Core:Qt5Core.dll
 0001:00010e04       ?tr@QMetaObject@@QBE?AVQString@@PBD0H@Z 10011e04 f   Qt5Core:Qt5Core.dll
 0001:00010e0a       ??1Connection@QMetaObject@@QAE@XZ 10011e0a f   Qt5Core:Qt5Core.dll
 0001:00010e10       ??0QChar@@QAE@UQLatin1Char@@@Z 10011e10 f   Qt5Core:Qt5Core.dll
 0001:00010e16       ?arg@QString@@QBE?AV1@ABV1@HVQChar@@@Z 10011e16 f   Qt5Core:Qt5Core.dll
 0001:00010e1c       ?connect@QObject@@QBE?AVConnection@QMetaObject@@PBV1@PBD1W4ConnectionType@Qt@@@Z 10011e1c f   Qt5Core:Qt5Core.dll
 0001:00010e22       ?childEvent@QObject@@MAEXPAVQChildEvent@@@Z 10011e22 f   Qt5Core:Qt5Core.dll
 0001:00010e28       ?connectNotify@QObject@@MAEXABVQMetaMethod@@@Z 10011e28 f   Qt5Core:Qt5Core.dll
 0001:00010e2e       ?customEvent@QObject@@MAEXPAVQEvent@@@Z 10011e2e f   Qt5Core:Qt5Core.dll
 0001:00010e34       ?disconnectNotify@QObject@@MAEXABVQMetaMethod@@@Z 10011e34 f   Qt5Core:Qt5Core.dll
 0001:00010e3a       ?event@QObject@@UAE_NPAVQEvent@@@Z 10011e3a f   Qt5Core:Qt5Core.dll
 0001:00010e40       ?eventFilter@QObject@@UAE_NPAV1@PAVQEvent@@@Z 10011e40 f   Qt5Core:Qt5Core.dll
 0001:00010e46       ?timerEvent@QObject@@MAEXPAVQTimerEvent@@@Z 10011e46 f   Qt5Core:Qt5Core.dll
 0001:00010e4c       ??4QString@@QAEAAV0@ABV0@@Z 10011e4c f   Qt5Core:Qt5Core.dll
 0001:00010e52       ??4QString@@QAEAAV0@$$QAV0@@Z 10011e52 f   Qt5Core:Qt5Core.dll
 0001:00010e58       ??4QString@@QAEAAV0@PBD@Z  10011e58 f   Qt5Core:Qt5Core.dll
 0001:00010e5e       ??0QRegExp@@QAE@ABVQString@@W4CaseSensitivity@Qt@@W4PatternSyntax@0@@Z 10011e5e f   Qt5Core:Qt5Core.dll
 0001:00010e64       ??1QRegExp@@QAE@XZ         10011e64 f   Qt5Core:Qt5Core.dll
 0001:00010e6a       ??4QRegExp@@QAEAAV0@$$QAV0@@Z 10011e6a f   Qt5Core:Qt5Core.dll
 0001:00010e70       ??0QFileInfo@@QAE@ABVQString@@@Z 10011e70 f   Qt5Core:Qt5Core.dll
 0001:00010e76       ??1QFileInfo@@QAE@XZ       10011e76 f   Qt5Core:Qt5Core.dll
 0001:00010e7c       ?exists@QFileInfo@@SA_NABVQString@@@Z 10011e7c f   Qt5Core:Qt5Core.dll
 0001:00010e82       ?absolutePath@QFileInfo@@QBE?AVQString@@XZ 10011e82 f   Qt5Core:Qt5Core.dll
 0001:00010e88       ?translate@QCoreApplication@@SA?AVQString@@PBD00H@Z 10011e88 f   Qt5Core:Qt5Core.dll
 0001:00010e8e       ??0QString@@QAE@XZ         10011e8e f   Qt5Core:Qt5Core.dll
 0001:00010e94       ??0QString@@QAE@$$QAV0@@Z  10011e94 f   Qt5Core:Qt5Core.dll
 0001:00010e9a       ?replace@QString@@QAEAAV1@ABV1@0W4CaseSensitivity@Qt@@@Z 10011e9a f   Qt5Core:Qt5Core.dll
 0001:00010ea0       ?number@QString@@SA?AV1@HH@Z 10011ea0 f   Qt5Core:Qt5Core.dll
 0001:00010ea6       ??8@YA_NABVQString@@0@Z    10011ea6 f   Qt5Core:Qt5Core.dll
 0001:00010eac       ??0QDir@@QAE@ABVQString@@@Z 10011eac f   Qt5Core:Qt5Core.dll
 0001:00010eb2       ??1QDir@@QAE@XZ            10011eb2 f   Qt5Core:Qt5Core.dll
 0001:00010eb8       ?toNativeSeparators@QDir@@SA?AVQString@@ABV2@@Z 10011eb8 f   Qt5Core:Qt5Core.dll
 0001:00010ebe       ?entryList@QDir@@QBE?AVQStringList@@ABV2@V?$QFlags@W4Filter@QDir@@@@V?$QFlags@W4SortFlag@QDir@@@@@Z 10011ebe f   Qt5Core:Qt5Core.dll
 0001:00010ec4       ?userType@QVariant@@QBEHXZ 10011ec4 f   Qt5Core:Qt5Core.dll
 0001:00010eca       ?constData@QVariant@@QBEPBXXZ 10011eca f   Qt5Core:Qt5Core.dll
 0001:00010ed0       ?convert@QVariant@@QBE_NHPAX@Z 10011ed0 f   Qt5Core:Qt5Core.dll
 0001:00010ed6       ?cast@QMetaObject@@QBEPAVQObject@@PAV2@@Z 10011ed6 f   Qt5Core:Qt5Core.dll
 0001:00010edc       ?arg@QString@@QBE?AV1@HHHVQChar@@@Z 10011edc f   Qt5Core:Qt5Core.dll
 0001:00010ee2       ?append@QString@@QAEAAV1@ABV1@@Z 10011ee2 f   Qt5Core:Qt5Core.dll
 0001:00010ee8       ??M@YA_NABVQString@@0@Z    10011ee8 f   Qt5Core:Qt5Core.dll
 0001:00010eee       ?realloc@QListData@@QAEXH@Z 10011eee f   Qt5Core:Qt5Core.dll
 0001:00010ef4       ??1QObject@@UAE@XZ         10011ef4 f   Qt5Core:Qt5Core.dll
 0001:00010efa       ?nextNode@QMapNodeBase@@QBEPBU1@XZ 10011efa f   Qt5Core:Qt5Core.dll
 0001:00010f00       ?freeNodeAndRebalance@QMapDataBase@@QAEXPAUQMapNodeBase@@@Z 10011f00 f   Qt5Core:Qt5Core.dll
 0001:00010f06       ?recalcMostLeftNode@QMapDataBase@@QAEXXZ 10011f06 f   Qt5Core:Qt5Core.dll
 0001:00010f0c       ?createNode@QMapDataBase@@QAEPAUQMapNodeBase@@HHPAU2@_N@Z 10011f0c f   Qt5Core:Qt5Core.dll
 0001:00010f12       ?freeTree@QMapDataBase@@QAEXPAUQMapNodeBase@@H@Z 10011f12 f   Qt5Core:Qt5Core.dll
 0001:00010f18       ?createData@QMapDataBase@@SAPAU1@XZ 10011f18 f   Qt5Core:Qt5Core.dll
 0001:00010f1e       ?freeData@QMapDataBase@@SAXPAU1@@Z 10011f1e f   Qt5Core:Qt5Core.dll
 0001:00010f24       ?free_helper@QHashData@@QAEXP6AXPAUNode@1@@Z@Z 10011f24 f   Qt5Core:Qt5Core.dll
 0001:00010f2a       ??0QVariant@@QAE@XZ        10011f2a f   Qt5Core:Qt5Core.dll
 0001:00010f30       ??1QVariant@@QAE@XZ        10011f30 f   Qt5Core:Qt5Core.dll
 0001:00010f36       ??0QVariant@@QAE@ABV0@@Z   10011f36 f   Qt5Core:Qt5Core.dll
 0001:00010f3c       ??4QVariant@@QAEAAV0@ABV0@@Z 10011f3c f   Qt5Core:Qt5Core.dll
 0001:00010f42       ?toString@QVariant@@QBE?AVQString@@XZ 10011f42 f   Qt5Core:Qt5Core.dll
 0001:00010f48       ?toMap@QVariant@@QBE?AV?$QMap@VQString@@VQVariant@@@@XZ 10011f48 f   Qt5Core:Qt5Core.dll
 0001:00010f4e       ?dir@QFileInfo@@QBE?AVQDir@@XZ 10011f4e f   Qt5Core:Qt5Core.dll
 0001:00010f54       ?absoluteDir@QFileInfo@@QBE?AVQDir@@XZ 10011f54 f   Qt5Core:Qt5Core.dll
 0001:00010f5a       ?path@QDir@@QBE?AVQString@@XZ 10011f5a f   Qt5Core:Qt5Core.dll
 0001:00010f60       ?mkpath@QDir@@QBE_NABVQString@@@Z 10011f60 f   Qt5Core:Qt5Core.dll
 0001:00010f66       ?fromUtf8@QString@@SA?AV1@PBDH@Z 10011f66 f   Qt5Core:Qt5Core.dll
 0001:00010f6c       ?idealThreadCount@QThread@@SAHXZ 10011f6c f   Qt5Core:Qt5Core.dll
 0001:00010f72       ??0QVariant@@QAE@H@Z       10011f72 f   Qt5Core:Qt5Core.dll
 0001:00010f78       ??0QVariant@@QAE@ABVQString@@@Z 10011f78 f   Qt5Core:Qt5Core.dll
 0001:00010f7e       ??4QVariant@@QAEAAV0@$$QAV0@@Z 10011f7e f   Qt5Core:Qt5Core.dll
 0001:00010f84       ?dynamicMetaObject@QObjectData@@QBEPAUQMetaObject@@XZ 10011f84 f   Qt5Core:Qt5Core.dll
 0001:00010f8a       ?className@QMetaObject@@QBEPBDXZ 10011f8a f   Qt5Core:Qt5Core.dll
 0001:00010f90       ??0QByteArray@@QAE@XZ      10011f90 f   Qt5Core:Qt5Core.dll
 0001:00010f96       ??1QByteArray@@QAE@XZ      10011f96 f   Qt5Core:Qt5Core.dll
 0001:00010f9c       ?reserve@QByteArray@@QAEXH@Z 10011f9c f   Qt5Core:Qt5Core.dll
 0001:00010fa2       ?append@QByteArray@@QAEAAV1@D@Z 10011fa2 f   Qt5Core:Qt5Core.dll
 0001:00010fa8       ?append@QByteArray@@QAEAAV1@PBD@Z 10011fa8 f   Qt5Core:Qt5Core.dll
 0001:00010fae       ?registerNormalizedType@QMetaType@@SAHABVQByteArray@@P6AXPAX@ZP6APAXPBX@Z2P6APAX13@ZHV?$QFlags@W4TypeFlag@QMetaType@@@@PBUQMetaObject@@@Z 10011fae f   Qt5Core:Qt5Core.dll
 0001:00010fb4       ?registerNormalizedTypedef@QMetaType@@SAHABVQByteArray@@H@Z 10011fb4 f   Qt5Core:Qt5Core.dll
 0001:00010fba       ?_Xbad_alloc@std@@YAXXZ    10011fba f   msvcprt:MSVCP120.dll
 0001:00010fc0       ?_Xlength_error@std@@YAXPBD@Z 10011fc0 f   msvcprt:MSVCP120.dll
 0001:00010fc6       ?_Xout_of_range@std@@YAXPBD@Z 10011fc6 f   msvcprt:MSVCP120.dll
 0001:00010fcc       ?_Syserror_map@std@@YAPBDH@Z 10011fcc f   msvcprt:MSVCP120.dll
 0001:00010fd2       ?_Winerror_map@std@@YAPBDH@Z 10011fd2 f   msvcprt:MSVCP120.dll
 0001:00010fd8       __purecall                 10011fd8 f   MSVCRT:MSVCR120.dll
 0001:00010fde       ??2@YAPAXI@Z               10011fde f   MSVCRT:MSVCR120.dll
 0001:00010fe4       ??3@YAXPAX@Z               10011fe4 f   MSVCRT:MSVCR120.dll
 0001:00010fed       ___atonexitinit            10011fed f   MSVCRT:atonexit.obj
 0001:00011029       __onexit                   10012029 f   MSVCRT:atonexit.obj
 0001:000110d2       _atexit                    100120d2 f   MSVCRT:atonexit.obj
 0001:000110e8       _memmove                   100120e8 f   MSVCRT:MSVCR120.dll
 0001:000110ee       __hypot                    100120ee f   MSVCRT:MSVCR120.dll
 0001:000110f4       @__security_check_cookie@4 100120f4 f   MSVCRT:secchk.obj
 0001:00011104       __CxxThrowException@8      10012104 f   MSVCRT:MSVCR120.dll
 0001:0001110a       ___CxxFrameHandler3        1001210a f   MSVCRT:MSVCR120.dll
 0001:00011110       _memcpy                    10012110 f   MSVCRT:MSVCR120.dll
 0001:00011116       ??0type_info@@AAE@ABV0@@Z  10012116 f   MSVCRT:ti_inst.obj
 0001:00011121       ??4type_info@@AAEAAV0@ABV0@@Z 10012121 f   MSVCRT:ti_inst.obj
 0001:00011126       ??_Etype_info@@UAEPAXI@Z   10012126 f i MSVCRT:ti_inst.obj
 0001:000111bc       _NtCurrentTeb              100121bc f i MSVCRT:crtdll.obj
 0001:000111c3       __CRT_INIT@12              100121c3 f   MSVCRT:crtdll.obj
 0001:000113ba       __DllMainCRTStartup@12     100123ba f   MSVCRT:crtdll.obj
 0001:00011510       __lock                     10012510 f   MSVCRT:MSVCR120.dll
 0001:00011516       __unlock                   10012516 f   MSVCRT:MSVCR120.dll
 0001:0001151c       __calloc_crt               1001251c f   MSVCRT:MSVCR120.dll
 0001:00011522       ___dllonexit               10012522 f   MSVCRT:MSVCR120.dll
 0001:00011530       __SEH_prolog4              10012530 f   MSVCRT:sehprolg4.obj
 0001:00011575       __SEH_epilog4              10012575 f   MSVCRT:sehprolg4.obj
 0001:00011589       __except_handler4          10012589 f   MSVCRT:chandler4gs.obj
 0001:000115ac       ___raise_securityfailure   100125ac f   MSVCRT:gs_report.obj
 0001:000115e9       ___report_gsfailure        100125e9 f   MSVCRT:gs_report.obj
 0001:000116e4       ___report_rangecheckfailure 100126e4 f   MSVCRT:gs_report.obj
 0001:000116f0       ___report_securityfailure  100126f0 f   MSVCRT:gs_report.obj
 0001:000117c0       ___report_securityfailureEx 100127c0 f   MSVCRT:gs_report.obj
 0001:000118d6       ??_M@YGXPAXIHP6EX0@Z@Z     100128d6 f   MSVCRT:ehvecdtr.obj
 0001:0001195e       ?__ArrayUnwind@@YGXPAXIHP6EX0@Z@Z 1001295e f   MSVCRT:ehvecdtr.obj
 0001:000119bc       ??1type_info@@UAE@XZ       100129bc f   MSVCRT:MSVCR120.dll
 0001:000119c2       ___CppXcptFilter           100129c2 f   MSVCRT:MSVCR120.dll
 0001:000119c8       __amsg_exit                100129c8 f   MSVCRT:MSVCR120.dll
 0001:000119d0       __FindPESection            100129d0 f   MSVCRT:pesect.obj
 0001:00011a20       __IsNonwritableInCurrentImage 10012a20 f   MSVCRT:pesect.obj
 0001:00011ae0       __ValidateImageBase        10012ae0 f   MSVCRT:pesect.obj
 0001:00011b12       _free                      10012b12 f   MSVCRT:MSVCR120.dll
 0001:00011b18       ___security_init_cookie    10012b18 f   MSVCRT:gs_support.obj
 0001:00011bb4       _DllMain@12                10012bb4 f   MSVCRT:dllmain.obj
 0001:00011bd6       __malloc_crt               10012bd6 f   MSVCRT:MSVCR120.dll
 0001:00011bdc       __RTC_Initialize           10012bdc f   MSVCRT:initsect.obj
 0001:00011bfc       __RTC_Terminate            10012bfc f   MSVCRT:initsect.obj
 0001:00011c1c       __initterm                 10012c1c f   MSVCRT:MSVCR120.dll
 0001:00011c22       __initterm_e               10012c22 f   MSVCRT:MSVCR120.dll
 0001:00011c28       ___clean_type_info_names   10012c28 f   MSVCRT:tncleanup.obj
 0001:00011c34       __except_handler4_common   10012c34 f   MSVCRT:MSVCR120.dll
 0001:00011c3a       __crt_debugger_hook        10012c3a f   MSVCRT:MSVCR120.dll
 0001:00011c40       ___crtUnhandledException   10012c40 f   MSVCRT:MSVCR120.dll
 0001:00011c46       ___crtTerminateProcess     10012c46 f   MSVCRT:MSVCR120.dll
 0001:00011c4c       ?terminate@@YAXXZ          10012c4c f   MSVCRT:MSVCR120.dll
 0001:00011c52       ___clean_type_info_names_internal 10012c52 f   MSVCRT:MSVCR120.dll
 0001:00011c58       _EncodePointer@4           10012c58 f   kernel32:KERNEL32.dll
 0001:00011c5e       _DecodePointer@4           10012c5e f   kernel32:KERNEL32.dll
 0001:00011c64       _IsDebuggerPresent@0       10012c64 f   kernel32:KERNEL32.dll
 0001:00011c6a       _IsProcessorFeaturePresent@4 10012c6a f   kernel32:KERNEL32.dll
 0001:00011c70       _QueryPerformanceCounter@4 10012c70 f   kernel32:KERNEL32.dll
 0001:00011c76       _GetCurrentProcessId@0     10012c76 f   kernel32:KERNEL32.dll
 0001:00011c7c       _GetCurrentThreadId@0      10012c7c f   kernel32:KERNEL32.dll
 0001:00011c82       _GetSystemTimeAsFileTime@4 10012c82 f   kernel32:KERNEL32.dll
 0001:00011c88       _DisableThreadLibraryCalls@4 10012c88 f   kernel32:KERNEL32.dll
 0002:00000000       __imp__DisableThreadLibraryCalls@4 10017000     kernel32:KERNEL32.dll
 0002:00000004       __imp__GetSystemTimeAsFileTime@4 10017004     kernel32:KERNEL32.dll
 0002:00000008       __imp__GetCurrentThreadId@0 10017008     kernel32:KERNEL32.dll
 0002:0000000c       __imp__GetCurrentProcessId@0 1001700c     kernel32:KERNEL32.dll
 0002:00000010       __imp__QueryPerformanceCounter@4 10017010     kernel32:KERNEL32.dll
 0002:00000014       __imp__IsProcessorFeaturePresent@4 10017014     kernel32:KERNEL32.dll
 0002:00000018       __imp__IsDebuggerPresent@0 10017018     kernel32:KERNEL32.dll
 0002:0000001c       __imp__EncodePointer@4     1001701c     kernel32:KERNEL32.dll
 0002:00000020       __imp__DecodePointer@4     10017020     kernel32:KERNEL32.dll
 0002:00000024       \177KERNEL32_NULL_THUNK_DATA 10017024     kernel32:KERNEL32.dll
 0002:00000028       __imp_?_Syserror_map@std@@YAPBDH@Z 10017028     msvcprt:MSVCP120.dll
 0002:0000002c       __imp_?_Xout_of_range@std@@YAXPBD@Z 1001702c     msvcprt:MSVCP120.dll
 0002:00000030       __imp_?_Xlength_error@std@@YAXPBD@Z 10017030     msvcprt:MSVCP120.dll
 0002:00000034       __imp_?_Xbad_alloc@std@@YAXXZ 10017034     msvcprt:MSVCP120.dll
 0002:00000038       __imp_?_Winerror_map@std@@YAPBDH@Z 10017038     msvcprt:MSVCP120.dll
 0002:0000003c       \177MSVCP120_NULL_THUNK_DATA 1001703c     msvcprt:MSVCP120.dll
 0002:00000040       __imp___initterm_e         10017040     MSVCRT:MSVCR120.dll
 0002:00000044       __imp___initterm           10017044     MSVCRT:MSVCR120.dll
 0002:00000048       __imp___malloc_crt         10017048     MSVCRT:MSVCR120.dll
 0002:0000004c       __imp___crt_debugger_hook  1001704c     MSVCRT:MSVCR120.dll
 0002:00000050       __imp___except_handler4_common 10017050     MSVCRT:MSVCR120.dll
 0002:00000054       __imp___CxxThrowException@8 10017054     MSVCRT:MSVCR120.dll
 0002:00000058       __imp___purecall           10017058     MSVCRT:MSVCR120.dll
 0002:0000005c       __imp_??2@YAPAXI@Z         1001705c     MSVCRT:MSVCR120.dll
 0002:00000060       __imp_??3@YAXPAX@Z         10017060     MSVCRT:MSVCR120.dll
 0002:00000064       __imp__memmove             10017064     MSVCRT:MSVCR120.dll
 0002:00000068       __imp___hypot              10017068     MSVCRT:MSVCR120.dll
 0002:0000006c       __imp____CxxFrameHandler3  1001706c     MSVCRT:MSVCR120.dll
 0002:00000070       __imp__memcpy              10017070     MSVCRT:MSVCR120.dll
 0002:00000074       __imp___lock               10017074     MSVCRT:MSVCR120.dll
 0002:00000078       __imp___unlock             10017078     MSVCRT:MSVCR120.dll
 0002:0000007c       __imp___calloc_crt         1001707c     MSVCRT:MSVCR120.dll
 0002:00000080       __imp____dllonexit         10017080     MSVCRT:MSVCR120.dll
 0002:00000084       __imp___onexit             10017084     MSVCRT:MSVCR120.dll
 0002:00000088       __imp_??1type_info@@UAE@XZ 10017088     MSVCRT:MSVCR120.dll
 0002:0000008c       __imp____CppXcptFilter     1001708c     MSVCRT:MSVCR120.dll
 0002:00000090       __imp___amsg_exit          10017090     MSVCRT:MSVCR120.dll
 0002:00000094       __imp____crtUnhandledException 10017094     MSVCRT:MSVCR120.dll
 0002:00000098       __imp____crtTerminateProcess 10017098     MSVCRT:MSVCR120.dll
 0002:0000009c       __imp_?terminate@@YAXXZ    1001709c     MSVCRT:MSVCR120.dll
 0002:000000a0       __imp____clean_type_info_names_internal 100170a0     MSVCRT:MSVCR120.dll
 0002:000000a4       __imp__free                100170a4     MSVCRT:MSVCR120.dll
 0002:000000a8       \177MSVCR120_NULL_THUNK_DATA 100170a8     MSVCRT:MSVCR120.dll
 0002:000000ac       __imp_?detach_grow@QListData@@QAEPAUData@1@PAHH@Z 100170ac     Qt5Core:Qt5Core.dll
 0002:000000b0       __imp_?dispose@QListData@@SAXPAUData@1@@Z 100170b0     Qt5Core:Qt5Core.dll
 0002:000000b4       __imp_?append@QListData@@QAEPAPAXXZ 100170b4     Qt5Core:Qt5Core.dll
 0002:000000b8       __imp_?shared_null@QListData@@2UData@1@B 100170b8     Qt5Core:Qt5Core.dll
 0002:000000bc       __imp_?tr@QMetaObject@@QBE?AVQString@@PBD0H@Z 100170bc     Qt5Core:Qt5Core.dll
 0002:000000c0       __imp_??1Connection@QMetaObject@@QAE@XZ 100170c0     Qt5Core:Qt5Core.dll
 0002:000000c4       __imp_??0QChar@@QAE@UQLatin1Char@@@Z 100170c4     Qt5Core:Qt5Core.dll
 0002:000000c8       __imp_?arg@QString@@QBE?AV1@ABV1@HVQChar@@@Z 100170c8     Qt5Core:Qt5Core.dll
 0002:000000cc       __imp_?connect@QObject@@QBE?AVConnection@QMetaObject@@PBV1@PBD1W4ConnectionType@Qt@@@Z 100170cc     Qt5Core:Qt5Core.dll
 0002:000000d0       __imp_?childEvent@QObject@@MAEXPAVQChildEvent@@@Z 100170d0     Qt5Core:Qt5Core.dll
 0002:000000d4       __imp_?connectNotify@QObject@@MAEXABVQMetaMethod@@@Z 100170d4     Qt5Core:Qt5Core.dll
 0002:000000d8       __imp_?customEvent@QObject@@MAEXPAVQEvent@@@Z 100170d8     Qt5Core:Qt5Core.dll
 0002:000000dc       __imp_?disconnectNotify@QObject@@MAEXABVQMetaMethod@@@Z 100170dc     Qt5Core:Qt5Core.dll
 0002:000000e0       __imp_?event@QObject@@UAE_NPAVQEvent@@@Z 100170e0     Qt5Core:Qt5Core.dll
 0002:000000e4       __imp_?eventFilter@QObject@@UAE_NPAV1@PAVQEvent@@@Z 100170e4     Qt5Core:Qt5Core.dll
 0002:000000e8       __imp_?timerEvent@QObject@@MAEXPAVQTimerEvent@@@Z 100170e8     Qt5Core:Qt5Core.dll
 0002:000000ec       __imp_??4QString@@QAEAAV0@ABV0@@Z 100170ec     Qt5Core:Qt5Core.dll
 0002:000000f0       __imp_??4QString@@QAEAAV0@$$QAV0@@Z 100170f0     Qt5Core:Qt5Core.dll
 0002:000000f4       __imp_??4QString@@QAEAAV0@PBD@Z 100170f4     Qt5Core:Qt5Core.dll
 0002:000000f8       __imp_??0QRegExp@@QAE@ABVQString@@W4CaseSensitivity@Qt@@W4PatternSyntax@0@@Z 100170f8     Qt5Core:Qt5Core.dll
 0002:000000fc       __imp_??1QRegExp@@QAE@XZ   100170fc     Qt5Core:Qt5Core.dll
 0002:00000100       __imp_??4QRegExp@@QAEAAV0@$$QAV0@@Z 10017100     Qt5Core:Qt5Core.dll
 0002:00000104       __imp_??0QFileInfo@@QAE@ABVQString@@@Z 10017104     Qt5Core:Qt5Core.dll
 0002:00000108       __imp_??1QFileInfo@@QAE@XZ 10017108     Qt5Core:Qt5Core.dll
 0002:0000010c       __imp_?exists@QFileInfo@@SA_NABVQString@@@Z 1001710c     Qt5Core:Qt5Core.dll
 0002:00000110       __imp_?detach@QListData@@QAEPAUData@1@H@Z 10017110     Qt5Core:Qt5Core.dll
 0002:00000114       __imp_?translate@QCoreApplication@@SA?AVQString@@PBD00H@Z 10017114     Qt5Core:Qt5Core.dll
 0002:00000118       __imp_??0QString@@QAE@XZ   10017118     Qt5Core:Qt5Core.dll
 0002:0000011c       __imp_??0QString@@QAE@$$QAV0@@Z 1001711c     Qt5Core:Qt5Core.dll
 0002:00000120       __imp_?replace@QString@@QAEAAV1@ABV1@0W4CaseSensitivity@Qt@@@Z 10017120     Qt5Core:Qt5Core.dll
 0002:00000124       __imp_?number@QString@@SA?AV1@HH@Z 10017124     Qt5Core:Qt5Core.dll
 0002:00000128       __imp_??8@YA_NABVQString@@0@Z 10017128     Qt5Core:Qt5Core.dll
 0002:0000012c       __imp_??0QDir@@QAE@ABVQString@@@Z 1001712c     Qt5Core:Qt5Core.dll
 0002:00000130       __imp_??1QDir@@QAE@XZ      10017130     Qt5Core:Qt5Core.dll
 0002:00000134       __imp_?toNativeSeparators@QDir@@SA?AVQString@@ABV2@@Z 10017134     Qt5Core:Qt5Core.dll
 0002:00000138       __imp_?entryList@QDir@@QBE?AVQStringList@@ABV2@V?$QFlags@W4Filter@QDir@@@@V?$QFlags@W4SortFlag@QDir@@@@@Z 10017138     Qt5Core:Qt5Core.dll
 0002:0000013c       __imp_?userType@QVariant@@QBEHXZ 1001713c     Qt5Core:Qt5Core.dll
 0002:00000140       __imp_?constData@QVariant@@QBEPBXXZ 10017140     Qt5Core:Qt5Core.dll
 0002:00000144       __imp_?convert@QVariant@@QBE_NHPAX@Z 10017144     Qt5Core:Qt5Core.dll
 0002:00000148       __imp_?cast@QMetaObject@@QBEPAVQObject@@PAV2@@Z 10017148     Qt5Core:Qt5Core.dll
 0002:0000014c       __imp_?arg@QString@@QBE?AV1@HHHVQChar@@@Z 1001714c     Qt5Core:Qt5Core.dll
 0002:00000150       __imp_?append@QString@@QAEAAV1@ABV1@@Z 10017150     Qt5Core:Qt5Core.dll
 0002:00000154       __imp_??M@YA_NABVQString@@0@Z 10017154     Qt5Core:Qt5Core.dll
 0002:00000158       __imp_?realloc@QListData@@QAEXH@Z 10017158     Qt5Core:Qt5Core.dll
 0002:0000015c       __imp_??1QObject@@UAE@XZ   1001715c     Qt5Core:Qt5Core.dll
 0002:00000160       __imp_?nextNode@QMapNodeBase@@QBEPBU1@XZ 10017160     Qt5Core:Qt5Core.dll
 0002:00000164       __imp_?freeNodeAndRebalance@QMapDataBase@@QAEXPAUQMapNodeBase@@@Z 10017164     Qt5Core:Qt5Core.dll
 0002:00000168       __imp_?recalcMostLeftNode@QMapDataBase@@QAEXXZ 10017168     Qt5Core:Qt5Core.dll
 0002:0000016c       __imp_?createNode@QMapDataBase@@QAEPAUQMapNodeBase@@HHPAU2@_N@Z 1001716c     Qt5Core:Qt5Core.dll
 0002:00000170       __imp_?freeTree@QMapDataBase@@QAEXPAUQMapNodeBase@@H@Z 10017170     Qt5Core:Qt5Core.dll
 0002:00000174       __imp_?createData@QMapDataBase@@SAPAU1@XZ 10017174     Qt5Core:Qt5Core.dll
 0002:00000178       __imp_?freeData@QMapDataBase@@SAXPAU1@@Z 10017178     Qt5Core:Qt5Core.dll
 0002:0000017c       __imp_?free_helper@QHashData@@QAEXP6AXPAUNode@1@@Z@Z 1001717c     Qt5Core:Qt5Core.dll
 0002:00000180       __imp_??0QVariant@@QAE@XZ  10017180     Qt5Core:Qt5Core.dll
 0002:00000184       __imp_??1QVariant@@QAE@XZ  10017184     Qt5Core:Qt5Core.dll
 0002:00000188       __imp_??0QVariant@@QAE@ABV0@@Z 10017188     Qt5Core:Qt5Core.dll
 0002:0000018c       __imp_??4QVariant@@QAEAAV0@ABV0@@Z 1001718c     Qt5Core:Qt5Core.dll
 0002:00000190       __imp_?toString@QVariant@@QBE?AVQString@@XZ 10017190     Qt5Core:Qt5Core.dll
 0002:00000194       __imp_?toMap@QVariant@@QBE?AV?$QMap@VQString@@VQVariant@@@@XZ 10017194     Qt5Core:Qt5Core.dll
 0002:00000198       __imp_?dir@QFileInfo@@QBE?AVQDir@@XZ 10017198     Qt5Core:Qt5Core.dll
 0002:0000019c       __imp_?absoluteDir@QFileInfo@@QBE?AVQDir@@XZ 1001719c     Qt5Core:Qt5Core.dll
 0002:000001a0       __imp_?path@QDir@@QBE?AVQString@@XZ 100171a0     Qt5Core:Qt5Core.dll
 0002:000001a4       __imp_?mkpath@QDir@@QBE_NABVQString@@@Z 100171a4     Qt5Core:Qt5Core.dll
 0002:000001a8       __imp_?shared_null@QMapDataBase@@2U1@B 100171a8     Qt5Core:Qt5Core.dll
 0002:000001ac       __imp_?shared_null@QHashData@@2U1@B 100171ac     Qt5Core:Qt5Core.dll
 0002:000001b0       __imp_?fromUtf8@QString@@SA?AV1@PBDH@Z 100171b0     Qt5Core:Qt5Core.dll
 0002:000001b4       __imp_?idealThreadCount@QThread@@SAHXZ 100171b4     Qt5Core:Qt5Core.dll
 0002:000001b8       __imp_??0QVariant@@QAE@H@Z 100171b8     Qt5Core:Qt5Core.dll
 0002:000001bc       __imp_??0QVariant@@QAE@ABVQString@@@Z 100171bc     Qt5Core:Qt5Core.dll
 0002:000001c0       __imp_??4QVariant@@QAEAAV0@$$QAV0@@Z 100171c0     Qt5Core:Qt5Core.dll
 0002:000001c4       __imp_?dynamicMetaObject@QObjectData@@QBEPAUQMetaObject@@XZ 100171c4     Qt5Core:Qt5Core.dll
 0002:000001c8       __imp_?className@QMetaObject@@QBEPBDXZ 100171c8     Qt5Core:Qt5Core.dll
 0002:000001cc       __imp_??0QByteArray@@QAE@XZ 100171cc     Qt5Core:Qt5Core.dll
 0002:000001d0       __imp_?fromAscii_helper@QString@@CAPAU?$QTypedArrayData@G@@PBDH@Z 100171d0     Qt5Core:Qt5Core.dll
 0002:000001d4       __imp_?indexOf@QString@@QBEHABV1@HW4CaseSensitivity@Qt@@@Z 100171d4     Qt5Core:Qt5Core.dll
 0002:000001d8       __imp_??1QString@@QAE@XZ   100171d8     Qt5Core:Qt5Core.dll
 0002:000001dc       __imp_??0QString@@QAE@ABV0@@Z 100171dc     Qt5Core:Qt5Core.dll
 0002:000001e0       __imp_?registerNormalizedTypedef@QMetaType@@SAHABVQByteArray@@H@Z 100171e0     Qt5Core:Qt5Core.dll
 0002:000001e4       __imp_?registerNormalizedType@QMetaType@@SAHABVQByteArray@@P6AXPAX@ZP6APAXPBX@Z2P6APAX13@ZHV?$QFlags@W4TypeFlag@QMetaType@@@@PBUQMetaObject@@@Z 100171e4     Qt5Core:Qt5Core.dll
 0002:000001e8       __imp_?append@QByteArray@@QAEAAV1@PBD@Z 100171e8     Qt5Core:Qt5Core.dll
 0002:000001ec       __imp_?append@QByteArray@@QAEAAV1@D@Z 100171ec     Qt5Core:Qt5Core.dll
 0002:000001f0       __imp_?reserve@QByteArray@@QAEXH@Z 100171f0     Qt5Core:Qt5Core.dll
 0002:000001f4       __imp_?absolutePath@QFileInfo@@QBE?AVQString@@XZ 100171f4     Qt5Core:Qt5Core.dll
 0002:000001f8       __imp_??1QByteArray@@QAE@XZ 100171f8     Qt5Core:Qt5Core.dll
 0002:000001fc       \177Qt5Core_NULL_THUNK_DATA 100171fc     Qt5Core:Qt5Core.dll
 0002:00000200       __imp_?clear@QTextDocument@@UAEXXZ 10017200     Qt5Gui:Qt5Gui.dll
 0002:00000204       __imp_?createObject@QTextDocument@@MAEPAVQTextObject@@ABVQTextFormat@@@Z 10017204     Qt5Gui:Qt5Gui.dll
 0002:00000208       __imp_?loadResource@QTextDocument@@MAE?AVQVariant@@HABVQUrl@@@Z 10017208     Qt5Gui:Qt5Gui.dll
 0002:0000020c       \177Qt5Gui_NULL_THUNK_DATA 1001720c     Qt5Gui:Qt5Gui.dll
 0002:00000210       __imp_?isString@QScriptValue@@QBE_NXZ 10017210     Qt5Script:Qt5Script.dll
 0002:00000214       __imp_?isNumber@QScriptValue@@QBE_NXZ 10017214     Qt5Script:Qt5Script.dll
 0002:00000218       __imp_??4QScriptValue@@QAEAAV0@ABV0@@Z 10017218     Qt5Script:Qt5Script.dll
 0002:0000021c       __imp_??0QScriptValue@@QAE@ABV0@@Z 1001721c     Qt5Script:Qt5Script.dll
 0002:00000220       __imp_??1QScriptValue@@QAE@XZ 10017220     Qt5Script:Qt5Script.dll
 0002:00000224       __imp_??0QScriptValue@@QAE@XZ 10017224     Qt5Script:Qt5Script.dll
 0002:00000228       __imp_?toString@QScriptValue@@QBE?AVQString@@XZ 10017228     Qt5Script:Qt5Script.dll
 0002:0000022c       __imp_?toInt32@QScriptValue@@QBEHXZ 1001722c     Qt5Script:Qt5Script.dll
 0002:00000230       __imp_??1QScriptEngine@@UAE@XZ 10017230     Qt5Script:Qt5Script.dll
 0002:00000234       __imp_?newVariant@QScriptEngine@@QAE?AVQScriptValue@@ABVQVariant@@@Z 10017234     Qt5Script:Qt5Script.dll
 0002:00000238       \177Qt5Script_NULL_THUNK_DATA 10017238     Qt5Script:Qt5Script.dll
 0002:0000023c       __imp_?destroyEditor@QAbstractItemDelegate@@UBEXPAVQWidget@@ABVQModelIndex@@@Z 1001723c     Qt5Widgets:Qt5Widgets.dll
 0002:00000240       __imp_?sizeHint@QItemDelegate@@UBE?AVQSize@@ABVQStyleOptionViewItem@@ABVQModelIndex@@@Z 10017240     Qt5Widgets:Qt5Widgets.dll
 0002:00000244       __imp_?paintingRoles@QAbstractItemDelegate@@UBE?AV?$QVector@H@@XZ 10017244     Qt5Widgets:Qt5Widgets.dll
 0002:00000248       __imp_?paint@QItemDelegate@@UBEXPAVQPainter@@ABVQStyleOptionViewItem@@ABVQModelIndex@@@Z 10017248     Qt5Widgets:Qt5Widgets.dll
 0002:0000024c       __imp_?helpEvent@QAbstractItemDelegate@@UAE_NPAVQHelpEvent@@PAVQAbstractItemView@@ABVQStyleOptionViewItem@@ABVQModelIndex@@@Z 1001724c     Qt5Widgets:Qt5Widgets.dll
 0002:00000250       __imp_?eventFilter@QItemDelegate@@MAE_NPAVQObject@@PAVQEvent@@@Z 10017250     Qt5Widgets:Qt5Widgets.dll
 0002:00000254       __imp_?editorEvent@QItemDelegate@@MAE_NPAVQEvent@@PAVQAbstractItemModel@@ABVQStyleOptionViewItem@@ABVQModelIndex@@@Z 10017254     Qt5Widgets:Qt5Widgets.dll
 0002:00000258       __imp_?drawFocus@QItemDelegate@@MBEXPAVQPainter@@ABVQStyleOptionViewItem@@ABVQRect@@@Z 10017258     Qt5Widgets:Qt5Widgets.dll
 0002:0000025c       __imp_?drawDisplay@QItemDelegate@@MBEXPAVQPainter@@ABVQStyleOptionViewItem@@ABVQRect@@ABVQString@@@Z 1001725c     Qt5Widgets:Qt5Widgets.dll
 0002:00000260       __imp_?drawDecoration@QItemDelegate@@MBEXPAVQPainter@@ABVQStyleOptionViewItem@@ABVQRect@@ABVQPixmap@@@Z 10017260     Qt5Widgets:Qt5Widgets.dll
 0002:00000264       __imp_?drawCheck@QItemDelegate@@MBEXPAVQPainter@@ABVQStyleOptionViewItem@@ABVQRect@@W4CheckState@Qt@@@Z 10017264     Qt5Widgets:Qt5Widgets.dll
 0002:00000268       __imp_?updateEditorGeometry@QItemDelegate@@UBEXPAVQWidget@@ABVQStyleOptionViewItem@@ABVQModelIndex@@@Z 10017268     Qt5Widgets:Qt5Widgets.dll
 0002:0000026c       \177Qt5Widgets_NULL_THUNK_DATA 1001726c     Qt5Widgets:Qt5Widgets.dll
 0002:00000270       __imp_?staticMetaObject@Task@U2@@2UQMetaObject@@B 10017270     U2Core:U2Core.dll
 0002:00000274       __imp_?staticMetaObject@Plugin@U2@@2UQMetaObject@@B 10017274     U2Core:U2Core.dll
 0002:00000278       __imp_?qt_metacall@Plugin@U2@@UAEHW4Call@QMetaObject@@HPAPAX@Z 10017278     U2Core:U2Core.dll
 0002:0000027c       __imp_?qt_metacast@Plugin@U2@@UAEPAXPBD@Z 1001727c     U2Core:U2Core.dll
 0002:00000280       __imp_?staticMetaObject@ExternalTool@U2@@2UQMetaObject@@B 10017280     U2Core:U2Core.dll
 0002:00000284       __imp_?qt_metacall@ExternalTool@U2@@UAEHW4Call@QMetaObject@@HPAPAX@Z 10017284     U2Core:U2Core.dll
 0002:00000288       __imp_?qt_metacast@ExternalTool@U2@@UAEPAXPBD@Z 10017288     U2Core:U2Core.dll
 0002:0000028c       __imp_?PLAIN_TEXT@BaseDocumentFormats@U2@@2VQString@@B 1001728c     U2Core:U2Core.dll
 0002:00000290       __imp_?getDataPathByName@U2DataPathRegistry@U2@@QAEPAVU2DataPath@2@ABVQString@@@Z 10017290     U2Core:U2Core.dll
 0002:00000294       __imp_?getPathByName@U2DataPath@U2@@QBE?AVQString@@ABV3@@Z 10017294     U2Core:U2Core.dll
 0002:00000298       __imp_?isValid@U2DataPath@U2@@QBE_NXZ 10017298     U2Core:U2Core.dll
 0002:0000029c       __imp_?getDataPathRegistry@AppContext@U2@@SAPAVU2DataPathRegistry@2@XZ 1001729c     U2Core:U2Core.dll
 0002:000002a0       __imp_?qt_metacast@TaskSignalMapper@U2@@UAEPAXPBD@Z 100172a0     U2Core:U2Core.dll
 0002:000002a4       __imp_?qt_metacast@FailTask@U2@@UAEPAXPBD@Z 100172a4     U2Core:U2Core.dll
 0002:000002a8       __imp_?qt_metacall@TaskSignalMapper@U2@@UAEHW4Call@QMetaObject@@HPAPAX@Z 100172a8     U2Core:U2Core.dll
 0002:000002ac       __imp_?qt_metacall@FailTask@U2@@UAEHW4Call@QMetaObject@@HPAPAX@Z 100172ac     U2Core:U2Core.dll
 0002:000002b0       __imp_?metaObject@TaskSignalMapper@U2@@UBEPBUQMetaObject@@XZ 100172b0     U2Core:U2Core.dll
 0002:000002b4       __imp_?metaObject@FailTask@U2@@UBEPBUQMetaObject@@XZ 100172b4     U2Core:U2Core.dll
 0002:000002b8       __imp_?runScript@ScriptTask@U2@@SA?AVQScriptValue@@PAVQScriptEngine@@ABV?$QMap@VQString@@VQScriptValue@@@@ABVQString@@AAVTaskStateInfo@2@@Z 100172b8     U2Core:U2Core.dll
 0002:000002bc       __imp_?addListeners@ExternalToolSupportTask@U2@@QAEXABV?$QList@PAVExternalToolListener@U2@@@@@Z 100172bc     U2Core:U2Core.dll
 0002:000002c0       __imp_?createCurrentProcessTemporarySubDir@UserAppsSettings@U2@@QBE?AVQString@@AAVU2OpStatus@2@ABV3@@Z 100172c0     U2Core:U2Core.dll
 0002:000002c4       __imp_??1U2OpStatus2Log@U2@@UAE@XZ 100172c4     U2Core:U2Core.dll
 0002:000002c8       __imp_??0U2OpStatus2Log@U2@@QAE@W4LogLevel@1@@Z 100172c8     U2Core:U2Core.dll
 0002:000002cc       __imp_?getError@U2OpStatusImpl@U2@@UBE?AVQString@@XZ 100172cc     U2Core:U2Core.dll
 0002:000002d0       __imp_??0TaskSignalMapper@U2@@QAE@PAVTask@1@@Z 100172d0     U2Core:U2Core.dll
 0002:000002d4       __imp_?rollFileName@GUrlUtils@U2@@SA?AVQString@@ABV3@0ABV?$QSet@VQString@@@@@Z 100172d4     U2Core:U2Core.dll
 0002:000002d8       __imp_?getWorkingDir@FileAndDirectoryUtils@U2@@SA?AVQString@@ABV3@H00@Z 100172d8     U2Core:U2Core.dll
 0002:000002dc       __imp_??1FailTask@U2@@UAE@XZ 100172dc     U2Core:U2Core.dll
 0002:000002e0       __imp_??0FailTask@U2@@QAE@ABVQString@@@Z 100172e0     U2Core:U2Core.dll
 0002:000002e4       __imp_??1TaskStateInfo@U2@@UAE@XZ 100172e4     U2Core:U2Core.dll
 0002:000002e8       __imp_?setError@TaskStateInfo@U2@@UAEXABVQString@@@Z 100172e8     U2Core:U2Core.dll
 0002:000002ec       __imp_?getError@TaskStateInfo@U2@@UBE?AVQString@@XZ 100172ec     U2Core:U2Core.dll
 0002:000002f0       __imp_??0TaskStateInfo@U2@@QAE@XZ 100172f0     U2Core:U2Core.dll
 0002:000002f4       __imp_?error@Logger@U2@@QAEXABVQString@@@Z 100172f4     U2Core:U2Core.dll
 0002:000002f8       __imp_?getAppSettings@AppContext@U2@@SAPAVAppSettings@2@XZ 100172f8     U2Core:U2Core.dll
 0002:000002fc       __imp_??_7SimpleEventCounter@U2@@6B@ 100172fc     U2Core:U2Core.dll
 0002:00000300       __imp_?FASTQ@BaseDocumentFormats@U2@@2VQString@@B 10017300     U2Core:U2Core.dll
 0002:00000304       __imp_?FASTA@BaseDocumentFormats@U2@@2VQString@@B 10017304     U2Core:U2Core.dll
 0002:00000308       __imp_?setReportingSupported@Task@U2@@UAEX_N@Z 10017308     U2Core:U2Core.dll
 0002:0000030c       __imp_?setReportingEnabled@Task@U2@@UAEX_N@Z 1001730c     U2Core:U2Core.dll
 0002:00000310       __imp_?setNotificationReport@Task@U2@@UAEX_N@Z 10017310     U2Core:U2Core.dll
 0002:00000314       __imp_?setNoAutoDelete@Task@U2@@UAEX_N@Z 10017314     U2Core:U2Core.dll
 0002:00000318       __imp_?setListenerForTask@ExternalToolSupportTask@U2@@MAEXPAVExternalToolRunTask@2@H@Z 10017318     U2Core:U2Core.dll
 0002:0000031c       __imp_?setListenerForHelper@ExternalToolSupportTask@U2@@MAEXPAVExternalToolRunTaskHelper@2@H@Z 1001731c     U2Core:U2Core.dll
 0002:00000320       __imp_?setLastError@ExternalToolLogParser@U2@@MAEXABVQString@@@Z 10017320     U2Core:U2Core.dll
 0002:00000324       __imp_?setCollectChildrensWarningsFlag@Task@U2@@UAEX_N@Z 10017324     U2Core:U2Core.dll
 0002:00000328       __imp_?run@Task@U2@@UAEXXZ 10017328     U2Core:U2Core.dll
 0002:0000032c       __imp_?run@ExternalToolRunTask@U2@@UAEXXZ 1001732c     U2Core:U2Core.dll
 0002:00000330       __imp_?report@Task@U2@@UAE?AW4ReportResult@12@XZ 10017330     U2Core:U2Core.dll
 0002:00000334       __imp_?qt_metacast@Task@U2@@UAEPAXPBD@Z 10017334     U2Core:U2Core.dll
 0002:00000338       __imp_?qt_metacast@ExternalToolRunTask@U2@@UAEPAXPBD@Z 10017338     U2Core:U2Core.dll
 0002:0000033c       __imp_?qt_metacast@ExternalToolLogParser@U2@@UAEPAXPBD@Z 1001733c     U2Core:U2Core.dll
 0002:00000340       __imp_?qt_metacall@Task@U2@@UAEHW4Call@QMetaObject@@HPAPAX@Z 10017340     U2Core:U2Core.dll
 0002:00000344       __imp_?qt_metacall@ExternalToolRunTask@U2@@UAEHW4Call@QMetaObject@@HPAPAX@Z 10017344     U2Core:U2Core.dll
 0002:00000348       __imp_?qt_metacall@ExternalToolLogParser@U2@@UAEHW4Call@QMetaObject@@HPAPAX@Z 10017348     U2Core:U2Core.dll
 0002:0000034c       __imp_?propagateSubtaskError@Task@U2@@UAE_NXZ 1001734c     U2Core:U2Core.dll
 0002:00000350       __imp_?processLine@ExternalToolLogParser@U2@@MAEXABVQString@@@Z 10017350     U2Core:U2Core.dll
 0002:00000354       __imp_?processErrLine@ExternalToolLogParser@U2@@MAEXABVQString@@@Z 10017354     U2Core:U2Core.dll
 0002:00000358       __imp_?prepare@Task@U2@@UAEXXZ 10017358     U2Core:U2Core.dll
 0002:0000035c       __imp_?parseOutput@ExternalToolLogParser@U2@@UAEXABVQString@@@Z 1001735c     U2Core:U2Core.dll
 0002:00000360       __imp_?parseErrOutput@ExternalToolLogParser@U2@@UAEXABVQString@@@Z 10017360     U2Core:U2Core.dll
 0002:00000364       __imp_?onSubTaskFinished@Task@U2@@MAE?AV?$QList@PAVTask@U2@@@@PAV12@@Z 10017364     U2Core:U2Core.dll
 0002:00000368       __imp_?metaObject@Task@U2@@UBEPBUQMetaObject@@XZ 10017368     U2Core:U2Core.dll
 0002:0000036c       __imp_?metaObject@ExternalToolRunTask@U2@@UBEPBUQMetaObject@@XZ 1001736c     U2Core:U2Core.dll
 0002:00000370       __imp_?metaObject@ExternalToolLogParser@U2@@UBEPBUQMetaObject@@XZ 10017370     U2Core:U2Core.dll
 0002:00000374       __imp_?isTopLevelTask@Task@U2@@UBE_NXZ 10017374     U2Core:U2Core.dll
 0002:00000378       __imp_?isReportingSupported@Task@U2@@UBE_NXZ 10017378     U2Core:U2Core.dll
 0002:0000037c       __imp_?isReportingEnabled@Task@U2@@UBE_NXZ 1001737c     U2Core:U2Core.dll
 0002:00000380       __imp_?isNotificationReport@Task@U2@@UBE_NXZ 10017380     U2Core:U2Core.dll
 0002:00000384       __imp_?hasWarning@Task@U2@@UBE_NXZ 10017384     U2Core:U2Core.dll
 0002:00000388       __imp_?hasSubtasksWithErrors@Task@U2@@UBE_NXZ 10017388     U2Core:U2Core.dll
 0002:0000038c       __imp_??1Logger@U2@@UAE@XZ 1001738c     U2Core:U2Core.dll
 0002:00000390       __imp_?getWarnings@Task@U2@@UBE?AVQStringList@@XZ 10017390     U2Core:U2Core.dll
 0002:00000394       __imp_?getTopLevelParentTask@Task@U2@@UAEPAV12@XZ 10017394     U2Core:U2Core.dll
 0002:00000398       __imp_?getTaskId@Task@U2@@UBE_JXZ 10017398     U2Core:U2Core.dll
 0002:0000039c       __imp_?getSubtaskWithErrors@Task@U2@@UBEPAV12@XZ 1001739c     U2Core:U2Core.dll
 0002:000003a0       __imp_??0Logger@U2@@QAE@ABVQString@@@Z 100173a0     U2Core:U2Core.dll
 0002:000003a4       __imp_?getProgress@ExternalToolLogParser@U2@@UAEHXZ 100173a4     U2Core:U2Core.dll
 0002:000003a8       __imp_?getParentTask@Task@U2@@UBEPAV12@XZ 100173a8     U2Core:U2Core.dll
 0002:000003ac       __imp_?getNumParallelSubtasks@Task@U2@@UBEHXZ 100173ac     U2Core:U2Core.dll
 0002:000003b0       __imp_?generateReport@Task@U2@@UBE?AVQString@@XZ 100173b0     U2Core:U2Core.dll
 0002:000003b4       __imp_?cleanup@Task@U2@@UAEXXZ 100173b4     U2Core:U2Core.dll
 0002:000003b8       __imp_??1ExternalToolLogParser@U2@@UAE@XZ 100173b8     U2Core:U2Core.dll
 0002:000003bc       __imp_??0ExternalToolLogParser@U2@@QAE@XZ 100173bc     U2Core:U2Core.dll
 0002:000003c0       __imp_??1ExternalToolSupportTask@U2@@UAE@XZ 100173c0     U2Core:U2Core.dll
 0002:000003c4       __imp_??0ExternalToolSupportTask@U2@@QAE@ABVQString@@V?$QFlags@W4TaskFlag@U2@@@@@Z 100173c4     U2Core:U2Core.dll
 0002:000003c8       __imp_??1ExternalToolRunTask@U2@@UAE@XZ 100173c8     U2Core:U2Core.dll
 0002:000003cc       __imp_??0ExternalToolRunTask@U2@@QAE@ABVQString@@ABVQStringList@@PAVExternalToolLogParser@1@010_N@Z 100173cc     U2Core:U2Core.dll
 0002:000003d0       __imp_?setError@Task@U2@@QAEXABVQString@@@Z 100173d0     U2Core:U2Core.dll
 0002:000003d4       __imp_?hasError@Task@U2@@QBE_NXZ 100173d4     U2Core:U2Core.dll
 0002:000003d8       __imp_?addSubTask@Task@U2@@QAEXPAV12@@Z 100173d8     U2Core:U2Core.dll
 0002:000003dc       __imp_?detectFormat@DocumentUtils@U2@@SA?AW4Detection@12@ABVGUrl@2@AAVQString@@@Z 100173dc     U2Core:U2Core.dll
 0002:000003e0       __imp_??1GUrl@U2@@QAE@XZ   100173e0     U2Core:U2Core.dll
 0002:000003e4       __imp_??0GUrl@U2@@QAE@ABVQString@@@Z 100173e4     U2Core:U2Core.dll
 0002:000003e8       __imp_??1SimpleEventCounter@U2@@UAE@XZ 100173e8     U2Core:U2Core.dll
 0002:000003ec       __imp_??0GReportableCounter@U2@@QAE@ABVQString@@0N@Z 100173ec     U2Core:U2Core.dll
 0002:000003f0       __imp_??1GCounter@U2@@UAE@XZ 100173f0     U2Core:U2Core.dll
 0002:000003f4       __imp_??1Plugin@U2@@UAE@XZ 100173f4     U2Core:U2Core.dll
 0002:000003f8       __imp_??0Plugin@U2@@QAE@ABVQString@@0_NW4PluginState@1@@Z 100173f8     U2Core:U2Core.dll
 0002:000003fc       __imp_?unregisterEntry@ExternalToolRegistry@U2@@QAEXABVQString@@@Z 100173fc     U2Core:U2Core.dll
 0002:00000400       __imp_?registerEntry@ExternalToolRegistry@U2@@QAE_NPAVExternalTool@2@@Z 10017400     U2Core:U2Core.dll
 0002:00000404       __imp_?getExternalToolRegistry@AppContext@U2@@SAPAVExternalToolRegistry@2@XZ 10017404     U2Core:U2Core.dll
 0002:00000408       __imp_?getToolRunnerAdditionalOptions@ExternalTool@U2@@UAE?BVQStringList@@XZ 10017408     U2Core:U2Core.dll
 0002:0000040c       __imp_?getAdditionalPaths@ExternalTool@U2@@UBE?AVQStringList@@XZ 1001740c     U2Core:U2Core.dll
 0002:00000410       __imp_?getAdditionalParameters@ExternalTool@U2@@UAEXABVQString@@@Z 10017410     U2Core:U2Core.dll
 0002:00000414       __imp_??1ExternalTool@U2@@UAE@XZ 10017414     U2Core:U2Core.dll
 0002:00000418       __imp_??0ExternalTool@U2@@QAE@VQString@@0@Z 10017418     U2Core:U2Core.dll
 0002:0000041c       \177U2Core_NULL_THUNK_DATA 1001741c     U2Core:U2Core.dll
 0002:00000420       __imp_??0SpinBoxDelegate@U2@@QAE@ABV?$QMap@VQString@@VQVariant@@@@PAVQObject@@@Z 10017420     U2Designer:U2Designer.dll
 0002:00000424       __imp_??1SpinBoxDelegate@U2@@UAE@XZ 10017424     U2Designer:U2Designer.dll
 0002:00000428       __imp_??0ComboBoxDelegate@U2@@QAE@ABV?$QMap@VQString@@VQVariant@@@@PAVQObject@@@Z 10017428     U2Designer:U2Designer.dll
 0002:0000042c       __imp_??1ComboBoxDelegate@U2@@UAE@XZ 1001742c     U2Designer:U2Designer.dll
 0002:00000430       __imp_?addDelegate@DelegateEditor@U2@@UAEXPAVPropertyDelegate@2@ABVQString@@@Z 10017430     U2Designer:U2Designer.dll
 0002:00000434       __imp_?clone@ComboBoxDelegate@U2@@UAEPAVPropertyDelegate@2@XZ 10017434     U2Designer:U2Designer.dll
 0002:00000438       __imp_?clone@DelegateEditor@U2@@UAEPAVConfigurationEditor@2@XZ 10017438     U2Designer:U2Designer.dll
 0002:0000043c       __imp_?clone@SpinBoxDelegate@U2@@UAEPAVPropertyDelegate@2@XZ 1001743c     U2Designer:U2Designer.dll
 0002:00000440       __imp_?clone@URLDelegate@U2@@UAEPAVPropertyDelegate@2@XZ 10017440     U2Designer:U2Designer.dll
 0002:00000444       __imp_?commit@DelegateEditor@U2@@UAEXXZ 10017444     U2Designer:U2Designer.dll
 0002:00000448       __imp_?createEditor@ComboBoxDelegate@U2@@UBEPAVQWidget@@PAV3@ABVQStyleOptionViewItem@@ABVQModelIndex@@@Z 10017448     U2Designer:U2Designer.dll
 0002:0000044c       __imp_?createEditor@SpinBoxDelegate@U2@@UBEPAVQWidget@@PAV3@ABVQStyleOptionViewItem@@ABVQModelIndex@@@Z 1001744c     U2Designer:U2Designer.dll
 0002:00000450       __imp_?createEditor@URLDelegate@U2@@UBEPAVQWidget@@PAV3@ABVQStyleOptionViewItem@@ABVQModelIndex@@@Z 10017450     U2Designer:U2Designer.dll
 0002:00000454       __imp_?createWizardWidget@ComboBoxDelegate@U2@@UBEPAVPropertyWidget@2@AAVU2OpStatus@2@PAVQWidget@@@Z 10017454     U2Designer:U2Designer.dll
 0002:00000458       __imp_?createWizardWidget@SpinBoxDelegate@U2@@UBEPAVPropertyWidget@2@AAVU2OpStatus@2@PAVQWidget@@@Z 10017458     U2Designer:U2Designer.dll
 0002:0000045c       __imp_?createWizardWidget@URLDelegate@U2@@UBEPAVPropertyWidget@2@AAVU2OpStatus@2@PAVQWidget@@@Z 1001745c     U2Designer:U2Designer.dll
 0002:00000460       __imp_?getDelegate@DelegateEditor@U2@@UAEPAVPropertyDelegate@2@ABVQString@@@Z 10017460     U2Designer:U2Designer.dll
 0002:00000464       __imp_?getDisplayValue@ComboBoxDelegate@U2@@UBE?AVQVariant@@ABV3@@Z 10017464     U2Designer:U2Designer.dll
 0002:00000468       __imp_?getDisplayValue@SpinBoxDelegate@U2@@UBE?AVQVariant@@ABV3@@Z 10017468     U2Designer:U2Designer.dll
 0002:0000046c       __imp_?getDisplayValue@URLDelegate@U2@@UBE?AVQVariant@@ABV3@@Z 1001746c     U2Designer:U2Designer.dll
 0002:00000470       __imp_?getItems@ComboBoxDelegate@U2@@UBEXAAV?$QMap@VQString@@VQVariant@@@@@Z 10017470     U2Designer:U2Designer.dll
 0002:00000474       __imp_?getItems@SpinBoxDelegate@U2@@UBEXAAV?$QMap@VQString@@VQVariant@@@@@Z 10017474     U2Designer:U2Designer.dll
 0002:00000478       __imp_?metaObject@ComboBoxDelegate@U2@@UBEPBUQMetaObject@@XZ 10017478     U2Designer:U2Designer.dll
 0002:0000047c       __imp_?metaObject@DelegateEditor@U2@@UBEPBUQMetaObject@@XZ 1001747c     U2Designer:U2Designer.dll
 0002:00000480       __imp_?metaObject@SpinBoxDelegate@U2@@UBEPBUQMetaObject@@XZ 10017480     U2Designer:U2Designer.dll
 0002:00000484       __imp_?metaObject@URLDelegate@U2@@UBEPBUQMetaObject@@XZ 10017484     U2Designer:U2Designer.dll
 0002:00000488       __imp_?qt_metacall@ComboBoxDelegate@U2@@UAEHW4Call@QMetaObject@@HPAPAX@Z 10017488     U2Designer:U2Designer.dll
 0002:0000048c       __imp_?qt_metacall@DelegateEditor@U2@@UAEHW4Call@QMetaObject@@HPAPAX@Z 1001748c     U2Designer:U2Designer.dll
 0002:00000490       __imp_?qt_metacall@SpinBoxDelegate@U2@@UAEHW4Call@QMetaObject@@HPAPAX@Z 10017490     U2Designer:U2Designer.dll
 0002:00000494       __imp_?qt_metacall@URLDelegate@U2@@UAEHW4Call@QMetaObject@@HPAPAX@Z 10017494     U2Designer:U2Designer.dll
 0002:00000498       __imp_?qt_metacast@ComboBoxDelegate@U2@@UAEPAXPBD@Z 10017498     U2Designer:U2Designer.dll
 0002:0000049c       __imp_?qt_metacast@DelegateEditor@U2@@UAEPAXPBD@Z 1001749c     U2Designer:U2Designer.dll
 0002:000004a0       __imp_?qt_metacast@SpinBoxDelegate@U2@@UAEPAXPBD@Z 100174a0     U2Designer:U2Designer.dll
 0002:000004a4       __imp_?qt_metacast@URLDelegate@U2@@UAEPAXPBD@Z 100174a4     U2Designer:U2Designer.dll
 0002:000004a8       __imp_?removeDelegate@DelegateEditor@U2@@UAEPAVPropertyDelegate@2@ABVQString@@@Z 100174a8     U2Designer:U2Designer.dll
 0002:000004ac       __imp_?setEditorData@ComboBoxDelegate@U2@@UBEXPAVQWidget@@ABVQModelIndex@@@Z 100174ac     U2Designer:U2Designer.dll
 0002:000004b0       __imp_?setEditorData@SpinBoxDelegate@U2@@UBEXPAVQWidget@@ABVQModelIndex@@@Z 100174b0     U2Designer:U2Designer.dll
 0002:000004b4       __imp_?setEditorData@URLDelegate@U2@@UBEXPAVQWidget@@ABVQModelIndex@@@Z 100174b4     U2Designer:U2Designer.dll
 0002:000004b8       __imp_?setModelData@ComboBoxDelegate@U2@@UBEXPAVQWidget@@PAVQAbstractItemModel@@ABVQModelIndex@@@Z 100174b8     U2Designer:U2Designer.dll
 0002:000004bc       __imp_?setModelData@SpinBoxDelegate@U2@@UBEXPAVQWidget@@PAVQAbstractItemModel@@ABVQModelIndex@@@Z 100174bc     U2Designer:U2Designer.dll
 0002:000004c0       __imp_?setModelData@URLDelegate@U2@@UBEXPAVQWidget@@PAVQAbstractItemModel@@ABVQModelIndex@@@Z 100174c0     U2Designer:U2Designer.dll
 0002:000004c4       __imp_?type@URLDelegate@U2@@UBE?AW4Type@PropertyDelegate@2@XZ 100174c4     U2Designer:U2Designer.dll
 0002:000004c8       __imp_?updateDelegate@DelegateEditor@U2@@UAEXABVQString@@@Z 100174c8     U2Designer:U2Designer.dll
 0002:000004cc       __imp_?updateDelegates@DelegateEditor@U2@@UAEXXZ 100174cc     U2Designer:U2Designer.dll
 0002:000004d0       __imp_??1URLDelegate@U2@@UAE@XZ 100174d0     U2Designer:U2Designer.dll
 0002:000004d4       __imp_??0URLDelegate@U2@@QAE@ABVDelegateTags@1@ABVQString@@_N22PAVQObject@@2@Z 100174d4     U2Designer:U2Designer.dll
 0002:000004d8       __imp_??1DelegateEditor@U2@@UAE@XZ 100174d8     U2Designer:U2Designer.dll
 0002:000004dc       __imp_??0DelegateEditor@U2@@QAE@ABV?$QMap@VQString@@PAVPropertyDelegate@U2@@@@@Z 100174dc     U2Designer:U2Designer.dll
 0002:000004e0       \177U2Designer_NULL_THUNK_DATA 100174e0     U2Designer:U2Designer.dll
 0002:000004e4       __imp_?getSequencesNumber@CalculateSequencesNumberTask@U2@@QBEHXZ 100174e4     U2Formats:U2Formats.dll
 0002:000004e8       __imp_??1CalculateSequencesNumberTask@U2@@UAE@XZ 100174e8     U2Formats:U2Formats.dll
 0002:000004ec       __imp_?run@CalculateSequencesNumberTask@U2@@EAEXXZ 100174ec     U2Formats:U2Formats.dll
 0002:000004f0       __imp_??0CalculateSequencesNumberTask@U2@@QAE@ABVQString@@@Z 100174f0     U2Formats:U2Formats.dll
 0002:000004f4       \177U2Formats_NULL_THUNK_DATA 100174f4     U2Formats:U2Formats.dll
 0002:000004f8       __imp_?prepareDocumentsFileFilter@DialogUtils@U2@@SA?AVQString@@ABV3@_NABVQStringList@@@Z 100174f8     U2Gui:U2Gui.dll
 0002:000004fc       \177U2Gui_NULL_THUNK_DATA  100174fc     U2Gui:U2Gui.dll
 0002:00000500       __imp_?FORMAT@DelegateTags@U2@@2VQString@@B 10017500     U2Lang:U2Lang.dll
 0002:00000504       __imp_?FILTER@DelegateTags@U2@@2VQString@@B 10017504     U2Lang:U2Lang.dll
 0002:00000508       __imp_?PLACEHOLDER_TEXT@DelegateTags@U2@@2VQString@@B 10017508     U2Lang:U2Lang.dll
 0002:0000050c       __imp_??_7ConfigurationValidator@U2@@6B@ 1001750c     U2Lang:U2Lang.dll
 0002:00000510       __imp_?valueChangingRelation@VisibilityRelation@U2@@UBE_NXZ 10017510     U2Lang:U2Lang.dll
 0002:00000514       __imp_?validate@PortValidator@Workflow@U2@@UBE_NPBVConfiguration@3@AAV?$QList@VWorkflowNotification@U2@@@@@Z 10017514     U2Lang:U2Lang.dll
 0002:00000518       __imp_?validate@PairedReadsPortValidator@Workflow@U2@@UBE_NPBVIntegralBusPort@23@AAV?$QList@VWorkflowNotification@U2@@@@@Z 10017518     U2Lang:U2Lang.dll
 0002:0000051c       __imp_?validate@Attribute@U2@@UAE_NAAV?$QList@VWorkflowNotification@U2@@@@@Z 1001751c     U2Lang:U2Lang.dll
 0002:00000520       __imp_?validate@ActorValidator@Workflow@U2@@UBE_NPBVConfiguration@3@AAV?$QList@VWorkflowNotification@U2@@@@@Z 10017520     U2Lang:U2Lang.dll
 0002:00000524       __imp_?updateDelegateTags@AttributeRelation@U2@@UBEXABVQVariant@@PAVDelegateTags@2@@Z 10017524     U2Lang:U2Lang.dll
 0002:00000528       __imp_?updateActorIds@Attribute@U2@@UAEXABV?$QMap@VQString@@V1@@@@Z 10017528     U2Lang:U2Lang.dll
 0002:0000052c       __imp_?update@PropertyDelegate@U2@@UAEXXZ 1001752c     U2Lang:U2Lang.dll
 0002:00000530       __imp_?unregisterEntry@?$IdRegistry@VDomainFactory@Workflow@U2@@@U2@@UAEPAVDomainFactory@Workflow@2@ABVQString@@@Z 10017530     U2Lang:U2Lang.dll
 0002:00000534       __imp_?type@PropertyDelegate@U2@@UBE?AW4Type@12@XZ 10017534     U2Lang:U2Lang.dll
 0002:00000538       __imp_?setVisibleSlot@PortDescriptor@Workflow@U2@@UAEXABVQString@@_N@Z 10017538     U2Lang:U2Lang.dll
 0002:0000053c       __imp_?setAttributeValue@Attribute@U2@@UAEXABVQVariant@@@Z 1001753c     U2Lang:U2Lang.dll
 0002:00000540       __imp_?registerEntry@?$IdRegistry@VDomainFactory@Workflow@U2@@@U2@@UAE_NPAVDomainFactory@Workflow@2@@Z 10017540     U2Lang:U2Lang.dll
 0002:00000544       __imp_?kind@MapDataType@U2@@UBE?AW4Kind@DataType@2@XZ 10017544     U2Lang:U2Lang.dll
 0002:00000548       __imp_?isSlotEnabled@SlotRelationDescriptor@U2@@UBE_NABVQVariant@@@Z 10017548     U2Lang:U2Lang.dll
 0002:0000054c       __imp_?isEmpty@Attribute@U2@@UBE_NXZ 1001754c     U2Lang:U2Lang.dll
 0002:00000550       __imp_?isDefaultValue@Attribute@U2@@UBE_NXZ 10017550     U2Lang:U2Lang.dll
 0002:00000554       __imp_?isAcceptableDrop@ActorPrototype@Workflow@U2@@UBE_NPBVQMimeData@@PAV?$QMap@VQString@@VQVariant@@@@@Z 10017554     U2Lang:U2Lang.dll
 0002:00000558       __imp_?getWidget@ConfigurationEditor@U2@@UAEPAVQWidget@@XZ 10017558     U2Lang:U2Lang.dll
 0002:0000055c       __imp_?getType@PortDescriptor@Workflow@U2@@UBE?AV?$QExplicitlySharedDataPointer@VDataType@U2@@@@XZ 1001755c     U2Lang:U2Lang.dll
 0002:00000560       __imp_?getItems@PropertyDelegate@U2@@UBEXAAV?$QMap@VQString@@VQVariant@@@@@Z 10017560     U2Lang:U2Lang.dll
 0002:00000564       __imp_?getGroup@Attribute@U2@@UAE?AW4AttributeGroup@2@XZ 10017564     U2Lang:U2Lang.dll
 0002:00000568       __imp_?getDefaultPureValue@Attribute@U2@@UBEABVQVariant@@XZ 10017568     U2Lang:U2Lang.dll
 0002:0000056c       __imp_?getDatatypesMap@MapDataType@U2@@UBE?AV?$QMap@VDescriptor@U2@@V?$QExplicitlySharedDataPointer@VDataType@U2@@@@@@XZ 1001756c     U2Lang:U2Lang.dll
 0002:00000570       __imp_?getDatatypeByDescriptor@MapDataType@U2@@UBE?AV?$QExplicitlySharedDataPointer@VDataType@U2@@@@ABVDescriptor@2@@Z 10017570     U2Lang:U2Lang.dll
 0002:00000574       __imp_?getById@?$IdRegistry@VDomainFactory@Workflow@U2@@@U2@@UAEPAVDomainFactory@Workflow@2@ABVQString@@@Z 10017574     U2Lang:U2Lang.dll
 0002:00000578       __imp_?getAttributePureValue@Attribute@U2@@UBEABVQVariant@@XZ 10017578     U2Lang:U2Lang.dll
 0002:0000057c       __imp_?getAllIds@?$IdRegistry@VDomainFactory@Workflow@U2@@@U2@@UBE?AV?$QList@VQString@@@@XZ 1001757c     U2Lang:U2Lang.dll
 0002:00000580       __imp_?getAllEntries@?$IdRegistry@VDomainFactory@Workflow@U2@@@U2@@UBE?AV?$QList@PAVDomainFactory@Workflow@U2@@@@XZ 10017580     U2Lang:U2Lang.dll
 0002:00000584       __imp_?getAllDescriptors@MapDataType@U2@@UBE?AV?$QList@VDescriptor@U2@@@@XZ 10017584     U2Lang:U2Lang.dll
 0002:00000588       __imp_?getAffectResult@VisibilityRelation@U2@@UBE?AVQVariant@@ABV3@0PAVDelegateTags@2@1@Z 10017588     U2Lang:U2Lang.dll
 0002:0000058c       __imp_?destroy@DomainFactory@Workflow@U2@@UAEXPAVScheduler@23@PAVSchema@23@@Z 1001758c     U2Lang:U2Lang.dll
 0002:00000590       __imp_?createScheduler@DomainFactory@Workflow@U2@@UAEPAVScheduler@23@PAVSchema@23@@Z 10017590     U2Lang:U2Lang.dll
 0002:00000594       __imp_?createPort@IntegralBusActorPrototype@Workflow@U2@@UAEPAVPort@23@ABVPortDescriptor@23@PAVActor@23@@Z 10017594     U2Lang:U2Lang.dll
 0002:00000598       __imp_?createInstance@ActorPrototype@Workflow@U2@@UAEPAVActor@23@ABVQString@@PAVAttributeScript@3@ABV?$QMap@VQString@@VQVariant@@@@@Z 10017598     U2Lang:U2Lang.dll
 0002:0000059c       __imp_?staticMetaObject@PrompterBaseImpl@U2@@2UQMetaObject@@B 1001759c     U2Lang:U2Lang.dll
 0002:000005a0       __imp_?clone@VisibilityRelation@U2@@UBEPAV12@XZ 100175a0     U2Lang:U2Lang.dll
 0002:000005a4       __imp_?clone@SlotRelationDescriptor@U2@@UBEPAV12@XZ 100175a4     U2Lang:U2Lang.dll
 0002:000005a8       __imp_?clone@Attribute@U2@@UAEPAV12@XZ 100175a8     U2Lang:U2Lang.dll
 0002:000005ac       __imp_?getInstance@WorkflowEnv@Workflow@U2@@KAPAV123@XZ 100175ac     U2Lang:U2Lang.dll
 0002:000005b0       __imp_??1PairedReadsPortValidator@Workflow@U2@@UAE@XZ 100175b0     U2Lang:U2Lang.dll
 0002:000005b4       __imp_??0PairedReadsPortValidator@Workflow@U2@@QAE@ABVQString@@0@Z 100175b4     U2Lang:U2Lang.dll
 0002:000005b8       __imp_?NUM_TYPE@BaseTypes@U2@@SA?AV?$QExplicitlySharedDataPointer@VDataType@U2@@@@XZ 100175b8     U2Lang:U2Lang.dll
 0002:000005bc       __imp_?STRING_TYPE@BaseTypes@U2@@SA?AV?$QExplicitlySharedDataPointer@VDataType@U2@@@@XZ 100175bc     U2Lang:U2Lang.dll
 0002:000005c0       __imp_?unregisterProto@ActorPrototypeRegistry@Workflow@U2@@QAEPAVActorPrototype@23@ABVQString@@@Z 100175c0     U2Lang:U2Lang.dll
 0002:000005c4       __imp_?registerProto@ActorPrototypeRegistry@Workflow@U2@@QAEXABVDescriptor@3@PAVActorPrototype@23@@Z 100175c4     U2Lang:U2Lang.dll
 0002:000005c8       __imp_??1DomainFactory@Workflow@U2@@UAE@XZ 100175c8     U2Lang:U2Lang.dll
 0002:000005cc       __imp_??0DomainFactory@Workflow@U2@@QAE@ABVQString@@@Z 100175cc     U2Lang:U2Lang.dll
 0002:000005d0       __imp_?addExternalTool@ActorPrototype@Workflow@U2@@QAEXABVQString@@0@Z 100175d0     U2Lang:U2Lang.dll
 0002:000005d4       __imp_?setPortValidator@ActorPrototype@Workflow@U2@@QAEXABVQString@@PAVConfigurationValidator@3@@Z 100175d4     U2Lang:U2Lang.dll
 0002:000005d8       __imp_?setPrompter@ActorPrototype@Workflow@U2@@QAEXPAVPrompter@23@@Z 100175d8     U2Lang:U2Lang.dll
 0002:000005dc       __imp_?setValidator@ActorPrototype@Workflow@U2@@QAEXPAVConfigurationValidator@3@@Z 100175dc     U2Lang:U2Lang.dll
 0002:000005e0       __imp_?setEditor@ActorPrototype@Workflow@U2@@QAEXPAVConfigurationEditor@3@@Z 100175e0     U2Lang:U2Lang.dll
 0002:000005e4       __imp_??1ActorPrototype@Workflow@U2@@UAE@XZ 100175e4     U2Lang:U2Lang.dll
 0002:000005e8       __imp_??0ActorPrototype@Workflow@U2@@QAE@ABVDescriptor@2@ABV?$QList@PAVPortDescriptor@Workflow@U2@@@@ABV?$QList@PAVAttribute@U2@@@@@Z 100175e8     U2Lang:U2Lang.dll
 0002:000005ec       __imp_??1PortDescriptor@Workflow@U2@@UAE@XZ 100175ec     U2Lang:U2Lang.dll
 0002:000005f0       __imp_??0PortDescriptor@Workflow@U2@@QAE@ABVDescriptor@2@V?$QExplicitlySharedDataPointer@VDataType@U2@@@@_N2I@Z 100175f0     U2Lang:U2Lang.dll
 0002:000005f4       __imp_??1DelegateTags@U2@@UAE@XZ 100175f4     U2Lang:U2Lang.dll
 0002:000005f8       __imp_?set@DelegateTags@U2@@QAEXABVQString@@ABVQVariant@@@Z 100175f8     U2Lang:U2Lang.dll
 0002:000005fc       __imp_??_7ActorValidator@Workflow@U2@@6B@ 100175fc     U2Lang:U2Lang.dll
 0002:00000600       __imp_?addSlotRelation@Attribute@U2@@QAEXPAVSlotRelationDescriptor@2@@Z 10017600     U2Lang:U2Lang.dll
 0002:00000604       __imp_?addRelation@Attribute@U2@@QAEXPBVAttributeRelation@2@@Z 10017604     U2Lang:U2Lang.dll
 0002:00000608       __imp_??1Attribute@U2@@UAE@XZ 10017608     U2Lang:U2Lang.dll
 0002:0000060c       __imp_??0Attribute@U2@@QAE@ABVDescriptor@1@V?$QExplicitlySharedDataPointer@VDataType@U2@@@@_NABVQVariant@@@Z 1001760c     U2Lang:U2Lang.dll
 0002:00000610       __imp_??0Attribute@U2@@QAE@ABVDescriptor@1@V?$QExplicitlySharedDataPointer@VDataType@U2@@@@V?$QFlags@W4Flag@Attribute@U2@@@@ABVQVariant@@@Z 10017610     U2Lang:U2Lang.dll
 0002:00000614       __imp_??1SlotRelationDescriptor@U2@@UAE@XZ 10017614     U2Lang:U2Lang.dll
 0002:00000618       __imp_??0SlotRelationDescriptor@U2@@QAE@ABVQString@@0ABV?$QList@VQVariant@@@@@Z 10017618     U2Lang:U2Lang.dll
 0002:0000061c       __imp_??1MapDataType@U2@@UAE@XZ 1001761c     U2Lang:U2Lang.dll
 0002:00000620       __imp_??0MapDataType@U2@@QAE@ABVDescriptor@1@ABV?$QMap@VDescriptor@U2@@V?$QExplicitlySharedDataPointer@VDataType@U2@@@@@@@Z 10017620     U2Lang:U2Lang.dll
 0002:00000624       __imp_??1VisibilityRelation@U2@@UAE@XZ 10017624     U2Lang:U2Lang.dll
 0002:00000628       __imp_??0VisibilityRelation@U2@@QAE@ABVQString@@ABV?$QList@VQVariant@@@@_N@Z 10017628     U2Lang:U2Lang.dll
 0002:0000062c       __imp_??0Descriptor@U2@@QAE@ABVQString@@@Z 1001762c     U2Lang:U2Lang.dll
 0002:00000630       __imp_??0Descriptor@U2@@QAE@ABVQString@@00@Z 10017630     U2Lang:U2Lang.dll
 0002:00000634       __imp_?setDone@BaseWorker@LocalWorkflow@U2@@UAEXXZ 10017634     U2Lang:U2Lang.dll
 0002:00000638       __imp_?isReady@BaseWorker@LocalWorkflow@U2@@UBE_NXZ 10017638     U2Lang:U2Lang.dll
 0002:0000063c       __imp_?isDone@BaseWorker@LocalWorkflow@U2@@UBE_NXZ 1001763c     U2Lang:U2Lang.dll
 0002:00000640       __imp_?getOutputFiles@BaseWorker@LocalWorkflow@U2@@UAE?AVQStringList@@XZ 10017640     U2Lang:U2Lang.dll
 0002:00000644       __imp_?getMessageAndSetupScriptValues@BaseWorker@LocalWorkflow@U2@@UAE?AVMessage@Workflow@3@PAVCommunicationChannel@53@@Z 10017644     U2Lang:U2Lang.dll
 0002:00000648       __imp_?getCommunication@BaseWorker@LocalWorkflow@U2@@UAEPAVCommunicationChannel@Workflow@3@ABVQString@@@Z 10017648     U2Lang:U2Lang.dll
 0002:0000064c       __imp_?getActorId@BaseWorker@LocalWorkflow@U2@@UBE?AVQString@@XZ 1001764c     U2Lang:U2Lang.dll
 0002:00000650       __imp_?canTaskBeCanceled@BaseWorker@LocalWorkflow@U2@@MBE_NPAVTask@3@@Z 10017650     U2Lang:U2Lang.dll
 0002:00000654       __imp_?addCommunication@BaseWorker@LocalWorkflow@U2@@UAE_NABVQString@@PAVCommunicationChannel@Workflow@3@@Z 10017654     U2Lang:U2Lang.dll
 0002:00000658       __imp_?createLogListeners@BaseWorker@LocalWorkflow@U2@@QAE?AV?$QList@PAVExternalToolListener@U2@@@@H@Z 10017658     U2Lang:U2Lang.dll
 0002:0000065c       __imp_??1BaseWorker@LocalWorkflow@U2@@UAE@XZ 1001765c     U2Lang:U2Lang.dll
 0002:00000660       __imp_??0BaseWorker@LocalWorkflow@U2@@QAE@PAVActor@Workflow@2@_N@Z 10017660     U2Lang:U2Lang.dll
 0002:00000664       __imp_?getExternalToolPath@WorkflowUtils@U2@@SA?AVQString@@ABV3@@Z 10017664     U2Lang:U2Lang.dll
 0002:00000668       __imp_?isOutUrlAttribute@RFSUtils@U2@@SA_NPAVAttribute@2@PAVActor@Workflow@2@AA_N@Z 10017668     U2Lang:U2Lang.dll
 0002:0000066c       __imp_?addOutputFile@WorkflowMonitor@Workflow@U2@@QAEXABVQString@@0_N@Z 1001766c     U2Lang:U2Lang.dll
 0002:00000670       __imp_??1Message@Workflow@U2@@QAE@XZ 10017670     U2Lang:U2Lang.dll
 0002:00000674       __imp_?getMetadataId@Message@Workflow@U2@@QBEHXZ 10017674     U2Lang:U2Lang.dll
 0002:00000678       __imp_?getData@Message@Workflow@U2@@QBE?AVQVariant@@XZ 10017678     U2Lang:U2Lang.dll
 0002:0000067c       __imp_?getScriptVars@AttributeScript@U2@@QBEABV?$QMap@VDescriptor@U2@@VQVariant@@@@XZ 1001767c     U2Lang:U2Lang.dll
 0002:00000680       __imp_?getScriptText@AttributeScript@U2@@QBEABVQString@@XZ 10017680     U2Lang:U2Lang.dll
 0002:00000684       __imp_?isEmpty@AttributeScript@U2@@QBE_NXZ 10017684     U2Lang:U2Lang.dll
 0002:00000688       __imp_??1WorkflowScriptEngine@U2@@UAE@XZ 10017688     U2Lang:U2Lang.dll
 0002:0000068c       __imp_??0WorkflowScriptEngine@U2@@QAE@PAVWorkflowContext@Workflow@1@@Z 1001768c     U2Lang:U2Lang.dll
 0002:00000690       __imp_?initEngine@WorkflowScriptLibrary@U2@@SAXPAVWorkflowScriptEngine@2@@Z 10017690     U2Lang:U2Lang.dll
 0002:00000694       __imp_?getMetadataStorage@WorkflowContext@Workflow@U2@@QAEAAVMessageMetadataStorage@3@XZ 10017694     U2Lang:U2Lang.dll
 0002:00000698       __imp_?absolutePath@WorkflowContext@Workflow@U2@@QBE?AVQString@@ABV4@@Z 10017698     U2Lang:U2Lang.dll
 0002:0000069c       __imp_?workingDir@WorkflowContext@Workflow@U2@@QBE?AVQString@@XZ 1001769c     U2Lang:U2Lang.dll
 0002:000006a0       __imp_?getMonitor@WorkflowContext@Workflow@U2@@QAEPAVWorkflowMonitor@23@XZ 100176a0     U2Lang:U2Lang.dll
 0002:000006a4       __imp_?get@MessageMetadataStorage@U2@@QBE?AVMessageMetadata@2@H@Z 100176a4     U2Lang:U2Lang.dll
 0002:000006a8       __imp_??1MessageMetadata@U2@@QAE@XZ 100176a8     U2Lang:U2Lang.dll
 0002:000006ac       __imp_?getFileUrl@MessageMetadata@U2@@QBEABVQString@@XZ 100176ac     U2Lang:U2Lang.dll
 0002:000006b0       __imp_??0Descriptor@U2@@QAE@ABV01@@Z 100176b0     U2Lang:U2Lang.dll
 0002:000006b4       __imp_?getId@Descriptor@U2@@QBE?AVQString@@XZ 100176b4     U2Lang:U2Lang.dll
 0002:000006b8       __imp_??1Descriptor@U2@@UAE@XZ 100176b8     U2Lang:U2Lang.dll
 0002:000006bc       __imp_?U2_ERROR@WorkflowNotification@U2@@2VQString@@B 100176bc     U2Lang:U2Lang.dll
 0002:000006c0       __imp_?getId@Actor@Workflow@U2@@QBE?AVQString@@XZ 100176c0     U2Lang:U2Lang.dll
 0002:000006c4       __imp_??0WorkflowNotification@U2@@QAE@ABV01@@Z 100176c4     U2Lang:U2Lang.dll
 0002:000006c8       __imp_??1WorkflowNotification@U2@@QAE@XZ 100176c8     U2Lang:U2Lang.dll
 0002:000006cc       __imp_??0WorkflowNotification@U2@@QAE@ABVQString@@00@Z 100176cc     U2Lang:U2Lang.dll
 0002:000006d0       __imp_?update@PrompterBaseImpl@U2@@UAEXABV?$QMap@VQString@@VQVariant@@@@@Z 100176d0     U2Lang:U2Lang.dll
 0002:000006d4       __imp_?sl_actorModified@PrompterBaseImpl@U2@@MAEXXZ 100176d4     U2Lang:U2Lang.dll
 0002:000006d8       __imp_?qt_metacast@PrompterBaseImpl@U2@@UAEPAXPBD@Z 100176d8     U2Lang:U2Lang.dll
 0002:000006dc       __imp_?qt_metacall@PrompterBaseImpl@U2@@UAEHW4Call@QMetaObject@@HPAPAX@Z 100176dc     U2Lang:U2Lang.dll
 0002:000006e0       __imp_?metaObject@PrompterBaseImpl@U2@@UBEPBUQMetaObject@@XZ 100176e0     U2Lang:U2Lang.dll
 0002:000006e4       __imp_??1PrompterBaseImpl@U2@@UAE@XZ 100176e4     U2Lang:U2Lang.dll
 0002:000006e8       __imp_?getHyperlink@PrompterBaseImpl@U2@@SA?AVQString@@ABV3@0@Z 100176e8     U2Lang:U2Lang.dll
 0002:000006ec       __imp_?getProducersOrUnset@PrompterBaseImpl@U2@@QAE?AVQString@@ABV3@0@Z 100176ec     U2Lang:U2Lang.dll
 0002:000006f0       __imp_?getURL@PrompterBaseImpl@U2@@QAE?AVQString@@ABV3@PA_N00@Z 100176f0     U2Lang:U2Lang.dll
 0002:000006f4       __imp_??0PrompterBaseImpl@U2@@QAE@PAVActor@Workflow@1@@Z 100176f4     U2Lang:U2Lang.dll
 0002:000006f8       __imp_?getOutputPorts@Actor@Workflow@U2@@QBE?AV?$QList@PAVPort@Workflow@U2@@@@XZ 100176f8     U2Lang:U2Lang.dll
 0002:000006fc       __imp_?getInputPorts@Actor@Workflow@U2@@QBE?AV?$QList@PAVPort@Workflow@U2@@@@XZ 100176fc     U2Lang:U2Lang.dll
 0002:00000700       __imp_??0DelegateTags@U2@@QAE@PAVQObject@@@Z 10017700     U2Lang:U2Lang.dll
 0002:00000704       __imp_?ID@LocalDomainFactory@LocalWorkflow@U2@@2VQString@@B 10017704     U2Lang:U2Lang.dll
 0002:00000708       __imp_?qt_metacast@BaseWorker@LocalWorkflow@U2@@UAEPAXPBD@Z 10017708     U2Lang:U2Lang.dll
 0002:0000070c       __imp_?qt_metacall@BaseWorker@LocalWorkflow@U2@@UAEHW4Call@QMetaObject@@HPAPAX@Z 1001770c     U2Lang:U2Lang.dll
 0002:00000710       __imp_?staticMetaObject@BaseWorker@LocalWorkflow@U2@@2UQMetaObject@@B 10017710     U2Lang:U2Lang.dll
 0002:00000714       __imp_?createConnection@DomainFactory@Workflow@U2@@UAEPAVCommunicationChannel@23@PAVLink@23@@Z 10017714     U2Lang:U2Lang.dll
 0002:00000718       __imp_?isEmpty@ConfigurationEditor@U2@@UBE_NXZ 10017718     U2Lang:U2Lang.dll
 0002:0000071c       __imp_?getType@VisibilityRelation@U2@@UBE?AW4RelationType@2@XZ 1001771c     U2Lang:U2Lang.dll
 0002:00000720       \177U2Lang_NULL_THUNK_DATA 10017720     U2Lang:U2Lang.dll
 0002:00000724       __imp_?WORKFLOW_ELEMENTS_GROUP@NgsReadsClassificationPlugin@U2@@2VQString@@B 10017724     ngs_reads_classification:ngs_reads_classification.dll
 0002:00000728       __imp_?METAPHLAN2_DATABASE_ITEM_ID@NgsReadsClassificationPlugin@U2@@2VQString@@B 10017728     ngs_reads_classification:ngs_reads_classification.dll
 0002:0000072c       __imp_?METAPHLAN2_DATABASE_DATA_ID@NgsReadsClassificationPlugin@U2@@2VQString@@B 1001772c     ngs_reads_classification:ngs_reads_classification.dll
 0002:00000730       __imp_?update@DatabaseDelegate@LocalWorkflow@U2@@UAEXXZ 10017730     ngs_reads_classification:ngs_reads_classification.dll
 0002:00000734       __imp_??1DatabaseDelegate@LocalWorkflow@U2@@UAE@XZ 10017734     ngs_reads_classification:ngs_reads_classification.dll
 0002:00000738       __imp_??0DatabaseDelegate@LocalWorkflow@U2@@QAE@ABVQString@@0ABV?$QList@U?$QPair@VQString@@V1@@@@@0_N@Z 10017738     ngs_reads_classification:ngs_reads_classification.dll
 0002:0000073c       __imp_?getBaseFileNameWithSuffixes@NgsReadsClassificationUtils@U2@@SA?AVQString@@ABV3@ABVQStringList@@0_N@Z 1001773c     ngs_reads_classification:ngs_reads_classification.dll
 0002:00000740       \177ngs_reads_classification_NULL_THUNK_DATA 10017740     ngs_reads_classification:ngs_reads_classification.dll
 0002:00000744       ___xc_a                    10017744     MSVCRT:cinitexe.obj
 0002:000009e8       ___xc_z                    100179e8     MSVCRT:cinitexe.obj
 0002:000009ec       ___xi_a                    100179ec     MSVCRT:cinitexe.obj
 0002:000009f8       ___xi_z                    100179f8     MSVCRT:cinitexe.obj
 0002:00000a3c       ??_7error_category@std@@6B@ 10017a3c     Metaphlan2LogParser.obj
 0002:00000a58       ??_7_Generic_error_category@std@@6B@ 10017a58     Metaphlan2LogParser.obj
 0002:00000a70       ??_C@_07DCLBNMLN@generic?$AA@ 10017a70     Metaphlan2LogParser.obj
 0002:00000a78       ??_C@_0O@BFJCFAAK@unknown?5error?$AA@ 10017a78     Metaphlan2LogParser.obj
 0002:00000a8c       ??_7_Iostream_error_category@std@@6B@ 10017a8c     Metaphlan2LogParser.obj
 0002:00000aa4       ??_C@_08LLGCOLLL@iostream?$AA@ 10017aa4     Metaphlan2LogParser.obj
 0002:00000ab0       ??_C@_0BG@PADBLCHM@iostream?5stream?5error?$AA@ 10017ab0     Metaphlan2LogParser.obj
 0002:00000acc       ??_7_System_error_category@std@@6B@ 10017acc     Metaphlan2LogParser.obj
 0002:00000ae4       ??_C@_06FHFOAHML@system?$AA@ 10017ae4     Metaphlan2LogParser.obj
 0002:00000aec       ??_C@_0L@JLHNEGIN@Algorithms?$AA@ 10017aec     Metaphlan2LogParser.obj
 0002:00000af8       ??_C@_07PGLPGHFC@Console?$AA@ 10017af8     Metaphlan2LogParser.obj
 0002:00000b00       ??_C@_0O@BOFHOPCF@Core?5Services?$AA@ 10017b00     Metaphlan2LogParser.obj
 0002:00000b10       ??_C@_0N@PPADAKBM@Input?1Output?$AA@ 10017b10     Metaphlan2LogParser.obj
 0002:00000b20       ??_C@_0M@KPPBKPKK@Performance?$AA@ 10017b20     Metaphlan2LogParser.obj
 0002:00000b2c       ??_C@_07BFDHHBBI@Scripts?$AA@ 10017b2c     Metaphlan2LogParser.obj
 0002:00000b34       ??_C@_05EEGKELMG@Tasks?$AA@ 10017b34     Metaphlan2LogParser.obj
 0002:00000b3c       ??_C@_0P@NIIOBHGA@User?5Interface?$AA@ 10017b3c     Metaphlan2LogParser.obj
 0002:00000b4c       ??_C@_0N@JINCGGMN@User?5Actions?$AA@ 10017b4c     Metaphlan2LogParser.obj
 0002:00000b5c       ??_C@_0BH@LBDHGFEP@ImportError?3?5No?5module?$AA@ 10017b5c     Metaphlan2LogParser.obj
 0002:00000b74       ??_C@_0BA@JFNIOLAK@string?5too?5long?$AA@ 10017b74     Metaphlan2LogParser.obj
 0002:00000b84       ??_C@_0BI@CFPLBAOH@invalid?5string?5position?$AA@ 10017b84     Metaphlan2LogParser.obj
 0002:00000b9c       ??_C@_00CNPNBAHC@?$AA@     10017b9c     Metaphlan2Prompter.obj
 0002:00000ba4       ??_7?$PrompterBase@VMetaphlan2Prompter@LocalWorkflow@U2@@@U2@@6BActorDocument@Workflow@1@@ 10017ba4     Metaphlan2Prompter.obj
 0002:00000bec       ??_7?$PrompterBase@VMetaphlan2Prompter@LocalWorkflow@U2@@@U2@@6BPrompter@Workflow@1@@ 10017bec     Metaphlan2Prompter.obj
 0002:00000bf8       ??_7Metaphlan2Prompter@LocalWorkflow@U2@@6BActorDocument@Workflow@2@@ 10017bf8     Metaphlan2Prompter.obj
 0002:00000c40       ??_7Metaphlan2Prompter@LocalWorkflow@U2@@6BPrompter@Workflow@2@@ 10017c40     Metaphlan2Prompter.obj
 0002:00000c48       ??_C@_0EE@IMEOCJAH@Classify?5sequences?5from?5?$DMu?$DO?$CF1?$DM?1u@ 10017c48     Metaphlan2Prompter.obj
 0002:00000c8c       ??_C@_0BE@LGBLLFOL@1sl_actorModified?$CI?$CJ?$AA@ 10017c8c     Metaphlan2Prompter.obj
 0002:00000ca0       ??_C@_0BD@FGIDJNMI@2si_labelChanged?$CI?$CJ?$AA@ 10017ca0     Metaphlan2Prompter.obj
 0002:00000cb4       ??_C@_0P@DIBOLHGA@2si_modified?$CI?$CJ?$AA@ 10017cb4     Metaphlan2Prompter.obj
 0002:00000cc4       ??_C@_0BC@HBGBGNIM@2bindingChanged?$CI?$CJ?$AA@ 10017cc4     Metaphlan2Prompter.obj
 0002:00000cdc       ??_7Metaphlan2Support@U2@@6B@ 10017cdc     Metaphlan2Support.obj
 0002:00000d18       ??_C@_0L@BIEFJEPM@MetaPhlAn2?$AA@ 10017d18     Metaphlan2Support.obj
 0002:00000d24       ??_C@_0BE@IGCFELA@utils?1read_fastx?4py?$AA@ 10017d24     Metaphlan2Support.obj
 0002:00000d38       ??_C@_0BB@OLPBINAP@Bowtie?52?5aligner?$AA@ 10017d38     Metaphlan2Support.obj
 0002:00000d4c       ??_C@_06OIODPPHE@python?$AA@ 10017d4c     Metaphlan2Support.obj
 0002:00000d54       ??_C@_03EKMFDHJC@Bio?$AA@  10017d54     Metaphlan2Support.obj
 0002:00000d58       ??_C@_05COLBNKPI@numpy?$AA@ 10017d58     Metaphlan2Support.obj
 0002:00000d60       ??_C@_09GAJKMFCA@?9?9version?$AA@ 10017d60     Metaphlan2Support.obj
 0002:00000d70       ??_C@_0ND@HNIDBKLE@?$DMi?$DOMetaPhlAn2?5?$CIMETAgenomic?5PHyLo@ 10017d70     Metaphlan2Support.obj
 0002:00000e44       ??_C@_0O@ICAEANL@metaphlan2?4py?$AA@ 10017e44     Metaphlan2Support.obj
 0002:00000e54       ??_C@_0BD@FCEENPGP@MetaPhlAn?5version?5?$AA@ 10017e54     Metaphlan2Support.obj
 0002:00000e68       ??_C@_0DD@EKCOGOLO@MetaPhlAn?5version?5?$CI?2d?$CL?2?4?2d?$CL?$CI?2?4?2d@ 10017e68     Metaphlan2Support.obj
 0002:00000e9c       ??_C@_05KOLKDEPN@?$CF1?1?$CF2?$AA@ 10017e9c     Metaphlan2Support.obj
 0002:00000ea4       ??_C@_0BP@JENDDBMI@?$CF1?5script?5?$CC?$CF2?$CC?5is?5not?5present?$CB?$AA@ 10017ea4     Metaphlan2Support.obj
 0002:00000ec8       ??_7MetaphlanSupportPlugin@U2@@6B@ 10017ec8     Metaphlan2SupportPlugin.obj
 0002:00000ef4       ??_C@_0CB@OENHBGMK@MetaPhlAn2?5external?5tool?5support@ 10017ef4     Metaphlan2SupportPlugin.obj
 0002:00000f18       ??_C@_0BH@LLODGJLJ@MetaphlanSupportPlugin?$AA@ 10017f18     Metaphlan2SupportPlugin.obj
 0002:00000f30       ??_C@_0MM@JMJAOIEI@MetaPhlAn2?5?$CIMETAgenomic?5PHyLogen@ 10017f30     Metaphlan2SupportPlugin.obj
 0002:00001004       ??_SCalculateSequencesNumberTask@U2@@6B@ 10018004     Metaphlan2Task.obj
 0002:00001094       ??_SExternalToolRunTask@U2@@6B@ 10018094     Metaphlan2Task.obj
 0002:00001124       ??_7Metaphlan2LogParser@U2@@6B@ 10018124     Metaphlan2Task.obj
 0002:00001170       ??_7Metaphlan2ClassifyTask@U2@@6B@ 10018170     Metaphlan2Task.obj
 0002:00001204       ??_C@_0BP@DANHGHJ@Classify?5reads?5with?5Metaphlan2?$AA@ 10018204     Metaphlan2Task.obj
 0002:00001224       ??_C@_0BH@ILDEFHHG@Metaphlan2ClassifyTask?$AA@ 10018224     Metaphlan2Task.obj
 0002:0000123c       ??_C@_0CC@JNENGDNH@Metaphlan2?5database?5URL?5is?5empty@ 1001823c     Metaphlan2Task.obj
 0002:00001260       ??_C@_0CC@PLDHPMAG@Bowtie2?5output?5file?5URL?5is?5empty@ 10018260     Metaphlan2Task.obj
 0002:00001284       ??_C@_0CF@DLAILHOJ@Metaphlan2?5output?5file?5URL?5is?5em@ 10018284     Metaphlan2Task.obj
 0002:000012ac       ??_C@_0BP@IPNCEEGL@Temporary?5folder?5URL?5is?5empty?4?$AA@ 100182ac     Metaphlan2Task.obj
 0002:000012cc       ??_C@_0BE@IIKOCLOP@Reads?5URL?5is?5empty?4?$AA@ 100182cc     Metaphlan2Task.obj
 0002:000012e0       ??_C@_05LMAPJLBD@?$CF1?0?$CF2?$AA@ 100182e0     Metaphlan2Task.obj
 0002:000012e8       ??_C@_07FBIFFNMG@?9?9nproc?$AA@ 100182e8     Metaphlan2Task.obj
 0002:000012f0       ??_C@_02HLHIEPKM@?9t?$AA@  100182f0     Metaphlan2Task.obj
 0002:000012f4       ??_C@_01IDAFKMJL@_?$AA@    100182f4     Metaphlan2Task.obj
 0002:000012f8       ??_C@_01JOAMLHOP@?9?$AA@   100182f8     Metaphlan2Task.obj
 0002:000012fc       ??_C@_09MLAIOKJA@?9?9tax_lev?$AA@ 100182fc     Metaphlan2Task.obj
 0002:00001308       ??_C@_08MNMEDMC@?9?9nreads?$AA@ 10018308     Metaphlan2Task.obj
 0002:00001314       ??_C@_09IJDGBAKO@?9?9pres_th?$AA@ 10018314     Metaphlan2Task.obj
 0002:00001320       ??_C@_09EIDJBGAG@?9?9tmp_dir?$AA@ 10018320     Metaphlan2Task.obj
 0002:0000132c       ??_C@_0N@MBACJIAO@?9?9input_type?$AA@ 1001832c     Metaphlan2Task.obj
 0002:0000133c       ??_C@_05GCFGHJPO@fasta?$AA@ 1001833c     Metaphlan2Task.obj
 0002:00001344       ??_C@_05CIJEGLKP@fastq?$AA@ 10018344     Metaphlan2Task.obj
 0002:0000134c       ??_C@_0N@PBBBIELH@?9?9bowtie2out?$AA@ 1001834c     Metaphlan2Task.obj
 0002:0000135c       ??_C@_05HAAOEJJP@?$CK?4pkl?$AA@ 1001835c     Metaphlan2Task.obj
 0002:00001364       ??_C@_0CM@CBBFHLAC@?4pkl?5file?5is?5absent?5in?5the?5datab@ 10018364     Metaphlan2Task.obj
 0002:00001390       ??_C@_0DG@KMBJMBDD@There?5is?51?5?4pkl?5file?5in?5the?5data@ 10018390     Metaphlan2Task.obj
 0002:000013c8       ??_C@_09ONPADLEP@?9?9mpa_pkl?$AA@ 100183c8     Metaphlan2Task.obj
 0002:000013d4       ??_C@_0M@JLNICLID@?9?9bowtie2db?$AA@ 100183d4     Metaphlan2Task.obj
 0002:000013e0       ??_C@_02NCEOIEDG@?9o?$AA@  100183e0     Metaphlan2Task.obj
 0002:000013e4       ??_C@_0DB@PHCOMDOE@Input?5files?5with?5PE?5reads?5have?5d@ 100183e4     Metaphlan2Task.obj
 0002:00001418       ??_C@_0CI@OLDDGDGI@Input?5file?5format?5couldn?8t?5be?5de@ 10018418     Metaphlan2Task.obj
 0002:00001440       ??_C@_0EE@BJHHEOPC@Unexpected?5input?5file?5format?5det@ 10018440     Metaphlan2Task.obj
 0002:00001488       __real@3ff0000000000000    10018488     Metaphlan2Task.obj
 0002:00001490       ??_C@_0BE@GNGPAMBM@Metaphlan2Validator?$AA@ 10018490     Metaphlan2Validator.obj
 0002:000014a4       ??_C@_0DK@JOINLCPL@The?5database?5folder?5should?5conta@ 100184a4     Metaphlan2Validator.obj
 0002:000014e0       ??_C@_05LJFMECBM@?$CK?4bt2?$AA@ 100184e0     Metaphlan2Validator.obj
 0002:000014e8       ??_C@_0EG@CAPKLBKE@The?5database?5folder?5should?5conta@ 100184e8     Metaphlan2Validator.obj
 0002:00001534       ??_SFailTask@U2@@6B@       10018534     Metaphlan2Worker.obj
 0002:000015c4       ??_STaskSignalMapper@U2@@6B@ 100185c4     Metaphlan2Worker.obj
 0002:000015f4       ??_SDescriptor@U2@@6B@     100185f4     Metaphlan2Worker.obj
 0002:000015f8       ??_C@_0BF@COKBMJP@Script?5task?5canceled?$AA@ 100185f8     Metaphlan2Worker.obj
 0002:00001614       ??_7Metaphlan2Worker@LocalWorkflow@U2@@6BQObject@@@ 10018614     Metaphlan2Worker.obj
 0002:00001658       ??_7Metaphlan2Worker@LocalWorkflow@U2@@6BWorker@Workflow@2@@ 10018658     Metaphlan2Worker.obj
 0002:00001674       ??_7Metaphlan2Worker@LocalWorkflow@U2@@6BCommunicationSubject@Workflow@2@@ 10018674     Metaphlan2Worker.obj
 0002:00001680       ??_C@_0L@OHCOICEE@bowtie2out?$AA@ 10018680     Metaphlan2Worker.obj
 0002:0000168c       ??_C@_08LKPBAFL@profiles?$AA@ 1001868c     Metaphlan2Worker.obj
 0002:00001698       ??_C@_07LNMDFKEJ@profile?$AA@ 10018698     Metaphlan2Worker.obj
 0002:000016a0       ??_C@_0CK@IGBIANDN@Trying?5to?5recover?5from?5error?3?5?$CF1@ 100186a0     Metaphlan2Worker.obj
 0002:000016cc       ??_C@_0BN@FODKIGFA@Port?5with?5id?5?8?$CF1?8?5is?5nullptr?$AA@ 100186cc     Metaphlan2Worker.obj
 0002:000016ec       ??_C@_0BJ@JNAODEJH@src?2Metaphlan2Worker?4cpp?$AA@ 100186ec     Metaphlan2Worker.obj
 0002:00001708       ??_C@_0BI@LFJECNHK@1sl_taskFinished?$CITask?$CK?$CJ?$AA@ 10018708     Metaphlan2Worker.obj
 0002:00001720       ??_C@_0BI@KGADHDJC@2si_taskFinished?$CITask?$CK?$CJ?$AA@ 10018720     Metaphlan2Worker.obj
 0002:00001738       ??_C@_07HDKMEHEP@Bowtie2?$AA@ 10018738     Metaphlan2Worker.obj
 0002:00001740       ??_C@_0CO@EAGCHLEN@Can?8t?5create?5a?5folder?5for?5the?5ou@ 10018740     Metaphlan2Worker.obj
 0002:00001770       ??_C@_0BM@JKCLCNKJ@Bowtie2?5aligner?5isn?8t?5found?$AA@ 10018770     Metaphlan2Worker.obj
 0002:0000178c       ??_C@_0BD@DDGCIKIJ@Python?5isn?8t?5found?$AA@ 1001878c     Metaphlan2Worker.obj
 0002:000017a0       ??_C@_03CLFHJCDC@txt?$AA@  100187a0     Metaphlan2Worker.obj
 0002:000017a4       ??_C@_0BN@KODHBDBE@?$CF1?5output?5file?5doesn?8t?5exist?$AA@ 100187a4     Metaphlan2Worker.obj
 0002:000017c8       ??_SVisibilityRelation@U2@@6B@ 100187c8     Metaphlan2WorkerFactory.obj
 0002:000017e4       ??_SMapDataType@U2@@6B@    100187e4     Metaphlan2WorkerFactory.obj
 0002:000017fc       ??_SSlotRelationDescriptor@U2@@6B@ 100187fc     Metaphlan2WorkerFactory.obj
 0002:0000180c       ??_SAttribute@U2@@6B@      1001880c     Metaphlan2WorkerFactory.obj
 0002:00001838       ??_SPortDescriptor@Workflow@U2@@6B@ 10018838     Metaphlan2WorkerFactory.obj
 0002:00001848       ??_SIntegralBusActorPrototype@Workflow@U2@@6B@ 10018848     Metaphlan2WorkerFactory.obj
 0002:0000185c       ??_7Metaphlan2Validator@Workflow@U2@@6B@ 1001885c     Metaphlan2WorkerFactory.obj
 0002:0000186c       ??_7Metaphlan2WorkerFactory@LocalWorkflow@U2@@6B?$IdRegistry@VDomainFactory@Workflow@U2@@@2@@ 1001886c     Metaphlan2WorkerFactory.obj
 0002:00001898       ??_7Metaphlan2WorkerFactory@LocalWorkflow@U2@@6BDescriptor@2@@ 10018898     Metaphlan2WorkerFactory.obj
 0002:0000189c       ??_C@_0BI@PLFCCFBJ@Metaphlan2WorkerFactory?$AA@ 1001889c     Metaphlan2WorkerFactory.obj
 0002:000018b8       ??_SPairedReadsPortValidator@Workflow@U2@@6B@ 100188b8     Metaphlan2WorkerFactory.obj
 0002:000018cc       ??_SDelegateEditor@U2@@6B@ 100188cc     Metaphlan2WorkerFactory.obj
 0002:00001924       ??_SURLDelegate@U2@@6B@    10018924     Metaphlan2WorkerFactory.obj
 0002:000019a4       ??_SSpinBoxDelegate@U2@@6B@ 100189a4     Metaphlan2WorkerFactory.obj
 0002:00001a24       ??_SComboBoxDelegate@U2@@6B@ 10018a24     Metaphlan2WorkerFactory.obj
 0002:00001aa4       ??_SDatabaseDelegate@LocalWorkflow@U2@@6B@ 10018aa4     Metaphlan2WorkerFactory.obj
 0002:00001b20       ??_C@_0BE@COIGNPFO@metaphlan2?9classify?$AA@ 10018b20     Metaphlan2WorkerFactory.obj
 0002:00001b34       ??_C@_02LMMGJAGL@in?$AA@   10018b34     Metaphlan2WorkerFactory.obj
 0002:00001b38       ??_C@_0L@LGHLPLD@reads?9url1?$AA@ 10018b38     Metaphlan2WorkerFactory.obj
 0002:00001b44       ??_C@_0L@CAEKOMHA@reads?9url2?$AA@ 10018b44     Metaphlan2WorkerFactory.obj
 0002:00001b50       ??_C@_0L@HPPLHBN@input?9data?$AA@ 10018b50     Metaphlan2WorkerFactory.obj
 0002:00001b5c       ??_C@_08PBOCEOLL@database?$AA@ 10018b5c     Metaphlan2WorkerFactory.obj
 0002:00001b68       ??_C@_07NFPADACG@threads?$AA@ 10018b68     Metaphlan2WorkerFactory.obj
 0002:00001b70       ??_C@_0O@BOMAHCDG@analysis?9type?$AA@ 10018b70     Metaphlan2WorkerFactory.obj
 0002:00001b80       ??_C@_09JOPEBAMJ@tax?9level?$AA@ 10018b80     Metaphlan2WorkerFactory.obj
 0002:00001b8c       ??_C@_0BC@LELCKANF@normalize?9by?9size?$AA@ 10018b8c     Metaphlan2WorkerFactory.obj
 0002:00001ba0       ??_C@_0BD@LAFAFBDN@presence?9threshold?$AA@ 10018ba0     Metaphlan2WorkerFactory.obj
 0002:00001bb4       ??_C@_0BD@LOLOAGMH@bowtie2?9output?9url?$AA@ 10018bb4     Metaphlan2WorkerFactory.obj
 0002:00001bc8       ??_C@_0L@JDEFPCKN@output?9url?$AA@ 10018bc8     Metaphlan2WorkerFactory.obj
 0002:00001bd4       ??_C@_0BE@IHKBOJBH@SE?5reads?5or?5contigs?$AA@ 10018bd4     Metaphlan2WorkerFactory.obj
 0002:00001be8       ??_C@_08BKAKNCGK@PE?5reads?$AA@ 10018be8     Metaphlan2WorkerFactory.obj
 0002:00001bf4       ??_C@_0BD@DCGHICLH@Relative?5abundance?$AA@ 10018bf4     Metaphlan2WorkerFactory.obj
 0002:00001c08       ??_C@_0CJ@FHGKBFKG@Relative?5abundance?5with?5reads?5st@ 10018c08     Metaphlan2WorkerFactory.obj
 0002:00001c34       ??_C@_0O@INIMCFFG@Reads?5mapping?$AA@ 10018c34     Metaphlan2WorkerFactory.obj
 0002:00001c44       ??_C@_0P@NBDEGFBE@Clade?5profiles?$AA@ 10018c44     Metaphlan2WorkerFactory.obj
 0002:00001c54       ??_C@_0BH@HMCFLFIM@Marker?5abundance?5table?$AA@ 10018c54     Metaphlan2WorkerFactory.obj
 0002:00001c6c       ??_C@_0BG@JOHJMHOH@Marker?5presence?5table?$AA@ 10018c6c     Metaphlan2WorkerFactory.obj
 0002:00001c84       ??_C@_06FBBJDKPH@rel?9ab?$AA@ 10018c84     Metaphlan2WorkerFactory.obj
 0002:00001c8c       ??_C@_0BE@FENODKJM@rel?9ab?9w?9read?9stats?$AA@ 10018c8c     Metaphlan2WorkerFactory.obj
 0002:00001ca0       ??_C@_09IAAEKNPB@reads?9map?$AA@ 10018ca0     Metaphlan2WorkerFactory.obj
 0002:00001cac       ??_C@_0P@KMAPNADK@clade?9profiles?$AA@ 10018cac     Metaphlan2WorkerFactory.obj
 0002:00001cbc       ??_C@_0BA@BNJIGGFJ@marker?9ab?9table?$AA@ 10018cbc     Metaphlan2WorkerFactory.obj
 0002:00001ccc       ??_C@_0BC@ICNFKCCI@marker?9pres?9table?$AA@ 10018ccc     Metaphlan2WorkerFactory.obj
 0002:00001ce0       ??_C@_03HFJGAJFE@All?$AA@  10018ce0     Metaphlan2WorkerFactory.obj
 0002:00001ce4       ??_C@_08PAHIBNP@Kingdoms?$AA@ 10018ce4     Metaphlan2WorkerFactory.obj
 0002:00001cf0       ??_C@_05MAONONJD@Phyla?$AA@ 10018cf0     Metaphlan2WorkerFactory.obj
 0002:00001cf8       ??_C@_07DPIHKJGF@Classes?$AA@ 10018cf8     Metaphlan2WorkerFactory.obj
 0002:00001d00       ??_C@_06KFBHMJGM@Orders?$AA@ 10018d00     Metaphlan2WorkerFactory.obj
 0002:00001d08       ??_C@_08DNEHEDHF@Families?$AA@ 10018d08     Metaphlan2WorkerFactory.obj
 0002:00001d14       ??_C@_06LKGPNNFK@Genera?$AA@ 10018d14     Metaphlan2WorkerFactory.obj
 0002:00001d1c       ??_C@_07CHJHAMJL@Species?$AA@ 10018d1c     Metaphlan2WorkerFactory.obj
 0002:00001d24       ??_C@_01MCMALHOG@a?$AA@    10018d24     Metaphlan2WorkerFactory.obj
 0002:00001d28       ??_C@_01DICPFPGM@k?$AA@    10018d28     Metaphlan2WorkerFactory.obj
 0002:00001d2c       ??_C@_01JBBJJEPG@p?$AA@    10018d2c     Metaphlan2WorkerFactory.obj
 0002:00001d30       ??_C@_01PAPGNFGE@c?$AA@    10018d30     Metaphlan2WorkerFactory.obj
 0002:00001d34       ??_C@_01FMEDJKGI@o?$AA@    10018d34     Metaphlan2WorkerFactory.obj
 0002:00001d38       ??_C@_01INIBCBCB@f?$AA@    10018d38     Metaphlan2WorkerFactory.obj
 0002:00001d3c       ??_C@_01JEJKBAGA@g?$AA@    10018d3c     Metaphlan2WorkerFactory.obj
 0002:00001d40       ??_C@_01LKDEMHDF@s?$AA@    10018d40     Metaphlan2WorkerFactory.obj
 0002:00001d44       ??_C@_04DLBGLKG@skip?$AA@  10018d44     Metaphlan2WorkerFactory.obj
 0002:00001d4c       ??_C@_09MMDNNKKJ@normalize?$AA@ 10018d4c     Metaphlan2WorkerFactory.obj
 0002:00001d58       ??_C@_0L@PCJLLKLK@single?9end?$AA@ 10018d58     Metaphlan2WorkerFactory.obj
 0002:00001d64       ??_C@_0L@HGFAFILP@paired?9end?$AA@ 10018d64     Metaphlan2WorkerFactory.obj
 0002:00001d70       ??_C@_0BAC@PKLLDIKN@URL?$CIs?$CJ?5to?5FASTQ?5or?5FASTA?5file?$CIs?$CJ@ 10018d70     Metaphlan2WorkerFactory.obj
 0002:00001e74       ??_C@_0BA@GLOOOALC@Input?5sequences?$AA@ 10018e74     Metaphlan2WorkerFactory.obj
 0002:00001e84       ??_C@_0N@JCLPICJJ@Input?5URL?51?4?$AA@ 10018e84     Metaphlan2WorkerFactory.obj
 0002:00001e94       ??_C@_0M@LBNKAPAD@Input?5URL?51?$AA@ 10018e94     Metaphlan2WorkerFactory.obj
 0002:00001ea0       ??_C@_0N@JAPJDMMA@Input?5URL?52?4?$AA@ 10018ea0     Metaphlan2WorkerFactory.obj
 0002:00001eb0       ??_C@_0M@JKPHFMMA@Input?5URL?52?$AA@ 10018eb0     Metaphlan2WorkerFactory.obj
 0002:00001ebc       ??_C@_03DAJLOBIG@?9in?$AA@ 10018ebc     Metaphlan2WorkerFactory.obj
 0002:00001ec0       ??_C@_0BKF@KENIEFCJ@To?5classify?5single?9end?5?$CISE?$CJ?5read@ 10018ec0     Metaphlan2WorkerFactory.obj
 0002:00002068       ??_C@_0L@DNPNCLBE@Input?5data?$AA@ 10019068     Metaphlan2WorkerFactory.obj
 0002:00002078       ??_C@_0BIN@HOKIPEJP@A?5path?5to?5a?5folder?5with?5MetaPhlA@ 10019078     Metaphlan2WorkerFactory.obj
 0002:00002208       ??_C@_08HDBDMMBI@Database?$AA@ 10019208     Metaphlan2WorkerFactory.obj
 0002:00002218       ??_C@_0ED@IOLHPCFJ@The?5number?5of?5CPUs?5to?5use?5for?5pa@ 10019218     Metaphlan2WorkerFactory.obj
 0002:0000225c       ??_C@_0BC@GJADDMKB@Number?5of?5threads?$AA@ 1001925c     Metaphlan2WorkerFactory.obj
 0002:00002270       ??_C@_0DJD@OFPEIAII@Specify?5type?5of?5analysis?5to?5perf@ 10019270     Metaphlan2WorkerFactory.obj
 0002:00002604       ??_C@_0O@GPDKBJDA@Analysis?5type?$AA@ 10019604     Metaphlan2WorkerFactory.obj
 0002:00002618       ??_C@_0IA@HAPDFBED@The?5taxonomic?5level?5for?5the?5rela@ 10019618     Metaphlan2WorkerFactory.obj
 0002:00002698       ??_C@_09LAHOHCNJ@Tax?5level?$AA@ 10019698     Metaphlan2WorkerFactory.obj
 0002:000026a8       ??_C@_0OK@BAMEECHB@If?5?$CCNormalize?$CC?5is?5selected?0?5the?5@ 100196a8     Metaphlan2WorkerFactory.obj
 0002:00002794       ??_C@_0BN@EMCNPPK@Normalize?5by?5metagenome?5size?$AA@ 10019794     Metaphlan2WorkerFactory.obj
 0002:000027b4       ??_C@_0CK@DPOFFFAP@Specify?5a?5threshold?5for?5calling?5@ 100197b4     Metaphlan2WorkerFactory.obj
 0002:000027e0       ??_C@_0BD@FNEAGKCO@Presence?5threshold?$AA@ 100197e0     Metaphlan2WorkerFactory.obj
 0002:000027f8       ??_C@_0HK@EMEEOJNJ@The?5file?5for?5saving?5the?5output?5o@ 100197f8     Metaphlan2WorkerFactory.obj
 0002:00002874       ??_C@_0BE@FMCCGIJA@Bowtie2?5output?5file?$AA@ 10019874     Metaphlan2WorkerFactory.obj
 0002:00002888       ??_C@_0JB@LOHPAGIO@MetaPhlAn2?5output?5depends?5on?5the@ 10019888     Metaphlan2WorkerFactory.obj
 0002:0000291c       ??_C@_0M@LEIJPAKP@Output?5file?$AA@ 1001991c     Metaphlan2WorkerFactory.obj
 0002:00002928       ??_C@_0BE@MKEBMNJJ@metaphlan2?1database?$AA@ 10019928     Metaphlan2WorkerFactory.obj
 0002:0000293c       ??_C@_07CCOEHHFD@minimum?$AA@ 1001993c     Metaphlan2WorkerFactory.obj
 0002:00002944       ??_C@_07MEIENILC@maximum?$AA@ 10019944     Metaphlan2WorkerFactory.obj
 0002:0000294c       ??_C@_04MCHAEEKC@Skip?$AA@ 1001994c     Metaphlan2WorkerFactory.obj
 0002:00002954       ??_C@_09IDGANJHJ@Normalize?$AA@ 10019954     Metaphlan2WorkerFactory.obj
 0002:00002960       ??_C@_04LBDCJOFB@Auto?$AA@ 10019960     Metaphlan2WorkerFactory.obj
 0002:00002968       ??_C@_0BJ@LMHKDEAE@metaphlan2?1bowtie2Output?$AA@ 10019968     Metaphlan2WorkerFactory.obj
 0002:00002984       ??_C@_0BC@EOGKMDNA@metaphlan2?1output?$AA@ 10019984     Metaphlan2WorkerFactory.obj
 0002:00002998       ??_C@_0BHN@POBBKHHM@MetaPhlAn2?5?$CIMETAgenomic?5PHyLogen@ 10019998     Metaphlan2WorkerFactory.obj
 0002:00002b18       ??_C@_0CD@MCCBCNEO@Classify?5Sequences?5with?5MetaPhlA@ 10019b18     Metaphlan2WorkerFactory.obj
 0002:00002dd4       ?value@?$integral_constant@_N$0A@@std@@2_NB 10019dd4     MSVCRT:ti_inst.obj
 0002:00002dd5       ?value@?$integral_constant@_N$00@std@@2_NB 10019dd5     MSVCRT:ti_inst.obj
 0002:00002ddc       ??_7type_info@@6B@         10019ddc     MSVCRT:ti_inst.obj
 0002:00002de0       __pDefaultRawDllMain       10019de0     MSVCRT:crtdll.obj
 0002:00002de0       __pRawDllMain              10019de0     MSVCRT:crtdll.obj
 0002:00002dec       ?ProcessDetach@NativeDll@<CrtImplementationDetails>@@0IB 10019dec     MSVCRT:initsect.obj
 0002:00002df0       ?ProcessAttach@NativeDll@<CrtImplementationDetails>@@0IB 10019df0     MSVCRT:initsect.obj
 0002:00002df4       ?ThreadAttach@NativeDll@<CrtImplementationDetails>@@0IB 10019df4     MSVCRT:initsect.obj
 0002:00002df8       ?ThreadDetach@NativeDll@<CrtImplementationDetails>@@0IB 10019df8     MSVCRT:initsect.obj
 0002:00002dfc       ?ProcessVerifier@NativeDll@<CrtImplementationDetails>@@0IB 10019dfc     MSVCRT:initsect.obj
 0002:00002e00       __load_config_used         10019e00     MSVCRT:loadcfg.obj
 0002:00002ec0       ??_R4error_category@std@@6B@ 10019ec0     Metaphlan2LogParser.obj
 0002:00002ed4       ??_R3error_category@std@@8 10019ed4     Metaphlan2LogParser.obj
 0002:00002ee4       ??_R2error_category@std@@8 10019ee4     Metaphlan2LogParser.obj
 0002:00002eec       ??_R1A@?0A@EA@error_category@std@@8 10019eec     Metaphlan2LogParser.obj
 0002:00002f08       ??_R4_Generic_error_category@std@@6B@ 10019f08     Metaphlan2LogParser.obj
 0002:00002f1c       ??_R3_Generic_error_category@std@@8 10019f1c     Metaphlan2LogParser.obj
 0002:00002f2c       ??_R2_Generic_error_category@std@@8 10019f2c     Metaphlan2LogParser.obj
 0002:00002f38       ??_R1A@?0A@EA@_Generic_error_category@std@@8 10019f38     Metaphlan2LogParser.obj
 0002:00002f54       ??_R4_Iostream_error_category@std@@6B@ 10019f54     Metaphlan2LogParser.obj
 0002:00002f68       ??_R3_Iostream_error_category@std@@8 10019f68     Metaphlan2LogParser.obj
 0002:00002f78       ??_R2_Iostream_error_category@std@@8 10019f78     Metaphlan2LogParser.obj
 0002:00002f88       ??_R1A@?0A@EA@_Iostream_error_category@std@@8 10019f88     Metaphlan2LogParser.obj
 0002:00002fa4       ??_R4_System_error_category@std@@6B@ 10019fa4     Metaphlan2LogParser.obj
 0002:00002fb8       ??_R3_System_error_category@std@@8 10019fb8     Metaphlan2LogParser.obj
 0002:00002fc8       ??_R2_System_error_category@std@@8 10019fc8     Metaphlan2LogParser.obj
 0002:00002fd8       ??_R1A@?0A@EA@_System_error_category@std@@8 10019fd8     Metaphlan2LogParser.obj
 0002:00002ff4       ??_R1A@?0A@EA@QObject@@8   10019ff4     Metaphlan2Prompter.obj
 0002:00003010       ??_R3QObject@@8            1001a010     Metaphlan2Prompter.obj
 0002:00003020       ??_R2QObject@@8            1001a020     Metaphlan2Prompter.obj
 0002:00003028       ??_R4Metaphlan2Prompter@LocalWorkflow@U2@@6BActorDocument@Workflow@2@@ 1001a028     Metaphlan2Prompter.obj
 0002:0000303c       ??_R3Metaphlan2Prompter@LocalWorkflow@U2@@8 1001a03c     Metaphlan2Prompter.obj
 0002:0000304c       ??_R2Metaphlan2Prompter@LocalWorkflow@U2@@8 1001a04c     Metaphlan2Prompter.obj
 0002:0000306c       ??_R1A@?0A@EA@Metaphlan2Prompter@LocalWorkflow@U2@@8 1001a06c     Metaphlan2Prompter.obj
 0002:00003088       ??_R1A@?0A@EA@?$PrompterBase@VMetaphlan2Prompter@LocalWorkflow@U2@@@U2@@8 1001a088     Metaphlan2Prompter.obj
 0002:000030a4       ??_R3?$PrompterBase@VMetaphlan2Prompter@LocalWorkflow@U2@@@U2@@8 1001a0a4     Metaphlan2Prompter.obj
 0002:000030b4       ??_R2?$PrompterBase@VMetaphlan2Prompter@LocalWorkflow@U2@@@U2@@8 1001a0b4     Metaphlan2Prompter.obj
 0002:000030d0       ??_R1A@?0A@EA@PrompterBaseImpl@U2@@8 1001a0d0     Metaphlan2Prompter.obj
 0002:000030ec       ??_R3PrompterBaseImpl@U2@@8 1001a0ec     Metaphlan2Prompter.obj
 0002:000030fc       ??_R2PrompterBaseImpl@U2@@8 1001a0fc     Metaphlan2Prompter.obj
 0002:00003114       ??_R1A@?0A@EA@ActorDocument@Workflow@U2@@8 1001a114     Metaphlan2Prompter.obj
 0002:00003130       ??_R3ActorDocument@Workflow@U2@@8 1001a130     Metaphlan2Prompter.obj
 0002:00003140       ??_R2ActorDocument@Workflow@U2@@8 1001a140     Metaphlan2Prompter.obj
 0002:00003150       ??_R1A@?0A@EA@QTextDocument@@8 1001a150     Metaphlan2Prompter.obj
 0002:0000316c       ??_R3QTextDocument@@8      1001a16c     Metaphlan2Prompter.obj
 0002:0000317c       ??_R2QTextDocument@@8      1001a17c     Metaphlan2Prompter.obj
 0002:00003188       ??_R1M@?0A@EA@Prompter@Workflow@U2@@8 1001a188     Metaphlan2Prompter.obj
 0002:000031a4       ??_R3Prompter@Workflow@U2@@8 1001a1a4     Metaphlan2Prompter.obj
 0002:000031b4       ??_R2Prompter@Workflow@U2@@8 1001a1b4     Metaphlan2Prompter.obj
 0002:000031bc       ??_R1A@?0A@EA@Prompter@Workflow@U2@@8 1001a1bc     Metaphlan2Prompter.obj
 0002:000031d8       ??_R4Metaphlan2Prompter@LocalWorkflow@U2@@6BPrompter@Workflow@2@@ 1001a1d8     Metaphlan2Prompter.obj
 0002:000031ec       ??_R4?$PrompterBase@VMetaphlan2Prompter@LocalWorkflow@U2@@@U2@@6BActorDocument@Workflow@1@@ 1001a1ec     Metaphlan2Prompter.obj
 0002:00003200       ??_R4?$PrompterBase@VMetaphlan2Prompter@LocalWorkflow@U2@@@U2@@6BPrompter@Workflow@1@@ 1001a200     Metaphlan2Prompter.obj
 0002:00003214       ??_R4Metaphlan2Support@U2@@6B@ 1001a214     Metaphlan2Support.obj
 0002:00003228       ??_R3Metaphlan2Support@U2@@8 1001a228     Metaphlan2Support.obj
 0002:00003238       ??_R2Metaphlan2Support@U2@@8 1001a238     Metaphlan2Support.obj
 0002:00003248       ??_R1A@?0A@EA@Metaphlan2Support@U2@@8 1001a248     Metaphlan2Support.obj
 0002:00003264       ??_R1A@?0A@EA@ExternalTool@U2@@8 1001a264     Metaphlan2Support.obj
 0002:00003280       ??_R3ExternalTool@U2@@8    1001a280     Metaphlan2Support.obj
 0002:00003290       ??_R2ExternalTool@U2@@8    1001a290     Metaphlan2Support.obj
 0002:0000329c       ??_R4MetaphlanSupportPlugin@U2@@6B@ 1001a29c     Metaphlan2SupportPlugin.obj
 0002:000032b0       ??_R3MetaphlanSupportPlugin@U2@@8 1001a2b0     Metaphlan2SupportPlugin.obj
 0002:000032c0       ??_R2MetaphlanSupportPlugin@U2@@8 1001a2c0     Metaphlan2SupportPlugin.obj
 0002:000032d0       ??_R1A@?0A@EA@MetaphlanSupportPlugin@U2@@8 1001a2d0     Metaphlan2SupportPlugin.obj
 0002:000032ec       ??_R1A@?0A@EA@Plugin@U2@@8 1001a2ec     Metaphlan2SupportPlugin.obj
 0002:00003308       ??_R3Plugin@U2@@8          1001a308     Metaphlan2SupportPlugin.obj
 0002:00003318       ??_R2Plugin@U2@@8          1001a318     Metaphlan2SupportPlugin.obj
 0002:00003324       ??_R4CalculateSequencesNumberTask@U2@@6B@ 1001a324     Metaphlan2Task.obj
 0002:00003338       ??_R3CalculateSequencesNumberTask@U2@@8 1001a338     Metaphlan2Task.obj
 0002:00003348       ??_R2CalculateSequencesNumberTask@U2@@8 1001a348     Metaphlan2Task.obj
 0002:00003358       ??_R1A@?0A@EA@CalculateSequencesNumberTask@U2@@8 1001a358     Metaphlan2Task.obj
 0002:00003374       ??_R1A@?0A@EA@Task@U2@@8   1001a374     Metaphlan2Task.obj
 0002:00003390       ??_R3Task@U2@@8            1001a390     Metaphlan2Task.obj
 0002:000033a0       ??_R2Task@U2@@8            1001a3a0     Metaphlan2Task.obj
 0002:000033ac       ??_R4ExternalToolRunTask@U2@@6B@ 1001a3ac     Metaphlan2Task.obj
 0002:000033c0       ??_R3ExternalToolRunTask@U2@@8 1001a3c0     Metaphlan2Task.obj
 0002:000033d0       ??_R2ExternalToolRunTask@U2@@8 1001a3d0     Metaphlan2Task.obj
 0002:000033e0       ??_R1A@?0A@EA@ExternalToolRunTask@U2@@8 1001a3e0     Metaphlan2Task.obj
 0002:000033fc       ??_R4Metaphlan2LogParser@U2@@6B@ 1001a3fc     Metaphlan2Task.obj
 0002:00003410       ??_R3Metaphlan2LogParser@U2@@8 1001a410     Metaphlan2Task.obj
 0002:00003420       ??_R2Metaphlan2LogParser@U2@@8 1001a420     Metaphlan2Task.obj
 0002:00003430       ??_R1A@?0A@EA@Metaphlan2LogParser@U2@@8 1001a430     Metaphlan2Task.obj
 0002:0000344c       ??_R1A@?0A@EA@ExternalToolLogParser@U2@@8 1001a44c     Metaphlan2Task.obj
 0002:00003468       ??_R3ExternalToolLogParser@U2@@8 1001a468     Metaphlan2Task.obj
 0002:00003478       ??_R2ExternalToolLogParser@U2@@8 1001a478     Metaphlan2Task.obj
 0002:00003484       ??_R4Metaphlan2ClassifyTask@U2@@6B@ 1001a484     Metaphlan2Task.obj
 0002:00003498       ??_R3Metaphlan2ClassifyTask@U2@@8 1001a498     Metaphlan2Task.obj
 0002:000034a8       ??_R2Metaphlan2ClassifyTask@U2@@8 1001a4a8     Metaphlan2Task.obj
 0002:000034bc       ??_R1A@?0A@EA@Metaphlan2ClassifyTask@U2@@8 1001a4bc     Metaphlan2Task.obj
 0002:000034d8       ??_R1A@?0A@EA@ExternalToolSupportTask@U2@@8 1001a4d8     Metaphlan2Task.obj
 0002:000034f4       ??_R3ExternalToolSupportTask@U2@@8 1001a4f4     Metaphlan2Task.obj
 0002:00003504       ??_R2ExternalToolSupportTask@U2@@8 1001a504     Metaphlan2Task.obj
 0002:00003514       ??_R4FailTask@U2@@6B@      1001a514     Metaphlan2Worker.obj
 0002:00003528       ??_R3FailTask@U2@@8        1001a528     Metaphlan2Worker.obj
 0002:00003538       ??_R2FailTask@U2@@8        1001a538     Metaphlan2Worker.obj
 0002:00003548       ??_R1A@?0A@EA@FailTask@U2@@8 1001a548     Metaphlan2Worker.obj
 0002:00003564       ??_R4TaskSignalMapper@U2@@6B@ 1001a564     Metaphlan2Worker.obj
 0002:00003578       ??_R3TaskSignalMapper@U2@@8 1001a578     Metaphlan2Worker.obj
 0002:00003588       ??_R2TaskSignalMapper@U2@@8 1001a588     Metaphlan2Worker.obj
 0002:00003594       ??_R1A@?0A@EA@TaskSignalMapper@U2@@8 1001a594     Metaphlan2Worker.obj
 0002:000035b0       ??_R4Descriptor@U2@@6B@    1001a5b0     Metaphlan2Worker.obj
 0002:000035c4       ??_R3Descriptor@U2@@8      1001a5c4     Metaphlan2Worker.obj
 0002:000035d4       ??_R2Descriptor@U2@@8      1001a5d4     Metaphlan2Worker.obj
 0002:000035dc       ??_R1A@?0A@EA@Descriptor@U2@@8 1001a5dc     Metaphlan2Worker.obj
 0002:000035f8       ??_R4Metaphlan2Worker@LocalWorkflow@U2@@6BQObject@@@ 1001a5f8     Metaphlan2Worker.obj
 0002:0000360c       ??_R3Metaphlan2Worker@LocalWorkflow@U2@@8 1001a60c     Metaphlan2Worker.obj
 0002:0000361c       ??_R2Metaphlan2Worker@LocalWorkflow@U2@@8 1001a61c     Metaphlan2Worker.obj
 0002:00003634       ??_R1A@?0A@EA@Metaphlan2Worker@LocalWorkflow@U2@@8 1001a634     Metaphlan2Worker.obj
 0002:00003650       ??_R1A@?0A@EA@BaseWorker@LocalWorkflow@U2@@8 1001a650     Metaphlan2Worker.obj
 0002:0000366c       ??_R3BaseWorker@LocalWorkflow@U2@@8 1001a66c     Metaphlan2Worker.obj
 0002:0000367c       ??_R2BaseWorker@LocalWorkflow@U2@@8 1001a67c     Metaphlan2Worker.obj
 0002:00003690       ??_R17?0A@EA@Worker@Workflow@U2@@8 1001a690     Metaphlan2Worker.obj
 0002:000036ac       ??_R3Worker@Workflow@U2@@8 1001a6ac     Metaphlan2Worker.obj
 0002:000036bc       ??_R2Worker@Workflow@U2@@8 1001a6bc     Metaphlan2Worker.obj
 0002:000036c4       ??_R1A@?0A@EA@Worker@Workflow@U2@@8 1001a6c4     Metaphlan2Worker.obj
 0002:000036e0       ??_R1BA@?0A@EA@CommunicationSubject@Workflow@U2@@8 1001a6e0     Metaphlan2Worker.obj
 0002:000036fc       ??_R3CommunicationSubject@Workflow@U2@@8 1001a6fc     Metaphlan2Worker.obj
 0002:0000370c       ??_R2CommunicationSubject@Workflow@U2@@8 1001a70c     Metaphlan2Worker.obj
 0002:00003714       ??_R1A@?0A@EA@CommunicationSubject@Workflow@U2@@8 1001a714     Metaphlan2Worker.obj
 0002:00003730       ??_R4Metaphlan2Worker@LocalWorkflow@U2@@6BWorker@Workflow@2@@ 1001a730     Metaphlan2Worker.obj
 0002:00003744       ??_R4Metaphlan2Worker@LocalWorkflow@U2@@6BCommunicationSubject@Workflow@2@@ 1001a744     Metaphlan2Worker.obj
 0002:00003758       ??_R4VisibilityRelation@U2@@6B@ 1001a758     Metaphlan2WorkerFactory.obj
 0002:0000376c       ??_R3VisibilityRelation@U2@@8 1001a76c     Metaphlan2WorkerFactory.obj
 0002:0000377c       ??_R2VisibilityRelation@U2@@8 1001a77c     Metaphlan2WorkerFactory.obj
 0002:00003788       ??_R1A@?0A@EA@VisibilityRelation@U2@@8 1001a788     Metaphlan2WorkerFactory.obj
 0002:000037a4       ??_R1A@?0A@EA@AttributeRelation@U2@@8 1001a7a4     Metaphlan2WorkerFactory.obj
 0002:000037c0       ??_R3AttributeRelation@U2@@8 1001a7c0     Metaphlan2WorkerFactory.obj
 0002:000037d0       ??_R2AttributeRelation@U2@@8 1001a7d0     Metaphlan2WorkerFactory.obj
 0002:000037d8       ??_R4MapDataType@U2@@6B@   1001a7d8     Metaphlan2WorkerFactory.obj
 0002:000037ec       ??_R3MapDataType@U2@@8     1001a7ec     Metaphlan2WorkerFactory.obj
 0002:000037fc       ??_R2MapDataType@U2@@8     1001a7fc     Metaphlan2WorkerFactory.obj
 0002:00003810       ??_R1A@?0A@EA@MapDataType@U2@@8 1001a810     Metaphlan2WorkerFactory.obj
 0002:0000382c       ??_R1A@?0A@EA@DataType@U2@@8 1001a82c     Metaphlan2WorkerFactory.obj
 0002:00003848       ??_R3DataType@U2@@8        1001a848     Metaphlan2WorkerFactory.obj
 0002:00003858       ??_R2DataType@U2@@8        1001a858     Metaphlan2WorkerFactory.obj
 0002:00003868       ??_R1BA@?0A@EA@QSharedData@@8 1001a868     Metaphlan2WorkerFactory.obj
 0002:00003884       ??_R3QSharedData@@8        1001a884     Metaphlan2WorkerFactory.obj
 0002:00003894       ??_R2QSharedData@@8        1001a894     Metaphlan2WorkerFactory.obj
 0002:0000389c       ??_R1A@?0A@EA@QSharedData@@8 1001a89c     Metaphlan2WorkerFactory.obj
 0002:000038b8       ??_R4SlotRelationDescriptor@U2@@6B@ 1001a8b8     Metaphlan2WorkerFactory.obj
 0002:000038cc       ??_R3SlotRelationDescriptor@U2@@8 1001a8cc     Metaphlan2WorkerFactory.obj
 0002:000038dc       ??_R2SlotRelationDescriptor@U2@@8 1001a8dc     Metaphlan2WorkerFactory.obj
 0002:000038e4       ??_R1A@?0A@EA@SlotRelationDescriptor@U2@@8 1001a8e4     Metaphlan2WorkerFactory.obj
 0002:00003900       ??_R4Attribute@U2@@6B@     1001a900     Metaphlan2WorkerFactory.obj
 0002:00003914       ??_R3Attribute@U2@@8       1001a914     Metaphlan2WorkerFactory.obj
 0002:00003924       ??_R2Attribute@U2@@8       1001a924     Metaphlan2WorkerFactory.obj
 0002:00003930       ??_R1A@?0A@EA@Attribute@U2@@8 1001a930     Metaphlan2WorkerFactory.obj
 0002:0000394c       ??_R3ConfigurationEditor@U2@@8 1001a94c     Metaphlan2WorkerFactory.obj
 0002:0000395c       ??_R2ConfigurationEditor@U2@@8 1001a95c     Metaphlan2WorkerFactory.obj
 0002:00003968       ??_R1A@?0A@EA@ConfigurationEditor@U2@@8 1001a968     Metaphlan2WorkerFactory.obj
 0002:00003984       ??_R4PortDescriptor@Workflow@U2@@6B@ 1001a984     Metaphlan2WorkerFactory.obj
 0002:00003998       ??_R3PortDescriptor@Workflow@U2@@8 1001a998     Metaphlan2WorkerFactory.obj
 0002:000039a8       ??_R2PortDescriptor@Workflow@U2@@8 1001a9a8     Metaphlan2WorkerFactory.obj
 0002:000039b4       ??_R1A@?0A@EA@PortDescriptor@Workflow@U2@@8 1001a9b4     Metaphlan2WorkerFactory.obj
 0002:000039d0       ??_R17?0A@EA@Descriptor@U2@@8 1001a9d0     Metaphlan2WorkerFactory.obj
 0002:000039ec       ??_R4IntegralBusActorPrototype@Workflow@U2@@6B@ 1001a9ec     Metaphlan2WorkerFactory.obj
 0002:00003a00       ??_R3IntegralBusActorPrototype@Workflow@U2@@8 1001aa00     Metaphlan2WorkerFactory.obj
 0002:00003a10       ??_R2IntegralBusActorPrototype@Workflow@U2@@8 1001aa10     Metaphlan2WorkerFactory.obj
 0002:00003a24       ??_R1A@?0A@EA@IntegralBusActorPrototype@Workflow@U2@@8 1001aa24     Metaphlan2WorkerFactory.obj
 0002:00003a40       ??_R1A@?0A@EA@ActorPrototype@Workflow@U2@@8 1001aa40     Metaphlan2WorkerFactory.obj
 0002:00003a5c       ??_R3ActorPrototype@Workflow@U2@@8 1001aa5c     Metaphlan2WorkerFactory.obj
 0002:00003a6c       ??_R2ActorPrototype@Workflow@U2@@8 1001aa6c     Metaphlan2WorkerFactory.obj
 0002:00003a7c       ??_R1A@?0A@EA@VisualDescriptor@U2@@8 1001aa7c     Metaphlan2WorkerFactory.obj
 0002:00003a98       ??_R3VisualDescriptor@U2@@8 1001aa98     Metaphlan2WorkerFactory.obj
 0002:00003aa8       ??_R2VisualDescriptor@U2@@8 1001aaa8     Metaphlan2WorkerFactory.obj
 0002:00003ab4       ??_R4Metaphlan2Validator@Workflow@U2@@6B@ 1001aab4     Metaphlan2WorkerFactory.obj
 0002:00003ac8       ??_R3Metaphlan2Validator@Workflow@U2@@8 1001aac8     Metaphlan2WorkerFactory.obj
 0002:00003ad8       ??_R2Metaphlan2Validator@Workflow@U2@@8 1001aad8     Metaphlan2WorkerFactory.obj
 0002:00003ae8       ??_R1A@?0A@EA@Metaphlan2Validator@Workflow@U2@@8 1001aae8     Metaphlan2WorkerFactory.obj
 0002:00003b04       ??_R1A@?0A@EA@ActorValidator@Workflow@U2@@8 1001ab04     Metaphlan2WorkerFactory.obj
 0002:00003b20       ??_R3ActorValidator@Workflow@U2@@8 1001ab20     Metaphlan2WorkerFactory.obj
 0002:00003b30       ??_R2ActorValidator@Workflow@U2@@8 1001ab30     Metaphlan2WorkerFactory.obj
 0002:00003b3c       ??_R1A@?0A@EA@ConfigurationValidator@U2@@8 1001ab3c     Metaphlan2WorkerFactory.obj
 0002:00003b58       ??_R3ConfigurationValidator@U2@@8 1001ab58     Metaphlan2WorkerFactory.obj
 0002:00003b68       ??_R2ConfigurationValidator@U2@@8 1001ab68     Metaphlan2WorkerFactory.obj
 0002:00003b70       ??_R4Metaphlan2WorkerFactory@LocalWorkflow@U2@@6B?$IdRegistry@VDomainFactory@Workflow@U2@@@2@@ 1001ab70     Metaphlan2WorkerFactory.obj
 0002:00003b84       ??_R3Metaphlan2WorkerFactory@LocalWorkflow@U2@@8 1001ab84     Metaphlan2WorkerFactory.obj
 0002:00003b94       ??_R2Metaphlan2WorkerFactory@LocalWorkflow@U2@@8 1001ab94     Metaphlan2WorkerFactory.obj
 0002:00003ba8       ??_R1A@?0A@EA@Metaphlan2WorkerFactory@LocalWorkflow@U2@@8 1001aba8     Metaphlan2WorkerFactory.obj
 0002:00003bc4       ??_R1A@?0A@EA@DomainFactory@Workflow@U2@@8 1001abc4     Metaphlan2WorkerFactory.obj
 0002:00003be0       ??_R3DomainFactory@Workflow@U2@@8 1001abe0     Metaphlan2WorkerFactory.obj
 0002:00003bf0       ??_R2DomainFactory@Workflow@U2@@8 1001abf0     Metaphlan2WorkerFactory.obj
 0002:00003c00       ??_R1A@?0A@EA@?$IdRegistry@VDomainFactory@Workflow@U2@@@U2@@8 1001ac00     Metaphlan2WorkerFactory.obj
 0002:00003c1c       ??_R3?$IdRegistry@VDomainFactory@Workflow@U2@@@U2@@8 1001ac1c     Metaphlan2WorkerFactory.obj
 0002:00003c2c       ??_R2?$IdRegistry@VDomainFactory@Workflow@U2@@@U2@@8 1001ac2c     Metaphlan2WorkerFactory.obj
 0002:00003c34       ??_R4Metaphlan2WorkerFactory@LocalWorkflow@U2@@6BDescriptor@2@@ 1001ac34     Metaphlan2WorkerFactory.obj
 0002:00003c48       ??_R4PairedReadsPortValidator@Workflow@U2@@6B@ 1001ac48     Metaphlan2WorkerFactory.obj
 0002:00003c5c       ??_R3PairedReadsPortValidator@Workflow@U2@@8 1001ac5c     Metaphlan2WorkerFactory.obj
 0002:00003c6c       ??_R2PairedReadsPortValidator@Workflow@U2@@8 1001ac6c     Metaphlan2WorkerFactory.obj
 0002:00003c7c       ??_R1A@?0A@EA@PairedReadsPortValidator@Workflow@U2@@8 1001ac7c     Metaphlan2WorkerFactory.obj
 0002:00003c98       ??_R1A@?0A@EA@PortValidator@Workflow@U2@@8 1001ac98     Metaphlan2WorkerFactory.obj
 0002:00003cb4       ??_R3PortValidator@Workflow@U2@@8 1001acb4     Metaphlan2WorkerFactory.obj
 0002:00003cc4       ??_R2PortValidator@Workflow@U2@@8 1001acc4     Metaphlan2WorkerFactory.obj
 0002:00003cd0       ??_R4DelegateEditor@U2@@6B@ 1001acd0     Metaphlan2WorkerFactory.obj
 0002:00003ce4       ??_R3DelegateEditor@U2@@8  1001ace4     Metaphlan2WorkerFactory.obj
 0002:00003cf4       ??_R2DelegateEditor@U2@@8  1001acf4     Metaphlan2WorkerFactory.obj
 0002:00003d04       ??_R1A@?0A@EA@DelegateEditor@U2@@8 1001ad04     Metaphlan2WorkerFactory.obj
 0002:00003d20       ??_R4URLDelegate@U2@@6B@   1001ad20     Metaphlan2WorkerFactory.obj
 0002:00003d34       ??_R3URLDelegate@U2@@8     1001ad34     Metaphlan2WorkerFactory.obj
 0002:00003d44       ??_R2URLDelegate@U2@@8     1001ad44     Metaphlan2WorkerFactory.obj
 0002:00003d5c       ??_R1A@?0A@EA@URLDelegate@U2@@8 1001ad5c     Metaphlan2WorkerFactory.obj
 0002:00003d78       ??_R1A@?0A@EA@PropertyDelegate@U2@@8 1001ad78     Metaphlan2WorkerFactory.obj
 0002:00003d94       ??_R3PropertyDelegate@U2@@8 1001ad94     Metaphlan2WorkerFactory.obj
 0002:00003da4       ??_R2PropertyDelegate@U2@@8 1001ada4     Metaphlan2WorkerFactory.obj
 0002:00003db8       ??_R1A@?0A@EA@QItemDelegate@@8 1001adb8     Metaphlan2WorkerFactory.obj
 0002:00003dd4       ??_R3QItemDelegate@@8      1001add4     Metaphlan2WorkerFactory.obj
 0002:00003de4       ??_R2QItemDelegate@@8      1001ade4     Metaphlan2WorkerFactory.obj
 0002:00003df4       ??_R1A@?0A@EA@QAbstractItemDelegate@@8 1001adf4     Metaphlan2WorkerFactory.obj
 0002:00003e10       ??_R3QAbstractItemDelegate@@8 1001ae10     Metaphlan2WorkerFactory.obj
 0002:00003e20       ??_R2QAbstractItemDelegate@@8 1001ae20     Metaphlan2WorkerFactory.obj
 0002:00003e2c       ??_R4SpinBoxDelegate@U2@@6B@ 1001ae2c     Metaphlan2WorkerFactory.obj
 0002:00003e40       ??_R3SpinBoxDelegate@U2@@8 1001ae40     Metaphlan2WorkerFactory.obj
 0002:00003e50       ??_R2SpinBoxDelegate@U2@@8 1001ae50     Metaphlan2WorkerFactory.obj
 0002:00003e68       ??_R1A@?0A@EA@SpinBoxDelegate@U2@@8 1001ae68     Metaphlan2WorkerFactory.obj
 0002:00003e84       ??_R4ComboBoxDelegate@U2@@6B@ 1001ae84     Metaphlan2WorkerFactory.obj
 0002:00003e98       ??_R3ComboBoxDelegate@U2@@8 1001ae98     Metaphlan2WorkerFactory.obj
 0002:00003ea8       ??_R2ComboBoxDelegate@U2@@8 1001aea8     Metaphlan2WorkerFactory.obj
 0002:00003ec0       ??_R1A@?0A@EA@ComboBoxDelegate@U2@@8 1001aec0     Metaphlan2WorkerFactory.obj
 0002:00003edc       ??_R4DatabaseDelegate@LocalWorkflow@U2@@6B@ 1001aedc     Metaphlan2WorkerFactory.obj
 0002:00003ef0       ??_R3DatabaseDelegate@LocalWorkflow@U2@@8 1001aef0     Metaphlan2WorkerFactory.obj
 0002:00003f00       ??_R2DatabaseDelegate@LocalWorkflow@U2@@8 1001af00     Metaphlan2WorkerFactory.obj
 0002:00003f1c       ??_R1A@?0A@EA@DatabaseDelegate@LocalWorkflow@U2@@8 1001af1c     Metaphlan2WorkerFactory.obj
 0002:00003f38       ??_R4type_info@@6B@        1001af38     MSVCRT:ti_inst.obj
 0002:00003f4c       ??_R3type_info@@8          1001af4c     MSVCRT:ti_inst.obj
 0002:00003f5c       ??_R2type_info@@8          1001af5c     MSVCRT:ti_inst.obj
 0002:00003f64       ??_R1A@?0A@EA@type_info@@8 1001af64     MSVCRT:ti_inst.obj
 0002:00003f80       ___safe_se_handler_table   1001af80     <linker-defined>
 0002:00004260       ___rtc_iaa                 1001b260     MSVCRT:initsect.obj
 0002:00004264       ___rtc_izz                 1001b264     MSVCRT:initsect.obj
 0002:00004268       ___rtc_taa                 1001b268     MSVCRT:initsect.obj
 0002:0000426c       ___rtc_tzz                 1001b26c     MSVCRT:initsect.obj
 0002:00007d0c       __IMPORT_DESCRIPTOR_ngs_reads_classification 1001ed0c     ngs_reads_classification:ngs_reads_classification.dll
 0002:00007d20       __IMPORT_DESCRIPTOR_U2Core 1001ed20     U2Core:U2Core.dll
 0002:00007d34       __IMPORT_DESCRIPTOR_U2Formats 1001ed34     U2Formats:U2Formats.dll
 0002:00007d48       __IMPORT_DESCRIPTOR_U2Gui  1001ed48     U2Gui:U2Gui.dll
 0002:00007d5c       __IMPORT_DESCRIPTOR_U2Lang 1001ed5c     U2Lang:U2Lang.dll
 0002:00007d70       __IMPORT_DESCRIPTOR_U2Designer 1001ed70     U2Designer:U2Designer.dll
 0002:00007d84       __IMPORT_DESCRIPTOR_Qt5Widgets 1001ed84     Qt5Widgets:Qt5Widgets.dll
 0002:00007d98       __IMPORT_DESCRIPTOR_Qt5Gui 1001ed98     Qt5Gui:Qt5Gui.dll
 0002:00007dac       __IMPORT_DESCRIPTOR_Qt5Script 1001edac     Qt5Script:Qt5Script.dll
 0002:00007dc0       __IMPORT_DESCRIPTOR_Qt5Core 1001edc0     Qt5Core:Qt5Core.dll
 0002:00007dd4       __IMPORT_DESCRIPTOR_MSVCP120 1001edd4     msvcprt:MSVCP120.dll
 0002:00007de8       __IMPORT_DESCRIPTOR_MSVCR120 1001ede8     MSVCRT:MSVCR120.dll
 0002:00007dfc       __IMPORT_DESCRIPTOR_KERNEL32 1001edfc     kernel32:KERNEL32.dll
 0002:00007e10       __NULL_IMPORT_DESCRIPTOR   1001ee10     ngs_reads_classification:ngs_reads_classification.dll
 0003:00000000       ?_Generic_object@?$_Error_objects@H@std@@2V_Generic_error_category@2@A 10026000     Metaphlan2LogParser.obj
 0003:00000004       ?_Iostream_object@?$_Error_objects@H@std@@2V_Iostream_error_category@2@A 10026004     Metaphlan2LogParser.obj
 0003:00000008       ?_System_object@?$_Error_objects@H@std@@2V_System_error_category@2@A 10026008     Metaphlan2LogParser.obj
 0003:0000000c       ?staticMetaObject@Metaphlan2Prompter@LocalWorkflow@U2@@2UQMetaObject@@B 1002600c     moc_Metaphlan2Prompter.obj
 0003:00000024       ?staticMetaObject@Metaphlan2Support@U2@@2UQMetaObject@@B 10026024     moc_Metaphlan2Support.obj
 0003:0000003c       ?staticMetaObject@MetaphlanSupportPlugin@U2@@2UQMetaObject@@B 1002603c     moc_Metaphlan2SupportPlugin.obj
 0003:00000054       ?staticMetaObject@Metaphlan2ClassifyTask@U2@@2UQMetaObject@@B 10026054     moc_Metaphlan2Task.obj
 0003:0000006c       ?staticMetaObject@Metaphlan2Worker@LocalWorkflow@U2@@2UQMetaObject@@B 1002606c     moc_Metaphlan2Worker.obj
 0003:00000084       ___security_cookie         10026084     MSVCRT:gs_cookie.obj
 0003:00000088       ___security_cookie_complement 10026088     MSVCRT:gs_cookie.obj
 0003:00000090       ___native_dllmain_reason   10026090     MSVCRT:natstart.obj
 0003:00000098       ??_R0?AVerror_category@std@@@8 10026098     Metaphlan2LogParser.obj
 0003:000000bc       ??_R0?AV_Generic_error_category@std@@@8 100260bc     Metaphlan2LogParser.obj
 0003:000000e8       ??_R0?AV_Iostream_error_category@std@@@8 100260e8     Metaphlan2LogParser.obj
 0003:00000114       ??_R0?AV_System_error_category@std@@@8 10026114     Metaphlan2LogParser.obj
 0003:00000140       ??_R0?AVQObject@@@8        10026140     Metaphlan2Prompter.obj
 0003:00000158       ??_R0?AVMetaphlan2Prompter@LocalWorkflow@U2@@@8 10026158     Metaphlan2Prompter.obj
 0003:00000190       ??_R0?AV?$PrompterBase@VMetaphlan2Prompter@LocalWorkflow@U2@@@U2@@@8 10026190     Metaphlan2Prompter.obj
 0003:000001d8       ??_R0?AVPrompterBaseImpl@U2@@@8 100261d8     Metaphlan2Prompter.obj
 0003:000001fc       ??_R0?AVActorDocument@Workflow@U2@@@8 100261fc     Metaphlan2Prompter.obj
 0003:00000224       ??_R0?AVQTextDocument@@@8  10026224     Metaphlan2Prompter.obj
 0003:00000240       ??_R0?AVPrompter@Workflow@U2@@@8 10026240     Metaphlan2Prompter.obj
 0003:00000264       ??_R0?AVMetaphlan2Support@U2@@@8 10026264     Metaphlan2Support.obj
 0003:00000288       ??_R0?AVExternalTool@U2@@@8 10026288     Metaphlan2Support.obj
 0003:000002a8       ??_R0?AVMetaphlanSupportPlugin@U2@@@8 100262a8     Metaphlan2SupportPlugin.obj
 0003:000002d0       ??_R0?AVPlugin@U2@@@8      100262d0     Metaphlan2SupportPlugin.obj
 0003:000002e8       ??_R0?AVCalculateSequencesNumberTask@U2@@@8 100262e8     Metaphlan2Task.obj
 0003:00000318       ??_R0?AVTask@U2@@@8        10026318     Metaphlan2Task.obj
 0003:00000330       ??_R0?AVExternalToolRunTask@U2@@@8 10026330     Metaphlan2Task.obj
 0003:00000358       ??_R0?AVMetaphlan2LogParser@U2@@@8 10026358     Metaphlan2Task.obj
 0003:00000380       ??_R0?AVExternalToolLogParser@U2@@@8 10026380     Metaphlan2Task.obj
 0003:000003a8       ??_R0?AVMetaphlan2ClassifyTask@U2@@@8 100263a8     Metaphlan2Task.obj
 0003:000003d0       ??_R0?AVExternalToolSupportTask@U2@@@8 100263d0     Metaphlan2Task.obj
 0003:000003fc       ??_R0?AVFailTask@U2@@@8    100263fc     Metaphlan2Worker.obj
 0003:00000418       ??_R0?AVTaskSignalMapper@U2@@@8 10026418     Metaphlan2Worker.obj
 0003:0000043c       ??_R0?AVDescriptor@U2@@@8  1002643c     Metaphlan2Worker.obj
 0003:00000458       ??_R0?AVMetaphlan2Worker@LocalWorkflow@U2@@@8 10026458     Metaphlan2Worker.obj
 0003:00000488       ??_R0?AVBaseWorker@LocalWorkflow@U2@@@8 10026488     Metaphlan2Worker.obj
 0003:000004b4       ??_R0?AVWorker@Workflow@U2@@@8 100264b4     Metaphlan2Worker.obj
 0003:000004d8       ??_R0?AVCommunicationSubject@Workflow@U2@@@8 100264d8     Metaphlan2Worker.obj
 0003:00000508       ??_R0?AVVisibilityRelation@U2@@@8 10026508     Metaphlan2WorkerFactory.obj
 0003:0000052c       ??_R0?AVAttributeRelation@U2@@@8 1002652c     Metaphlan2WorkerFactory.obj
 0003:00000550       ??_R0?AVMapDataType@U2@@@8 10026550     Metaphlan2WorkerFactory.obj
 0003:00000570       ??_R0?AVDataType@U2@@@8    10026570     Metaphlan2WorkerFactory.obj
 0003:0000058c       ??_R0?AVQSharedData@@@8    1002658c     Metaphlan2WorkerFactory.obj
 0003:000005a8       ??_R0?AVSlotRelationDescriptor@U2@@@8 100265a8     Metaphlan2WorkerFactory.obj
 0003:000005d0       ??_R0?AVAttribute@U2@@@8   100265d0     Metaphlan2WorkerFactory.obj
 0003:000005ec       ??_R0?AVConfigurationEditor@U2@@@8 100265ec     Metaphlan2WorkerFactory.obj
 0003:00000614       ??_R0?AVPortDescriptor@Workflow@U2@@@8 10026614     Metaphlan2WorkerFactory.obj
 0003:00000640       ??_R0?AVIntegralBusActorPrototype@Workflow@U2@@@8 10026640     Metaphlan2WorkerFactory.obj
 0003:00000674       ??_R0?AVActorPrototype@Workflow@U2@@@8 10026674     Metaphlan2WorkerFactory.obj
 0003:000006a0       ??_R0?AVVisualDescriptor@U2@@@8 100266a0     Metaphlan2WorkerFactory.obj
 0003:000006c4       ??_R0?AVMetaphlan2Validator@Workflow@U2@@@8 100266c4     Metaphlan2WorkerFactory.obj
 0003:000006f4       ??_R0?AVActorValidator@Workflow@U2@@@8 100266f4     Metaphlan2WorkerFactory.obj
 0003:00000720       ??_R0?AVConfigurationValidator@U2@@@8 10026720     Metaphlan2WorkerFactory.obj
 0003:00000748       ??_R0?AVMetaphlan2WorkerFactory@LocalWorkflow@U2@@@8 10026748     Metaphlan2WorkerFactory.obj
 0003:00000780       ??_R0?AVDomainFactory@Workflow@U2@@@8 10026780     Metaphlan2WorkerFactory.obj
 0003:000007a8       ??_R0?AV?$IdRegistry@VDomainFactory@Workflow@U2@@@U2@@@8 100267a8     Metaphlan2WorkerFactory.obj
 0003:000007e4       ??_R0?AVPairedReadsPortValidator@Workflow@U2@@@8 100267e4     Metaphlan2WorkerFactory.obj
 0003:00000818       ??_R0?AVPortValidator@Workflow@U2@@@8 10026818     Metaphlan2WorkerFactory.obj
 0003:00000840       ??_R0?AVDelegateEditor@U2@@@8 10026840     Metaphlan2WorkerFactory.obj
 0003:00000860       ??_R0?AVURLDelegate@U2@@@8 10026860     Metaphlan2WorkerFactory.obj
 0003:00000880       ??_R0?AVPropertyDelegate@U2@@@8 10026880     Metaphlan2WorkerFactory.obj
 0003:000008a4       ??_R0?AVQItemDelegate@@@8  100268a4     Metaphlan2WorkerFactory.obj
 0003:000008c0       ??_R0?AVQAbstractItemDelegate@@@8 100268c0     Metaphlan2WorkerFactory.obj
 0003:000008e4       ??_R0?AVSpinBoxDelegate@U2@@@8 100268e4     Metaphlan2WorkerFactory.obj
 0003:00000908       ??_R0?AVComboBoxDelegate@U2@@@8 10026908     Metaphlan2WorkerFactory.obj
 0003:0000092c       ??_R0?AVDatabaseDelegate@LocalWorkflow@U2@@@8 1002692c     Metaphlan2WorkerFactory.obj
 0003:0000095c       ??_R0?AVtype_info@@@8      1002695c     MSVCRT:ti_inst.obj
 0003:0000098c       ?wellKnownErrors@Metaphlan2LogParser@U2@@0VQStringList@@B 1002698c     Metaphlan2LogParser.obj
 0003:000009c8       ?id@?$num_put@DV?$back_insert_iterator@V?$basic_string@DU?$char_traits@D@std@@V?$allocator@D@2@@std@@@std@@@std@@2V0locale@2@A 100269c8     Metaphlan2LogParser.obj
 0003:000009cc       ?id@?$num_put@_WV?$back_insert_iterator@V?$basic_string@_WU?$char_traits@_W@std@@V?$allocator@_W@2@@std@@@std@@@std@@2V0locale@2@A 100269cc     Metaphlan2LogParser.obj
 0003:00000a58       ?UTIL_SCRIPT@Metaphlan2Support@U2@@2VQString@@B 10026a58     Metaphlan2Support.obj
 0003:00000a64       ?ET_BOWTIE_2_ALIGNER@Metaphlan2Support@U2@@2VQString@@B 10026a64     Metaphlan2Support.obj
 0003:00000a68       ?ET_PYTHON_BIO@Metaphlan2Support@U2@@2VQString@@B 10026a68     Metaphlan2Support.obj
 0003:00000a6c       ?ET_PYTHON_NUMPY@Metaphlan2Support@U2@@2VQString@@B 10026a6c     Metaphlan2Support.obj
 0003:00000a78       ?TOOL_NAME@Metaphlan2Support@U2@@2VQString@@B 10026a78     Metaphlan2Support.obj
 0003:00000a7c       ?ET_PYTHON@Metaphlan2Support@U2@@2VQString@@B 10026a7c     Metaphlan2Support.obj
 0003:00000a84       ?PLUGIN_NAME@MetaphlanSupportPlugin@U2@@2VQString@@B 10026a84     Metaphlan2SupportPlugin.obj
 0003:00000ad0       ?PLUGIN_DESCRIPRION@MetaphlanSupportPlugin@U2@@2VQString@@B 10026ad0     Metaphlan2SupportPlugin.obj
 0003:00000b9c       ?PROFILE_SUFFIX@Metaphlan2Worker@LocalWorkflow@U2@@0VQString@@B 10026b9c     Metaphlan2Worker.obj
 0003:00000ba0       ?PROFILE_DIR@Metaphlan2Worker@LocalWorkflow@U2@@0VQString@@B 10026ba0     Metaphlan2Worker.obj
 0003:00000ba4       ?BOWTIE2OUT_DIR@Metaphlan2Worker@LocalWorkflow@U2@@0VQString@@B 10026ba4     Metaphlan2Worker.obj
 0003:00000be0       ?METAPHLAN2_ROOT_DIR@Metaphlan2Worker@LocalWorkflow@U2@@0VQString@@B 10026be0     Metaphlan2Worker.obj
 0003:00000be4       ?BOWTIE2OUT_SUFFIX@Metaphlan2Worker@LocalWorkflow@U2@@0VQString@@B 10026be4     Metaphlan2Worker.obj
 0003:00000bfc       ?TAX_LEVEL_ORDERS_VALUE@Metaphlan2WorkerFactory@LocalWorkflow@U2@@2VQString@@B 10026bfc     Metaphlan2WorkerFactory.obj
 0003:00000c00       ?TAX_LEVEL_FAMILIES_TEXT@Metaphlan2WorkerFactory@LocalWorkflow@U2@@2VQString@@B 10026c00     Metaphlan2WorkerFactory.obj
 0003:00000c04       ?DB_URL@Metaphlan2WorkerFactory@LocalWorkflow@U2@@2VQString@@B 10026c04     Metaphlan2WorkerFactory.obj
 0003:00000c08       ?INPUT_SLOT@Metaphlan2WorkerFactory@LocalWorkflow@U2@@2VQString@@B 10026c08     Metaphlan2WorkerFactory.obj
 0003:00000c0c       ?TAX_LEVEL_GENERA_TEXT@Metaphlan2WorkerFactory@LocalWorkflow@U2@@2VQString@@B 10026c0c     Metaphlan2WorkerFactory.obj
 0003:00000c10       ?TAX_LEVEL_SPECIES_VALUE@Metaphlan2WorkerFactory@LocalWorkflow@U2@@2VQString@@B 10026c10     Metaphlan2WorkerFactory.obj
 0003:00000c14       ?PAIRED_END@Metaphlan2WorkerFactory@LocalWorkflow@U2@@2VQString@@B 10026c14     Metaphlan2WorkerFactory.obj
 0003:00000c40       ?TAX_LEVEL@Metaphlan2WorkerFactory@LocalWorkflow@U2@@2VQString@@B 10026c40     Metaphlan2WorkerFactory.obj
 0003:00000c44       ?SEQUENCING_READS@Metaphlan2WorkerFactory@LocalWorkflow@U2@@2VQString@@B 10026c44     Metaphlan2WorkerFactory.obj
 0003:00000c48       ?NORMALIZE@Metaphlan2WorkerFactory@LocalWorkflow@U2@@2VQString@@B 10026c48     Metaphlan2WorkerFactory.obj
 0003:00000c4c       ?TAX_LEVEL_FAMILIES_VALUE@Metaphlan2WorkerFactory@LocalWorkflow@U2@@2VQString@@B 10026c4c     Metaphlan2WorkerFactory.obj
 0003:00000c50       ?TAX_LEVEL_KINGDOMS_TEXT@Metaphlan2WorkerFactory@LocalWorkflow@U2@@2VQString@@B 10026c50     Metaphlan2WorkerFactory.obj
 0003:00000c54       ?PAIRED_END_TEXT@Metaphlan2WorkerFactory@LocalWorkflow@U2@@2VQString@@B 10026c54     Metaphlan2WorkerFactory.obj
 0003:00000c58       ?TAX_LEVEL_PHYLA_TEXT@Metaphlan2WorkerFactory@LocalWorkflow@U2@@2VQString@@B 10026c58     Metaphlan2WorkerFactory.obj
 0003:00000c5c       ?ANALYSIS_TYPE_REL_AB_W_READ_STATS_VALUE@Metaphlan2WorkerFactory@LocalWorkflow@U2@@2VQString@@B 10026c5c     Metaphlan2WorkerFactory.obj
 0003:00000c60       ?TAX_LEVEL_GENERA_VALUE@Metaphlan2WorkerFactory@LocalWorkflow@U2@@2VQString@@B 10026c60     Metaphlan2WorkerFactory.obj
 0003:00000c74       ?TAX_LEVEL_ALL_VALUE@Metaphlan2WorkerFactory@LocalWorkflow@U2@@2VQString@@B 10026c74     Metaphlan2WorkerFactory.obj
 0003:00000c78       ?ANALYSIS_TYPE_READS_MAP_TEXT@Metaphlan2WorkerFactory@LocalWorkflow@U2@@2VQString@@B 10026c78     Metaphlan2WorkerFactory.obj
 0003:00000c7c       ?TAX_LEVEL_SPECIES_TEXT@Metaphlan2WorkerFactory@LocalWorkflow@U2@@2VQString@@B 10026c7c     Metaphlan2WorkerFactory.obj
 0003:00000c80       ?SKIP_NORMILIZE_BY_SIZE@Metaphlan2WorkerFactory@LocalWorkflow@U2@@2VQString@@B 10026c80     Metaphlan2WorkerFactory.obj
 0003:00000c84       ?ANALYSIS_TYPE_CLADE_PROFILES_TEXT@Metaphlan2WorkerFactory@LocalWorkflow@U2@@2VQString@@B 10026c84     Metaphlan2WorkerFactory.obj
 0003:00000c88       ?TAX_LEVEL_ALL_TEXT@Metaphlan2WorkerFactory@LocalWorkflow@U2@@2VQString@@B 10026c88     Metaphlan2WorkerFactory.obj
 0003:00000c94       ?ANALYSIS_TYPE_MARKER_AB_TABLE_TEXT@Metaphlan2WorkerFactory@LocalWorkflow@U2@@2VQString@@B 10026c94     Metaphlan2WorkerFactory.obj
 0003:00000c98       ?ANALYSIS_TYPE_REL_AB_VALUE@Metaphlan2WorkerFactory@LocalWorkflow@U2@@2VQString@@B 10026c98     Metaphlan2WorkerFactory.obj
 0003:00000c9c       ?INPUT_PORT_ID@Metaphlan2WorkerFactory@LocalWorkflow@U2@@2VQString@@B 10026c9c     Metaphlan2WorkerFactory.obj
 0003:00000ca0       ?ANALYSIS_TYPE_READS_MAP_VALUE@Metaphlan2WorkerFactory@LocalWorkflow@U2@@2VQString@@B 10026ca0     Metaphlan2WorkerFactory.obj
 0003:00000cac       ?SINGLE_END_TEXT@Metaphlan2WorkerFactory@LocalWorkflow@U2@@2VQString@@B 10026cac     Metaphlan2WorkerFactory.obj
 0003:00000cb0       ?BOWTIE2_OUTPUT_URL@Metaphlan2WorkerFactory@LocalWorkflow@U2@@2VQString@@B 10026cb0     Metaphlan2WorkerFactory.obj
 0003:00000cb4       ?TAX_LEVEL_KINGDOMS_VALUE@Metaphlan2WorkerFactory@LocalWorkflow@U2@@2VQString@@B 10026cb4     Metaphlan2WorkerFactory.obj
 0003:00000cb8       ?TAX_LEVEL_PHYLA_VALUE@Metaphlan2WorkerFactory@LocalWorkflow@U2@@2VQString@@B 10026cb8     Metaphlan2WorkerFactory.obj
 0003:00000cbc       ?ACTOR_ID@Metaphlan2WorkerFactory@LocalWorkflow@U2@@2VQString@@B 10026cbc     Metaphlan2WorkerFactory.obj
 0003:00000cc0       ?PAIRED_INPUT_SLOT@Metaphlan2WorkerFactory@LocalWorkflow@U2@@2VQString@@B 10026cc0     Metaphlan2WorkerFactory.obj
 0003:00000cc4       ?ANALYSIS_TYPE_MARKER_PRES_TABLE_TEXT@Metaphlan2WorkerFactory@LocalWorkflow@U2@@2VQString@@B 10026cc4     Metaphlan2WorkerFactory.obj
 0003:00000cc8       ?ANALYSIS_TYPE_REL_AB_W_READ_STATS_TEXT@Metaphlan2WorkerFactory@LocalWorkflow@U2@@2VQString@@B 10026cc8     Metaphlan2WorkerFactory.obj
 0003:00000ccc       ?ANALYSIS_TYPE_CLADE_PROFILES_VALUE@Metaphlan2WorkerFactory@LocalWorkflow@U2@@2VQString@@B 10026ccc     Metaphlan2WorkerFactory.obj
 0003:00000cd0       ?ANALYSIS_TYPE_MARKER_PRES_TABLE_VALUE@Metaphlan2WorkerFactory@LocalWorkflow@U2@@2VQString@@B 10026cd0     Metaphlan2WorkerFactory.obj
 0003:00000cd4       ?TAX_LEVEL_CLASSES_TEXT@Metaphlan2WorkerFactory@LocalWorkflow@U2@@2VQString@@B 10026cd4     Metaphlan2WorkerFactory.obj
 0003:00000cd8       ?ANALYSIS_TYPE_REL_AB_TEXT@Metaphlan2WorkerFactory@LocalWorkflow@U2@@2VQString@@B 10026cd8     Metaphlan2WorkerFactory.obj
 0003:00000cdc       ?SINGLE_END@Metaphlan2WorkerFactory@LocalWorkflow@U2@@2VQString@@B 10026cdc     Metaphlan2WorkerFactory.obj
 0003:00000ce0       ?NUM_THREADS@Metaphlan2WorkerFactory@LocalWorkflow@U2@@2VQString@@B 10026ce0     Metaphlan2WorkerFactory.obj
 0003:00000ce4       ?ANALYSIS_TYPE@Metaphlan2WorkerFactory@LocalWorkflow@U2@@2VQString@@B 10026ce4     Metaphlan2WorkerFactory.obj
 0003:00000ce8       ?NOT_SKIP_NORMILIZE_BY_SIZE@Metaphlan2WorkerFactory@LocalWorkflow@U2@@2VQString@@B 10026ce8     Metaphlan2WorkerFactory.obj
 0003:00000cec       ?PRESENCE_THRESHOLD@Metaphlan2WorkerFactory@LocalWorkflow@U2@@2VQString@@B 10026cec     Metaphlan2WorkerFactory.obj
 0003:00000cf0       ?TAX_LEVEL_CLASSES_VALUE@Metaphlan2WorkerFactory@LocalWorkflow@U2@@2VQString@@B 10026cf0     Metaphlan2WorkerFactory.obj
 0003:00000cf4       ?OUTPUT_URL@Metaphlan2WorkerFactory@LocalWorkflow@U2@@2VQString@@B 10026cf4     Metaphlan2WorkerFactory.obj
 0003:00000cf8       ?ANALYSIS_TYPE_MARKER_AB_TABLE_VALUE@Metaphlan2WorkerFactory@LocalWorkflow@U2@@2VQString@@B 10026cf8     Metaphlan2WorkerFactory.obj
 0003:00000cfc       ?TAX_LEVEL_ORDERS_TEXT@Metaphlan2WorkerFactory@LocalWorkflow@U2@@2VQString@@B 10026cfc     Metaphlan2WorkerFactory.obj
 0003:00000dec       ?metatype_id@?1??qt_metatype_id@?$QMetaTypeIdQObject@PAVTask@U2@@$00@@SAHXZ@4V?$QBasicAtomicInteger@H@@A 10026dec     moc_Metaphlan2Worker.obj
 0003:00001118       ?__type_info_root_node@@3U__type_info_node@@A 10027118     MSVCRT:tncleanup.obj
 0003:00001120       ___native_startup_lock     10027120     <common>
 0003:00001124       ___native_startup_state    10027124     <common>
 0003:00001128       ___dyn_tls_init_callback   10027128     <common>
 0003:0000112c       ___onexitend               1002712c     <common>
 0003:00001130       ___onexitbegin             10027130     <common>

 entry point at        0001:000113ba

 Static symbols

 0000:fffd3000       .debug$S                   10000000     MSVCRT:MSVCR120.dll
 0000:fffd3000       .debug$S                   10000000     MSVCRT:MSVCR120.dll
 0000:fffd3000       .debug$S                   10000000     MSVCRT:MSVCR120.dll
 0000:fffd3000       .debug$S                   10000000     MSVCRT:MSVCR120.dll
 0000:fffd3000       .debug$S                   10000000     MSVCRT:MSVCR120.dll
 0000:fffd3000       .debug$S                   10000000     MSVCRT:MSVCR120.dll
 0000:fffd3000       .debug$S                   10000000     MSVCRT:MSVCR120.dll
 0000:fffd3000       .debug$S                   10000000     MSVCRT:MSVCR120.dll
 0000:fffd3000       .debug$S                   10000000     MSVCRT:MSVCR120.dll
 0000:fffd3000       .debug$S                   10000000     MSVCRT:MSVCR120.dll
 0000:fffd3000       .debug$S                   10000000     MSVCRT:MSVCR120.dll
 0000:fffd3000       .debug$S                   10000000     MSVCRT:MSVCR120.dll
 0000:fffd3000       .debug$S                   10000000     MSVCRT:MSVCR120.dll
 0000:fffd3000       .debug$S                   10000000     MSVCRT:MSVCR120.dll
 0000:fffd3000       .debug$S                   10000000     MSVCRT:MSVCR120.dll
 0000:fffd3000       .debug$S                   10000000     MSVCRT:MSVCR120.dll
 0000:fffd3000       .debug$S                   10000000     MSVCRT:MSVCR120.dll
 0000:fffd3000       .debug$S                   10000000     MSVCRT:MSVCR120.dll
 0000:fffd3000       .debug$S                   10000000     MSVCRT:MSVCR120.dll
 0000:fffd3000       .debug$S                   10000000     MSVCRT:MSVCR120.dll
 0000:fffd3000       .debug$S                   10000000     MSVCRT:MSVCR120.dll
 0000:fffd3000       .debug$S                   10000000     MSVCRT:MSVCR120.dll
 0000:fffd3000       .debug$S                   10000000     MSVCRT:MSVCR120.dll
 0000:fffd3000       .debug$S                   10000000     MSVCRT:MSVCR120.dll
 0000:fffd3000       .debug$S                   10000000     MSVCRT:MSVCR120.dll
 0000:fffd3000       .debug$S                   10000000     MSVCRT:MSVCR120.dll
 0000:fffd3000       .debug$S                   10000000     msvcprt:MSVCP120.dll
 0000:fffd3000       .debug$S                   10000000     msvcprt:MSVCP120.dll
 0000:fffd3000       .debug$S                   10000000     msvcprt:MSVCP120.dll
 0000:fffd3000       .debug$S                   10000000     msvcprt:MSVCP120.dll
 0000:fffd3000       .debug$S                   10000000     msvcprt:MSVCP120.dll
 0000:fffd3000       .debug$S                   10000000     kernel32:KERNEL32.dll
 0000:fffd3000       .debug$S                   10000000     kernel32:KERNEL32.dll
 0000:fffd3000       .debug$S                   10000000     kernel32:KERNEL32.dll
 0001:fffff000       __ehhandler$?_Copy@?$basic_string@DU?$char_traits@D@std@@V?$allocator@D@2@@std@@QAEXII@Z 10000000 f   moc_Metaphlan2Worker.obj
 0000:fffd3000       .debug$S                   10000000     kernel32:KERNEL32.dll
 0000:fffd3000       .debug$S                   10000000     kernel32:KERNEL32.dll
 0000:fffd3000       .debug$S                   10000000     kernel32:KERNEL32.dll
 0000:fffd3000       .debug$S                   10000000     kernel32:KERNEL32.dll
 0000:fffd3000       .debug$S                   10000000     kernel32:KERNEL32.dll
 0000:fffd3000       .debug$S                   10000000     kernel32:KERNEL32.dll
 0000:fffd3000       .debug$S                   10000000     Qt5Core:Qt5Core.dll
 0000:fffd3000       .debug$S                   10000000     Qt5Core:Qt5Core.dll
 0000:fffd3000       .debug$S                   10000000     Qt5Core:Qt5Core.dll
 0000:fffd3000       .debug$S                   10000000     Qt5Core:Qt5Core.dll
 0000:fffd3000       .debug$S                   10000000     Qt5Core:Qt5Core.dll
 0000:fffd3000       .debug$S                   10000000     Qt5Core:Qt5Core.dll
 0000:fffd3000       .debug$S                   10000000     Qt5Core:Qt5Core.dll
 0000:fffd3000       .debug$S                   10000000     Qt5Core:Qt5Core.dll
 0000:fffd3000       .debug$S                   10000000     Qt5Core:Qt5Core.dll
 0000:fffd3000       .debug$S                   10000000     Qt5Core:Qt5Core.dll
 0000:fffd3000       .debug$S                   10000000     Qt5Core:Qt5Core.dll
 0000:fffd3000       .debug$S                   10000000     Qt5Core:Qt5Core.dll
 0000:fffd3000       .debug$S                   10000000     Qt5Core:Qt5Core.dll
 0000:fffd3000       .debug$S                   10000000     Qt5Core:Qt5Core.dll
 0000:fffd3000       .debug$S                   10000000     Qt5Core:Qt5Core.dll
 0000:fffd3000       .debug$S                   10000000     Qt5Core:Qt5Core.dll
 0000:fffd3000       .debug$S                   10000000     Qt5Core:Qt5Core.dll
 0000:fffd3000       .debug$S                   10000000     Qt5Core:Qt5Core.dll
 0000:fffd3000       .debug$S                   10000000     Qt5Core:Qt5Core.dll
 0002:fffe9000       __catchsym$?_Copy@?$basic_string@DU?$char_traits@D@std@@V?$allocator@D@2@@std@@QAEXII@Z$5 10000000     Metaphlan2WorkerFactory.obj
 0002:fffe9000       __catchsym$?_Copy@?$basic_string@DU?$char_traits@D@std@@V?$allocator@D@2@@std@@QAEXII@Z$5 10000000     moc_Metaphlan2Worker.obj
 0000:fffd3000       .debug$S                   10000000     Qt5Core:Qt5Core.dll
 0000:fffd3000       .debug$S                   10000000     Qt5Core:Qt5Core.dll
 0000:fffd3000       .debug$S                   10000000     Qt5Core:Qt5Core.dll
 0000:fffd3000       .debug$S                   10000000     Qt5Core:Qt5Core.dll
 0000:fffd3000       .debug$S                   10000000     Qt5Core:Qt5Core.dll
 0000:fffd3000       .debug$S                   10000000     Qt5Core:Qt5Core.dll
 0000:fffd3000       .debug$S                   10000000     Qt5Core:Qt5Core.dll
 0000:fffd3000       .debug$S                   10000000     Qt5Core:Qt5Core.dll
 0000:fffd3000       .debug$S                   10000000     Qt5Core:Qt5Core.dll
 0000:fffd3000       .debug$S                   10000000     Qt5Core:Qt5Core.dll
 0000:fffd3000       .debug$S                   10000000     Qt5Core:Qt5Core.dll
 0000:fffd3000       .debug$S                   10000000     Qt5Core:Qt5Core.dll
 0000:fffd3000       .debug$S                   10000000     Qt5Core:Qt5Core.dll
 0000:fffd3000       .debug$S                   10000000     Qt5Core:Qt5Core.dll
 0000:fffd3000       .debug$S                   10000000     Qt5Core:Qt5Core.dll
 0000:fffd3000       .debug$S                   10000000     Qt5Core:Qt5Core.dll
 0000:fffd3000       .debug$S                   10000000     Qt5Core:Qt5Core.dll
 0000:fffd3000       .debug$S                   10000000     Qt5Core:Qt5Core.dll
 0000:fffd3000       .debug$S                   10000000     Qt5Core:Qt5Core.dll
 0000:fffd3000       .debug$S                   10000000     Qt5Core:Qt5Core.dll
 0000:fffd3000       .debug$S                   10000000     Qt5Core:Qt5Core.dll
 0000:fffd3000       .debug$S                   10000000     Qt5Core:Qt5Core.dll
 0000:fffd3000       .debug$S                   10000000     Qt5Core:Qt5Core.dll
 0000:fffd3000       .debug$S                   10000000     Qt5Core:Qt5Core.dll
 0000:fffd3000       .debug$S                   10000000     Qt5Core:Qt5Core.dll
 0000:fffd3000       .debug$S                   10000000     Qt5Core:Qt5Core.dll
 0000:fffd3000       .debug$S                   10000000     Qt5Core:Qt5Core.dll
 0000:fffd3000       .debug$S                   10000000     Qt5Core:Qt5Core.dll
 0000:fffd3000       .debug$S                   10000000     Qt5Core:Qt5Core.dll
 0000:fffd3000       .debug$S                   10000000     Qt5Core:Qt5Core.dll
 0000:fffd3000       .debug$S                   10000000     Qt5Core:Qt5Core.dll
 0000:fffd3000       .debug$S                   10000000     Qt5Core:Qt5Core.dll
 0000:fffd3000       .debug$S                   10000000     Qt5Core:Qt5Core.dll
 0000:fffd3000       .debug$S                   10000000     Qt5Core:Qt5Core.dll
 0000:fffd3000       .debug$S                   10000000     Qt5Core:Qt5Core.dll
 0000:fffd3000       .debug$S                   10000000     Qt5Core:Qt5Core.dll
 0000:fffd3000       .debug$S                   10000000     Qt5Core:Qt5Core.dll
 0000:fffd3000       .debug$S                   10000000     Qt5Core:Qt5Core.dll
 0000:fffd3000       .debug$S                   10000000     Qt5Core:Qt5Core.dll
 0000:fffd3000       .debug$S                   10000000     Qt5Core:Qt5Core.dll
 0000:fffd3000       .debug$S                   10000000     Qt5Core:Qt5Core.dll
 0000:fffd3000       .debug$S                   10000000     Qt5Core:Qt5Core.dll
 0000:fffd3000       .debug$S                   10000000     Qt5Core:Qt5Core.dll
 0002:fffe9000       ?_Generic_object$initializer$@?$_Error_objects@H@std@@2P6AXXZA 10000000     moc_Metaphlan2Worker.obj
 0002:fffe9000       ?_Iostream_object$initializer$@?$_Error_objects@H@std@@2P6AXXZA 10000000     moc_Metaphlan2Worker.obj
 0002:fffe9000       ?_System_object$initializer$@?$_Error_objects@H@std@@2P6AXXZA 10000000     moc_Metaphlan2Worker.obj
 0000:fffd3000       .debug$S                   10000000     Qt5Core:Qt5Core.dll
 0000:fffd3000       .debug$S                   10000000     Qt5Core:Qt5Core.dll
 0000:fffd3000       .debug$S                   10000000     Qt5Core:Qt5Core.dll
 0000:fffd3000       .debug$S                   10000000     Qt5Core:Qt5Core.dll
 0000:fffd3000       .debug$S                   10000000     Qt5Core:Qt5Core.dll
 0000:fffd3000       .debug$S                   10000000     Qt5Core:Qt5Core.dll
 0000:fffd3000       .debug$S                   10000000     Qt5Core:Qt5Core.dll
 0000:fffd3000       .debug$S                   10000000     Qt5Core:Qt5Core.dll
 0000:fffd3000       .debug$S                   10000000     Qt5Core:Qt5Core.dll
 0000:fffd3000       .debug$S                   10000000     Qt5Core:Qt5Core.dll
 0000:fffd3000       .debug$S                   10000000     Qt5Core:Qt5Core.dll
 0000:fffd3000       .debug$S                   10000000     Qt5Core:Qt5Core.dll
 0000:fffd3000       .debug$S                   10000000     Qt5Core:Qt5Core.dll
 0000:fffd3000       .debug$S                   10000000     Qt5Core:Qt5Core.dll
 0000:fffd3000       .debug$S                   10000000     Qt5Core:Qt5Core.dll
 0000:fffd3000       .debug$S                   10000000     Qt5Core:Qt5Core.dll
 0000:fffd3000       .debug$S                   10000000     Qt5Core:Qt5Core.dll
 0000:fffd3000       .debug$S                   10000000     Qt5Core:Qt5Core.dll
 0000:fffd3000       .debug$S                   10000000     Qt5Core:Qt5Core.dll
 0000:fffd3000       .debug$S                   10000000     Qt5Core:Qt5Core.dll
 0000:fffd3000       .debug$S                   10000000     Qt5Core:Qt5Core.dll
 0000:fffd3000       .debug$S                   10000000     Qt5Core:Qt5Core.dll
 0000:fffd3000       .debug$S                   10000000     Qt5Script:Qt5Script.dll
 0000:fffd3000       .debug$S                   10000000     Qt5Script:Qt5Script.dll
 0000:fffd3000       .debug$S                   10000000     Qt5Script:Qt5Script.dll
 0000:fffd3000       .debug$S                   10000000     Qt5Script:Qt5Script.dll
 0000:fffd3000       .debug$S                   10000000     Qt5Script:Qt5Script.dll
 0001:fffff000       __ehhandler$?_Copy@?$basic_string@DU?$char_traits@D@std@@V?$allocator@D@2@@std@@QAEXII@Z 10000000 f   moc_Metaphlan2Task.obj
 0000:fffd3000       .debug$S                   10000000     Qt5Script:Qt5Script.dll
 0000:fffd3000       .debug$S                   10000000     Qt5Script:Qt5Script.dll
 0000:fffd3000       .debug$S                   10000000     Qt5Script:Qt5Script.dll
 0000:fffd3000       .debug$S                   10000000     Qt5Script:Qt5Script.dll
 0000:fffd3000       .debug$S                   10000000     Qt5Script:Qt5Script.dll
 0000:fffd3000       .debug$S                   10000000     Qt5Gui:Qt5Gui.dll
 0000:fffd3000       .debug$S                   10000000     Qt5Gui:Qt5Gui.dll
 0000:fffd3000       .debug$S                   10000000     Qt5Gui:Qt5Gui.dll
 0000:fffd3000       .debug$S                   10000000     Qt5Widgets:Qt5Widgets.dll
 0000:fffd3000       .debug$S                   10000000     Qt5Widgets:Qt5Widgets.dll
 0000:fffd3000       .debug$S                   10000000     Qt5Widgets:Qt5Widgets.dll
 0000:fffd3000       .debug$S                   10000000     Qt5Widgets:Qt5Widgets.dll
 0000:fffd3000       .debug$S                   10000000     Qt5Widgets:Qt5Widgets.dll
 0000:fffd3000       .debug$S                   10000000     Qt5Widgets:Qt5Widgets.dll
 0000:fffd3000       .debug$S                   10000000     Qt5Widgets:Qt5Widgets.dll
 0000:fffd3000       .debug$S                   10000000     Qt5Widgets:Qt5Widgets.dll
 0000:fffd3000       .debug$S                   10000000     Qt5Widgets:Qt5Widgets.dll
 0000:fffd3000       .debug$S                   10000000     Qt5Widgets:Qt5Widgets.dll
 0000:fffd3000       .debug$S                   10000000     Qt5Widgets:Qt5Widgets.dll
 0000:fffd3000       .debug$S                   10000000     Qt5Widgets:Qt5Widgets.dll
 0000:fffd3000       .debug$S                   10000000     U2Designer:U2Designer.dll
 0000:fffd3000       .debug$S                   10000000     U2Designer:U2Designer.dll
 0000:fffd3000       .debug$S                   10000000     U2Designer:U2Designer.dll
 0002:fffe9000       __unwindtable$??A?$QMap@VQString@@VQVariant@@@@QAEAAVQVariant@@ABVQString@@@Z 10000000     Metaphlan2WorkerFactory.obj
 0002:fffe9000       __catchsym$?_Copy@?$basic_string@DU?$char_traits@D@std@@V?$allocator@D@2@@std@@QAEXII@Z$5 10000000     moc_Metaphlan2Task.obj
 0000:fffd3000       .debug$S                   10000000     U2Designer:U2Designer.dll
 0000:fffd3000       .debug$S                   10000000     U2Designer:U2Designer.dll
 0000:fffd3000       .debug$S                   10000000     U2Designer:U2Designer.dll
 0000:fffd3000       .debug$S                   10000000     U2Designer:U2Designer.dll
 0000:fffd3000       .debug$S                   10000000     U2Designer:U2Designer.dll
 0000:fffd3000       .debug$S                   10000000     U2Designer:U2Designer.dll
 0000:fffd3000       .debug$S                   10000000     U2Designer:U2Designer.dll
 0000:fffd3000       .debug$S                   10000000     U2Designer:U2Designer.dll
 0000:fffd3000       .debug$S                   10000000     U2Designer:U2Designer.dll
 0000:fffd3000       .debug$S                   10000000     U2Designer:U2Designer.dll
 0000:fffd3000       .debug$S                   10000000     U2Designer:U2Designer.dll
 0000:fffd3000       .debug$S                   10000000     U2Designer:U2Designer.dll
 0000:fffd3000       .debug$S                   10000000     U2Designer:U2Designer.dll
 0000:fffd3000       .debug$S                   10000000     U2Designer:U2Designer.dll
 0000:fffd3000       .debug$S                   10000000     U2Designer:U2Designer.dll
 0000:fffd3000       .debug$S                   10000000     U2Designer:U2Designer.dll
 0000:fffd3000       .debug$S                   10000000     U2Designer:U2Designer.dll
 0000:fffd3000       .debug$S                   10000000     U2Designer:U2Designer.dll
 0000:fffd3000       .debug$S                   10000000     U2Designer:U2Designer.dll
 0000:fffd3000       .debug$S                   10000000     U2Designer:U2Designer.dll
 0000:fffd3000       .debug$S                   10000000     U2Designer:U2Designer.dll
 0000:fffd3000       .debug$S                   10000000     U2Designer:U2Designer.dll
 0000:fffd3000       .debug$S                   10000000     U2Designer:U2Designer.dll
 0000:fffd3000       .debug$S                   10000000     U2Designer:U2Designer.dll
 0000:fffd3000       .debug$S                   10000000     U2Designer:U2Designer.dll
 0000:fffd3000       .debug$S                   10000000     U2Designer:U2Designer.dll
 0000:fffd3000       .debug$S                   10000000     U2Designer:U2Designer.dll
 0000:fffd3000       .debug$S                   10000000     U2Designer:U2Designer.dll
 0000:fffd3000       .debug$S                   10000000     U2Designer:U2Designer.dll
 0000:fffd3000       .debug$S                   10000000     U2Designer:U2Designer.dll
 0000:fffd3000       .debug$S                   10000000     U2Designer:U2Designer.dll
 0000:fffd3000       .debug$S                   10000000     U2Designer:U2Designer.dll
 0000:fffd3000       .debug$S                   10000000     U2Designer:U2Designer.dll
 0000:fffd3000       .debug$S                   10000000     U2Designer:U2Designer.dll
 0000:fffd3000       .debug$S                   10000000     U2Designer:U2Designer.dll
 0000:fffd3000       .debug$S                   10000000     U2Designer:U2Designer.dll
 0000:fffd3000       .debug$S                   10000000     U2Designer:U2Designer.dll
 0000:fffd3000       .debug$S                   10000000     U2Designer:U2Designer.dll
 0000:fffd3000       .debug$S                   10000000     U2Designer:U2Designer.dll
 0000:fffd3000       .debug$S                   10000000     U2Designer:U2Designer.dll
 0000:fffd3000       .debug$S                   10000000     U2Designer:U2Designer.dll
 0002:fffe9000       ?_Generic_object$initializer$@?$_Error_objects@H@std@@2P6AXXZA 10000000     moc_Metaphlan2Task.obj
 0002:fffe9000       ?_Iostream_object$initializer$@?$_Error_objects@H@std@@2P6AXXZA 10000000     moc_Metaphlan2Task.obj
 0002:fffe9000       ?_System_object$initializer$@?$_Error_objects@H@std@@2P6AXXZA 10000000     moc_Metaphlan2Task.obj
 0000:fffd3000       .debug$S                   10000000     U2Designer:U2Designer.dll
 0000:fffd3000       .debug$S                   10000000     U2Designer:U2Designer.dll
 0000:fffd3000       .debug$S                   10000000     U2Designer:U2Designer.dll
 0000:fffd3000       .debug$S                   10000000     U2Designer:U2Designer.dll
 0000:fffd3000       .debug$S                   10000000     U2Lang:U2Lang.dll
 0000:fffd3000       .debug$S                   10000000     U2Lang:U2Lang.dll
 0000:fffd3000       .debug$S                   10000000     U2Lang:U2Lang.dll
 0000:fffd3000       .debug$S                   10000000     U2Lang:U2Lang.dll
 0000:fffd3000       .debug$S                   10000000     U2Lang:U2Lang.dll
 0001:fffff000       __ehhandler$?_Copy@?$basic_string@DU?$char_traits@D@std@@V?$allocator@D@2@@std@@QAEXII@Z 10000000 f   moc_Metaphlan2SupportPlugin.obj
 0000:fffd3000       .debug$S                   10000000     U2Lang:U2Lang.dll
 0000:fffd3000       .debug$S                   10000000     U2Lang:U2Lang.dll
 0000:fffd3000       .debug$S                   10000000     U2Lang:U2Lang.dll
 0000:fffd3000       .debug$S                   10000000     U2Lang:U2Lang.dll
 0000:fffd3000       .debug$S                   10000000     U2Lang:U2Lang.dll
 0002:fffe9000       __catchsym$?createNode@?$QMapData@VQString@@VQVariant@@@@QAEPAU?$QMapNode@VQString@@VQVariant@@@@ABVQString@@ABVQVariant@@PAU2@_N@Z$7 10000000     Metaphlan2WorkerFactory.obj
 0002:fffe9000       __catchsym$?_Copy@?$basic_string@DU?$char_traits@D@std@@V?$allocator@D@2@@std@@QAEXII@Z$5 10000000     moc_Metaphlan2SupportPlugin.obj
 0000:fffd3000       .debug$S                   10000000     U2Lang:U2Lang.dll
 0000:fffd3000       .debug$S                   10000000     U2Lang:U2Lang.dll
 0000:fffd3000       .debug$S                   10000000     U2Lang:U2Lang.dll
 0000:fffd3000       .debug$S                   10000000     U2Lang:U2Lang.dll
 0000:fffd3000       .debug$S                   10000000     U2Lang:U2Lang.dll
 0002:fffe9000       ?_Generic_object$initializer$@?$_Error_objects@H@std@@2P6AXXZA 10000000     moc_Metaphlan2SupportPlugin.obj
 0002:fffe9000       ?_Iostream_object$initializer$@?$_Error_objects@H@std@@2P6AXXZA 10000000     moc_Metaphlan2SupportPlugin.obj
 0002:fffe9000       ?_System_object$initializer$@?$_Error_objects@H@std@@2P6AXXZA 10000000     moc_Metaphlan2SupportPlugin.obj
 0000:fffd3000       .debug$S                   10000000     U2Lang:U2Lang.dll
 0000:fffd3000       .debug$S                   10000000     U2Lang:U2Lang.dll
 0000:fffd3000       .debug$S                   10000000     U2Lang:U2Lang.dll
 0000:fffd3000       .debug$S                   10000000     U2Lang:U2Lang.dll
 0000:fffd3000       .debug$S                   10000000     U2Lang:U2Lang.dll
 0000:fffd3000       .debug$S                   10000000     U2Lang:U2Lang.dll
 0000:fffd3000       .debug$S                   10000000     U2Lang:U2Lang.dll
 0000:fffd3000       .debug$S                   10000000     U2Lang:U2Lang.dll
 0000:fffd3000       .debug$S                   10000000     U2Lang:U2Lang.dll
 0001:fffff000       __ehhandler$?_Copy@?$basic_string@DU?$char_traits@D@std@@V?$allocator@D@2@@std@@QAEXII@Z 10000000 f   moc_Metaphlan2Support.obj
 0000:fffd3000       .debug$S                   10000000     U2Lang:U2Lang.dll
 0000:fffd3000       .debug$S                   10000000     U2Lang:U2Lang.dll
 0000:fffd3000       .debug$S                   10000000     U2Lang:U2Lang.dll
 0000:fffd3000       .debug$S                   10000000     U2Lang:U2Lang.dll
 0000:fffd3000       .debug$S                   10000000     U2Lang:U2Lang.dll
 0002:fffe9000       ?_Generic_object$initializer$@?$_Error_objects@H@std@@2P6AXXZA 10000000     Metaphlan2WorkerFactory.obj
 0002:fffe9000       __catchsym$?_Copy@?$basic_string@DU?$char_traits@D@std@@V?$allocator@D@2@@std@@QAEXII@Z$5 10000000     moc_Metaphlan2Support.obj
 0000:fffd3000       .debug$S                   10000000     U2Lang:U2Lang.dll
 0000:fffd3000       .debug$S                   10000000     U2Lang:U2Lang.dll
 0000:fffd3000       .debug$S                   10000000     U2Lang:U2Lang.dll
 0000:fffd3000       .debug$S                   10000000     U2Lang:U2Lang.dll
 0000:fffd3000       .debug$S                   10000000     U2Lang:U2Lang.dll
 0002:fffe9000       ?_Generic_object$initializer$@?$_Error_objects@H@std@@2P6AXXZA 10000000     moc_Metaphlan2Support.obj
 0002:fffe9000       ?_Iostream_object$initializer$@?$_Error_objects@H@std@@2P6AXXZA 10000000     moc_Metaphlan2Support.obj
 0002:fffe9000       ?_System_object$initializer$@?$_Error_objects@H@std@@2P6AXXZA 10000000     moc_Metaphlan2Support.obj
 0000:fffd3000       .debug$S                   10000000     U2Lang:U2Lang.dll
 0000:fffd3000       .debug$S                   10000000     U2Lang:U2Lang.dll
 0000:fffd3000       .debug$S                   10000000     U2Lang:U2Lang.dll
 0000:fffd3000       .debug$S                   10000000     U2Lang:U2Lang.dll
 0000:fffd3000       .debug$S                   10000000     U2Lang:U2Lang.dll
 0000:fffd3000       .debug$S                   10000000     U2Lang:U2Lang.dll
 0000:fffd3000       .debug$S                   10000000     U2Lang:U2Lang.dll
 0000:fffd3000       .debug$S                   10000000     U2Lang:U2Lang.dll
 0000:fffd3000       .debug$S                   10000000     U2Lang:U2Lang.dll
 0000:fffd3000       .debug$S                   10000000     U2Lang:U2Lang.dll
 0000:fffd3000       .debug$S                   10000000     U2Lang:U2Lang.dll
 0000:fffd3000       .debug$S                   10000000     U2Lang:U2Lang.dll
 0000:fffd3000       .debug$S                   10000000     U2Lang:U2Lang.dll
 0000:fffd3000       .debug$S                   10000000     U2Lang:U2Lang.dll
 0000:fffd3000       .debug$S                   10000000     U2Lang:U2Lang.dll
 0000:fffd3000       .debug$S                   10000000     U2Lang:U2Lang.dll
 0000:fffd3000       .debug$S                   10000000     U2Lang:U2Lang.dll
 0000:fffd3000       .debug$S                   10000000     U2Lang:U2Lang.dll
 0000:fffd3000       .debug$S                   10000000     U2Lang:U2Lang.dll
 0000:fffd3000       .debug$S                   10000000     U2Lang:U2Lang.dll
 0000:fffd3000       .debug$S                   10000000     U2Lang:U2Lang.dll
 0000:fffd3000       .debug$S                   10000000     U2Lang:U2Lang.dll
 0000:fffd3000       .debug$S                   10000000     U2Lang:U2Lang.dll
 0000:fffd3000       .debug$S                   10000000     U2Lang:U2Lang.dll
 0000:fffd3000       .debug$S                   10000000     U2Lang:U2Lang.dll
 0000:fffd3000       .debug$S                   10000000     U2Lang:U2Lang.dll
 0000:fffd3000       .debug$S                   10000000     U2Lang:U2Lang.dll
 0001:fffff000       __ehhandler$?_Copy@?$basic_string@DU?$char_traits@D@std@@V?$allocator@D@2@@std@@QAEXII@Z 10000000 f   moc_Metaphlan2Prompter.obj
 0000:fffd3000       .debug$S                   10000000     U2Lang:U2Lang.dll
 0000:fffd3000       .debug$S                   10000000     U2Lang:U2Lang.dll
 0000:fffd3000       .debug$S                   10000000     U2Lang:U2Lang.dll
 0000:fffd3000       .debug$S                   10000000     U2Lang:U2Lang.dll
 0000:fffd3000       .debug$S                   10000000     U2Lang:U2Lang.dll
 0000:fffd3000       .debug$S                   10000000     U2Lang:U2Lang.dll
 0000:fffd3000       .debug$S                   10000000     U2Lang:U2Lang.dll
 0000:fffd3000       .debug$S                   10000000     U2Lang:U2Lang.dll
 0000:fffd3000       .debug$S                   10000000     U2Lang:U2Lang.dll
 0000:fffd3000       .debug$S                   10000000     U2Lang:U2Lang.dll
 0000:fffd3000       .debug$S                   10000000     U2Lang:U2Lang.dll
 0000:fffd3000       .debug$S                   10000000     U2Lang:U2Lang.dll
 0000:fffd3000       .debug$S                   10000000     U2Lang:U2Lang.dll
 0000:fffd3000       .debug$S                   10000000     U2Lang:U2Lang.dll
 0000:fffd3000       .debug$S                   10000000     U2Lang:U2Lang.dll
 0000:fffd3000       .debug$S                   10000000     U2Lang:U2Lang.dll
 0000:fffd3000       .debug$S                   10000000     U2Lang:U2Lang.dll
 0000:fffd3000       .debug$S                   10000000     U2Lang:U2Lang.dll
 0000:fffd3000       .debug$S                   10000000     U2Lang:U2Lang.dll
 0000:fffd3000       .debug$S                   10000000     U2Lang:U2Lang.dll
 0000:fffd3000       .debug$S                   10000000     U2Lang:U2Lang.dll
 0000:fffd3000       .debug$S                   10000000     U2Lang:U2Lang.dll
 0000:fffd3000       .debug$S                   10000000     U2Lang:U2Lang.dll
 0002:fffe9000       ?_Iostream_object$initializer$@?$_Error_objects@H@std@@2P6AXXZA 10000000     Metaphlan2WorkerFactory.obj
 0002:fffe9000       __catchsym$?_Copy@?$basic_string@DU?$char_traits@D@std@@V?$allocator@D@2@@std@@QAEXII@Z$5 10000000     moc_Metaphlan2Prompter.obj
 0000:fffd3000       .debug$S                   10000000     U2Lang:U2Lang.dll
 0000:fffd3000       .debug$S                   10000000     U2Lang:U2Lang.dll
 0000:fffd3000       .debug$S                   10000000     U2Lang:U2Lang.dll
 0000:fffd3000       .debug$S                   10000000     U2Lang:U2Lang.dll
 0000:fffd3000       .debug$S                   10000000     U2Lang:U2Lang.dll
 0000:fffd3000       .debug$S                   10000000     U2Lang:U2Lang.dll
 0000:fffd3000       .debug$S                   10000000     U2Lang:U2Lang.dll
 0000:fffd3000       .debug$S                   10000000     U2Lang:U2Lang.dll
 0000:fffd3000       .debug$S                   10000000     U2Lang:U2Lang.dll
 0000:fffd3000       .debug$S                   10000000     U2Lang:U2Lang.dll
 0000:fffd3000       .debug$S                   10000000     U2Lang:U2Lang.dll
 0000:fffd3000       .debug$S                   10000000     U2Lang:U2Lang.dll
 0000:fffd3000       .debug$S                   10000000     U2Lang:U2Lang.dll
 0000:fffd3000       .debug$S                   10000000     U2Lang:U2Lang.dll
 0000:fffd3000       .debug$S                   10000000     U2Lang:U2Lang.dll
 0000:fffd3000       .debug$S                   10000000     U2Lang:U2Lang.dll
 0000:fffd3000       .debug$S                   10000000     U2Lang:U2Lang.dll
 0000:fffd3000       .debug$S                   10000000     U2Lang:U2Lang.dll
 0000:fffd3000       .debug$S                   10000000     U2Lang:U2Lang.dll
 0000:fffd3000       .debug$S                   10000000     U2Lang:U2Lang.dll
 0000:fffd3000       .debug$S                   10000000     U2Lang:U2Lang.dll
 0000:fffd3000       .debug$S                   10000000     U2Lang:U2Lang.dll
 0000:fffd3000       .debug$S                   10000000     U2Lang:U2Lang.dll
 0000:fffd3000       .debug$S                   10000000     U2Lang:U2Lang.dll
 0000:fffd3000       .debug$S                   10000000     U2Lang:U2Lang.dll
 0000:fffd3000       .debug$S                   10000000     U2Lang:U2Lang.dll
 0000:fffd3000       .debug$S                   10000000     U2Lang:U2Lang.dll
 0000:fffd3000       .debug$S                   10000000     U2Lang:U2Lang.dll
 0000:fffd3000       .debug$S                   10000000     U2Lang:U2Lang.dll
 0000:fffd3000       .debug$S                   10000000     U2Lang:U2Lang.dll
 0000:fffd3000       .debug$S                   10000000     U2Lang:U2Lang.dll
 0000:fffd3000       .debug$S                   10000000     U2Lang:U2Lang.dll
 0000:fffd3000       .debug$S                   10000000     U2Lang:U2Lang.dll
 0000:fffd3000       .debug$S                   10000000     U2Lang:U2Lang.dll
 0000:fffd3000       .debug$S                   10000000     U2Lang:U2Lang.dll
 0000:fffd3000       .debug$S                   10000000     U2Lang:U2Lang.dll
 0000:fffd3000       .debug$S                   10000000     U2Lang:U2Lang.dll
 0000:fffd3000       .debug$S                   10000000     U2Lang:U2Lang.dll
 0000:fffd3000       .debug$S                   10000000     U2Lang:U2Lang.dll
 0000:fffd3000       .debug$S                   10000000     U2Lang:U2Lang.dll
 0000:fffd3000       .debug$S                   10000000     U2Lang:U2Lang.dll
 0002:fffe9000       ?_Generic_object$initializer$@?$_Error_objects@H@std@@2P6AXXZA 10000000     moc_Metaphlan2Prompter.obj
 0002:fffe9000       ?_Iostream_object$initializer$@?$_Error_objects@H@std@@2P6AXXZA 10000000     moc_Metaphlan2Prompter.obj
 0002:fffe9000       ?_System_object$initializer$@?$_Error_objects@H@std@@2P6AXXZA 10000000     moc_Metaphlan2Prompter.obj
 0000:fffd3000       .debug$S                   10000000     U2Lang:U2Lang.dll
 0000:fffd3000       .debug$S                   10000000     U2Lang:U2Lang.dll
 0000:fffd3000       .debug$S                   10000000     U2Lang:U2Lang.dll
 0000:fffd3000       .debug$S                   10000000     U2Lang:U2Lang.dll
 0000:fffd3000       .debug$S                   10000000     U2Lang:U2Lang.dll
 0000:fffd3000       .debug$S                   10000000     U2Lang:U2Lang.dll
 0000:fffd3000       .debug$S                   10000000     U2Lang:U2Lang.dll
 0000:fffd3000       .debug$S                   10000000     U2Lang:U2Lang.dll
 0000:fffd3000       .debug$S                   10000000     U2Lang:U2Lang.dll
 0000:fffd3000       .debug$S                   10000000     U2Lang:U2Lang.dll
 0000:fffd3000       .debug$S                   10000000     U2Lang:U2Lang.dll
 0000:fffd3000       .debug$S                   10000000     U2Gui:U2Gui.dll
 0000:fffd3000       .debug$S                   10000000     U2Formats:U2Formats.dll
 0000:fffd3000       .debug$S                   10000000     U2Formats:U2Formats.dll
 0000:fffd3000       .debug$S                   10000000     U2Formats:U2Formats.dll
 0000:fffd3000       .debug$S                   10000000     U2Formats:U2Formats.dll
 0000:fffd3000       .debug$S                   10000000     U2Core:U2Core.dll
 0000:fffd3000       .debug$S                   10000000     U2Core:U2Core.dll
 0000:fffd3000       .debug$S                   10000000     U2Core:U2Core.dll
 0000:fffd3000       .debug$S                   10000000     U2Core:U2Core.dll
 0000:fffd3000       .debug$S                   10000000     U2Core:U2Core.dll
 0000:fffd3000       .debug$S                   10000000     U2Core:U2Core.dll
 0000:fffd3000       .debug$S                   10000000     U2Core:U2Core.dll
 0000:fffd3000       .debug$S                   10000000     U2Core:U2Core.dll
 0000:fffd3000       .debug$S                   10000000     U2Core:U2Core.dll
 0000:fffd3000       .debug$S                   10000000     U2Core:U2Core.dll
 0000:fffd3000       .debug$S                   10000000     U2Core:U2Core.dll
 0000:fffd3000       .debug$S                   10000000     U2Core:U2Core.dll
 0000:fffd3000       .debug$S                   10000000     U2Core:U2Core.dll
 0000:fffd3000       .debug$S                   10000000     U2Core:U2Core.dll
 0000:fffd3000       .debug$S                   10000000     U2Core:U2Core.dll
 0000:fffd3000       .debug$S                   10000000     U2Core:U2Core.dll
 0000:fffd3000       .debug$S                   10000000     U2Core:U2Core.dll
 0000:fffd3000       .debug$S                   10000000     U2Core:U2Core.dll
 0000:fffd3000       .debug$S                   10000000     U2Core:U2Core.dll
 0000:fffd3000       .debug$S                   10000000     U2Core:U2Core.dll
 0000:fffd3000       .debug$S                   10000000     U2Core:U2Core.dll
 0000:fffd3000       .debug$S                   10000000     U2Core:U2Core.dll
 0000:fffd3000       .debug$S                   10000000     U2Core:U2Core.dll
 0000:fffd3000       .debug$S                   10000000     U2Core:U2Core.dll
 0000:fffd3000       .debug$S                   10000000     U2Core:U2Core.dll
 0000:fffd3000       .debug$S                   10000000     U2Core:U2Core.dll
 0000:fffd3000       .debug$S                   10000000     U2Core:U2Core.dll
 0000:fffd3000       .debug$S                   10000000     U2Core:U2Core.dll
 0000:fffd3000       .debug$S                   10000000     U2Core:U2Core.dll
 0000:fffd3000       .debug$S                   10000000     U2Core:U2Core.dll
 0000:fffd3000       .debug$S                   10000000     U2Core:U2Core.dll
 0000:fffd3000       .debug$S                   10000000     U2Core:U2Core.dll
 0000:fffd3000       .debug$S                   10000000     U2Core:U2Core.dll
 0000:fffd3000       .debug$S                   10000000     U2Core:U2Core.dll
 0000:fffd3000       .debug$S                   10000000     U2Core:U2Core.dll
 0000:fffd3000       .debug$S                   10000000     U2Core:U2Core.dll
 0000:fffd3000       .debug$S                   10000000     U2Core:U2Core.dll
 0000:fffd3000       .debug$S                   10000000     U2Core:U2Core.dll
 0000:fffd3000       .debug$S                   10000000     U2Core:U2Core.dll
 0000:fffd3000       .debug$S                   10000000     U2Core:U2Core.dll
 0000:fffd3000       .debug$S                   10000000     U2Core:U2Core.dll
 0000:fffd3000       .debug$S                   10000000     U2Core:U2Core.dll
 0000:fffd3000       .debug$S                   10000000     U2Core:U2Core.dll
 0000:fffd3000       .debug$S                   10000000     U2Core:U2Core.dll
 0000:fffd3000       .debug$S                   10000000     U2Core:U2Core.dll
 0000:fffd3000       .debug$S                   10000000     U2Core:U2Core.dll
 0000:fffd3000       .debug$S                   10000000     U2Core:U2Core.dll
 0000:fffd3000       .debug$S                   10000000     U2Core:U2Core.dll
 0000:fffd3000       .debug$S                   10000000     U2Core:U2Core.dll
 0000:fffd3000       .debug$S                   10000000     U2Core:U2Core.dll
 0000:fffd3000       .debug$S                   10000000     U2Core:U2Core.dll
 0000:fffd3000       .debug$S                   10000000     U2Core:U2Core.dll
 0000:fffd3000       .debug$S                   10000000     U2Core:U2Core.dll
 0000:fffd3000       .debug$S                   10000000     U2Core:U2Core.dll
 0000:fffd3000       .debug$S                   10000000     U2Core:U2Core.dll
 0000:fffd3000       .debug$S                   10000000     U2Core:U2Core.dll
 0000:fffd3000       .debug$S                   10000000     U2Core:U2Core.dll
 0000:fffd3000       .debug$S                   10000000     U2Core:U2Core.dll
 0000:fffd3000       .debug$S                   10000000     U2Core:U2Core.dll
 0000:fffd3000       .debug$S                   10000000     U2Core:U2Core.dll
 0000:fffd3000       .debug$S                   10000000     U2Core:U2Core.dll
 0000:fffd3000       .debug$S                   10000000     U2Core:U2Core.dll
 0000:fffd3000       .debug$S                   10000000     U2Core:U2Core.dll
 0000:fffd3000       .debug$S                   10000000     U2Core:U2Core.dll
 0000:fffd3000       .debug$S                   10000000     U2Core:U2Core.dll
 0000:fffd3000       .debug$S                   10000000     U2Core:U2Core.dll
 0000:fffd3000       .debug$S                   10000000     U2Core:U2Core.dll
 0000:fffd3000       .debug$S                   10000000     U2Core:U2Core.dll
 0000:fffd3000       .debug$S                   10000000     U2Core:U2Core.dll
 0000:fffd3000       .debug$S                   10000000     U2Core:U2Core.dll
 0000:fffd3000       .debug$S                   10000000     U2Core:U2Core.dll
 0000:fffd3000       .debug$S                   10000000     U2Core:U2Core.dll
 0000:fffd3000       .debug$S                   10000000     U2Core:U2Core.dll
 0000:fffd3000       .debug$S                   10000000     U2Core:U2Core.dll
 0000:fffd3000       .debug$S                   10000000     U2Core:U2Core.dll
 0000:fffd3000       .debug$S                   10000000     U2Core:U2Core.dll
 0000:fffd3000       .debug$S                   10000000     U2Core:U2Core.dll
 0000:fffd3000       .debug$S                   10000000     U2Core:U2Core.dll
 0000:fffd3000       .debug$S                   10000000     U2Core:U2Core.dll
 0000:fffd3000       .debug$S                   10000000     U2Core:U2Core.dll
 0000:fffd3000       .debug$S                   10000000     U2Core:U2Core.dll
 0000:fffd3000       .debug$S                   10000000     U2Core:U2Core.dll
 0000:fffd3000       .debug$S                   10000000     U2Core:U2Core.dll
 0000:fffd3000       .debug$S                   10000000     U2Core:U2Core.dll
 0000:fffd3000       .debug$S                   10000000     U2Core:U2Core.dll
 0000:fffd3000       .debug$S                   10000000     U2Core:U2Core.dll
 0000:fffd3000       .debug$S                   10000000     U2Core:U2Core.dll
 0000:fffd3000       .debug$S                   10000000     U2Core:U2Core.dll
 0000:fffd3000       .debug$S                   10000000     U2Core:U2Core.dll
 0000:fffd3000       .debug$S                   10000000     U2Core:U2Core.dll
 0000:fffd3000       .debug$S                   10000000     U2Core:U2Core.dll
 0000:fffd3000       .debug$S                   10000000     U2Core:U2Core.dll
 0000:fffd3000       .debug$S                   10000000     U2Core:U2Core.dll
 0000:fffd3000       .debug$S                   10000000     U2Core:U2Core.dll
 0000:fffd3000       .debug$S                   10000000     U2Core:U2Core.dll
 0000:fffd3000       .debug$S                   10000000     U2Core:U2Core.dll
 0000:fffd3000       .debug$S                   10000000     U2Core:U2Core.dll
 0000:fffd3000       .debug$S                   10000000     U2Core:U2Core.dll
 0000:fffd3000       .debug$S                   10000000     U2Core:U2Core.dll
 0000:fffd3000       .debug$S                   10000000     U2Core:U2Core.dll
 0000:fffd3000       .debug$S                   10000000     U2Core:U2Core.dll
 0000:fffd3000       .debug$S                   10000000     U2Core:U2Core.dll
 0001:fffff000       __ehhandler$?_Copy@?$basic_string@DU?$char_traits@D@std@@V?$allocator@D@2@@std@@QAEXII@Z 10000000 f   Metaphlan2WorkerFactory.obj
 0000:fffd3000       .debug$S                   10000000     U2Core:U2Core.dll
 0000:fffd3000       .debug$S                   10000000     U2Core:U2Core.dll
 0000:fffd3000       .debug$S                   10000000     U2Core:U2Core.dll
 0000:fffd3000       .debug$S                   10000000     U2Core:U2Core.dll
 0000:fffd3000       .debug$S                   10000000     U2Core:U2Core.dll
 0002:fffe9000       ?_System_object$initializer$@?$_Error_objects@H@std@@2P6AXXZA 10000000     Metaphlan2WorkerFactory.obj
 0001:fffff000       __unwindfunclet$??A?$QMap@VQString@@VQVariant@@@@QAEAAVQVariant@@ABVQString@@@Z$0 10000000 f   Metaphlan2WorkerFactory.obj
 0000:fffd3000       .debug$S                   10000000     ngs_reads_classification:ngs_reads_classification.dll
 0000:fffd3000       .debug$S                   10000000     ngs_reads_classification:ngs_reads_classification.dll
 0000:fffd3000       .debug$S                   10000000     ngs_reads_classification:ngs_reads_classification.dll
 0000:fffd3000       .debug$S                   10000000     ngs_reads_classification:ngs_reads_classification.dll
 0000:fffd3000       .debug$S                   10000000     ngs_reads_classification:ngs_reads_classification.dll
 0000:fffd3000       .debug$S                   10000000     ngs_reads_classification:ngs_reads_classification.dll
 0000:fffd3000       .debug$S                   10000000     ngs_reads_classification:ngs_reads_classification.dll
 0002:fffe9000       ?_System_object$initializer$@?$_Error_objects@H@std@@2P6AXXZA 10000000     Metaphlan2Prompter.obj
 0002:fffe9000       ?_Iostream_object$initializer$@?$_Error_objects@H@std@@2P6AXXZA 10000000     Metaphlan2Prompter.obj
 0002:fffe9000       ?_Generic_object$initializer$@?$_Error_objects@H@std@@2P6AXXZA 10000000     Metaphlan2Prompter.obj
 0002:fffe9000       __catchsym$?_Copy@?$basic_string@DU?$char_traits@D@std@@V?$allocator@D@2@@std@@QAEXII@Z$5 10000000     Metaphlan2Prompter.obj
 0001:fffff000       __ehhandler$?_Copy@?$basic_string@DU?$char_traits@D@std@@V?$allocator@D@2@@std@@QAEXII@Z 10000000 f   Metaphlan2Worker.obj
 0001:fffff000       __ehhandler$?_Copy@?$basic_string@DU?$char_traits@D@std@@V?$allocator@D@2@@std@@QAEXII@Z 10000000 f   Metaphlan2Prompter.obj
 0002:fffe9000       ?_System_object$initializer$@?$_Error_objects@H@std@@2P6AXXZA 10000000     Metaphlan2Support.obj
 0002:fffe9000       ?_Iostream_object$initializer$@?$_Error_objects@H@std@@2P6AXXZA 10000000     Metaphlan2Support.obj
 0002:fffe9000       ?_Generic_object$initializer$@?$_Error_objects@H@std@@2P6AXXZA 10000000     Metaphlan2Support.obj
 0002:fffe9000       __catchsym$?node_copy@?$QList@VQString@@@@AAEXPAUNode@1@00@Z$6 10000000     Metaphlan2Support.obj
 0001:fffff000       __unwindfunclet$?append@?$QList@VQString@@@@QAEXABVQString@@@Z$7 10000000 f   Metaphlan2Worker.obj
 0002:fffe9000       __unwindtable$?node_construct@?$QList@VQString@@@@AAEXPAUNode@1@ABVQString@@@Z 10000000     Metaphlan2Support.obj
 0001:fffff000       __ehhandler$?detach_helper_grow@?$QList@VQString@@@@AAEPAUNode@1@HH@Z 10000000 f   Metaphlan2Worker.obj
 0002:fffe9000       __catchsym$?detach_helper_grow@?$QList@VQString@@@@AAEPAUNode@1@HH@Z$5 10000000     Metaphlan2Support.obj
 0001:fffff000       __unwindfunclet$?node_construct@?$QList@VQString@@@@AAEXPAUNode@1@ABVQString@@@Z$1 10000000 f   Metaphlan2Worker.obj
 0002:fffe9000       __catchsym$?append@?$QList@VQString@@@@QAEXABVQString@@@Z$13 10000000     Metaphlan2Support.obj
 0001:fffff000       __unwindfunclet$?node_copy@?$QList@VQString@@@@AAEXPAUNode@1@00@Z$5 10000000 f   Metaphlan2Worker.obj
 0002:fffe9000       __catchsym$?_Copy@?$basic_string@DU?$char_traits@D@std@@V?$allocator@D@2@@std@@QAEXII@Z$5 10000000     Metaphlan2Support.obj
 0001:fffff000       __unwindfunclet$??1Metaphlan2TaskSettings@U2@@QAE@XZ$0 10000000 f   Metaphlan2Worker.obj
 0001:fffff000       __unwindfunclet$?node_copy@?$QList@VQString@@@@AAEXPAUNode@1@00@Z$5 10000000 f   Metaphlan2Support.obj
 0001:fffff000       __unwindfunclet$?node_construct@?$QList@VQString@@@@AAEXPAUNode@1@ABVQString@@@Z$1 10000000 f   Metaphlan2Support.obj
 0001:fffff000       __ehhandler$?detach_helper_grow@?$QList@VQString@@@@AAEPAUNode@1@HH@Z 10000000 f   Metaphlan2Support.obj
 0001:fffff000       __unwindfunclet$?append@?$QList@VQString@@@@QAEXABVQString@@@Z$7 10000000 f   Metaphlan2Support.obj
 0001:fffff000       __ehhandler$?_Copy@?$basic_string@DU?$char_traits@D@std@@V?$allocator@D@2@@std@@QAEXII@Z 10000000 f   Metaphlan2Support.obj
 0002:fffe9000       ?_System_object$initializer$@?$_Error_objects@H@std@@2P6AXXZA 10000000     Metaphlan2SupportPlugin.obj
 0002:fffe9000       ?_Iostream_object$initializer$@?$_Error_objects@H@std@@2P6AXXZA 10000000     Metaphlan2SupportPlugin.obj
 0002:fffe9000       ?_Generic_object$initializer$@?$_Error_objects@H@std@@2P6AXXZA 10000000     Metaphlan2SupportPlugin.obj
 0002:fffe9000       __catchsym$?_Copy@?$basic_string@DU?$char_traits@D@std@@V?$allocator@D@2@@std@@QAEXII@Z$5 10000000     Metaphlan2SupportPlugin.obj
 0001:fffff000       __unwindfunclet$??0Metaphlan2TaskSettings@U2@@QAE@ABU01@@Z$0 10000000 f   Metaphlan2Worker.obj
 0001:fffff000       __ehhandler$?_Copy@?$basic_string@DU?$char_traits@D@std@@V?$allocator@D@2@@std@@QAEXII@Z 10000000 f   Metaphlan2SupportPlugin.obj
 0002:fffe9000       ?_System_object$initializer$@?$_Error_objects@H@std@@2P6AXXZA 10000000     Metaphlan2Task.obj
 0002:fffe9000       ?_Iostream_object$initializer$@?$_Error_objects@H@std@@2P6AXXZA 10000000     Metaphlan2Task.obj
 0002:fffe9000       ?_Generic_object$initializer$@?$_Error_objects@H@std@@2P6AXXZA 10000000     Metaphlan2Task.obj
 0002:fffe9000       __catchsym$?node_copy@?$QList@VQString@@@@AAEXPAUNode@1@00@Z$6 10000000     Metaphlan2Task.obj
 0001:fffff000       __unwindfunclet$?metaType@?$QVariantValueHelper@VQString@@@QtPrivate@@SA?AVQString@@ABVQVariant@@@Z$0 10000000 f   Metaphlan2Worker.obj
 0002:fffe9000       __unwindtable$?node_construct@?$QList@VQString@@@@AAEXPAUNode@1@ABVQString@@@Z 10000000     Metaphlan2Task.obj
 0002:fffe9000       __catchsym$?_Copy@?$basic_string@DU?$char_traits@D@std@@V?$allocator@D@2@@std@@QAEXII@Z$5 10000000     Metaphlan2Worker.obj
 0002:fffe9000       __catchsym$?detach_helper_grow@?$QList@VQString@@@@AAEPAUNode@1@HH@Z$5 10000000     Metaphlan2Task.obj
 0002:fffe9000       __catchsym$?append@?$QList@VQString@@@@QAEXABVQString@@@Z$13 10000000     Metaphlan2Worker.obj
 0002:fffe9000       __catchsym$?append@?$QList@VQString@@@@QAEXABVQString@@@Z$13 10000000     Metaphlan2Task.obj
 0002:fffe9000       __catchsym$?detach_helper_grow@?$QList@VQString@@@@AAEPAUNode@1@HH@Z$5 10000000     Metaphlan2Worker.obj
 0002:fffe9000       __catchsym$??0?$QList@VQString@@@@QAE@ABV0@@Z$2 10000000     Metaphlan2Task.obj
 0002:fffe9000       __unwindtable$?node_construct@?$QList@VQString@@@@AAEXPAUNode@1@ABVQString@@@Z 10000000     Metaphlan2Worker.obj
 0002:fffe9000       __catchsym$?_Copy@?$basic_string@DU?$char_traits@D@std@@V?$allocator@D@2@@std@@QAEXII@Z$5 10000000     Metaphlan2Task.obj
 0002:fffe9000       __catchsym$?node_copy@?$QList@VQString@@@@AAEXPAUNode@1@00@Z$6 10000000     Metaphlan2Worker.obj
 0001:fffff000       __unwindfunclet$?node_copy@?$QList@VQString@@@@AAEXPAUNode@1@00@Z$5 10000000 f   Metaphlan2Task.obj
 0001:fffff000       __unwindfunclet$?node_construct@?$QList@VQString@@@@AAEXPAUNode@1@ABVQString@@@Z$1 10000000 f   Metaphlan2Task.obj
 0001:fffff000       __ehhandler$?detach_helper_grow@?$QList@VQString@@@@AAEPAUNode@1@HH@Z 10000000 f   Metaphlan2Task.obj
 0001:fffff000       __unwindfunclet$?append@?$QList@VQString@@@@QAEXABVQString@@@Z$7 10000000 f   Metaphlan2Task.obj
 0001:fffff000       __ehhandler$??0?$QList@VQString@@@@QAE@ABV0@@Z 10000000 f   Metaphlan2Task.obj
 0001:fffff000       __ehhandler$?_Copy@?$basic_string@DU?$char_traits@D@std@@V?$allocator@D@2@@std@@QAEXII@Z 10000000 f   Metaphlan2Task.obj
 0002:fffe9000       ?_System_object$initializer$@?$_Error_objects@H@std@@2P6AXXZA 10000000     Metaphlan2Validator.obj
 0002:fffe9000       ?_Iostream_object$initializer$@?$_Error_objects@H@std@@2P6AXXZA 10000000     Metaphlan2Validator.obj
 0002:fffe9000       ?_Generic_object$initializer$@?$_Error_objects@H@std@@2P6AXXZA 10000000     Metaphlan2Validator.obj
 0002:fffe9000       __catchsym$?node_copy@?$QList@VQString@@@@AAEXPAUNode@1@00@Z$6 10000000     Metaphlan2Validator.obj
 0002:fffe9000       __ehfuncinfo$??1Metaphlan2TaskSettings@U2@@QAE@XZ 10000000     Metaphlan2Worker.obj
 0002:fffe9000       __unwindtable$?node_construct@?$QList@VQString@@@@AAEXPAUNode@1@ABVQString@@@Z 10000000     Metaphlan2Validator.obj
 0002:fffe9000       __ehfuncinfo$??0Metaphlan2TaskSettings@U2@@QAE@ABU01@@Z 10000000     Metaphlan2Worker.obj
 0002:fffe9000       __catchsym$?detach_helper_grow@?$QList@VQString@@@@AAEPAUNode@1@HH@Z$5 10000000     Metaphlan2Validator.obj
 0002:fffe9000       __unwindtable$?metaType@?$QVariantValueHelper@VQString@@@QtPrivate@@SA?AVQString@@ABVQVariant@@@Z 10000000     Metaphlan2Worker.obj
 0002:fffe9000       __catchsym$?append@?$QList@VQString@@@@QAEXABVQString@@@Z$13 10000000     Metaphlan2Validator.obj
 0002:fffe9000       ?_Generic_object$initializer$@?$_Error_objects@H@std@@2P6AXXZA 10000000     Metaphlan2Worker.obj
 0002:fffe9000       __catchsym$??0?$QList@VQString@@@@QAE@ABV0@@Z$2 10000000     Metaphlan2Validator.obj
 0002:fffe9000       ?_Iostream_object$initializer$@?$_Error_objects@H@std@@2P6AXXZA 10000000     Metaphlan2Worker.obj
 0002:fffe9000       __catchsym$?_Copy@?$basic_string@DU?$char_traits@D@std@@V?$allocator@D@2@@std@@QAEXII@Z$5 10000000     Metaphlan2Validator.obj
 0002:fffe9000       ?_System_object$initializer$@?$_Error_objects@H@std@@2P6AXXZA 10000000     Metaphlan2Worker.obj
 0001:fffff000       __unwindfunclet$?node_copy@?$QList@VQString@@@@AAEXPAUNode@1@00@Z$5 10000000 f   Metaphlan2Validator.obj
 0001:fffff000       __unwindfunclet$?node_construct@?$QList@VQString@@@@AAEXPAUNode@1@ABVQString@@@Z$1 10000000 f   Metaphlan2Validator.obj
 0001:fffff000       __ehhandler$?detach_helper_grow@?$QList@VQString@@@@AAEPAUNode@1@HH@Z 10000000 f   Metaphlan2Validator.obj
 0001:fffff000       __unwindfunclet$?append@?$QList@VQString@@@@QAEXABVQString@@@Z$7 10000000 f   Metaphlan2Validator.obj
 0001:fffff000       __ehhandler$??0?$QList@VQString@@@@QAE@ABV0@@Z 10000000 f   Metaphlan2Validator.obj
 0001:fffff000       __ehhandler$?_Copy@?$basic_string@DU?$char_traits@D@std@@V?$allocator@D@2@@std@@QAEXII@Z 10000000 f   Metaphlan2Validator.obj
 0001:fffff000       __unwindfunclet$?createNode@?$QMapData@VQString@@VQVariant@@@@QAEPAU?$QMapNode@VQString@@VQVariant@@@@ABVQString@@ABVQVariant@@PAU2@_N@Z$4 10000000 f   Metaphlan2WorkerFactory.obj
 0002:fffe9008       __ehfuncinfo$??A?$QMap@VQString@@VQVariant@@@@QAEAAVQVariant@@ABVQString@@@Z 10000008     Metaphlan2WorkerFactory.obj
 0001:fffff009       __ehhandler$??A?$QMap@VQString@@VQVariant@@@@QAEAAVQVariant@@ABVQString@@@Z 10000009 f   Metaphlan2WorkerFactory.obj
 0001:fffff00c       __unwindfunclet$??1Metaphlan2TaskSettings@U2@@QAE@XZ$1 1000000c f   Metaphlan2Worker.obj
 0001:fffff00c       __unwindfunclet$??0Metaphlan2TaskSettings@U2@@QAE@ABU01@@Z$1 1000000c f   Metaphlan2Worker.obj
 0002:fffe9010       __ehfuncinfo$?node_construct@?$QList@VQString@@@@AAEXPAUNode@1@ABVQString@@@Z 10000010     Metaphlan2Validator.obj
 0002:fffe9010       __tryblocktable$?node_copy@?$QList@VQString@@@@AAEXPAUNode@1@00@Z 10000010     Metaphlan2Validator.obj
 0002:fffe9010       __catchsym$?_Copy@?$basic_string@DU?$char_traits@D@std@@V?$allocator@D@2@@std@@QAEXII@Z$4 10000010     Metaphlan2Task.obj
 0002:fffe9010       __tryblocktable$?node_copy@?$QList@VQString@@@@AAEXPAUNode@1@00@Z 10000010     Metaphlan2Worker.obj
 0002:fffe9010       __unwindtable$??0?$QList@VQString@@@@QAE@ABV0@@Z 10000010     Metaphlan2Task.obj
 0002:fffe9010       __ehfuncinfo$?node_construct@?$QList@VQString@@@@AAEXPAUNode@1@ABVQString@@@Z 10000010     Metaphlan2Worker.obj
 0002:fffe9010       __catchsym$?append@?$QList@VQString@@@@QAEXABVQString@@@Z$12 10000010     Metaphlan2Task.obj
 0002:fffe9010       __catchsym$?detach_helper_grow@?$QList@VQString@@@@AAEPAUNode@1@HH@Z$4 10000010     Metaphlan2Worker.obj
 0002:fffe9010       __catchsym$?detach_helper_grow@?$QList@VQString@@@@AAEPAUNode@1@HH@Z$4 10000010     Metaphlan2Task.obj
 0002:fffe9010       __catchsym$?append@?$QList@VQString@@@@QAEXABVQString@@@Z$12 10000010     Metaphlan2Worker.obj
 0002:fffe9010       __ehfuncinfo$?node_construct@?$QList@VQString@@@@AAEXPAUNode@1@ABVQString@@@Z 10000010     Metaphlan2Task.obj
 0002:fffe9010       __catchsym$?_Copy@?$basic_string@DU?$char_traits@D@std@@V?$allocator@D@2@@std@@QAEXII@Z$4 10000010     Metaphlan2Worker.obj
 0002:fffe9010       __tryblocktable$?node_copy@?$QList@VQString@@@@AAEXPAUNode@1@00@Z 10000010     Metaphlan2Task.obj
 0002:fffe9010       __ehfuncinfo$?metaType@?$QVariantValueHelper@VQString@@@QtPrivate@@SA?AVQString@@ABVQVariant@@@Z 10000010     Metaphlan2Worker.obj
 0002:fffe9010       __catchsym$?_Copy@?$basic_string@DU?$char_traits@D@std@@V?$allocator@D@2@@std@@QAEXII@Z$4 10000010     Metaphlan2SupportPlugin.obj
 0002:fffe9010       __catchsym$?detach_helper_grow@?$QList@VQString@@@@AAEPAUNode@1@HH@Z$4 10000010     Metaphlan2Validator.obj
 0002:fffe9010       __catchsym$?_Copy@?$basic_string@DU?$char_traits@D@std@@V?$allocator@D@2@@std@@QAEXII@Z$4 10000010     Metaphlan2Support.obj
 0002:fffe9010       __catchsym$?append@?$QList@VQString@@@@QAEXABVQString@@@Z$12 10000010     Metaphlan2Support.obj
 0002:fffe9010       __catchsym$?detach_helper_grow@?$QList@VQString@@@@AAEPAUNode@1@HH@Z$4 10000010     Metaphlan2Support.obj
 0002:fffe9010       __ehfuncinfo$?node_construct@?$QList@VQString@@@@AAEXPAUNode@1@ABVQString@@@Z 10000010     Metaphlan2Support.obj
 0002:fffe9010       __tryblocktable$?node_copy@?$QList@VQString@@@@AAEXPAUNode@1@00@Z 10000010     Metaphlan2Support.obj
 0002:fffe9010       __catchsym$?_Copy@?$basic_string@DU?$char_traits@D@std@@V?$allocator@D@2@@std@@QAEXII@Z$4 10000010     Metaphlan2Prompter.obj
 0002:fffe9010       __catchsym$?append@?$QList@VQString@@@@QAEXABVQString@@@Z$12 10000010     Metaphlan2Validator.obj
 0002:fffe9010       __catchsym$?_Copy@?$basic_string@DU?$char_traits@D@std@@V?$allocator@D@2@@std@@QAEXII@Z$4 10000010     moc_Metaphlan2Prompter.obj
 0002:fffe9010       __catchsym$?_Copy@?$basic_string@DU?$char_traits@D@std@@V?$allocator@D@2@@std@@QAEXII@Z$4 10000010     moc_Metaphlan2Support.obj
 0002:fffe9010       __catchsym$?_Copy@?$basic_string@DU?$char_traits@D@std@@V?$allocator@D@2@@std@@QAEXII@Z$4 10000010     moc_Metaphlan2SupportPlugin.obj
 0002:fffe9010       __catchsym$?createNode@?$QMapData@VQString@@VQVariant@@@@QAEPAU?$QMapNode@VQString@@VQVariant@@@@ABVQString@@ABVQVariant@@PAU2@_N@Z$6 10000010     Metaphlan2WorkerFactory.obj
 0002:fffe9010       __catchsym$?_Copy@?$basic_string@DU?$char_traits@D@std@@V?$allocator@D@2@@std@@QAEXII@Z$4 10000010     moc_Metaphlan2Task.obj
 0002:fffe9010       __unwindtable$??0?$QList@VQString@@@@QAE@ABV0@@Z 10000010     Metaphlan2Validator.obj
 0002:fffe9010       __catchsym$?_Copy@?$basic_string@DU?$char_traits@D@std@@V?$allocator@D@2@@std@@QAEXII@Z$4 10000010     moc_Metaphlan2Worker.obj
 0002:fffe9010       __catchsym$?_Copy@?$basic_string@DU?$char_traits@D@std@@V?$allocator@D@2@@std@@QAEXII@Z$4 10000010     Metaphlan2WorkerFactory.obj
 0002:fffe9010       __catchsym$?_Copy@?$basic_string@DU?$char_traits@D@std@@V?$allocator@D@2@@std@@QAEXII@Z$4 10000010     Metaphlan2Validator.obj
 0001:fffff011       __unwindfunclet$?append@?$QList@VQString@@@@QAEXABVQString@@@Z$11 10000011 f   Metaphlan2Validator.obj
 0001:fffff011       __unwindfunclet$?append@?$QList@VQString@@@@QAEXABVQString@@@Z$11 10000011 f   Metaphlan2Task.obj
 0001:fffff011       __ehhandler$?node_copy@?$QList@VQString@@@@AAEXPAUNode@1@00@Z 10000011 f   Metaphlan2Task.obj
 0001:fffff011       __unwindfunclet$?append@?$QList@VQString@@@@QAEXABVQString@@@Z$11 10000011 f   Metaphlan2Support.obj
 0001:fffff011       __ehhandler$?node_construct@?$QList@VQString@@@@AAEXPAUNode@1@ABVQString@@@Z 10000011 f   Metaphlan2Worker.obj
 0001:fffff011       __ehhandler$?node_copy@?$QList@VQString@@@@AAEXPAUNode@1@00@Z 10000011 f   Metaphlan2Support.obj
 0001:fffff011       __ehhandler$?node_construct@?$QList@VQString@@@@AAEXPAUNode@1@ABVQString@@@Z 10000011 f   Metaphlan2Validator.obj
 0001:fffff011       __ehhandler$?node_construct@?$QList@VQString@@@@AAEXPAUNode@1@ABVQString@@@Z 10000011 f   Metaphlan2Support.obj
 0001:fffff011       __ehhandler$?node_copy@?$QList@VQString@@@@AAEXPAUNode@1@00@Z 10000011 f   Metaphlan2Validator.obj
 0001:fffff011       __unwindfunclet$?append@?$QList@VQString@@@@QAEXABVQString@@@Z$11 10000011 f   Metaphlan2Worker.obj
 0001:fffff011       __ehhandler$?node_copy@?$QList@VQString@@@@AAEXPAUNode@1@00@Z 10000011 f   Metaphlan2Worker.obj
 0001:fffff011       __ehhandler$?node_construct@?$QList@VQString@@@@AAEXPAUNode@1@ABVQString@@@Z 10000011 f   Metaphlan2Task.obj
 0001:fffff014       __unwindfunclet$?createNode@?$QMapData@VQString@@VQVariant@@@@QAEPAU?$QMapNode@VQString@@VQVariant@@@@ABVQString@@ABVQVariant@@PAU2@_N@Z$5 10000014 f   Metaphlan2WorkerFactory.obj
 0001:fffff018       __unwindfunclet$??0Metaphlan2TaskSettings@U2@@QAE@ABU01@@Z$2 10000018 f   Metaphlan2Worker.obj
 0001:fffff018       __unwindfunclet$??1Metaphlan2TaskSettings@U2@@QAE@XZ$2 10000018 f   Metaphlan2Worker.obj
 0001:fffff01a       __unwindfunclet$?metaType@?$QVariantValueHelper@VQString@@@QtPrivate@@SA?AVQString@@ABVQVariant@@@Z$1 1000001a f   Metaphlan2Worker.obj
 0002:fffe9020       __ehfuncinfo$?append@?$QList@VQString@@@@QAEXABVQString@@@Z 10000020     Metaphlan2Support.obj
 0002:fffe9020       __unwindtable$?detach_helper_grow@?$QList@VQString@@@@AAEPAUNode@1@HH@Z 10000020     Metaphlan2Worker.obj
 0002:fffe9020       __tryblocktable$??0?$QList@VQString@@@@QAE@ABV0@@Z 10000020     Metaphlan2Task.obj
 0002:fffe9020       __unwindtable$?_Copy@?$basic_string@DU?$char_traits@D@std@@V?$allocator@D@2@@std@@QAEXII@Z 10000020     Metaphlan2Worker.obj
 0002:fffe9020       __unwindtable$?_Copy@?$basic_string@DU?$char_traits@D@std@@V?$allocator@D@2@@std@@QAEXII@Z 10000020     Metaphlan2Prompter.obj
 0002:fffe9020       __unwindtable$?_Copy@?$basic_string@DU?$char_traits@D@std@@V?$allocator@D@2@@std@@QAEXII@Z 10000020     Metaphlan2Task.obj
 0002:fffe9020       __unwindtable$?detach_helper_grow@?$QList@VQString@@@@AAEPAUNode@1@HH@Z 10000020     Metaphlan2Validator.obj
 0002:fffe9020       __unwindtable$?detach_helper_grow@?$QList@VQString@@@@AAEPAUNode@1@HH@Z 10000020     Metaphlan2Support.obj
 0002:fffe9020       __unwindtable$?_Copy@?$basic_string@DU?$char_traits@D@std@@V?$allocator@D@2@@std@@QAEXII@Z 10000020     moc_Metaphlan2Support.obj
 0002:fffe9020       __unwindtable$?_Copy@?$basic_string@DU?$char_traits@D@std@@V?$allocator@D@2@@std@@QAEXII@Z 10000020     Metaphlan2Validator.obj
 0002:fffe9020       __unwindtable$?_Copy@?$basic_string@DU?$char_traits@D@std@@V?$allocator@D@2@@std@@QAEXII@Z 10000020     moc_Metaphlan2Task.obj
 0002:fffe9020       __unwindtable$?detach_helper_grow@?$QList@VQString@@@@AAEPAUNode@1@HH@Z 10000020     Metaphlan2Task.obj
 0002:fffe9020       __unwindtable$?_Copy@?$basic_string@DU?$char_traits@D@std@@V?$allocator@D@2@@std@@QAEXII@Z 10000020     moc_Metaphlan2Worker.obj
 0002:fffe9020       __ehfuncinfo$?createNode@?$QMapData@VQString@@VQVariant@@@@QAEPAU?$QMapNode@VQString@@VQVariant@@@@ABVQString@@ABVQVariant@@PAU2@_N@Z 10000020     Metaphlan2WorkerFactory.obj
 0002:fffe9020       __ehfuncinfo$?append@?$QList@VQString@@@@QAEXABVQString@@@Z 10000020     Metaphlan2Validator.obj
 0002:fffe9020       __unwindtable$?_Copy@?$basic_string@DU?$char_traits@D@std@@V?$allocator@D@2@@std@@QAEXII@Z 10000020     moc_Metaphlan2SupportPlugin.obj
 0002:fffe9020       __unwindtable$?_Copy@?$basic_string@DU?$char_traits@D@std@@V?$allocator@D@2@@std@@QAEXII@Z 10000020     moc_Metaphlan2Prompter.obj
 0002:fffe9020       __unwindtable$?_Copy@?$basic_string@DU?$char_traits@D@std@@V?$allocator@D@2@@std@@QAEXII@Z 10000020     Metaphlan2Support.obj
 0002:fffe9020       __tryblocktable$??0?$QList@VQString@@@@QAE@ABV0@@Z 10000020     Metaphlan2Validator.obj
 0002:fffe9020       __unwindtable$?_Copy@?$basic_string@DU?$char_traits@D@std@@V?$allocator@D@2@@std@@QAEXII@Z 10000020     Metaphlan2WorkerFactory.obj
 0002:fffe9020       __ehfuncinfo$?append@?$QList@VQString@@@@QAEXABVQString@@@Z 10000020     Metaphlan2Worker.obj
 0002:fffe9020       __ehfuncinfo$?append@?$QList@VQString@@@@QAEXABVQString@@@Z 10000020     Metaphlan2Task.obj
 0002:fffe9020       __unwindtable$?_Copy@?$basic_string@DU?$char_traits@D@std@@V?$allocator@D@2@@std@@QAEXII@Z 10000020     Metaphlan2SupportPlugin.obj
 0001:fffff022       __ehhandler$?append@?$QList@VQString@@@@QAEXABVQString@@@Z 10000022 f   Metaphlan2Support.obj
 0001:fffff022       __ehhandler$?append@?$QList@VQString@@@@QAEXABVQString@@@Z 10000022 f   Metaphlan2Worker.obj
 0001:fffff022       __ehhandler$?append@?$QList@VQString@@@@QAEXABVQString@@@Z 10000022 f   Metaphlan2Validator.obj
 0001:fffff022       __ehhandler$?append@?$QList@VQString@@@@QAEXABVQString@@@Z 10000022 f   Metaphlan2Task.obj
 0001:fffff023       __ehhandler$?metaType@?$QVariantValueHelper@VQString@@@QtPrivate@@SA?AVQString@@ABVQVariant@@@Z 10000023 f   Metaphlan2Worker.obj
 0002:fffe9024       __ehfuncinfo$?node_copy@?$QList@VQString@@@@AAEXPAUNode@1@00@Z 10000024     Metaphlan2Worker.obj
 0001:fffff024       __unwindfunclet$??0Metaphlan2TaskSettings@U2@@QAE@ABU01@@Z$3 10000024 f   Metaphlan2Worker.obj
 0002:fffe9024       __ehfuncinfo$?node_copy@?$QList@VQString@@@@AAEXPAUNode@1@00@Z 10000024     Metaphlan2Validator.obj
 0002:fffe9024       __ehfuncinfo$?node_copy@?$QList@VQString@@@@AAEXPAUNode@1@00@Z 10000024     Metaphlan2Support.obj
 0002:fffe9024       __ehfuncinfo$?node_copy@?$QList@VQString@@@@AAEXPAUNode@1@00@Z 10000024     Metaphlan2Task.obj
 0002:fffe9024       __unwindtable$??0Metaphlan2TaskSettings@U2@@QAE@ABU01@@Z 10000024     Metaphlan2Worker.obj
 0002:fffe9024       __unwindtable$??1Metaphlan2TaskSettings@U2@@QAE@XZ 10000024     Metaphlan2Worker.obj
 0001:fffff024       __unwindfunclet$??1Metaphlan2TaskSettings@U2@@QAE@XZ$3 10000024 f   Metaphlan2Worker.obj
 0001:fffff028       __ehhandler$?createNode@?$QMapData@VQString@@VQVariant@@@@QAEPAU?$QMapNode@VQString@@VQVariant@@@@ABVQString@@ABVQVariant@@PAU2@_N@Z 10000028 f   Metaphlan2WorkerFactory.obj
 0001:fffff030       __unwindfunclet$??0Metaphlan2TaskSettings@U2@@QAE@ABU01@@Z$4 10000030 f   Metaphlan2Worker.obj
 0001:fffff030       __unwindfunclet$??1Metaphlan2TaskSettings@U2@@QAE@XZ$4 10000030 f   Metaphlan2Worker.obj
 0002:fffe9034       __ehfuncinfo$??0?$QList@VQString@@@@QAE@ABV0@@Z 10000034     Metaphlan2Validator.obj
 0002:fffe9034       __ehfuncinfo$??0?$QList@VQString@@@@QAE@ABV0@@Z 10000034     Metaphlan2Task.obj
 0001:fffff03c       __unwindfunclet$??0Metaphlan2TaskSettings@U2@@QAE@ABU01@@Z$5 1000003c f   Metaphlan2Worker.obj
 0001:fffff03c       __unwindfunclet$??1Metaphlan2TaskSettings@U2@@QAE@XZ$5 1000003c f   Metaphlan2Worker.obj
 0002:fffe9040       __ehfuncinfo$?_Copy@?$basic_string@DU?$char_traits@D@std@@V?$allocator@D@2@@std@@QAEXII@Z 10000040     Metaphlan2WorkerFactory.obj
 0002:fffe9040       __ehfuncinfo$?_Copy@?$basic_string@DU?$char_traits@D@std@@V?$allocator@D@2@@std@@QAEXII@Z 10000040     Metaphlan2Task.obj
 0002:fffe9040       __ehfuncinfo$?detach_helper_grow@?$QList@VQString@@@@AAEPAUNode@1@HH@Z 10000040     Metaphlan2Validator.obj
 0002:fffe9040       __ehfuncinfo$?_Copy@?$basic_string@DU?$char_traits@D@std@@V?$allocator@D@2@@std@@QAEXII@Z 10000040     moc_Metaphlan2Support.obj
 0002:fffe9040       __ehfuncinfo$?_Copy@?$basic_string@DU?$char_traits@D@std@@V?$allocator@D@2@@std@@QAEXII@Z 10000040     moc_Metaphlan2Task.obj
 0002:fffe9040       __ehfuncinfo$?_Copy@?$basic_string@DU?$char_traits@D@std@@V?$allocator@D@2@@std@@QAEXII@Z 10000040     Metaphlan2Prompter.obj
 0002:fffe9040       __ehfuncinfo$?_Copy@?$basic_string@DU?$char_traits@D@std@@V?$allocator@D@2@@std@@QAEXII@Z 10000040     Metaphlan2Worker.obj
 0002:fffe9040       __ehfuncinfo$?detach_helper_grow@?$QList@VQString@@@@AAEPAUNode@1@HH@Z 10000040     Metaphlan2Worker.obj
 0002:fffe9040       __ehfuncinfo$?_Copy@?$basic_string@DU?$char_traits@D@std@@V?$allocator@D@2@@std@@QAEXII@Z 10000040     moc_Metaphlan2SupportPlugin.obj
 0002:fffe9040       __ehfuncinfo$?_Copy@?$basic_string@DU?$char_traits@D@std@@V?$allocator@D@2@@std@@QAEXII@Z 10000040     moc_Metaphlan2Worker.obj
 0002:fffe9040       __ehfuncinfo$?_Copy@?$basic_string@DU?$char_traits@D@std@@V?$allocator@D@2@@std@@QAEXII@Z 10000040     Metaphlan2Support.obj
 0002:fffe9040       __ehfuncinfo$?detach_helper_grow@?$QList@VQString@@@@AAEPAUNode@1@HH@Z 10000040     Metaphlan2Task.obj
 0002:fffe9040       __ehfuncinfo$?_Copy@?$basic_string@DU?$char_traits@D@std@@V?$allocator@D@2@@std@@QAEXII@Z 10000040     moc_Metaphlan2Prompter.obj
 0002:fffe9040       __ehfuncinfo$?detach_helper_grow@?$QList@VQString@@@@AAEPAUNode@1@HH@Z 10000040     Metaphlan2Support.obj
 0002:fffe9040       __ehfuncinfo$?_Copy@?$basic_string@DU?$char_traits@D@std@@V?$allocator@D@2@@std@@QAEXII@Z 10000040     Metaphlan2SupportPlugin.obj
 0002:fffe9040       __ehfuncinfo$?_Copy@?$basic_string@DU?$char_traits@D@std@@V?$allocator@D@2@@std@@QAEXII@Z 10000040     Metaphlan2Validator.obj
 0002:fffe9044       __tryblocktable$?append@?$QList@VQString@@@@QAEXABVQString@@@Z 10000044     Metaphlan2Support.obj
 0002:fffe9044       __tryblocktable$?createNode@?$QMapData@VQString@@VQVariant@@@@QAEPAU?$QMapNode@VQString@@VQVariant@@@@ABVQString@@ABVQVariant@@PAU2@_N@Z 10000044     Metaphlan2WorkerFactory.obj
 0002:fffe9044       __tryblocktable$?append@?$QList@VQString@@@@QAEXABVQString@@@Z 10000044     Metaphlan2Worker.obj
 0002:fffe9044       __tryblocktable$?append@?$QList@VQString@@@@QAEXABVQString@@@Z 10000044     Metaphlan2Validator.obj
 0002:fffe9044       __tryblocktable$?append@?$QList@VQString@@@@QAEXABVQString@@@Z 10000044     Metaphlan2Task.obj
 0002:fffe9048       __unwindtable$?node_copy@?$QList@VQString@@@@AAEXPAUNode@1@00@Z 10000048     Metaphlan2Task.obj
 0002:fffe9048       __unwindtable$?node_copy@?$QList@VQString@@@@AAEXPAUNode@1@00@Z 10000048     Metaphlan2Validator.obj
 0002:fffe9048       __unwindtable$?node_copy@?$QList@VQString@@@@AAEXPAUNode@1@00@Z 10000048     Metaphlan2Support.obj
 0002:fffe9048       __unwindtable$?node_copy@?$QList@VQString@@@@AAEXPAUNode@1@00@Z 10000048     Metaphlan2Worker.obj
 0001:fffff048       __unwindfunclet$??1Metaphlan2TaskSettings@U2@@QAE@XZ$6 10000048 f   Metaphlan2Worker.obj
 0001:fffff048       __unwindfunclet$??0Metaphlan2TaskSettings@U2@@QAE@ABU01@@Z$6 10000048 f   Metaphlan2Worker.obj
 0001:fffff054       __unwindfunclet$??0Metaphlan2TaskSettings@U2@@QAE@ABU01@@Z$7 10000054 f   Metaphlan2Worker.obj
 0001:fffff054       __unwindfunclet$??1Metaphlan2TaskSettings@U2@@QAE@XZ$7 10000054 f   Metaphlan2Worker.obj
 0001:fffff060       __unwindfunclet$??1Metaphlan2TaskSettings@U2@@QAE@XZ$8 10000060 f   Metaphlan2Worker.obj
 0001:fffff060       __unwindfunclet$??0Metaphlan2TaskSettings@U2@@QAE@ABU01@@Z$8 10000060 f   Metaphlan2Worker.obj
 0001:fffff062       __catch$?node_copy@?$QList@VQString@@@@AAEXPAUNode@1@00@Z$2 10000062 f   Metaphlan2Worker.obj
 0001:fffff062       __catch$?node_copy@?$QList@VQString@@@@AAEXPAUNode@1@00@Z$2 10000062 f   Metaphlan2Task.obj
 0001:fffff062       __catch$?node_copy@?$QList@VQString@@@@AAEXPAUNode@1@00@Z$2 10000062 f   Metaphlan2Validator.obj
 0001:fffff062       __catch$?node_copy@?$QList@VQString@@@@AAEXPAUNode@1@00@Z$2 10000062 f   Metaphlan2Support.obj
 0002:fffe9064       __tryblocktable$?_Copy@?$basic_string@DU?$char_traits@D@std@@V?$allocator@D@2@@std@@QAEXII@Z 10000064     Metaphlan2Task.obj
 0002:fffe9064       __tryblocktable$?detach_helper_grow@?$QList@VQString@@@@AAEPAUNode@1@HH@Z 10000064     Metaphlan2Worker.obj
 0002:fffe9064       __tryblocktable$?_Copy@?$basic_string@DU?$char_traits@D@std@@V?$allocator@D@2@@std@@QAEXII@Z 10000064     moc_Metaphlan2Prompter.obj
 0002:fffe9064       __tryblocktable$?_Copy@?$basic_string@DU?$char_traits@D@std@@V?$allocator@D@2@@std@@QAEXII@Z 10000064     Metaphlan2Validator.obj
 0002:fffe9064       __tryblocktable$?_Copy@?$basic_string@DU?$char_traits@D@std@@V?$allocator@D@2@@std@@QAEXII@Z 10000064     Metaphlan2Prompter.obj
 0002:fffe9064       __tryblocktable$?detach_helper_grow@?$QList@VQString@@@@AAEPAUNode@1@HH@Z 10000064     Metaphlan2Task.obj
 0002:fffe9064       __tryblocktable$?_Copy@?$basic_string@DU?$char_traits@D@std@@V?$allocator@D@2@@std@@QAEXII@Z 10000064     Metaphlan2SupportPlugin.obj
 0002:fffe9064       __tryblocktable$?_Copy@?$basic_string@DU?$char_traits@D@std@@V?$allocator@D@2@@std@@QAEXII@Z 10000064     moc_Metaphlan2Support.obj
 0002:fffe9064       __tryblocktable$?detach_helper_grow@?$QList@VQString@@@@AAEPAUNode@1@HH@Z 10000064     Metaphlan2Support.obj
 0002:fffe9064       __tryblocktable$?_Copy@?$basic_string@DU?$char_traits@D@std@@V?$allocator@D@2@@std@@QAEXII@Z 10000064     Metaphlan2Worker.obj
 0002:fffe9064       __tryblocktable$?_Copy@?$basic_string@DU?$char_traits@D@std@@V?$allocator@D@2@@std@@QAEXII@Z 10000064     Metaphlan2Support.obj
 0002:fffe9064       __tryblocktable$?_Copy@?$basic_string@DU?$char_traits@D@std@@V?$allocator@D@2@@std@@QAEXII@Z 10000064     moc_Metaphlan2Task.obj
 0002:fffe9064       __tryblocktable$?_Copy@?$basic_string@DU?$char_traits@D@std@@V?$allocator@D@2@@std@@QAEXII@Z 10000064     Metaphlan2WorkerFactory.obj
 0002:fffe9064       __tryblocktable$?detach_helper_grow@?$QList@VQString@@@@AAEPAUNode@1@HH@Z 10000064     Metaphlan2Validator.obj
 0002:fffe9064       __tryblocktable$?_Copy@?$basic_string@DU?$char_traits@D@std@@V?$allocator@D@2@@std@@QAEXII@Z 10000064     moc_Metaphlan2SupportPlugin.obj
 0002:fffe9064       __tryblocktable$?_Copy@?$basic_string@DU?$char_traits@D@std@@V?$allocator@D@2@@std@@QAEXII@Z 10000064     moc_Metaphlan2Worker.obj
 0002:fffe906c       __unwindtable$?append@?$QList@VQString@@@@QAEXABVQString@@@Z 1000006c     Metaphlan2Support.obj
 0001:fffff06c       __ehhandler$??0Metaphlan2TaskSettings@U2@@QAE@ABU01@@Z 1000006c f   Metaphlan2Worker.obj
 0002:fffe906c       __unwindtable$?append@?$QList@VQString@@@@QAEXABVQString@@@Z 1000006c     Metaphlan2Validator.obj
 0002:fffe906c       __unwindtable$?append@?$QList@VQString@@@@QAEXABVQString@@@Z 1000006c     Metaphlan2Task.obj
 0002:fffe906c       __unwindtable$?append@?$QList@VQString@@@@QAEXABVQString@@@Z 1000006c     Metaphlan2Worker.obj
 0001:fffff06c       __ehhandler$??1Metaphlan2TaskSettings@U2@@QAE@XZ 1000006c f   Metaphlan2Worker.obj
 0002:fffe906c       __unwindtable$?createNode@?$QMapData@VQString@@VQVariant@@@@QAEPAU?$QMapNode@VQString@@VQVariant@@@@ABVQString@@ABVQVariant@@PAU2@_N@Z 1000006c     Metaphlan2WorkerFactory.obj
 0001:fffff07d       __catch$?append@?$QList@VQString@@@@QAEXABVQString@@@Z$0 1000007d f   Metaphlan2Task.obj
 0001:fffff07d       __catch$?append@?$QList@VQString@@@@QAEXABVQString@@@Z$0 1000007d f   Metaphlan2Support.obj
 0001:fffff07d       __catch$?append@?$QList@VQString@@@@QAEXABVQString@@@Z$0 1000007d f   Metaphlan2Validator.obj
 0001:fffff07d       __catch$?append@?$QList@VQString@@@@QAEXABVQString@@@Z$0 1000007d f   Metaphlan2Worker.obj
 0001:fffff08e       __catch$?createNode@?$QMapData@VQString@@VQVariant@@@@QAEPAU?$QMapNode@VQString@@VQVariant@@@@ABVQString@@ABVQVariant@@PAU2@_N@Z$0 1000008e f   Metaphlan2WorkerFactory.obj
 0001:fffff096       __catch$?_Copy@?$basic_string@DU?$char_traits@D@std@@V?$allocator@D@2@@std@@QAEXII@Z$0 10000096 f   moc_Metaphlan2SupportPlugin.obj
 0001:fffff096       __catch$?_Copy@?$basic_string@DU?$char_traits@D@std@@V?$allocator@D@2@@std@@QAEXII@Z$0 10000096 f   moc_Metaphlan2Support.obj
 0001:fffff096       __catch$?_Copy@?$basic_string@DU?$char_traits@D@std@@V?$allocator@D@2@@std@@QAEXII@Z$0 10000096 f   moc_Metaphlan2Task.obj
 0001:fffff096       __catch$?_Copy@?$basic_string@DU?$char_traits@D@std@@V?$allocator@D@2@@std@@QAEXII@Z$0 10000096 f   Metaphlan2Support.obj
 0001:fffff096       __catch$?_Copy@?$basic_string@DU?$char_traits@D@std@@V?$allocator@D@2@@std@@QAEXII@Z$0 10000096 f   Metaphlan2Prompter.obj
 0001:fffff096       __catch$?_Copy@?$basic_string@DU?$char_traits@D@std@@V?$allocator@D@2@@std@@QAEXII@Z$0 10000096 f   Metaphlan2Worker.obj
 0001:fffff096       __catch$?_Copy@?$basic_string@DU?$char_traits@D@std@@V?$allocator@D@2@@std@@QAEXII@Z$0 10000096 f   Metaphlan2WorkerFactory.obj
 0001:fffff096       __catch$?_Copy@?$basic_string@DU?$char_traits@D@std@@V?$allocator@D@2@@std@@QAEXII@Z$0 10000096 f   moc_Metaphlan2Prompter.obj
 0001:fffff096       __catch$?_Copy@?$basic_string@DU?$char_traits@D@std@@V?$allocator@D@2@@std@@QAEXII@Z$0 10000096 f   Metaphlan2Validator.obj
 0001:fffff096       __catch$?_Copy@?$basic_string@DU?$char_traits@D@std@@V?$allocator@D@2@@std@@QAEXII@Z$0 10000096 f   Metaphlan2Task.obj
 0001:fffff096       __catch$?_Copy@?$basic_string@DU?$char_traits@D@std@@V?$allocator@D@2@@std@@QAEXII@Z$0 10000096 f   Metaphlan2SupportPlugin.obj
 0001:fffff096       __catch$?_Copy@?$basic_string@DU?$char_traits@D@std@@V?$allocator@D@2@@std@@QAEXII@Z$0 10000096 f   moc_Metaphlan2Worker.obj
 0001:fffff09e       __catch$??0?$QList@VQString@@@@QAE@ABV0@@Z$0 1000009e f   Metaphlan2Validator.obj
 0001:fffff09e       __catch$??0?$QList@VQString@@@@QAE@ABV0@@Z$0 1000009e f   Metaphlan2Task.obj
 0001:fffff0a3       __catch$?createNode@?$QMapData@VQString@@VQVariant@@@@QAEPAU?$QMapNode@VQString@@VQVariant@@@@ABVQString@@ABVQVariant@@PAU2@_N@Z$2 100000a3 f   Metaphlan2WorkerFactory.obj
 0001:fffff0ce       __catch$?append@?$QList@VQString@@@@QAEXABVQString@@@Z$4 100000ce f   Metaphlan2Task.obj
 0001:fffff0ce       __catch$?append@?$QList@VQString@@@@QAEXABVQString@@@Z$4 100000ce f   Metaphlan2Worker.obj
 0001:fffff0ce       __catch$?append@?$QList@VQString@@@@QAEXABVQString@@@Z$4 100000ce f   Metaphlan2Support.obj
 0001:fffff0ce       __catch$?append@?$QList@VQString@@@@QAEXABVQString@@@Z$4 100000ce f   Metaphlan2Validator.obj
 0001:fffff0d3       __catch$?_Copy@?$basic_string@DU?$char_traits@D@std@@V?$allocator@D@2@@std@@QAEXII@Z$1 100000d3 f   Metaphlan2Task.obj
 0001:fffff0d3       __catch$?_Copy@?$basic_string@DU?$char_traits@D@std@@V?$allocator@D@2@@std@@QAEXII@Z$1 100000d3 f   Metaphlan2WorkerFactory.obj
 0001:fffff0d3       __catch$?_Copy@?$basic_string@DU?$char_traits@D@std@@V?$allocator@D@2@@std@@QAEXII@Z$1 100000d3 f   Metaphlan2Worker.obj
 0001:fffff0d3       __catch$?_Copy@?$basic_string@DU?$char_traits@D@std@@V?$allocator@D@2@@std@@QAEXII@Z$1 100000d3 f   moc_Metaphlan2Worker.obj
 0001:fffff0d3       __catch$?_Copy@?$basic_string@DU?$char_traits@D@std@@V?$allocator@D@2@@std@@QAEXII@Z$1 100000d3 f   moc_Metaphlan2Task.obj
 0001:fffff0d3       __catch$?_Copy@?$basic_string@DU?$char_traits@D@std@@V?$allocator@D@2@@std@@QAEXII@Z$1 100000d3 f   Metaphlan2Validator.obj
 0001:fffff0d3       __catch$?_Copy@?$basic_string@DU?$char_traits@D@std@@V?$allocator@D@2@@std@@QAEXII@Z$1 100000d3 f   moc_Metaphlan2Prompter.obj
 0001:fffff0d3       __catch$?_Copy@?$basic_string@DU?$char_traits@D@std@@V?$allocator@D@2@@std@@QAEXII@Z$1 100000d3 f   moc_Metaphlan2Support.obj
 0001:fffff0d3       __catch$?_Copy@?$basic_string@DU?$char_traits@D@std@@V?$allocator@D@2@@std@@QAEXII@Z$1 100000d3 f   Metaphlan2SupportPlugin.obj
 0001:fffff0d3       __catch$?_Copy@?$basic_string@DU?$char_traits@D@std@@V?$allocator@D@2@@std@@QAEXII@Z$1 100000d3 f   Metaphlan2Prompter.obj
 0001:fffff0d3       __catch$?_Copy@?$basic_string@DU?$char_traits@D@std@@V?$allocator@D@2@@std@@QAEXII@Z$1 100000d3 f   moc_Metaphlan2SupportPlugin.obj
 0001:fffff0d3       __catch$?_Copy@?$basic_string@DU?$char_traits@D@std@@V?$allocator@D@2@@std@@QAEXII@Z$1 100000d3 f   Metaphlan2Support.obj
 0001:fffff11e       __catch$?detach_helper_grow@?$QList@VQString@@@@AAEPAUNode@1@HH@Z$2 1000011e f   Metaphlan2Support.obj
 0001:fffff11e       __catch$?detach_helper_grow@?$QList@VQString@@@@AAEPAUNode@1@HH@Z$2 1000011e f   Metaphlan2Worker.obj
 0001:fffff11e       __catch$?detach_helper_grow@?$QList@VQString@@@@AAEPAUNode@1@HH@Z$2 1000011e f   Metaphlan2Validator.obj
 0001:fffff11e       __catch$?detach_helper_grow@?$QList@VQString@@@@AAEPAUNode@1@HH@Z$2 1000011e f   Metaphlan2Task.obj
 0001:fffff159       __catch$?detach_helper_grow@?$QList@VQString@@@@AAEPAUNode@1@HH@Z$0 10000159 f   Metaphlan2Task.obj
 0001:fffff159       __catch$?detach_helper_grow@?$QList@VQString@@@@AAEPAUNode@1@HH@Z$0 10000159 f   Metaphlan2Worker.obj
 0001:fffff159       __catch$?detach_helper_grow@?$QList@VQString@@@@AAEPAUNode@1@HH@Z$0 10000159 f   Metaphlan2Support.obj
 0001:fffff159       __catch$?detach_helper_grow@?$QList@VQString@@@@AAEPAUNode@1@HH@Z$0 10000159 f   Metaphlan2Validator.obj
 0001:00000000       ??__E?_Generic_object@?$_Error_objects@H@std@@2V_Generic_error_category@2@A@@YAXXZ 10001000 f   Metaphlan2LogParser.obj
 0001:00000010       ??__E?_Iostream_object@?$_Error_objects@H@std@@2V_Iostream_error_category@2@A@@YAXXZ 10001010 f   Metaphlan2LogParser.obj
 0001:00000020       ??__E?_System_object@?$_Error_objects@H@std@@2V_System_error_category@2@A@@YAXXZ 10001020 f   Metaphlan2LogParser.obj
 0001:00000030       ??__E?wellKnownErrors@Metaphlan2LogParser@U2@@0VQStringList@@B@@YAXXZ 10001030 f   Metaphlan2LogParser.obj
 0001:00000050       ??__EalgoLog@U2@@YAXXZ     10001050 f   Metaphlan2LogParser.obj
 0001:000000d0       ??__EcmdLog@U2@@YAXXZ      100010d0 f   Metaphlan2LogParser.obj
 0001:00000150       ??__EcoreLog@U2@@YAXXZ     10001150 f   Metaphlan2LogParser.obj
 0001:000001d0       ??__EioLog@U2@@YAXXZ       100011d0 f   Metaphlan2LogParser.obj
 0001:00000250       ??__EperfLog@U2@@YAXXZ     10001250 f   Metaphlan2LogParser.obj
 0001:000002d0       ??__EscriptLog@U2@@YAXXZ   100012d0 f   Metaphlan2LogParser.obj
 0001:00000350       ??__EtaskLog@U2@@YAXXZ     10001350 f   Metaphlan2LogParser.obj
 0001:000003d0       ??__EuiLog@U2@@YAXXZ       100013d0 f   Metaphlan2LogParser.obj
 0001:00000450       ??__EuserActLog@U2@@YAXXZ  10001450 f   Metaphlan2LogParser.obj
 0001:000004d0       ??__E?_Generic_object@?$_Error_objects@H@std@@2V_Generic_error_category@2@A@@YAXXZ 100014d0 f   Metaphlan2Prompter.obj
 0001:000004e0       ??__E?_Iostream_object@?$_Error_objects@H@std@@2V_Iostream_error_category@2@A@@YAXXZ 100014e0 f   Metaphlan2Prompter.obj
 0001:000004f0       ??__E?_System_object@?$_Error_objects@H@std@@2V_System_error_category@2@A@@YAXXZ 100014f0 f   Metaphlan2Prompter.obj
 0001:00000500       ??__EalgoLog@U2@@YAXXZ     10001500 f   Metaphlan2Prompter.obj
 0001:00000580       ??__EcmdLog@U2@@YAXXZ      10001580 f   Metaphlan2Prompter.obj
 0001:00000600       ??__EcoreLog@U2@@YAXXZ     10001600 f   Metaphlan2Prompter.obj
 0001:00000680       ??__EioLog@U2@@YAXXZ       10001680 f   Metaphlan2Prompter.obj
 0001:00000700       ??__EperfLog@U2@@YAXXZ     10001700 f   Metaphlan2Prompter.obj
 0001:00000780       ??__EscriptLog@U2@@YAXXZ   10001780 f   Metaphlan2Prompter.obj
 0001:00000800       ??__EtaskLog@U2@@YAXXZ     10001800 f   Metaphlan2Prompter.obj
 0001:00000880       ??__EuiLog@U2@@YAXXZ       10001880 f   Metaphlan2Prompter.obj
 0001:00000900       ??__EuserActLog@U2@@YAXXZ  10001900 f   Metaphlan2Prompter.obj
 0001:00000980       ??__E?ET_BOWTIE_2_ALIGNER@Metaphlan2Support@U2@@2VQString@@B@@YAXXZ 10001980 f   Metaphlan2Support.obj
 0001:000009a0       ??__E?ET_PYTHON@Metaphlan2Support@U2@@2VQString@@B@@YAXXZ 100019a0 f   Metaphlan2Support.obj
 0001:000009c0       ??__E?ET_PYTHON_BIO@Metaphlan2Support@U2@@2VQString@@B@@YAXXZ 100019c0 f   Metaphlan2Support.obj
 0001:000009e0       ??__E?ET_PYTHON_NUMPY@Metaphlan2Support@U2@@2VQString@@B@@YAXXZ 100019e0 f   Metaphlan2Support.obj
 0001:00000a00       ??__E?TOOL_NAME@Metaphlan2Support@U2@@2VQString@@B@@YAXXZ 10001a00 f   Metaphlan2Support.obj
 0001:00000a20       ??__E?UTIL_SCRIPT@Metaphlan2Support@U2@@2VQString@@B@@YAXXZ 10001a20 f   Metaphlan2Support.obj
 0001:00000a40       ??__E?_Generic_object@?$_Error_objects@H@std@@2V_Generic_error_category@2@A@@YAXXZ 10001a40 f   Metaphlan2Support.obj
 0001:00000a50       ??__E?_Iostream_object@?$_Error_objects@H@std@@2V_Iostream_error_category@2@A@@YAXXZ 10001a50 f   Metaphlan2Support.obj
 0001:00000a60       ??__E?_System_object@?$_Error_objects@H@std@@2V_System_error_category@2@A@@YAXXZ 10001a60 f   Metaphlan2Support.obj
 0001:00000a70       ??__EalgoLog@U2@@YAXXZ     10001a70 f   Metaphlan2Support.obj
 0001:00000af0       ??__EcmdLog@U2@@YAXXZ      10001af0 f   Metaphlan2Support.obj
 0001:00000b70       ??__EcoreLog@U2@@YAXXZ     10001b70 f   Metaphlan2Support.obj
 0001:00000bf0       ??__EioLog@U2@@YAXXZ       10001bf0 f   Metaphlan2Support.obj
 0001:00000c70       ??__EperfLog@U2@@YAXXZ     10001c70 f   Metaphlan2Support.obj
 0001:00000cf0       ??__EscriptLog@U2@@YAXXZ   10001cf0 f   Metaphlan2Support.obj
 0001:00000d70       ??__EtaskLog@U2@@YAXXZ     10001d70 f   Metaphlan2Support.obj
 0001:00000df0       ??__EuiLog@U2@@YAXXZ       10001df0 f   Metaphlan2Support.obj
 0001:00000e70       ??__EuserActLog@U2@@YAXXZ  10001e70 f   Metaphlan2Support.obj
 0001:00000ef0       ??__E?PLUGIN_DESCRIPRION@MetaphlanSupportPlugin@U2@@2VQString@@B@@YAXXZ 10001ef0 f   Metaphlan2SupportPlugin.obj
 0001:00000f20       ??__E?PLUGIN_NAME@MetaphlanSupportPlugin@U2@@2VQString@@B@@YAXXZ 10001f20 f   Metaphlan2SupportPlugin.obj
 0001:00000f50       ??__E?_Generic_object@?$_Error_objects@H@std@@2V_Generic_error_category@2@A@@YAXXZ 10001f50 f   Metaphlan2SupportPlugin.obj
 0001:00000f60       ??__E?_Iostream_object@?$_Error_objects@H@std@@2V_Iostream_error_category@2@A@@YAXXZ 10001f60 f   Metaphlan2SupportPlugin.obj
 0001:00000f70       ??__E?_System_object@?$_Error_objects@H@std@@2V_System_error_category@2@A@@YAXXZ 10001f70 f   Metaphlan2SupportPlugin.obj
 0001:00000f80       ??__EalgoLog@U2@@YAXXZ     10001f80 f   Metaphlan2SupportPlugin.obj
 0001:00001000       ??__EcmdLog@U2@@YAXXZ      10002000 f   Metaphlan2SupportPlugin.obj
 0001:00001080       ??__EcoreLog@U2@@YAXXZ     10002080 f   Metaphlan2SupportPlugin.obj
 0001:00001100       ??__EioLog@U2@@YAXXZ       10002100 f   Metaphlan2SupportPlugin.obj
 0001:00001180       ??__EperfLog@U2@@YAXXZ     10002180 f   Metaphlan2SupportPlugin.obj
 0001:00001200       ??__EscriptLog@U2@@YAXXZ   10002200 f   Metaphlan2SupportPlugin.obj
 0001:00001280       ??__EtaskLog@U2@@YAXXZ     10002280 f   Metaphlan2SupportPlugin.obj
 0001:00001300       ??__EuiLog@U2@@YAXXZ       10002300 f   Metaphlan2SupportPlugin.obj
 0001:00001380       ??__EuserActLog@U2@@YAXXZ  10002380 f   Metaphlan2SupportPlugin.obj
 0001:00001400       ??__E?_Generic_object@?$_Error_objects@H@std@@2V_Generic_error_category@2@A@@YAXXZ 10002400 f   Metaphlan2Task.obj
 0001:00001410       ??__E?_Iostream_object@?$_Error_objects@H@std@@2V_Iostream_error_category@2@A@@YAXXZ 10002410 f   Metaphlan2Task.obj
 0001:00001420       ??__E?_System_object@?$_Error_objects@H@std@@2V_System_error_category@2@A@@YAXXZ 10002420 f   Metaphlan2Task.obj
 0001:00001430       ??__EalgoLog@U2@@YAXXZ     10002430 f   Metaphlan2Task.obj
 0001:000014b0       ??__EcmdLog@U2@@YAXXZ      100024b0 f   Metaphlan2Task.obj
 0001:00001530       ??__EcoreLog@U2@@YAXXZ     10002530 f   Metaphlan2Task.obj
 0001:000015b0       ??__EioLog@U2@@YAXXZ       100025b0 f   Metaphlan2Task.obj
 0001:00001630       ??__EperfLog@U2@@YAXXZ     10002630 f   Metaphlan2Task.obj
 0001:000016b0       ??__EscriptLog@U2@@YAXXZ   100026b0 f   Metaphlan2Task.obj
 0001:00001730       ??__EtaskLog@U2@@YAXXZ     10002730 f   Metaphlan2Task.obj
 0001:000017b0       ??__EuiLog@U2@@YAXXZ       100027b0 f   Metaphlan2Task.obj
 0001:00001830       ??__EuserActLog@U2@@YAXXZ  10002830 f   Metaphlan2Task.obj
 0001:000018b0       ??__E?_Generic_object@?$_Error_objects@H@std@@2V_Generic_error_category@2@A@@YAXXZ 100028b0 f   Metaphlan2Validator.obj
 0001:000018c0       ??__E?_Iostream_object@?$_Error_objects@H@std@@2V_Iostream_error_category@2@A@@YAXXZ 100028c0 f   Metaphlan2Validator.obj
 0001:000018d0       ??__E?_System_object@?$_Error_objects@H@std@@2V_System_error_category@2@A@@YAXXZ 100028d0 f   Metaphlan2Validator.obj
 0001:000018e0       ??__EalgoLog@U2@@YAXXZ     100028e0 f   Metaphlan2Validator.obj
 0001:00001960       ??__EcmdLog@U2@@YAXXZ      10002960 f   Metaphlan2Validator.obj
 0001:000019e0       ??__EcoreLog@U2@@YAXXZ     100029e0 f   Metaphlan2Validator.obj
 0001:00001a60       ??__EioLog@U2@@YAXXZ       10002a60 f   Metaphlan2Validator.obj
 0001:00001ae0       ??__EperfLog@U2@@YAXXZ     10002ae0 f   Metaphlan2Validator.obj
 0001:00001b60       ??__EscriptLog@U2@@YAXXZ   10002b60 f   Metaphlan2Validator.obj
 0001:00001be0       ??__EtaskLog@U2@@YAXXZ     10002be0 f   Metaphlan2Validator.obj
 0001:00001c60       ??__EuiLog@U2@@YAXXZ       10002c60 f   Metaphlan2Validator.obj
 0001:00001ce0       ??__EuserActLog@U2@@YAXXZ  10002ce0 f   Metaphlan2Validator.obj
 0001:00001d60       ??__E?BOWTIE2OUT_DIR@Metaphlan2Worker@LocalWorkflow@U2@@0VQString@@B@@YAXXZ 10002d60 f   Metaphlan2Worker.obj
 0001:00001d80       ??__E?BOWTIE2OUT_SUFFIX@Metaphlan2Worker@LocalWorkflow@U2@@0VQString@@B@@YAXXZ 10002d80 f   Metaphlan2Worker.obj
 0001:00001da0       ??__E?METAPHLAN2_ROOT_DIR@Metaphlan2Worker@LocalWorkflow@U2@@0VQString@@B@@YAXXZ 10002da0 f   Metaphlan2Worker.obj
 0001:00001dc0       ??__E?PROFILE_DIR@Metaphlan2Worker@LocalWorkflow@U2@@0VQString@@B@@YAXXZ 10002dc0 f   Metaphlan2Worker.obj
 0001:00001de0       ??__E?PROFILE_SUFFIX@Metaphlan2Worker@LocalWorkflow@U2@@0VQString@@B@@YAXXZ 10002de0 f   Metaphlan2Worker.obj
 0001:00001e00       ??__E?_Generic_object@?$_Error_objects@H@std@@2V_Generic_error_category@2@A@@YAXXZ 10002e00 f   Metaphlan2Worker.obj
 0001:00001e10       ??__E?_Iostream_object@?$_Error_objects@H@std@@2V_Iostream_error_category@2@A@@YAXXZ 10002e10 f   Metaphlan2Worker.obj
 0001:00001e20       ??__E?_System_object@?$_Error_objects@H@std@@2V_System_error_category@2@A@@YAXXZ 10002e20 f   Metaphlan2Worker.obj
 0001:00001e30       ??__EalgoLog@U2@@YAXXZ     10002e30 f   Metaphlan2Worker.obj
 0001:00001eb0       ??__EcmdLog@U2@@YAXXZ      10002eb0 f   Metaphlan2Worker.obj
 0001:00001f30       ??__EcoreLog@U2@@YAXXZ     10002f30 f   Metaphlan2Worker.obj
 0001:00001fb0       ??__EioLog@U2@@YAXXZ       10002fb0 f   Metaphlan2Worker.obj
 0001:00002030       ??__EperfLog@U2@@YAXXZ     10003030 f   Metaphlan2Worker.obj
 0001:000020b0       ??__EscriptLog@U2@@YAXXZ   100030b0 f   Metaphlan2Worker.obj
 0001:00002130       ??__EtaskLog@U2@@YAXXZ     10003130 f   Metaphlan2Worker.obj
 0001:000021b0       ??__EuiLog@U2@@YAXXZ       100031b0 f   Metaphlan2Worker.obj
 0001:00002230       ??__EuserActLog@U2@@YAXXZ  10003230 f   Metaphlan2Worker.obj
 0001:000022b0       ??__E?ACTOR_ID@Metaphlan2WorkerFactory@LocalWorkflow@U2@@2VQString@@B@@YAXXZ 100032b0 f   Metaphlan2WorkerFactory.obj
 0001:000022d0       ??__E?ANALYSIS_TYPE@Metaphlan2WorkerFactory@LocalWorkflow@U2@@2VQString@@B@@YAXXZ 100032d0 f   Metaphlan2WorkerFactory.obj
 0001:000022f0       ??__E?ANALYSIS_TYPE_CLADE_PROFILES_TEXT@Metaphlan2WorkerFactory@LocalWorkflow@U2@@2VQString@@B@@YAXXZ 100032f0 f   Metaphlan2WorkerFactory.obj
 0001:00002320       ??__E?ANALYSIS_TYPE_CLADE_PROFILES_VALUE@Metaphlan2WorkerFactory@LocalWorkflow@U2@@2VQString@@B@@YAXXZ 10003320 f   Metaphlan2WorkerFactory.obj
 0001:00002340       ??__E?ANALYSIS_TYPE_MARKER_AB_TABLE_TEXT@Metaphlan2WorkerFactory@LocalWorkflow@U2@@2VQString@@B@@YAXXZ 10003340 f   Metaphlan2WorkerFactory.obj
 0001:00002370       ??__E?ANALYSIS_TYPE_MARKER_AB_TABLE_VALUE@Metaphlan2WorkerFactory@LocalWorkflow@U2@@2VQString@@B@@YAXXZ 10003370 f   Metaphlan2WorkerFactory.obj
 0001:00002390       ??__E?ANALYSIS_TYPE_MARKER_PRES_TABLE_TEXT@Metaphlan2WorkerFactory@LocalWorkflow@U2@@2VQString@@B@@YAXXZ 10003390 f   Metaphlan2WorkerFactory.obj
 0001:000023c0       ??__E?ANALYSIS_TYPE_MARKER_PRES_TABLE_VALUE@Metaphlan2WorkerFactory@LocalWorkflow@U2@@2VQString@@B@@YAXXZ 100033c0 f   Metaphlan2WorkerFactory.obj
 0001:000023e0       ??__E?ANALYSIS_TYPE_READS_MAP_TEXT@Metaphlan2WorkerFactory@LocalWorkflow@U2@@2VQString@@B@@YAXXZ 100033e0 f   Metaphlan2WorkerFactory.obj
 0001:00002410       ??__E?ANALYSIS_TYPE_READS_MAP_VALUE@Metaphlan2WorkerFactory@LocalWorkflow@U2@@2VQString@@B@@YAXXZ 10003410 f   Metaphlan2WorkerFactory.obj
 0001:00002430       ??__E?ANALYSIS_TYPE_REL_AB_TEXT@Metaphlan2WorkerFactory@LocalWorkflow@U2@@2VQString@@B@@YAXXZ 10003430 f   Metaphlan2WorkerFactory.obj
 0001:00002460       ??__E?ANALYSIS_TYPE_REL_AB_VALUE@Metaphlan2WorkerFactory@LocalWorkflow@U2@@2VQString@@B@@YAXXZ 10003460 f   Metaphlan2WorkerFactory.obj
 0001:00002480       ??__E?ANALYSIS_TYPE_REL_AB_W_READ_STATS_TEXT@Metaphlan2WorkerFactory@LocalWorkflow@U2@@2VQString@@B@@YAXXZ 10003480 f   Metaphlan2WorkerFactory.obj
 0001:000024b0       ??__E?ANALYSIS_TYPE_REL_AB_W_READ_STATS_VALUE@Metaphlan2WorkerFactory@LocalWorkflow@U2@@2VQString@@B@@YAXXZ 100034b0 f   Metaphlan2WorkerFactory.obj
 0001:000024d0       ??__E?BOWTIE2_OUTPUT_URL@Metaphlan2WorkerFactory@LocalWorkflow@U2@@2VQString@@B@@YAXXZ 100034d0 f   Metaphlan2WorkerFactory.obj
 0001:000024f0       ??__E?DB_URL@Metaphlan2WorkerFactory@LocalWorkflow@U2@@2VQString@@B@@YAXXZ 100034f0 f   Metaphlan2WorkerFactory.obj
 0001:00002510       ??__E?INPUT_PORT_ID@Metaphlan2WorkerFactory@LocalWorkflow@U2@@2VQString@@B@@YAXXZ 10003510 f   Metaphlan2WorkerFactory.obj
 0001:00002530       ??__E?INPUT_SLOT@Metaphlan2WorkerFactory@LocalWorkflow@U2@@2VQString@@B@@YAXXZ 10003530 f   Metaphlan2WorkerFactory.obj
 0001:00002550       ??__E?NORMALIZE@Metaphlan2WorkerFactory@LocalWorkflow@U2@@2VQString@@B@@YAXXZ 10003550 f   Metaphlan2WorkerFactory.obj
 0001:00002570       ??__E?NOT_SKIP_NORMILIZE_BY_SIZE@Metaphlan2WorkerFactory@LocalWorkflow@U2@@2VQString@@B@@YAXXZ 10003570 f   Metaphlan2WorkerFactory.obj
 0001:00002590       ??__E?NUM_THREADS@Metaphlan2WorkerFactory@LocalWorkflow@U2@@2VQString@@B@@YAXXZ 10003590 f   Metaphlan2WorkerFactory.obj
 0001:000025b0       ??__E?OUTPUT_URL@Metaphlan2WorkerFactory@LocalWorkflow@U2@@2VQString@@B@@YAXXZ 100035b0 f   Metaphlan2WorkerFactory.obj
 0001:000025d0       ??__E?PAIRED_END@Metaphlan2WorkerFactory@LocalWorkflow@U2@@2VQString@@B@@YAXXZ 100035d0 f   Metaphlan2WorkerFactory.obj
 0001:000025f0       ??__E?PAIRED_END_TEXT@Metaphlan2WorkerFactory@LocalWorkflow@U2@@2VQString@@B@@YAXXZ 100035f0 f   Metaphlan2WorkerFactory.obj
 0001:00002620       ??__E?PAIRED_INPUT_SLOT@Metaphlan2WorkerFactory@LocalWorkflow@U2@@2VQString@@B@@YAXXZ 10003620 f   Metaphlan2WorkerFactory.obj
 0001:00002640       ??__E?PRESENCE_THRESHOLD@Metaphlan2WorkerFactory@LocalWorkflow@U2@@2VQString@@B@@YAXXZ 10003640 f   Metaphlan2WorkerFactory.obj
 0001:00002660       ??__E?SEQUENCING_READS@Metaphlan2WorkerFactory@LocalWorkflow@U2@@2VQString@@B@@YAXXZ 10003660 f   Metaphlan2WorkerFactory.obj
 0001:00002680       ??__E?SINGLE_END@Metaphlan2WorkerFactory@LocalWorkflow@U2@@2VQString@@B@@YAXXZ 10003680 f   Metaphlan2WorkerFactory.obj
 0001:000026a0       ??__E?SINGLE_END_TEXT@Metaphlan2WorkerFactory@LocalWorkflow@U2@@2VQString@@B@@YAXXZ 100036a0 f   Metaphlan2WorkerFactory.obj
 0001:000026d0       ??__E?SKIP_NORMILIZE_BY_SIZE@Metaphlan2WorkerFactory@LocalWorkflow@U2@@2VQString@@B@@YAXXZ 100036d0 f   Metaphlan2WorkerFactory.obj
 0001:000026f0       ??__E?TAX_LEVEL@Metaphlan2WorkerFactory@LocalWorkflow@U2@@2VQString@@B@@YAXXZ 100036f0 f   Metaphlan2WorkerFactory.obj
 0001:00002710       ??__E?TAX_LEVEL_ALL_TEXT@Metaphlan2WorkerFactory@LocalWorkflow@U2@@2VQString@@B@@YAXXZ 10003710 f   Metaphlan2WorkerFactory.obj
 0001:00002730       ??__E?TAX_LEVEL_ALL_VALUE@Metaphlan2WorkerFactory@LocalWorkflow@U2@@2VQString@@B@@YAXXZ 10003730 f   Metaphlan2WorkerFactory.obj
 0001:00002750       ??__E?TAX_LEVEL_CLASSES_TEXT@Metaphlan2WorkerFactory@LocalWorkflow@U2@@2VQString@@B@@YAXXZ 10003750 f   Metaphlan2WorkerFactory.obj
 0001:00002770       ??__E?TAX_LEVEL_CLASSES_VALUE@Metaphlan2WorkerFactory@LocalWorkflow@U2@@2VQString@@B@@YAXXZ 10003770 f   Metaphlan2WorkerFactory.obj
 0001:00002790       ??__E?TAX_LEVEL_FAMILIES_TEXT@Metaphlan2WorkerFactory@LocalWorkflow@U2@@2VQString@@B@@YAXXZ 10003790 f   Metaphlan2WorkerFactory.obj
 0001:000027b0       ??__E?TAX_LEVEL_FAMILIES_VALUE@Metaphlan2WorkerFactory@LocalWorkflow@U2@@2VQString@@B@@YAXXZ 100037b0 f   Metaphlan2WorkerFactory.obj
 0001:000027d0       ??__E?TAX_LEVEL_GENERA_TEXT@Metaphlan2WorkerFactory@LocalWorkflow@U2@@2VQString@@B@@YAXXZ 100037d0 f   Metaphlan2WorkerFactory.obj
 0001:000027f0       ??__E?TAX_LEVEL_GENERA_VALUE@Metaphlan2WorkerFactory@LocalWorkflow@U2@@2VQString@@B@@YAXXZ 100037f0 f   Metaphlan2WorkerFactory.obj
 0001:00002810       ??__E?TAX_LEVEL_KINGDOMS_TEXT@Metaphlan2WorkerFactory@LocalWorkflow@U2@@2VQString@@B@@YAXXZ 10003810 f   Metaphlan2WorkerFactory.obj
 0001:00002830       ??__E?TAX_LEVEL_KINGDOMS_VALUE@Metaphlan2WorkerFactory@LocalWorkflow@U2@@2VQString@@B@@YAXXZ 10003830 f   Metaphlan2WorkerFactory.obj
 0001:00002850       ??__E?TAX_LEVEL_ORDERS_TEXT@Metaphlan2WorkerFactory@LocalWorkflow@U2@@2VQString@@B@@YAXXZ 10003850 f   Metaphlan2WorkerFactory.obj
 0001:00002870       ??__E?TAX_LEVEL_ORDERS_VALUE@Metaphlan2WorkerFactory@LocalWorkflow@U2@@2VQString@@B@@YAXXZ 10003870 f   Metaphlan2WorkerFactory.obj
 0001:00002890       ??__E?TAX_LEVEL_PHYLA_TEXT@Metaphlan2WorkerFactory@LocalWorkflow@U2@@2VQString@@B@@YAXXZ 10003890 f   Metaphlan2WorkerFactory.obj
 0001:000028b0       ??__E?TAX_LEVEL_PHYLA_VALUE@Metaphlan2WorkerFactory@LocalWorkflow@U2@@2VQString@@B@@YAXXZ 100038b0 f   Metaphlan2WorkerFactory.obj
 0001:000028d0       ??__E?TAX_LEVEL_SPECIES_TEXT@Metaphlan2WorkerFactory@LocalWorkflow@U2@@2VQString@@B@@YAXXZ 100038d0 f   Metaphlan2WorkerFactory.obj
 0001:000028f0       ??__E?TAX_LEVEL_SPECIES_VALUE@Metaphlan2WorkerFactory@LocalWorkflow@U2@@2VQString@@B@@YAXXZ 100038f0 f   Metaphlan2WorkerFactory.obj
 0001:00002910       ??__E?_Generic_object@?$_Error_objects@H@std@@2V_Generic_error_category@2@A@@YAXXZ 10003910 f   Metaphlan2WorkerFactory.obj
 0001:00002920       ??__E?_Iostream_object@?$_Error_objects@H@std@@2V_Iostream_error_category@2@A@@YAXXZ 10003920 f   Metaphlan2WorkerFactory.obj
 0001:00002930       ??__E?_System_object@?$_Error_objects@H@std@@2V_System_error_category@2@A@@YAXXZ 10003930 f   Metaphlan2WorkerFactory.obj
 0001:00002940       ??__EalgoLog@U2@@YAXXZ     10003940 f   Metaphlan2WorkerFactory.obj
 0001:000029c0       ??__EcmdLog@U2@@YAXXZ      100039c0 f   Metaphlan2WorkerFactory.obj
 0001:00002a40       ??__EcoreLog@U2@@YAXXZ     10003a40 f   Metaphlan2WorkerFactory.obj
 0001:00002ac0       ??__EioLog@U2@@YAXXZ       10003ac0 f   Metaphlan2WorkerFactory.obj
 0001:00002b40       ??__EperfLog@U2@@YAXXZ     10003b40 f   Metaphlan2WorkerFactory.obj
 0001:00002bc0       ??__EscriptLog@U2@@YAXXZ   10003bc0 f   Metaphlan2WorkerFactory.obj
 0001:00002c40       ??__EtaskLog@U2@@YAXXZ     10003c40 f   Metaphlan2WorkerFactory.obj
 0001:00002cc0       ??__EuiLog@U2@@YAXXZ       10003cc0 f   Metaphlan2WorkerFactory.obj
 0001:00002d40       ??__EuserActLog@U2@@YAXXZ  10003d40 f   Metaphlan2WorkerFactory.obj
 0001:00002dc0       ??__E?_Generic_object@?$_Error_objects@H@std@@2V_Generic_error_category@2@A@@YAXXZ 10003dc0 f   moc_Metaphlan2Prompter.obj
 0001:00002dd0       ??__E?_Iostream_object@?$_Error_objects@H@std@@2V_Iostream_error_category@2@A@@YAXXZ 10003dd0 f   moc_Metaphlan2Prompter.obj
 0001:00002de0       ??__E?_System_object@?$_Error_objects@H@std@@2V_System_error_category@2@A@@YAXXZ 10003de0 f   moc_Metaphlan2Prompter.obj
 0001:00002df0       ??__E?staticMetaObject@Metaphlan2Prompter@LocalWorkflow@U2@@2UQMetaObject@@B@@YAXXZ 10003df0 f   moc_Metaphlan2Prompter.obj
 0001:00002e00       ??__EalgoLog@U2@@YAXXZ     10003e00 f   moc_Metaphlan2Prompter.obj
 0001:00002e80       ??__EcmdLog@U2@@YAXXZ      10003e80 f   moc_Metaphlan2Prompter.obj
 0001:00002f00       ??__EcoreLog@U2@@YAXXZ     10003f00 f   moc_Metaphlan2Prompter.obj
 0001:00002f80       ??__EioLog@U2@@YAXXZ       10003f80 f   moc_Metaphlan2Prompter.obj
 0001:00003000       ??__EperfLog@U2@@YAXXZ     10004000 f   moc_Metaphlan2Prompter.obj
 0001:00003080       ??__EscriptLog@U2@@YAXXZ   10004080 f   moc_Metaphlan2Prompter.obj
 0001:00003100       ??__EtaskLog@U2@@YAXXZ     10004100 f   moc_Metaphlan2Prompter.obj
 0001:00003180       ??__EuiLog@U2@@YAXXZ       10004180 f   moc_Metaphlan2Prompter.obj
 0001:00003200       ??__EuserActLog@U2@@YAXXZ  10004200 f   moc_Metaphlan2Prompter.obj
 0001:00003280       ??__E?_Generic_object@?$_Error_objects@H@std@@2V_Generic_error_category@2@A@@YAXXZ 10004280 f   moc_Metaphlan2Support.obj
 0001:00003290       ??__E?_Iostream_object@?$_Error_objects@H@std@@2V_Iostream_error_category@2@A@@YAXXZ 10004290 f   moc_Metaphlan2Support.obj
 0001:000032a0       ??__E?_System_object@?$_Error_objects@H@std@@2V_System_error_category@2@A@@YAXXZ 100042a0 f   moc_Metaphlan2Support.obj
 0001:000032b0       ??__E?staticMetaObject@Metaphlan2Support@U2@@2UQMetaObject@@B@@YAXXZ 100042b0 f   moc_Metaphlan2Support.obj
 0001:000032c0       ??__E?_Generic_object@?$_Error_objects@H@std@@2V_Generic_error_category@2@A@@YAXXZ 100042c0 f   moc_Metaphlan2SupportPlugin.obj
 0001:000032d0       ??__E?_Iostream_object@?$_Error_objects@H@std@@2V_Iostream_error_category@2@A@@YAXXZ 100042d0 f   moc_Metaphlan2SupportPlugin.obj
 0001:000032e0       ??__E?_System_object@?$_Error_objects@H@std@@2V_System_error_category@2@A@@YAXXZ 100042e0 f   moc_Metaphlan2SupportPlugin.obj
 0001:000032f0       ??__E?staticMetaObject@MetaphlanSupportPlugin@U2@@2UQMetaObject@@B@@YAXXZ 100042f0 f   moc_Metaphlan2SupportPlugin.obj
 0001:00003300       ??__E?_Generic_object@?$_Error_objects@H@std@@2V_Generic_error_category@2@A@@YAXXZ 10004300 f   moc_Metaphlan2Task.obj
 0001:00003310       ??__E?_Iostream_object@?$_Error_objects@H@std@@2V_Iostream_error_category@2@A@@YAXXZ 10004310 f   moc_Metaphlan2Task.obj
 0001:00003320       ??__E?_System_object@?$_Error_objects@H@std@@2V_System_error_category@2@A@@YAXXZ 10004320 f   moc_Metaphlan2Task.obj
 0001:00003330       ??__E?staticMetaObject@Metaphlan2ClassifyTask@U2@@2UQMetaObject@@B@@YAXXZ 10004330 f   moc_Metaphlan2Task.obj
 0001:00003340       ??__EalgoLog@U2@@YAXXZ     10004340 f   moc_Metaphlan2Task.obj
 0001:000033c0       ??__EcmdLog@U2@@YAXXZ      100043c0 f   moc_Metaphlan2Task.obj
 0001:00003440       ??__EcoreLog@U2@@YAXXZ     10004440 f   moc_Metaphlan2Task.obj
 0001:000034c0       ??__EioLog@U2@@YAXXZ       100044c0 f   moc_Metaphlan2Task.obj
 0001:00003540       ??__EperfLog@U2@@YAXXZ     10004540 f   moc_Metaphlan2Task.obj
 0001:000035c0       ??__EscriptLog@U2@@YAXXZ   100045c0 f   moc_Metaphlan2Task.obj
 0001:00003640       ??__EtaskLog@U2@@YAXXZ     10004640 f   moc_Metaphlan2Task.obj
 0001:000036c0       ??__EuiLog@U2@@YAXXZ       100046c0 f   moc_Metaphlan2Task.obj
 0001:00003740       ??__EuserActLog@U2@@YAXXZ  10004740 f   moc_Metaphlan2Task.obj
 0001:000037c0       ??__E?_Generic_object@?$_Error_objects@H@std@@2V_Generic_error_category@2@A@@YAXXZ 100047c0 f   moc_Metaphlan2Worker.obj
 0001:000037d0       ??__E?_Iostream_object@?$_Error_objects@H@std@@2V_Iostream_error_category@2@A@@YAXXZ 100047d0 f   moc_Metaphlan2Worker.obj
 0001:000037e0       ??__E?_System_object@?$_Error_objects@H@std@@2V_System_error_category@2@A@@YAXXZ 100047e0 f   moc_Metaphlan2Worker.obj
 0001:000037f0       ??__E?staticMetaObject@Metaphlan2Worker@LocalWorkflow@U2@@2UQMetaObject@@B@@YAXXZ 100047f0 f   moc_Metaphlan2Worker.obj
 0001:00003800       ??__EalgoLog@U2@@YAXXZ     10004800 f   moc_Metaphlan2Worker.obj
 0001:00003880       ??__EcmdLog@U2@@YAXXZ      10004880 f   moc_Metaphlan2Worker.obj
 0001:00003900       ??__EcoreLog@U2@@YAXXZ     10004900 f   moc_Metaphlan2Worker.obj
 0001:00003980       ??__EioLog@U2@@YAXXZ       10004980 f   moc_Metaphlan2Worker.obj
 0001:00003a00       ??__EperfLog@U2@@YAXXZ     10004a00 f   moc_Metaphlan2Worker.obj
 0001:00003a80       ??__EscriptLog@U2@@YAXXZ   10004a80 f   moc_Metaphlan2Worker.obj
 0001:00003b00       ??__EtaskLog@U2@@YAXXZ     10004b00 f   moc_Metaphlan2Worker.obj
 0001:00003b80       ??__EuiLog@U2@@YAXXZ       10004b80 f   moc_Metaphlan2Worker.obj
 0001:00003c00       ??__EuserActLog@U2@@YAXXZ  10004c00 f   moc_Metaphlan2Worker.obj
 0001:00003e9e       __catch$??0?$QList@VQString@@@@QAE@ABV0@@Z$0 10004e9e f i Metaphlan2LogParser.obj
 0001:00004366       __catch$?_Copy@?$basic_string@DU?$char_traits@D@std@@V?$allocator@D@2@@std@@QAEXII@Z$0 10005366 f i Metaphlan2LogParser.obj
 0001:000043a3       __catch$?_Copy@?$basic_string@DU?$char_traits@D@std@@V?$allocator@D@2@@std@@QAEXII@Z$1 100053a3 f i Metaphlan2LogParser.obj
 0001:000046bd       __catch$?append@?$QList@VQString@@@@QAEXABVQString@@@Z$0 100056bd f i Metaphlan2LogParser.obj
 0001:0000470e       __catch$?append@?$QList@VQString@@@@QAEXABVQString@@@Z$4 1000570e f i Metaphlan2LogParser.obj
 0001:00004c2e       __catch$?detach_helper_grow@?$QList@VQString@@@@AAEPAUNode@1@HH@Z$2 10005c2e f i Metaphlan2LogParser.obj
 0001:00004c69       __catch$?detach_helper_grow@?$QList@VQString@@@@AAEPAUNode@1@HH@Z$0 10005c69 f i Metaphlan2LogParser.obj
 0001:000052e2       __catch$?node_copy@?$QList@VQString@@@@AAEXPAUNode@1@00@Z$2 100062e2 f i Metaphlan2LogParser.obj
 0001:0000552e       __catch$??0?$QList@PAVPort@Workflow@U2@@@@QAE@ABV0@@Z$0 1000652e f i Metaphlan2Prompter.obj
 0001:00006a05       __catch$?append@?$QList@PAVTask@U2@@@@QAEXABQAVTask@U2@@@Z$4 10007a05 f i Metaphlan2Task.obj
 0001:00006b61       __catch$?detach_helper@?$QList@VQString@@@@AAEXH@Z$0 10007b61 f i Metaphlan2Task.obj
 0001:00006c81       __catch$?detach_helper_grow@?$QList@PAVTask@U2@@@@AAEPAUNode@1@HH@Z$0 10007c81 f i Metaphlan2Task.obj
 0001:00006c81       __catch$?detach_helper_grow@?$QList@PAVTask@U2@@@@AAEPAUNode@1@HH@Z$2 10007c81 f i Metaphlan2Task.obj
 0001:00007dc0       __catch$?append@?$QList@VWorkflowNotification@U2@@@@QAEXABVWorkflowNotification@U2@@@Z$2 10008dc0 f i Metaphlan2Validator.obj
 0001:00007dc0       __catch$?append@?$QList@VWorkflowNotification@U2@@@@QAEXABVWorkflowNotification@U2@@@Z$0 10008dc0 f i Metaphlan2Validator.obj
 0001:00007f4f       __catch$?detach_helper_grow@?$QList@VWorkflowNotification@U2@@@@AAEPAUNode@1@HH@Z$2 10008f4f f i Metaphlan2Validator.obj
 0001:00007f8a       __catch$?detach_helper_grow@?$QList@VWorkflowNotification@U2@@@@AAEPAUNode@1@HH@Z$0 10008f8a f i Metaphlan2Validator.obj
 0001:0000818e       __catch$?node_copy@?$QList@VWorkflowNotification@U2@@@@AAEXPAUNode@1@00@Z$0 1000918e f i Metaphlan2Validator.obj
 0001:0000904e       __catch$??0?$QList@VDescriptor@U2@@@@QAE@ABV0@@Z$0 1000a04e f i Metaphlan2Worker.obj
 0001:0000982c       __catch$?append@?$QList@VDescriptor@U2@@@@QAEXABVDescriptor@U2@@@Z$0 1000a82c f i Metaphlan2Worker.obj
 0001:0000982c       __catch$?append@?$QList@VDescriptor@U2@@@@QAEXABVDescriptor@U2@@@Z$2 1000a82c f i Metaphlan2Worker.obj
 0001:00009bae       __catch$?createNode@?$QMapData@VQString@@VQScriptValue@@@@QAEPAU?$QMapNode@VQString@@VQScriptValue@@@@ABVQString@@ABVQScriptValue@@PAU2@_N@Z$0 1000abae f i Metaphlan2Worker.obj
 0001:00009bc3       __catch$?createNode@?$QMapData@VQString@@VQScriptValue@@@@QAEPAU?$QMapNode@VQString@@VQScriptValue@@@@ABVQString@@ABVQScriptValue@@PAU2@_N@Z$2 1000abc3 f i Metaphlan2Worker.obj
 0001:00009c6e       __catch$?createNode@?$QMapData@VQString@@VQVariant@@@@QAEPAU?$QMapNode@VQString@@VQVariant@@@@ABVQString@@ABVQVariant@@PAU2@_N@Z$0 1000ac6e f i Metaphlan2Worker.obj
 0001:00009c83       __catch$?createNode@?$QMapData@VQString@@VQVariant@@@@QAEPAU?$QMapNode@VQString@@VQVariant@@@@ABVQString@@ABVQVariant@@PAU2@_N@Z$2 1000ac83 f i Metaphlan2Worker.obj
 0001:0000a14a       __catch$?detach_helper@?$QList@VDescriptor@U2@@@@AAEXH@Z$0 1000b14a f i Metaphlan2Worker.obj
 0001:0000a35f       __catch$?detach_helper_grow@?$QList@VDescriptor@U2@@@@AAEPAUNode@1@HH@Z$2 1000b35f f i Metaphlan2Worker.obj
 0001:0000a39a       __catch$?detach_helper_grow@?$QList@VDescriptor@U2@@@@AAEPAUNode@1@HH@Z$0 1000b39a f i Metaphlan2Worker.obj
 0001:0000b665       __catch$?node_copy@?$QList@VDescriptor@U2@@@@AAEXPAUNode@1@00@Z$0 1000c665 f i Metaphlan2Worker.obj
 0001:0000c845       __catch$?append@?$QList@PAVAttribute@U2@@@@QAEXABQAVAttribute@U2@@@Z$4 1000d845 f i Metaphlan2WorkerFactory.obj
 0001:0000c8d5       __catch$?append@?$QList@PAVPortDescriptor@Workflow@U2@@@@QAEXABQAVPortDescriptor@Workflow@U2@@@Z$4 1000d8d5 f i Metaphlan2WorkerFactory.obj
 0001:0000c932       __catch$?append@?$QList@U?$QPair@VQString@@V1@@@@@QAEXABU?$QPair@VQString@@V1@@@@Z$2 1000d932 f i Metaphlan2WorkerFactory.obj
 0001:0000c932       __catch$?append@?$QList@U?$QPair@VQString@@V1@@@@@QAEXABU?$QPair@VQString@@V1@@@@Z$0 1000d932 f i Metaphlan2WorkerFactory.obj
 0001:0000ca10       __catch$?append@?$QList@VQVariant@@@@QAEXABVQVariant@@@Z$2 1000da10 f i Metaphlan2WorkerFactory.obj
 0001:0000ca10       __catch$?append@?$QList@VQVariant@@@@QAEXABVQVariant@@@Z$0 1000da10 f i Metaphlan2WorkerFactory.obj
 0001:0000cc7d       __catch$?createNode@?$QMapData@VDescriptor@U2@@V?$QExplicitlySharedDataPointer@VDataType@U2@@@@@@QAEPAU?$QMapNode@VDescriptor@U2@@V?$QExplicitlySharedDataPointer@VDataType@U2@@@@@@ABVDescriptor@U2@@ABV?$QExplicitlySharedDataPointer@VDataType@U2@@@@PAU2@_N@Z$2 1000dc7d f i Metaphlan2WorkerFactory.obj
 0001:0000cd25       __catch$?createNode@?$QMapData@VQString@@PAVPropertyDelegate@U2@@@@QAEPAU?$QMapNode@VQString@@PAVPropertyDelegate@U2@@@@ABVQString@@ABQAVPropertyDelegate@U2@@PAU2@_N@Z$2 1000dd25 f i Metaphlan2WorkerFactory.obj
 0001:0000d1e1       __catch$?detach_helper_grow@?$QList@PAVAttribute@U2@@@@AAEPAUNode@1@HH@Z$2 1000e1e1 f i Metaphlan2WorkerFactory.obj
 0001:0000d1e1       __catch$?detach_helper_grow@?$QList@PAVAttribute@U2@@@@AAEPAUNode@1@HH@Z$0 1000e1e1 f i Metaphlan2WorkerFactory.obj
 0001:0000d2f1       __catch$?detach_helper_grow@?$QList@PAVPortDescriptor@Workflow@U2@@@@AAEPAUNode@1@HH@Z$0 1000e2f1 f i Metaphlan2WorkerFactory.obj
 0001:0000d2f1       __catch$?detach_helper_grow@?$QList@PAVPortDescriptor@Workflow@U2@@@@AAEPAUNode@1@HH@Z$2 1000e2f1 f i Metaphlan2WorkerFactory.obj
 0001:0000d41c       __catch$?detach_helper_grow@?$QList@U?$QPair@VQString@@V1@@@@@AAEPAUNode@1@HH@Z$2 1000e41c f i Metaphlan2WorkerFactory.obj
 0001:0000d457       __catch$?detach_helper_grow@?$QList@U?$QPair@VQString@@V1@@@@@AAEPAUNode@1@HH@Z$0 1000e457 f i Metaphlan2WorkerFactory.obj
 0001:0000d56f       __catch$?detach_helper_grow@?$QList@VQVariant@@@@AAEPAUNode@1@HH@Z$2 1000e56f f i Metaphlan2WorkerFactory.obj
 0001:0000d5aa       __catch$?detach_helper_grow@?$QList@VQVariant@@@@AAEPAUNode@1@HH@Z$0 1000e5aa f i Metaphlan2WorkerFactory.obj
 0001:0000fc9b       __catch$?node_copy@?$QList@U?$QPair@VQString@@V1@@@@@AAEXPAUNode@1@00@Z$0 10010c9b f i Metaphlan2WorkerFactory.obj
 0001:0000fd7e       __catch$?node_copy@?$QList@VQVariant@@@@AAEXPAUNode@1@00@Z$0 10010d7e f i Metaphlan2WorkerFactory.obj
 0001:00011170       _pre_c_init                10012170 f   MSVCRT:crtdll.obj
 0001:000113dd       ___DllMainCRTStartup       100123dd f   MSVCRT:crtdll.obj
 0001:00011530       $$000000                   10012530     MSVCRT:sehprolg4.obj
 0001:00011945       ?ArrayUnwindFilter@@YAHPAU_EXCEPTION_POINTERS@@@Z 10012945 f   MSVCRT:ehvecdtr.obj
 0001:00011c90       __ehhandler$??0?$QList@VQString@@@@QAE@ABV0@@Z 10012c90 f   Metaphlan2LogParser.obj
 0001:00011cb0       __unwindfunclet$??__EalgoLog@U2@@YAXXZ$0 10012cb0 f   Metaphlan2LogParser.obj
 0001:00011cb9       __ehhandler$??__EalgoLog@U2@@YAXXZ 10012cb9 f   Metaphlan2LogParser.obj
 0001:00011ce0       __unwindfunclet$??__EcmdLog@U2@@YAXXZ$0 10012ce0 f   Metaphlan2LogParser.obj
 0001:00011ce9       __ehhandler$??__EcmdLog@U2@@YAXXZ 10012ce9 f   Metaphlan2LogParser.obj
 0001:00011d10       __unwindfunclet$??__EcoreLog@U2@@YAXXZ$0 10012d10 f   Metaphlan2LogParser.obj
 0001:00011d19       __ehhandler$??__EcoreLog@U2@@YAXXZ 10012d19 f   Metaphlan2LogParser.obj
 0001:00011d40       __unwindfunclet$??__EioLog@U2@@YAXXZ$0 10012d40 f   Metaphlan2LogParser.obj
 0001:00011d49       __ehhandler$??__EioLog@U2@@YAXXZ 10012d49 f   Metaphlan2LogParser.obj
 0001:00011d70       __unwindfunclet$??__EperfLog@U2@@YAXXZ$0 10012d70 f   Metaphlan2LogParser.obj
 0001:00011d79       __ehhandler$??__EperfLog@U2@@YAXXZ 10012d79 f   Metaphlan2LogParser.obj
 0001:00011da0       __unwindfunclet$??__EscriptLog@U2@@YAXXZ$0 10012da0 f   Metaphlan2LogParser.obj
 0001:00011da9       __ehhandler$??__EscriptLog@U2@@YAXXZ 10012da9 f   Metaphlan2LogParser.obj
 0001:00011dd0       __unwindfunclet$??__EtaskLog@U2@@YAXXZ$0 10012dd0 f   Metaphlan2LogParser.obj
 0001:00011dd9       __ehhandler$??__EtaskLog@U2@@YAXXZ 10012dd9 f   Metaphlan2LogParser.obj
 0001:00011e00       __unwindfunclet$??__EuiLog@U2@@YAXXZ$0 10012e00 f   Metaphlan2LogParser.obj
 0001:00011e09       __ehhandler$??__EuiLog@U2@@YAXXZ 10012e09 f   Metaphlan2LogParser.obj
 0001:00011e30       __unwindfunclet$??__EuserActLog@U2@@YAXXZ$0 10012e30 f   Metaphlan2LogParser.obj
 0001:00011e39       __ehhandler$??__EuserActLog@U2@@YAXXZ 10012e39 f   Metaphlan2LogParser.obj
 0001:00011e60       __ehhandler$?_Copy@?$basic_string@DU?$char_traits@D@std@@V?$allocator@D@2@@std@@QAEXII@Z 10012e60 f   Metaphlan2LogParser.obj
 0001:00011e80       __unwindfunclet$?append@?$QList@VQString@@@@QAEXABVQString@@@Z$7 10012e80 f   Metaphlan2LogParser.obj
 0001:00011e91       __unwindfunclet$?append@?$QList@VQString@@@@QAEXABVQString@@@Z$11 10012e91 f   Metaphlan2LogParser.obj
 0001:00011ea2       __ehhandler$?append@?$QList@VQString@@@@QAEXABVQString@@@Z 10012ea2 f   Metaphlan2LogParser.obj
 0001:00011ec0       __ehhandler$?detach_helper_grow@?$QList@VQString@@@@AAEPAUNode@1@HH@Z 10012ec0 f   Metaphlan2LogParser.obj
 0001:00011ee0       __unwindfunclet$?initWellKnownErrors@Metaphlan2LogParser@U2@@CA?AVQStringList@@XZ$0 10012ee0 f   Metaphlan2LogParser.obj
 0001:00011ef9       __unwindfunclet$?initWellKnownErrors@Metaphlan2LogParser@U2@@CA?AVQStringList@@XZ$1 10012ef9 f   Metaphlan2LogParser.obj
 0001:00011f02       __ehhandler$?initWellKnownErrors@Metaphlan2LogParser@U2@@CA?AVQStringList@@XZ 10012f02 f   Metaphlan2LogParser.obj
 0001:00011f20       __unwindfunclet$?isError@Metaphlan2LogParser@U2@@EBE_NABVQString@@@Z$0 10012f20 f   Metaphlan2LogParser.obj
 0001:00011f28       __ehhandler$?isError@Metaphlan2LogParser@U2@@EBE_NABVQString@@@Z 10012f28 f   Metaphlan2LogParser.obj
 0001:00011f50       __unwindfunclet$?node_construct@?$QList@VQString@@@@AAEXPAUNode@1@ABVQString@@@Z$1 10012f50 f   Metaphlan2LogParser.obj
 0001:00011f61       __ehhandler$?node_construct@?$QList@VQString@@@@AAEXPAUNode@1@ABVQString@@@Z 10012f61 f   Metaphlan2LogParser.obj
 0001:00011f80       __unwindfunclet$?node_copy@?$QList@VQString@@@@AAEXPAUNode@1@00@Z$5 10012f80 f   Metaphlan2LogParser.obj
 0001:00011f91       __ehhandler$?node_copy@?$QList@VQString@@@@AAEXPAUNode@1@00@Z 10012f91 f   Metaphlan2LogParser.obj
 0001:00011fb0       __ehhandler$??0?$QList@PAVPort@Workflow@U2@@@@QAE@ABV0@@Z 10012fb0 f   Metaphlan2Prompter.obj
 0001:00011fd0       __unwindfunclet$??__EalgoLog@U2@@YAXXZ$0 10012fd0 f   Metaphlan2Prompter.obj
 0001:00011fd9       __ehhandler$??__EalgoLog@U2@@YAXXZ 10012fd9 f   Metaphlan2Prompter.obj
 0001:00012000       __unwindfunclet$??__EcmdLog@U2@@YAXXZ$0 10013000 f   Metaphlan2Prompter.obj
 0001:00012009       __ehhandler$??__EcmdLog@U2@@YAXXZ 10013009 f   Metaphlan2Prompter.obj
 0001:00012030       __unwindfunclet$??__EcoreLog@U2@@YAXXZ$0 10013030 f   Metaphlan2Prompter.obj
 0001:00012039       __ehhandler$??__EcoreLog@U2@@YAXXZ 10013039 f   Metaphlan2Prompter.obj
 0001:00012060       __unwindfunclet$??__EioLog@U2@@YAXXZ$0 10013060 f   Metaphlan2Prompter.obj
 0001:00012069       __ehhandler$??__EioLog@U2@@YAXXZ 10013069 f   Metaphlan2Prompter.obj
 0001:00012090       __unwindfunclet$??__EperfLog@U2@@YAXXZ$0 10013090 f   Metaphlan2Prompter.obj
 0001:00012099       __ehhandler$??__EperfLog@U2@@YAXXZ 10013099 f   Metaphlan2Prompter.obj
 0001:000120c0       __unwindfunclet$??__EscriptLog@U2@@YAXXZ$0 100130c0 f   Metaphlan2Prompter.obj
 0001:000120c9       __ehhandler$??__EscriptLog@U2@@YAXXZ 100130c9 f   Metaphlan2Prompter.obj
 0001:000120f0       __unwindfunclet$??__EtaskLog@U2@@YAXXZ$0 100130f0 f   Metaphlan2Prompter.obj
 0001:000120f9       __ehhandler$??__EtaskLog@U2@@YAXXZ 100130f9 f   Metaphlan2Prompter.obj
 0001:00012120       __unwindfunclet$??__EuiLog@U2@@YAXXZ$0 10013120 f   Metaphlan2Prompter.obj
 0001:00012129       __ehhandler$??__EuiLog@U2@@YAXXZ 10013129 f   Metaphlan2Prompter.obj
 0001:00012150       __unwindfunclet$??__EuserActLog@U2@@YAXXZ$0 10013150 f   Metaphlan2Prompter.obj
 0001:00012159       __ehhandler$??__EuserActLog@U2@@YAXXZ 10013159 f   Metaphlan2Prompter.obj
 0001:00012180       __unwindfunclet$?composeRichDoc@Metaphlan2Prompter@LocalWorkflow@U2@@EAE?AVQString@@XZ$0 10013180 f   Metaphlan2Prompter.obj
 0001:00012189       __unwindfunclet$?composeRichDoc@Metaphlan2Prompter@LocalWorkflow@U2@@EAE?AVQString@@XZ$1 10013189 f   Metaphlan2Prompter.obj
 0001:00012192       __unwindfunclet$?composeRichDoc@Metaphlan2Prompter@LocalWorkflow@U2@@EAE?AVQString@@XZ$2 10013192 f   Metaphlan2Prompter.obj
 0001:0001219b       __unwindfunclet$?composeRichDoc@Metaphlan2Prompter@LocalWorkflow@U2@@EAE?AVQString@@XZ$3 1001319b f   Metaphlan2Prompter.obj
 0001:000121a4       __unwindfunclet$?composeRichDoc@Metaphlan2Prompter@LocalWorkflow@U2@@EAE?AVQString@@XZ$4 100131a4 f   Metaphlan2Prompter.obj
 0001:000121ad       __unwindfunclet$?composeRichDoc@Metaphlan2Prompter@LocalWorkflow@U2@@EAE?AVQString@@XZ$5 100131ad f   Metaphlan2Prompter.obj
 0001:000121b6       __unwindfunclet$?composeRichDoc@Metaphlan2Prompter@LocalWorkflow@U2@@EAE?AVQString@@XZ$6 100131b6 f   Metaphlan2Prompter.obj
 0001:000121bf       __unwindfunclet$?composeRichDoc@Metaphlan2Prompter@LocalWorkflow@U2@@EAE?AVQString@@XZ$7 100131bf f   Metaphlan2Prompter.obj
 0001:000121d9       __ehhandler$?composeRichDoc@Metaphlan2Prompter@LocalWorkflow@U2@@EAE?AVQString@@XZ 100131d9 f   Metaphlan2Prompter.obj
 0001:00012200       __unwindfunclet$?createDescription@?$PrompterBase@VMetaphlan2Prompter@LocalWorkflow@U2@@@U2@@UAEPAVActorDocument@Workflow@2@PAVActor@42@@Z$0 10013200 f   Metaphlan2Prompter.obj
 0001:0001220b       __unwindfunclet$?createDescription@?$PrompterBase@VMetaphlan2Prompter@LocalWorkflow@U2@@@U2@@UAEPAVActorDocument@Workflow@2@PAVActor@42@@Z$3 1001320b f   Metaphlan2Prompter.obj
 0001:00012213       __unwindfunclet$?createDescription@?$PrompterBase@VMetaphlan2Prompter@LocalWorkflow@U2@@@U2@@UAEPAVActorDocument@Workflow@2@PAVActor@42@@Z$4 10013213 f   Metaphlan2Prompter.obj
 0001:0001221b       __unwindfunclet$?createDescription@?$PrompterBase@VMetaphlan2Prompter@LocalWorkflow@U2@@@U2@@UAEPAVActorDocument@Workflow@2@PAVActor@42@@Z$6 1001321b f   Metaphlan2Prompter.obj
 0001:00012223       __unwindfunclet$?createDescription@?$PrompterBase@VMetaphlan2Prompter@LocalWorkflow@U2@@@U2@@UAEPAVActorDocument@Workflow@2@PAVActor@42@@Z$7 10013223 f   Metaphlan2Prompter.obj
 0001:0001222b       __ehhandler$?createDescription@?$PrompterBase@VMetaphlan2Prompter@LocalWorkflow@U2@@@U2@@UAEPAVActorDocument@Workflow@2@PAVActor@42@@Z 1001322b f   Metaphlan2Prompter.obj
 0001:00012250       __unwindfunclet$??0Metaphlan2Support@U2@@QAE@ABVQString@@0@Z$0 10013250 f   Metaphlan2Support.obj
 0001:00012259       __unwindfunclet$??0Metaphlan2Support@U2@@QAE@ABVQString@@0@Z$2 10013259 f   Metaphlan2Support.obj
 0001:00012262       __unwindfunclet$??0Metaphlan2Support@U2@@QAE@ABVQString@@0@Z$3 10013262 f   Metaphlan2Support.obj
 0001:0001226b       __unwindfunclet$??0Metaphlan2Support@U2@@QAE@ABVQString@@0@Z$4 1001326b f   Metaphlan2Support.obj
 0001:00012274       __unwindfunclet$??0Metaphlan2Support@U2@@QAE@ABVQString@@0@Z$5 10013274 f   Metaphlan2Support.obj
 0001:0001227d       __unwindfunclet$??0Metaphlan2Support@U2@@QAE@ABVQString@@0@Z$6 1001327d f   Metaphlan2Support.obj
 0001:00012286       __ehhandler$??0Metaphlan2Support@U2@@QAE@ABVQString@@0@Z 10013286 f   Metaphlan2Support.obj
 0001:000122b0       __unwindfunclet$??__EalgoLog@U2@@YAXXZ$0 100132b0 f   Metaphlan2Support.obj
 0001:000122b9       __ehhandler$??__EalgoLog@U2@@YAXXZ 100132b9 f   Metaphlan2Support.obj
 0001:000122e0       __unwindfunclet$??__EcmdLog@U2@@YAXXZ$0 100132e0 f   Metaphlan2Support.obj
 0001:000122e9       __ehhandler$??__EcmdLog@U2@@YAXXZ 100132e9 f   Metaphlan2Support.obj
 0001:00012310       __unwindfunclet$??__EcoreLog@U2@@YAXXZ$0 10013310 f   Metaphlan2Support.obj
 0001:00012319       __ehhandler$??__EcoreLog@U2@@YAXXZ 10013319 f   Metaphlan2Support.obj
 0001:00012340       __unwindfunclet$??__EioLog@U2@@YAXXZ$0 10013340 f   Metaphlan2Support.obj
 0001:00012349       __ehhandler$??__EioLog@U2@@YAXXZ 10013349 f   Metaphlan2Support.obj
 0001:00012370       __unwindfunclet$??__EperfLog@U2@@YAXXZ$0 10013370 f   Metaphlan2Support.obj
 0001:00012379       __ehhandler$??__EperfLog@U2@@YAXXZ 10013379 f   Metaphlan2Support.obj
 0001:000123a0       __unwindfunclet$??__EscriptLog@U2@@YAXXZ$0 100133a0 f   Metaphlan2Support.obj
 0001:000123a9       __ehhandler$??__EscriptLog@U2@@YAXXZ 100133a9 f   Metaphlan2Support.obj
 0001:000123d0       __unwindfunclet$??__EtaskLog@U2@@YAXXZ$0 100133d0 f   Metaphlan2Support.obj
 0001:000123d9       __ehhandler$??__EtaskLog@U2@@YAXXZ 100133d9 f   Metaphlan2Support.obj
 0001:00012400       __unwindfunclet$??__EuiLog@U2@@YAXXZ$0 10013400 f   Metaphlan2Support.obj
 0001:00012409       __ehhandler$??__EuiLog@U2@@YAXXZ 10013409 f   Metaphlan2Support.obj
 0001:00012430       __unwindfunclet$??__EuserActLog@U2@@YAXXZ$0 10013430 f   Metaphlan2Support.obj
 0001:00012439       __ehhandler$??__EuserActLog@U2@@YAXXZ 10013439 f   Metaphlan2Support.obj
 0001:00012460       __unwindfunclet$?performAdditionalChecks@Metaphlan2Support@U2@@UAEXABVQString@@@Z$0 10013460 f   Metaphlan2Support.obj
 0001:00012469       __unwindfunclet$?performAdditionalChecks@Metaphlan2Support@U2@@UAEXABVQString@@@Z$1 10013469 f   Metaphlan2Support.obj
 0001:00012472       __unwindfunclet$?performAdditionalChecks@Metaphlan2Support@U2@@UAEXABVQString@@@Z$2 10013472 f   Metaphlan2Support.obj
 0001:0001247b       __unwindfunclet$?performAdditionalChecks@Metaphlan2Support@U2@@UAEXABVQString@@@Z$3 1001347b f   Metaphlan2Support.obj
 0001:00012484       __unwindfunclet$?performAdditionalChecks@Metaphlan2Support@U2@@UAEXABVQString@@@Z$4 10013484 f   Metaphlan2Support.obj
 0001:0001248d       __unwindfunclet$?performAdditionalChecks@Metaphlan2Support@U2@@UAEXABVQString@@@Z$5 1001348d f   Metaphlan2Support.obj
 0001:00012496       __unwindfunclet$?performAdditionalChecks@Metaphlan2Support@U2@@UAEXABVQString@@@Z$6 10013496 f   Metaphlan2Support.obj
 0001:0001249f       __unwindfunclet$?performAdditionalChecks@Metaphlan2Support@U2@@UAEXABVQString@@@Z$7 1001349f f   Metaphlan2Support.obj
 0001:000124a8       __ehhandler$?performAdditionalChecks@Metaphlan2Support@U2@@UAEXABVQString@@@Z 100134a8 f   Metaphlan2Support.obj
 0001:000124d0       __unwindfunclet$??0MetaphlanSupportPlugin@U2@@QAE@XZ$0 100134d0 f   Metaphlan2SupportPlugin.obj
 0001:000124d9       __unwindfunclet$??0MetaphlanSupportPlugin@U2@@QAE@XZ$1 100134d9 f   Metaphlan2SupportPlugin.obj
 0001:000124e4       __unwindfunclet$??0MetaphlanSupportPlugin@U2@@QAE@XZ$2 100134e4 f   Metaphlan2SupportPlugin.obj
 0001:000124fe       __ehhandler$??0MetaphlanSupportPlugin@U2@@QAE@XZ 100134fe f   Metaphlan2SupportPlugin.obj
 0001:00012520       __unwindfunclet$??1MetaphlanSupportPlugin@U2@@UAE@XZ$0 10013520 f   Metaphlan2SupportPlugin.obj
 0001:00012529       __ehhandler$??1MetaphlanSupportPlugin@U2@@UAE@XZ 10013529 f   Metaphlan2SupportPlugin.obj
 0001:00012550       __unwindfunclet$??_GMetaphlanSupportPlugin@U2@@UAEPAXI@Z$0 10013550 f   Metaphlan2SupportPlugin.obj
 0001:00012559       __ehhandler$??_GMetaphlanSupportPlugin@U2@@UAEPAXI@Z 10013559 f   Metaphlan2SupportPlugin.obj
 0001:00012580       __unwindfunclet$??__EalgoLog@U2@@YAXXZ$0 10013580 f   Metaphlan2SupportPlugin.obj
 0001:00012589       __ehhandler$??__EalgoLog@U2@@YAXXZ 10013589 f   Metaphlan2SupportPlugin.obj
 0001:000125b0       __unwindfunclet$??__EcmdLog@U2@@YAXXZ$0 100135b0 f   Metaphlan2SupportPlugin.obj
 0001:000125b9       __ehhandler$??__EcmdLog@U2@@YAXXZ 100135b9 f   Metaphlan2SupportPlugin.obj
 0001:000125e0       __unwindfunclet$??__EcoreLog@U2@@YAXXZ$0 100135e0 f   Metaphlan2SupportPlugin.obj
 0001:000125e9       __ehhandler$??__EcoreLog@U2@@YAXXZ 100135e9 f   Metaphlan2SupportPlugin.obj
 0001:00012610       __unwindfunclet$??__EioLog@U2@@YAXXZ$0 10013610 f   Metaphlan2SupportPlugin.obj
 0001:00012619       __ehhandler$??__EioLog@U2@@YAXXZ 10013619 f   Metaphlan2SupportPlugin.obj
 0001:00012640       __unwindfunclet$??__EperfLog@U2@@YAXXZ$0 10013640 f   Metaphlan2SupportPlugin.obj
 0001:00012649       __ehhandler$??__EperfLog@U2@@YAXXZ 10013649 f   Metaphlan2SupportPlugin.obj
 0001:00012670       __unwindfunclet$??__EscriptLog@U2@@YAXXZ$0 10013670 f   Metaphlan2SupportPlugin.obj
 0001:00012679       __ehhandler$??__EscriptLog@U2@@YAXXZ 10013679 f   Metaphlan2SupportPlugin.obj
 0001:000126a0       __unwindfunclet$??__EtaskLog@U2@@YAXXZ$0 100136a0 f   Metaphlan2SupportPlugin.obj
 0001:000126a9       __ehhandler$??__EtaskLog@U2@@YAXXZ 100136a9 f   Metaphlan2SupportPlugin.obj
 0001:000126d0       __unwindfunclet$??__EuiLog@U2@@YAXXZ$0 100136d0 f   Metaphlan2SupportPlugin.obj
 0001:000126d9       __ehhandler$??__EuiLog@U2@@YAXXZ 100136d9 f   Metaphlan2SupportPlugin.obj
 0001:00012700       __unwindfunclet$??__EuserActLog@U2@@YAXXZ$0 10013700 f   Metaphlan2SupportPlugin.obj
 0001:00012709       __ehhandler$??__EuserActLog@U2@@YAXXZ 10013709 f   Metaphlan2SupportPlugin.obj
 0001:00012730       __unwindfunclet$??0Metaphlan2ClassifyTask@U2@@QAE@ABUMetaphlan2TaskSettings@1@@Z$0 10013730 f   Metaphlan2Task.obj
 0001:00012739       __unwindfunclet$??0Metaphlan2ClassifyTask@U2@@QAE@ABUMetaphlan2TaskSettings@1@@Z$1 10013739 f   Metaphlan2Task.obj
 0001:00012742       __unwindfunclet$??0Metaphlan2ClassifyTask@U2@@QAE@ABUMetaphlan2TaskSettings@1@@Z$2 10013742 f   Metaphlan2Task.obj
 0001:00012750       __unwindfunclet$??0Metaphlan2ClassifyTask@U2@@QAE@ABUMetaphlan2TaskSettings@1@@Z$3 10013750 f   Metaphlan2Task.obj
 0001:0001275e       __unwindfunclet$??0Metaphlan2ClassifyTask@U2@@QAE@ABUMetaphlan2TaskSettings@1@@Z$4 1001375e f   Metaphlan2Task.obj
 0001:00012767       __unwindfunclet$??0Metaphlan2ClassifyTask@U2@@QAE@ABUMetaphlan2TaskSettings@1@@Z$5 10013767 f   Metaphlan2Task.obj
 0001:00012770       __unwindfunclet$??0Metaphlan2ClassifyTask@U2@@QAE@ABUMetaphlan2TaskSettings@1@@Z$6 10013770 f   Metaphlan2Task.obj
 0001:00012779       __unwindfunclet$??0Metaphlan2ClassifyTask@U2@@QAE@ABUMetaphlan2TaskSettings@1@@Z$7 10013779 f   Metaphlan2Task.obj
 0001:00012782       __unwindfunclet$??0Metaphlan2ClassifyTask@U2@@QAE@ABUMetaphlan2TaskSettings@1@@Z$8 10013782 f   Metaphlan2Task.obj
 0001:0001278b       __unwindfunclet$??0Metaphlan2ClassifyTask@U2@@QAE@ABUMetaphlan2TaskSettings@1@@Z$9 1001378b f   Metaphlan2Task.obj
 0001:00012794       __unwindfunclet$??0Metaphlan2ClassifyTask@U2@@QAE@ABUMetaphlan2TaskSettings@1@@Z$10 10013794 f   Metaphlan2Task.obj
 0001:0001279d       __unwindfunclet$??0Metaphlan2ClassifyTask@U2@@QAE@ABUMetaphlan2TaskSettings@1@@Z$11 1001379d f   Metaphlan2Task.obj
 0001:000127a6       __ehhandler$??0Metaphlan2ClassifyTask@U2@@QAE@ABUMetaphlan2TaskSettings@1@@Z 100137a6 f   Metaphlan2Task.obj
 0001:000127d0       __unwindfunclet$??0Metaphlan2TaskSettings@U2@@QAE@ABU01@@Z$0 100137d0 f   Metaphlan2Task.obj
 0001:000127dc       __unwindfunclet$??0Metaphlan2TaskSettings@U2@@QAE@ABU01@@Z$1 100137dc f   Metaphlan2Task.obj
 0001:000127e8       __unwindfunclet$??0Metaphlan2TaskSettings@U2@@QAE@ABU01@@Z$2 100137e8 f   Metaphlan2Task.obj
 0001:000127f4       __unwindfunclet$??0Metaphlan2TaskSettings@U2@@QAE@ABU01@@Z$3 100137f4 f   Metaphlan2Task.obj
 0001:00012800       __unwindfunclet$??0Metaphlan2TaskSettings@U2@@QAE@ABU01@@Z$4 10013800 f   Metaphlan2Task.obj
 0001:0001280c       __unwindfunclet$??0Metaphlan2TaskSettings@U2@@QAE@ABU01@@Z$5 1001380c f   Metaphlan2Task.obj
 0001:00012818       __unwindfunclet$??0Metaphlan2TaskSettings@U2@@QAE@ABU01@@Z$6 10013818 f   Metaphlan2Task.obj
 0001:00012824       __unwindfunclet$??0Metaphlan2TaskSettings@U2@@QAE@ABU01@@Z$7 10013824 f   Metaphlan2Task.obj
 0001:00012830       __unwindfunclet$??0Metaphlan2TaskSettings@U2@@QAE@ABU01@@Z$8 10013830 f   Metaphlan2Task.obj
 0001:0001283c       __ehhandler$??0Metaphlan2TaskSettings@U2@@QAE@ABU01@@Z 1001383c f   Metaphlan2Task.obj
 0001:00012860       __unwindfunclet$??0Metaphlan2TaskSettings@U2@@QAE@XZ$0 10013860 f   Metaphlan2Task.obj
 0001:0001286c       __unwindfunclet$??0Metaphlan2TaskSettings@U2@@QAE@XZ$1 1001386c f   Metaphlan2Task.obj
 0001:00012878       __unwindfunclet$??0Metaphlan2TaskSettings@U2@@QAE@XZ$2 10013878 f   Metaphlan2Task.obj
 0001:00012884       __unwindfunclet$??0Metaphlan2TaskSettings@U2@@QAE@XZ$3 10013884 f   Metaphlan2Task.obj
 0001:00012890       __unwindfunclet$??0Metaphlan2TaskSettings@U2@@QAE@XZ$4 10013890 f   Metaphlan2Task.obj
 0001:0001289c       __unwindfunclet$??0Metaphlan2TaskSettings@U2@@QAE@XZ$5 1001389c f   Metaphlan2Task.obj
 0001:000128a8       __unwindfunclet$??0Metaphlan2TaskSettings@U2@@QAE@XZ$6 100138a8 f   Metaphlan2Task.obj
 0001:000128b4       __unwindfunclet$??0Metaphlan2TaskSettings@U2@@QAE@XZ$7 100138b4 f   Metaphlan2Task.obj
 0001:000128c0       __unwindfunclet$??0Metaphlan2TaskSettings@U2@@QAE@XZ$8 100138c0 f   Metaphlan2Task.obj
 0001:000128cc       __ehhandler$??0Metaphlan2TaskSettings@U2@@QAE@XZ 100138cc f   Metaphlan2Task.obj
 0001:000128f0       __unwindfunclet$??1Metaphlan2ClassifyTask@U2@@UAE@XZ$0 100138f0 f   Metaphlan2Task.obj
 0001:000128f9       __ehhandler$??1Metaphlan2ClassifyTask@U2@@UAE@XZ 100138f9 f   Metaphlan2Task.obj
 0001:00012920       __unwindfunclet$??1Metaphlan2TaskSettings@U2@@QAE@XZ$0 10013920 f   Metaphlan2Task.obj
 0001:0001292c       __unwindfunclet$??1Metaphlan2TaskSettings@U2@@QAE@XZ$1 1001392c f   Metaphlan2Task.obj
 0001:00012938       __unwindfunclet$??1Metaphlan2TaskSettings@U2@@QAE@XZ$2 10013938 f   Metaphlan2Task.obj
 0001:00012944       __unwindfunclet$??1Metaphlan2TaskSettings@U2@@QAE@XZ$3 10013944 f   Metaphlan2Task.obj
 0001:00012950       __unwindfunclet$??1Metaphlan2TaskSettings@U2@@QAE@XZ$4 10013950 f   Metaphlan2Task.obj
 0001:0001295c       __unwindfunclet$??1Metaphlan2TaskSettings@U2@@QAE@XZ$5 1001395c f   Metaphlan2Task.obj
 0001:00012968       __unwindfunclet$??1Metaphlan2TaskSettings@U2@@QAE@XZ$6 10013968 f   Metaphlan2Task.obj
 0001:00012974       __unwindfunclet$??1Metaphlan2TaskSettings@U2@@QAE@XZ$7 10013974 f   Metaphlan2Task.obj
 0001:00012980       __unwindfunclet$??1Metaphlan2TaskSettings@U2@@QAE@XZ$8 10013980 f   Metaphlan2Task.obj
 0001:0001298c       __ehhandler$??1Metaphlan2TaskSettings@U2@@QAE@XZ 1001398c f   Metaphlan2Task.obj
 0001:000129b0       __unwindfunclet$??_GMetaphlan2ClassifyTask@U2@@UAEPAXI@Z$0 100139b0 f   Metaphlan2Task.obj
 0001:000129b9       __ehhandler$??_GMetaphlan2ClassifyTask@U2@@UAEPAXI@Z 100139b9 f   Metaphlan2Task.obj
 0001:000129e0       __unwindfunclet$??__EalgoLog@U2@@YAXXZ$0 100139e0 f   Metaphlan2Task.obj
 0001:000129e9       __ehhandler$??__EalgoLog@U2@@YAXXZ 100139e9 f   Metaphlan2Task.obj
 0001:00012a10       __unwindfunclet$??__EcmdLog@U2@@YAXXZ$0 10013a10 f   Metaphlan2Task.obj
 0001:00012a19       __ehhandler$??__EcmdLog@U2@@YAXXZ 10013a19 f   Metaphlan2Task.obj
 0001:00012a40       __unwindfunclet$??__EcoreLog@U2@@YAXXZ$0 10013a40 f   Metaphlan2Task.obj
 0001:00012a49       __ehhandler$??__EcoreLog@U2@@YAXXZ 10013a49 f   Metaphlan2Task.obj
 0001:00012a70       __unwindfunclet$??__EioLog@U2@@YAXXZ$0 10013a70 f   Metaphlan2Task.obj
 0001:00012a79       __ehhandler$??__EioLog@U2@@YAXXZ 10013a79 f   Metaphlan2Task.obj
 0001:00012aa0       __unwindfunclet$??__EperfLog@U2@@YAXXZ$0 10013aa0 f   Metaphlan2Task.obj
 0001:00012aa9       __ehhandler$??__EperfLog@U2@@YAXXZ 10013aa9 f   Metaphlan2Task.obj
 0001:00012ad0       __unwindfunclet$??__EscriptLog@U2@@YAXXZ$0 10013ad0 f   Metaphlan2Task.obj
 0001:00012ad9       __ehhandler$??__EscriptLog@U2@@YAXXZ 10013ad9 f   Metaphlan2Task.obj
 0001:00012b00       __unwindfunclet$??__EtaskLog@U2@@YAXXZ$0 10013b00 f   Metaphlan2Task.obj
 0001:00012b09       __ehhandler$??__EtaskLog@U2@@YAXXZ 10013b09 f   Metaphlan2Task.obj
 0001:00012b30       __unwindfunclet$??__EuiLog@U2@@YAXXZ$0 10013b30 f   Metaphlan2Task.obj
 0001:00012b39       __ehhandler$??__EuiLog@U2@@YAXXZ 10013b39 f   Metaphlan2Task.obj
 0001:00012b60       __unwindfunclet$??__EuserActLog@U2@@YAXXZ$0 10013b60 f   Metaphlan2Task.obj
 0001:00012b69       __ehhandler$??__EuserActLog@U2@@YAXXZ 10013b69 f   Metaphlan2Task.obj
 0001:00012b90       __ehhandler$?append@?$QList@PAVTask@U2@@@@QAEXABQAVTask@U2@@@Z 10013b90 f   Metaphlan2Task.obj
 0001:00012bb0       __ehhandler$?detach_helper@?$QList@VQString@@@@AAEXH@Z 10013bb0 f   Metaphlan2Task.obj
 0001:00012bd0       __ehhandler$?detach_helper_grow@?$QList@PAVTask@U2@@@@AAEPAUNode@1@HH@Z 10013bd0 f   Metaphlan2Task.obj
 0001:00012bf0       __unwindfunclet$?detectFormat@Metaphlan2ClassifyTask@U2@@AAE?AVQString@@ABVGUrl@2@@Z$0 10013bf0 f   Metaphlan2Task.obj
 0001:00012bf9       __unwindfunclet$?detectFormat@Metaphlan2ClassifyTask@U2@@AAE?AVQString@@ABVGUrl@2@@Z$1 10013bf9 f   Metaphlan2Task.obj
 0001:00012c02       __unwindfunclet$?detectFormat@Metaphlan2ClassifyTask@U2@@AAE?AVQString@@ABVGUrl@2@@Z$2 10013c02 f   Metaphlan2Task.obj
 0001:00012c1c       __unwindfunclet$?detectFormat@Metaphlan2ClassifyTask@U2@@AAE?AVQString@@ABVGUrl@2@@Z$3 10013c1c f   Metaphlan2Task.obj
 0001:00012c25       __ehhandler$?detectFormat@Metaphlan2ClassifyTask@U2@@AAE?AVQString@@ABVGUrl@2@@Z 10013c25 f   Metaphlan2Task.obj
 0001:00012c40       __unwindfunclet$?detectInputFormats@Metaphlan2ClassifyTask@U2@@AAE?AVQString@@XZ$0 10013c40 f   Metaphlan2Task.obj
 0001:00012c49       __unwindfunclet$?detectInputFormats@Metaphlan2ClassifyTask@U2@@AAE?AVQString@@XZ$1 10013c49 f   Metaphlan2Task.obj
 0001:00012c52       __unwindfunclet$?detectInputFormats@Metaphlan2ClassifyTask@U2@@AAE?AVQString@@XZ$2 10013c52 f   Metaphlan2Task.obj
 0001:00012c5b       __unwindfunclet$?detectInputFormats@Metaphlan2ClassifyTask@U2@@AAE?AVQString@@XZ$3 10013c5b f   Metaphlan2Task.obj
 0001:00012c64       __unwindfunclet$?detectInputFormats@Metaphlan2ClassifyTask@U2@@AAE?AVQString@@XZ$4 10013c64 f   Metaphlan2Task.obj
 0001:00012c6d       __unwindfunclet$?detectInputFormats@Metaphlan2ClassifyTask@U2@@AAE?AVQString@@XZ$5 10013c6d f   Metaphlan2Task.obj
 0001:00012c87       __ehhandler$?detectInputFormats@Metaphlan2ClassifyTask@U2@@AAE?AVQString@@XZ 10013c87 f   Metaphlan2Task.obj
 0001:00012cb0       __unwindfunclet$?getArguments@Metaphlan2ClassifyTask@U2@@AAE?AVQStringList@@XZ$0 10013cb0 f   Metaphlan2Task.obj
 0001:00012cb8       __unwindfunclet$?getArguments@Metaphlan2ClassifyTask@U2@@AAE?AVQStringList@@XZ$1 10013cb8 f   Metaphlan2Task.obj
 0001:00012cc1       __unwindfunclet$?getArguments@Metaphlan2ClassifyTask@U2@@AAE?AVQStringList@@XZ$2 10013cc1 f   Metaphlan2Task.obj
 0001:00012cca       __unwindfunclet$?getArguments@Metaphlan2ClassifyTask@U2@@AAE?AVQStringList@@XZ$3 10013cca f   Metaphlan2Task.obj
 0001:00012cd3       __unwindfunclet$?getArguments@Metaphlan2ClassifyTask@U2@@AAE?AVQStringList@@XZ$4 10013cd3 f   Metaphlan2Task.obj
 0001:00012cdc       __unwindfunclet$?getArguments@Metaphlan2ClassifyTask@U2@@AAE?AVQStringList@@XZ$5 10013cdc f   Metaphlan2Task.obj
 0001:00012ce5       __unwindfunclet$?getArguments@Metaphlan2ClassifyTask@U2@@AAE?AVQStringList@@XZ$6 10013ce5 f   Metaphlan2Task.obj
 0001:00012cee       __unwindfunclet$?getArguments@Metaphlan2ClassifyTask@U2@@AAE?AVQStringList@@XZ$7 10013cee f   Metaphlan2Task.obj
 0001:00012cf7       __unwindfunclet$?getArguments@Metaphlan2ClassifyTask@U2@@AAE?AVQStringList@@XZ$8 10013cf7 f   Metaphlan2Task.obj
 0001:00012d00       __unwindfunclet$?getArguments@Metaphlan2ClassifyTask@U2@@AAE?AVQStringList@@XZ$9 10013d00 f   Metaphlan2Task.obj
 0001:00012d09       __unwindfunclet$?getArguments@Metaphlan2ClassifyTask@U2@@AAE?AVQStringList@@XZ$10 10013d09 f   Metaphlan2Task.obj
 0001:00012d12       __unwindfunclet$?getArguments@Metaphlan2ClassifyTask@U2@@AAE?AVQStringList@@XZ$11 10013d12 f   Metaphlan2Task.obj
 0001:00012d1b       __unwindfunclet$?getArguments@Metaphlan2ClassifyTask@U2@@AAE?AVQStringList@@XZ$12 10013d1b f   Metaphlan2Task.obj
 0001:00012d24       __unwindfunclet$?getArguments@Metaphlan2ClassifyTask@U2@@AAE?AVQStringList@@XZ$14 10013d24 f   Metaphlan2Task.obj
 0001:00012d2d       __unwindfunclet$?getArguments@Metaphlan2ClassifyTask@U2@@AAE?AVQStringList@@XZ$15 10013d2d f   Metaphlan2Task.obj
 0001:00012d36       __unwindfunclet$?getArguments@Metaphlan2ClassifyTask@U2@@AAE?AVQStringList@@XZ$16 10013d36 f   Metaphlan2Task.obj
 0001:00012d3f       __unwindfunclet$?getArguments@Metaphlan2ClassifyTask@U2@@AAE?AVQStringList@@XZ$17 10013d3f f   Metaphlan2Task.obj
 0001:00012d48       __unwindfunclet$?getArguments@Metaphlan2ClassifyTask@U2@@AAE?AVQStringList@@XZ$13 10013d48 f   Metaphlan2Task.obj
 0001:00012d51       __unwindfunclet$?getArguments@Metaphlan2ClassifyTask@U2@@AAE?AVQStringList@@XZ$18 10013d51 f   Metaphlan2Task.obj
 0001:00012d5a       __unwindfunclet$?getArguments@Metaphlan2ClassifyTask@U2@@AAE?AVQStringList@@XZ$19 10013d5a f   Metaphlan2Task.obj
 0001:00012d63       __unwindfunclet$?getArguments@Metaphlan2ClassifyTask@U2@@AAE?AVQStringList@@XZ$20 10013d63 f   Metaphlan2Task.obj
 0001:00012d6c       __unwindfunclet$?getArguments@Metaphlan2ClassifyTask@U2@@AAE?AVQStringList@@XZ$21 10013d6c f   Metaphlan2Task.obj
 0001:00012d85       __unwindfunclet$?getArguments@Metaphlan2ClassifyTask@U2@@AAE?AVQStringList@@XZ$22 10013d85 f   Metaphlan2Task.obj
 0001:00012d8e       __unwindfunclet$?getArguments@Metaphlan2ClassifyTask@U2@@AAE?AVQStringList@@XZ$23 10013d8e f   Metaphlan2Task.obj
 0001:00012d97       __unwindfunclet$?getArguments@Metaphlan2ClassifyTask@U2@@AAE?AVQStringList@@XZ$24 10013d97 f   Metaphlan2Task.obj
 0001:00012da0       __unwindfunclet$?getArguments@Metaphlan2ClassifyTask@U2@@AAE?AVQStringList@@XZ$25 10013da0 f   Metaphlan2Task.obj
 0001:00012da9       __unwindfunclet$?getArguments@Metaphlan2ClassifyTask@U2@@AAE?AVQStringList@@XZ$26 10013da9 f   Metaphlan2Task.obj
 0001:00012db2       __unwindfunclet$?getArguments@Metaphlan2ClassifyTask@U2@@AAE?AVQStringList@@XZ$27 10013db2 f   Metaphlan2Task.obj
 0001:00012dbb       __unwindfunclet$?getArguments@Metaphlan2ClassifyTask@U2@@AAE?AVQStringList@@XZ$28 10013dbb f   Metaphlan2Task.obj
 0001:00012dc4       __unwindfunclet$?getArguments@Metaphlan2ClassifyTask@U2@@AAE?AVQStringList@@XZ$29 10013dc4 f   Metaphlan2Task.obj
 0001:00012dcc       __unwindfunclet$?getArguments@Metaphlan2ClassifyTask@U2@@AAE?AVQStringList@@XZ$30 10013dcc f   Metaphlan2Task.obj
 0001:00012dd4       __unwindfunclet$?getArguments@Metaphlan2ClassifyTask@U2@@AAE?AVQStringList@@XZ$31 10013dd4 f   Metaphlan2Task.obj
 0001:00012ddc       __unwindfunclet$?getArguments@Metaphlan2ClassifyTask@U2@@AAE?AVQStringList@@XZ$32 10013ddc f   Metaphlan2Task.obj
 0001:00012de5       __unwindfunclet$?getArguments@Metaphlan2ClassifyTask@U2@@AAE?AVQStringList@@XZ$33 10013de5 f   Metaphlan2Task.obj
 0001:00012dee       __unwindfunclet$?getArguments@Metaphlan2ClassifyTask@U2@@AAE?AVQStringList@@XZ$34 10013dee f   Metaphlan2Task.obj
 0001:00012df7       __unwindfunclet$?getArguments@Metaphlan2ClassifyTask@U2@@AAE?AVQStringList@@XZ$35 10013df7 f   Metaphlan2Task.obj
 0001:00012e00       __unwindfunclet$?getArguments@Metaphlan2ClassifyTask@U2@@AAE?AVQStringList@@XZ$36 10013e00 f   Metaphlan2Task.obj
 0001:00012e09       __unwindfunclet$?getArguments@Metaphlan2ClassifyTask@U2@@AAE?AVQStringList@@XZ$37 10013e09 f   Metaphlan2Task.obj
 0001:00012e12       __unwindfunclet$?getArguments@Metaphlan2ClassifyTask@U2@@AAE?AVQStringList@@XZ$38 10013e12 f   Metaphlan2Task.obj
 0001:00012e1b       __unwindfunclet$?getArguments@Metaphlan2ClassifyTask@U2@@AAE?AVQStringList@@XZ$39 10013e1b f   Metaphlan2Task.obj
 0001:00012e24       __unwindfunclet$?getArguments@Metaphlan2ClassifyTask@U2@@AAE?AVQStringList@@XZ$40 10013e24 f   Metaphlan2Task.obj
 0001:00012e2d       __unwindfunclet$?getArguments@Metaphlan2ClassifyTask@U2@@AAE?AVQStringList@@XZ$41 10013e2d f   Metaphlan2Task.obj
 0001:00012e36       __unwindfunclet$?getArguments@Metaphlan2ClassifyTask@U2@@AAE?AVQStringList@@XZ$42 10013e36 f   Metaphlan2Task.obj
 0001:00012e3f       __ehhandler$?getArguments@Metaphlan2ClassifyTask@U2@@AAE?AVQStringList@@XZ 10013e3f f   Metaphlan2Task.obj
 0001:00012e60       __unwindfunclet$?onSubTaskFinished@Metaphlan2ClassifyTask@U2@@EAE?AV?$QList@PAVTask@U2@@@@PAVTask@2@@Z$0 10013e60 f   Metaphlan2Task.obj
 0001:00012e68       __unwindfunclet$?onSubTaskFinished@Metaphlan2ClassifyTask@U2@@EAE?AV?$QList@PAVTask@U2@@@@PAVTask@2@@Z$1 10013e68 f   Metaphlan2Task.obj
 0001:00012e81       __ehhandler$?onSubTaskFinished@Metaphlan2ClassifyTask@U2@@EAE?AV?$QList@PAVTask@U2@@@@PAVTask@2@@Z 10013e81 f   Metaphlan2Task.obj
 0001:00012ea0       __unwindfunclet$?prepare@Metaphlan2ClassifyTask@U2@@EAEXXZ$0 10013ea0 f   Metaphlan2Task.obj
 0001:00012eab       __ehhandler$?prepare@Metaphlan2ClassifyTask@U2@@EAEXXZ 10013eab f   Metaphlan2Task.obj
 0001:00012ed0       __unwindfunclet$?prepareClassifyTask@Metaphlan2ClassifyTask@U2@@AAEXXZ$0 10013ed0 f   Metaphlan2Task.obj
 0001:00012edb       __unwindfunclet$?prepareClassifyTask@Metaphlan2ClassifyTask@U2@@AAEXXZ$1 10013edb f   Metaphlan2Task.obj
 0001:00012ee6       __unwindfunclet$?prepareClassifyTask@Metaphlan2ClassifyTask@U2@@AAEXXZ$2 10013ee6 f   Metaphlan2Task.obj
 0001:00012f00       __unwindfunclet$?prepareClassifyTask@Metaphlan2ClassifyTask@U2@@AAEXXZ$3 10013f00 f   Metaphlan2Task.obj
 0001:00012f19       __unwindfunclet$?prepareClassifyTask@Metaphlan2ClassifyTask@U2@@AAEXXZ$4 10013f19 f   Metaphlan2Task.obj
 0001:00012f33       __unwindfunclet$?prepareClassifyTask@Metaphlan2ClassifyTask@U2@@AAEXXZ$5 10013f33 f   Metaphlan2Task.obj
 0001:00012f4c       __ehhandler$?prepareClassifyTask@Metaphlan2ClassifyTask@U2@@AAEXXZ 10013f4c f   Metaphlan2Task.obj
 0001:00012f70       __unwindfunclet$??__EalgoLog@U2@@YAXXZ$0 10013f70 f   Metaphlan2Validator.obj
 0001:00012f79       __ehhandler$??__EalgoLog@U2@@YAXXZ 10013f79 f   Metaphlan2Validator.obj
 0001:00012fa0       __unwindfunclet$??__EcmdLog@U2@@YAXXZ$0 10013fa0 f   Metaphlan2Validator.obj
 0001:00012fa9       __ehhandler$??__EcmdLog@U2@@YAXXZ 10013fa9 f   Metaphlan2Validator.obj
 0001:00012fd0       __unwindfunclet$??__EcoreLog@U2@@YAXXZ$0 10013fd0 f   Metaphlan2Validator.obj
 0001:00012fd9       __ehhandler$??__EcoreLog@U2@@YAXXZ 10013fd9 f   Metaphlan2Validator.obj
 0001:00013000       __unwindfunclet$??__EioLog@U2@@YAXXZ$0 10014000 f   Metaphlan2Validator.obj
 0001:00013009       __ehhandler$??__EioLog@U2@@YAXXZ 10014009 f   Metaphlan2Validator.obj
 0001:00013030       __unwindfunclet$??__EperfLog@U2@@YAXXZ$0 10014030 f   Metaphlan2Validator.obj
 0001:00013039       __ehhandler$??__EperfLog@U2@@YAXXZ 10014039 f   Metaphlan2Validator.obj
 0001:00013060       __unwindfunclet$??__EscriptLog@U2@@YAXXZ$0 10014060 f   Metaphlan2Validator.obj
 0001:00013069       __ehhandler$??__EscriptLog@U2@@YAXXZ 10014069 f   Metaphlan2Validator.obj
 0001:00013090       __unwindfunclet$??__EtaskLog@U2@@YAXXZ$0 10014090 f   Metaphlan2Validator.obj
 0001:00013099       __ehhandler$??__EtaskLog@U2@@YAXXZ 10014099 f   Metaphlan2Validator.obj
 0001:000130c0       __unwindfunclet$??__EuiLog@U2@@YAXXZ$0 100140c0 f   Metaphlan2Validator.obj
 0001:000130c9       __ehhandler$??__EuiLog@U2@@YAXXZ 100140c9 f   Metaphlan2Validator.obj
 0001:000130f0       __unwindfunclet$??__EuserActLog@U2@@YAXXZ$0 100140f0 f   Metaphlan2Validator.obj
 0001:000130f9       __ehhandler$??__EuserActLog@U2@@YAXXZ 100140f9 f   Metaphlan2Validator.obj
 0001:00013120       __unwindfunclet$?append@?$QList@VWorkflowNotification@U2@@@@QAEXABVWorkflowNotification@U2@@@Z$6 10014120 f   Metaphlan2Validator.obj
 0001:0001312b       __ehhandler$?append@?$QList@VWorkflowNotification@U2@@@@QAEXABVWorkflowNotification@U2@@@Z 1001412b f   Metaphlan2Validator.obj
 0001:00013150       __ehhandler$?detach_helper_grow@?$QList@VWorkflowNotification@U2@@@@AAEPAUNode@1@HH@Z 10014150 f   Metaphlan2Validator.obj
 0001:00013170       __unwindfunclet$?metaType@?$QVariantValueHelper@VQString@@@QtPrivate@@SA?AVQString@@ABVQVariant@@@Z$0 10014170 f   Metaphlan2Validator.obj
 0001:0001318a       __unwindfunclet$?metaType@?$QVariantValueHelper@VQString@@@QtPrivate@@SA?AVQString@@ABVQVariant@@@Z$1 1001418a f   Metaphlan2Validator.obj
 0001:00013193       __ehhandler$?metaType@?$QVariantValueHelper@VQString@@@QtPrivate@@SA?AVQString@@ABVQVariant@@@Z 10014193 f   Metaphlan2Validator.obj
 0001:000131b0       __unwindfunclet$?node_construct@?$QList@VWorkflowNotification@U2@@@@AAEXPAUNode@1@ABVWorkflowNotification@U2@@@Z$0 100141b0 f   Metaphlan2Validator.obj
 0001:000131bb       __ehhandler$?node_construct@?$QList@VWorkflowNotification@U2@@@@AAEXPAUNode@1@ABVWorkflowNotification@U2@@@Z 100141bb f   Metaphlan2Validator.obj
 0001:000131e0       __unwindfunclet$?node_copy@?$QList@VWorkflowNotification@U2@@@@AAEXPAUNode@1@00@Z$4 100141e0 f   Metaphlan2Validator.obj
 0001:000131eb       __ehhandler$?node_copy@?$QList@VWorkflowNotification@U2@@@@AAEXPAUNode@1@00@Z 100141eb f   Metaphlan2Validator.obj
 0001:00013210       __unwindfunclet$?validateDatabase@Metaphlan2Validator@Workflow@U2@@ABE_NPBVActor@23@AAV?$QList@VWorkflowNotification@U2@@@@@Z$0 10014210 f   Metaphlan2Validator.obj
 0001:00013219       __unwindfunclet$?validateDatabase@Metaphlan2Validator@Workflow@U2@@ABE_NPBVActor@23@AAV?$QList@VWorkflowNotification@U2@@@@@Z$1 10014219 f   Metaphlan2Validator.obj
 0001:00013222       __unwindfunclet$?validateDatabase@Metaphlan2Validator@Workflow@U2@@ABE_NPBVActor@23@AAV?$QList@VWorkflowNotification@U2@@@@@Z$2 10014222 f   Metaphlan2Validator.obj
 0001:0001322b       __unwindfunclet$?validateDatabase@Metaphlan2Validator@Workflow@U2@@ABE_NPBVActor@23@AAV?$QList@VWorkflowNotification@U2@@@@@Z$3 1001422b f   Metaphlan2Validator.obj
 0001:00013233       __unwindfunclet$?validateDatabase@Metaphlan2Validator@Workflow@U2@@ABE_NPBVActor@23@AAV?$QList@VWorkflowNotification@U2@@@@@Z$4 10014233 f   Metaphlan2Validator.obj
 0001:0001323b       __unwindfunclet$?validateDatabase@Metaphlan2Validator@Workflow@U2@@ABE_NPBVActor@23@AAV?$QList@VWorkflowNotification@U2@@@@@Z$5 1001423b f   Metaphlan2Validator.obj
 0001:00013243       __unwindfunclet$?validateDatabase@Metaphlan2Validator@Workflow@U2@@ABE_NPBVActor@23@AAV?$QList@VWorkflowNotification@U2@@@@@Z$6 10014243 f   Metaphlan2Validator.obj
 0001:0001324c       __unwindfunclet$?validateDatabase@Metaphlan2Validator@Workflow@U2@@ABE_NPBVActor@23@AAV?$QList@VWorkflowNotification@U2@@@@@Z$7 1001424c f   Metaphlan2Validator.obj
 0001:00013255       __unwindfunclet$?validateDatabase@Metaphlan2Validator@Workflow@U2@@ABE_NPBVActor@23@AAV?$QList@VWorkflowNotification@U2@@@@@Z$8 10014255 f   Metaphlan2Validator.obj
 0001:0001325e       __unwindfunclet$?validateDatabase@Metaphlan2Validator@Workflow@U2@@ABE_NPBVActor@23@AAV?$QList@VWorkflowNotification@U2@@@@@Z$9 1001425e f   Metaphlan2Validator.obj
 0001:00013267       __unwindfunclet$?validateDatabase@Metaphlan2Validator@Workflow@U2@@ABE_NPBVActor@23@AAV?$QList@VWorkflowNotification@U2@@@@@Z$10 10014267 f   Metaphlan2Validator.obj
 0001:0001326f       __unwindfunclet$?validateDatabase@Metaphlan2Validator@Workflow@U2@@ABE_NPBVActor@23@AAV?$QList@VWorkflowNotification@U2@@@@@Z$11 1001426f f   Metaphlan2Validator.obj
 0001:00013277       __unwindfunclet$?validateDatabase@Metaphlan2Validator@Workflow@U2@@ABE_NPBVActor@23@AAV?$QList@VWorkflowNotification@U2@@@@@Z$12 10014277 f   Metaphlan2Validator.obj
 0001:0001327f       __unwindfunclet$?validateDatabase@Metaphlan2Validator@Workflow@U2@@ABE_NPBVActor@23@AAV?$QList@VWorkflowNotification@U2@@@@@Z$13 1001427f f   Metaphlan2Validator.obj
 0001:00013288       __unwindfunclet$?validateDatabase@Metaphlan2Validator@Workflow@U2@@ABE_NPBVActor@23@AAV?$QList@VWorkflowNotification@U2@@@@@Z$14 10014288 f   Metaphlan2Validator.obj
 0001:00013291       __unwindfunclet$?validateDatabase@Metaphlan2Validator@Workflow@U2@@ABE_NPBVActor@23@AAV?$QList@VWorkflowNotification@U2@@@@@Z$15 10014291 f   Metaphlan2Validator.obj
 0001:0001329a       __ehhandler$?validateDatabase@Metaphlan2Validator@Workflow@U2@@ABE_NPBVActor@23@AAV?$QList@VWorkflowNotification@U2@@@@@Z 1001429a f   Metaphlan2Validator.obj
 0001:000132c0       __unwindfunclet$??$getAttributeValue@H@Attribute@U2@@QBEHPAVWorkflowContext@Workflow@1@@Z$0 100142c0 f   Metaphlan2Worker.obj
 0001:000132c9       __unwindfunclet$??$getAttributeValue@H@Attribute@U2@@QBEHPAVWorkflowContext@Workflow@1@@Z$1 100142c9 f   Metaphlan2Worker.obj
 0001:000132d1       __unwindfunclet$??$getAttributeValue@H@Attribute@U2@@QBEHPAVWorkflowContext@Workflow@1@@Z$2 100142d1 f   Metaphlan2Worker.obj
 0001:000132d9       __unwindfunclet$??$getAttributeValue@H@Attribute@U2@@QBEHPAVWorkflowContext@Workflow@1@@Z$3 100142d9 f   Metaphlan2Worker.obj
 0001:000132e1       __unwindfunclet$??$getAttributeValue@H@Attribute@U2@@QBEHPAVWorkflowContext@Workflow@1@@Z$4 100142e1 f   Metaphlan2Worker.obj
 0001:000132ea       __unwindfunclet$??$getAttributeValue@H@Attribute@U2@@QBEHPAVWorkflowContext@Workflow@1@@Z$5 100142ea f   Metaphlan2Worker.obj
 0001:000132f3       __unwindfunclet$??$getAttributeValue@H@Attribute@U2@@QBEHPAVWorkflowContext@Workflow@1@@Z$6 100142f3 f   Metaphlan2Worker.obj
 0001:000132fc       __unwindfunclet$??$getAttributeValue@H@Attribute@U2@@QBEHPAVWorkflowContext@Workflow@1@@Z$7 100142fc f   Metaphlan2Worker.obj
 0001:00013305       __unwindfunclet$??$getAttributeValue@H@Attribute@U2@@QBEHPAVWorkflowContext@Workflow@1@@Z$8 10014305 f   Metaphlan2Worker.obj
 0001:0001330e       __unwindfunclet$??$getAttributeValue@H@Attribute@U2@@QBEHPAVWorkflowContext@Workflow@1@@Z$9 1001430e f   Metaphlan2Worker.obj
 0001:00013317       __unwindfunclet$??$getAttributeValue@H@Attribute@U2@@QBEHPAVWorkflowContext@Workflow@1@@Z$10 10014317 f   Metaphlan2Worker.obj
 0001:00013320       __unwindfunclet$??$getAttributeValue@H@Attribute@U2@@QBEHPAVWorkflowContext@Workflow@1@@Z$11 10014320 f   Metaphlan2Worker.obj
 0001:00013329       __ehhandler$??$getAttributeValue@H@Attribute@U2@@QBEHPAVWorkflowContext@Workflow@1@@Z 10014329 f   Metaphlan2Worker.obj
 0001:00013350       __unwindfunclet$??$getAttributeValue@VQString@@@Attribute@U2@@QBE?AVQString@@PAVWorkflowContext@Workflow@1@@Z$0 10014350 f   Metaphlan2Worker.obj
 0001:0001336a       __unwindfunclet$??$getAttributeValue@VQString@@@Attribute@U2@@QBE?AVQString@@PAVWorkflowContext@Workflow@1@@Z$1 1001436a f   Metaphlan2Worker.obj
 0001:00013373       __unwindfunclet$??$getAttributeValue@VQString@@@Attribute@U2@@QBE?AVQString@@PAVWorkflowContext@Workflow@1@@Z$2 10014373 f   Metaphlan2Worker.obj
 0001:0001337b       __unwindfunclet$??$getAttributeValue@VQString@@@Attribute@U2@@QBE?AVQString@@PAVWorkflowContext@Workflow@1@@Z$3 1001437b f   Metaphlan2Worker.obj
 0001:00013383       __unwindfunclet$??$getAttributeValue@VQString@@@Attribute@U2@@QBE?AVQString@@PAVWorkflowContext@Workflow@1@@Z$4 10014383 f   Metaphlan2Worker.obj
 0001:0001338b       __unwindfunclet$??$getAttributeValue@VQString@@@Attribute@U2@@QBE?AVQString@@PAVWorkflowContext@Workflow@1@@Z$5 1001438b f   Metaphlan2Worker.obj
 0001:00013394       __unwindfunclet$??$getAttributeValue@VQString@@@Attribute@U2@@QBE?AVQString@@PAVWorkflowContext@Workflow@1@@Z$6 10014394 f   Metaphlan2Worker.obj
 0001:0001339d       __unwindfunclet$??$getAttributeValue@VQString@@@Attribute@U2@@QBE?AVQString@@PAVWorkflowContext@Workflow@1@@Z$7 1001439d f   Metaphlan2Worker.obj
 0001:000133a6       __unwindfunclet$??$getAttributeValue@VQString@@@Attribute@U2@@QBE?AVQString@@PAVWorkflowContext@Workflow@1@@Z$8 100143a6 f   Metaphlan2Worker.obj
 0001:000133af       __unwindfunclet$??$getAttributeValue@VQString@@@Attribute@U2@@QBE?AVQString@@PAVWorkflowContext@Workflow@1@@Z$9 100143af f   Metaphlan2Worker.obj
 0001:000133b8       __unwindfunclet$??$getAttributeValue@VQString@@@Attribute@U2@@QBE?AVQString@@PAVWorkflowContext@Workflow@1@@Z$10 100143b8 f   Metaphlan2Worker.obj
 0001:000133c1       __unwindfunclet$??$getAttributeValue@VQString@@@Attribute@U2@@QBE?AVQString@@PAVWorkflowContext@Workflow@1@@Z$11 100143c1 f   Metaphlan2Worker.obj
 0001:000133ca       __unwindfunclet$??$getAttributeValue@VQString@@@Attribute@U2@@QBE?AVQString@@PAVWorkflowContext@Workflow@1@@Z$12 100143ca f   Metaphlan2Worker.obj
 0001:000133d3       __ehhandler$??$getAttributeValue@VQString@@@Attribute@U2@@QBE?AVQString@@PAVWorkflowContext@Workflow@1@@Z 100143d3 f   Metaphlan2Worker.obj
 0001:00013400       __unwindfunclet$??$getValue@VQString@@@BaseWorker@LocalWorkflow@U2@@IBE?AVQString@@ABV3@@Z$0 10014400 f   Metaphlan2Worker.obj
 0001:0001341a       __unwindfunclet$??$getValue@VQString@@@BaseWorker@LocalWorkflow@U2@@IBE?AVQString@@ABV3@@Z$1 1001441a f   Metaphlan2Worker.obj
 0001:00013423       __ehhandler$??$getValue@VQString@@@BaseWorker@LocalWorkflow@U2@@IBE?AVQString@@ABV3@@Z 10014423 f   Metaphlan2Worker.obj
 0001:00013440       __ehhandler$??0?$QList@VDescriptor@U2@@@@QAE@ABV0@@Z 10014440 f   Metaphlan2Worker.obj
 0001:00013460       __unwindfunclet$??A?$QMap@VQString@@VQScriptValue@@@@QAEAAVQScriptValue@@ABVQString@@@Z$0 10014460 f   Metaphlan2Worker.obj
 0001:00013469       __ehhandler$??A?$QMap@VQString@@VQScriptValue@@@@QAEAAVQScriptValue@@ABVQString@@@Z 10014469 f   Metaphlan2Worker.obj
 0001:00013490       __unwindfunclet$??A?$QMap@VQString@@VQVariant@@@@QAEAAVQVariant@@ABVQString@@@Z$0 10014490 f   Metaphlan2Worker.obj
 0001:00013499       __ehhandler$??A?$QMap@VQString@@VQVariant@@@@QAEAAVQVariant@@ABVQString@@@Z 10014499 f   Metaphlan2Worker.obj
 0001:000134c0       __unwindfunclet$??__EalgoLog@U2@@YAXXZ$0 100144c0 f   Metaphlan2Worker.obj
 0001:000134c9       __ehhandler$??__EalgoLog@U2@@YAXXZ 100144c9 f   Metaphlan2Worker.obj
 0001:000134f0       __unwindfunclet$??__EcmdLog@U2@@YAXXZ$0 100144f0 f   Metaphlan2Worker.obj
 0001:000134f9       __ehhandler$??__EcmdLog@U2@@YAXXZ 100144f9 f   Metaphlan2Worker.obj
 0001:00013520       __unwindfunclet$??__EcoreLog@U2@@YAXXZ$0 10014520 f   Metaphlan2Worker.obj
 0001:00013529       __ehhandler$??__EcoreLog@U2@@YAXXZ 10014529 f   Metaphlan2Worker.obj
 0001:00013550       __unwindfunclet$??__EioLog@U2@@YAXXZ$0 10014550 f   Metaphlan2Worker.obj
 0001:00013559       __ehhandler$??__EioLog@U2@@YAXXZ 10014559 f   Metaphlan2Worker.obj
 0001:00013580       __unwindfunclet$??__EperfLog@U2@@YAXXZ$0 10014580 f   Metaphlan2Worker.obj
 0001:00013589       __ehhandler$??__EperfLog@U2@@YAXXZ 10014589 f   Metaphlan2Worker.obj
 0001:000135b0       __unwindfunclet$??__EscriptLog@U2@@YAXXZ$0 100145b0 f   Metaphlan2Worker.obj
 0001:000135b9       __ehhandler$??__EscriptLog@U2@@YAXXZ 100145b9 f   Metaphlan2Worker.obj
 0001:000135e0       __unwindfunclet$??__EtaskLog@U2@@YAXXZ$0 100145e0 f   Metaphlan2Worker.obj
 0001:000135e9       __ehhandler$??__EtaskLog@U2@@YAXXZ 100145e9 f   Metaphlan2Worker.obj
 0001:00013610       __unwindfunclet$??__EuiLog@U2@@YAXXZ$0 10014610 f   Metaphlan2Worker.obj
 0001:00013619       __ehhandler$??__EuiLog@U2@@YAXXZ 10014619 f   Metaphlan2Worker.obj
 0001:00013640       __unwindfunclet$??__EuserActLog@U2@@YAXXZ$0 10014640 f   Metaphlan2Worker.obj
 0001:00013649       __ehhandler$??__EuserActLog@U2@@YAXXZ 10014649 f   Metaphlan2Worker.obj
 0001:00013670       __unwindfunclet$?addOutputToDashboard@Metaphlan2Worker@LocalWorkflow@U2@@ABEXABVQString@@0@Z$0 10014670 f   Metaphlan2Worker.obj
 0001:00013679       __unwindfunclet$?addOutputToDashboard@Metaphlan2Worker@LocalWorkflow@U2@@ABEXABVQString@@0@Z$1 10014679 f   Metaphlan2Worker.obj
 0001:00013682       __unwindfunclet$?addOutputToDashboard@Metaphlan2Worker@LocalWorkflow@U2@@ABEXABVQString@@0@Z$2 10014682 f   Metaphlan2Worker.obj
 0001:0001368b       __ehhandler$?addOutputToDashboard@Metaphlan2Worker@LocalWorkflow@U2@@ABEXABVQString@@0@Z 1001468b f   Metaphlan2Worker.obj
 0001:000136b0       __unwindfunclet$?append@?$QList@VDescriptor@U2@@@@QAEXABVDescriptor@U2@@@Z$6 100146b0 f   Metaphlan2Worker.obj
 0001:000136bb       __ehhandler$?append@?$QList@VDescriptor@U2@@@@QAEXABVDescriptor@U2@@@Z 100146bb f   Metaphlan2Worker.obj
 0001:000136e0       __unwindfunclet$?createDirectory@Metaphlan2Worker@LocalWorkflow@U2@@ABEXAAVQString@@@Z$0 100146e0 f   Metaphlan2Worker.obj
 0001:000136e9       __unwindfunclet$?createDirectory@Metaphlan2Worker@LocalWorkflow@U2@@ABEXAAVQString@@@Z$1 100146e9 f   Metaphlan2Worker.obj
 0001:000136f1       __unwindfunclet$?createDirectory@Metaphlan2Worker@LocalWorkflow@U2@@ABEXAAVQString@@@Z$2 100146f1 f   Metaphlan2Worker.obj
 0001:000136fa       __unwindfunclet$?createDirectory@Metaphlan2Worker@LocalWorkflow@U2@@ABEXAAVQString@@@Z$3 100146fa f   Metaphlan2Worker.obj
 0001:00013703       __ehhandler$?createDirectory@Metaphlan2Worker@LocalWorkflow@U2@@ABEXAAVQString@@@Z 10014703 f   Metaphlan2Worker.obj
 0001:00013720       __unwindfunclet$?createNode@?$QMapData@VQString@@VQScriptValue@@@@QAEPAU?$QMapNode@VQString@@VQScriptValue@@@@ABVQString@@ABVQScriptValue@@PAU2@_N@Z$4 10014720 f   Metaphlan2Worker.obj
 0001:00013734       __unwindfunclet$?createNode@?$QMapData@VQString@@VQScriptValue@@@@QAEPAU?$QMapNode@VQString@@VQScriptValue@@@@ABVQString@@ABVQScriptValue@@PAU2@_N@Z$5 10014734 f   Metaphlan2Worker.obj
 0001:00013748       __ehhandler$?createNode@?$QMapData@VQString@@VQScriptValue@@@@QAEPAU?$QMapNode@VQString@@VQScriptValue@@@@ABVQString@@ABVQScriptValue@@PAU2@_N@Z 10014748 f   Metaphlan2Worker.obj
 0001:00013770       __unwindfunclet$?createNode@?$QMapData@VQString@@VQVariant@@@@QAEPAU?$QMapNode@VQString@@VQVariant@@@@ABVQString@@ABVQVariant@@PAU2@_N@Z$4 10014770 f   Metaphlan2Worker.obj
 0001:00013784       __unwindfunclet$?createNode@?$QMapData@VQString@@VQVariant@@@@QAEPAU?$QMapNode@VQString@@VQVariant@@@@ABVQString@@ABVQVariant@@PAU2@_N@Z$5 10014784 f   Metaphlan2Worker.obj
 0001:00013798       __ehhandler$?createNode@?$QMapData@VQString@@VQVariant@@@@QAEPAU?$QMapNode@VQString@@VQVariant@@@@ABVQString@@ABVQVariant@@PAU2@_N@Z 10014798 f   Metaphlan2Worker.obj
 0001:000137c0       __unwindfunclet$?createOutputToolDirectory@Metaphlan2Worker@LocalWorkflow@U2@@ABE?AVQString@@ABV4@ABVMessage@Workflow@3@_NW4Output@123@@Z$0 100147c0 f   Metaphlan2Worker.obj
 0001:000137c8       __unwindfunclet$?createOutputToolDirectory@Metaphlan2Worker@LocalWorkflow@U2@@ABE?AVQString@@ABV4@ABVMessage@Workflow@3@_NW4Output@123@@Z$1 100147c8 f   Metaphlan2Worker.obj
 0001:000137d1       __unwindfunclet$?createOutputToolDirectory@Metaphlan2Worker@LocalWorkflow@U2@@ABE?AVQString@@ABV4@ABVMessage@Workflow@3@_NW4Output@123@@Z$2 100147d1 f   Metaphlan2Worker.obj
 0001:000137da       __unwindfunclet$?createOutputToolDirectory@Metaphlan2Worker@LocalWorkflow@U2@@ABE?AVQString@@ABV4@ABVMessage@Workflow@3@_NW4Output@123@@Z$3 100147da f   Metaphlan2Worker.obj
 0001:000137e3       __unwindfunclet$?createOutputToolDirectory@Metaphlan2Worker@LocalWorkflow@U2@@ABE?AVQString@@ABV4@ABVMessage@Workflow@3@_NW4Output@123@@Z$4 100147e3 f   Metaphlan2Worker.obj
 0001:000137ec       __unwindfunclet$?createOutputToolDirectory@Metaphlan2Worker@LocalWorkflow@U2@@ABE?AVQString@@ABV4@ABVMessage@Workflow@3@_NW4Output@123@@Z$5 100147ec f   Metaphlan2Worker.obj
 0001:000137f5       __unwindfunclet$?createOutputToolDirectory@Metaphlan2Worker@LocalWorkflow@U2@@ABE?AVQString@@ABV4@ABVMessage@Workflow@3@_NW4Output@123@@Z$6 100147f5 f   Metaphlan2Worker.obj
 0001:000137fe       __unwindfunclet$?createOutputToolDirectory@Metaphlan2Worker@LocalWorkflow@U2@@ABE?AVQString@@ABV4@ABVMessage@Workflow@3@_NW4Output@123@@Z$7 100147fe f   Metaphlan2Worker.obj
 0001:00013807       __unwindfunclet$?createOutputToolDirectory@Metaphlan2Worker@LocalWorkflow@U2@@ABE?AVQString@@ABV4@ABVMessage@Workflow@3@_NW4Output@123@@Z$8 10014807 f   Metaphlan2Worker.obj
 0001:00013810       __unwindfunclet$?createOutputToolDirectory@Metaphlan2Worker@LocalWorkflow@U2@@ABE?AVQString@@ABV4@ABVMessage@Workflow@3@_NW4Output@123@@Z$9 10014810 f   Metaphlan2Worker.obj
 0001:00013819       __unwindfunclet$?createOutputToolDirectory@Metaphlan2Worker@LocalWorkflow@U2@@ABE?AVQString@@ABV4@ABVMessage@Workflow@3@_NW4Output@123@@Z$10 10014819 f   Metaphlan2Worker.obj
 0001:00013833       __ehhandler$?createOutputToolDirectory@Metaphlan2Worker@LocalWorkflow@U2@@ABE?AVQString@@ABV4@ABVMessage@Workflow@3@_NW4Output@123@@Z 10014833 f   Metaphlan2Worker.obj
 0001:00013850       __ehhandler$?detach_helper@?$QList@VDescriptor@U2@@@@AAEXH@Z 10014850 f   Metaphlan2Worker.obj
 0001:00013870       __ehhandler$?detach_helper_grow@?$QList@VDescriptor@U2@@@@AAEPAUNode@1@HH@Z 10014870 f   Metaphlan2Worker.obj
 0001:00013890       __unwindfunclet$?getDefaultOutputDir@Metaphlan2Worker@LocalWorkflow@U2@@ABE?AVQString@@XZ$0 10014890 f   Metaphlan2Worker.obj
 0001:00013899       __unwindfunclet$?getDefaultOutputDir@Metaphlan2Worker@LocalWorkflow@U2@@ABE?AVQString@@XZ$1 10014899 f   Metaphlan2Worker.obj
 0001:000138a2       __unwindfunclet$?getDefaultOutputDir@Metaphlan2Worker@LocalWorkflow@U2@@ABE?AVQString@@XZ$2 100148a2 f   Metaphlan2Worker.obj
 0001:000138ab       __unwindfunclet$?getDefaultOutputDir@Metaphlan2Worker@LocalWorkflow@U2@@ABE?AVQString@@XZ$3 100148ab f   Metaphlan2Worker.obj
 0001:000138b4       __unwindfunclet$?getDefaultOutputDir@Metaphlan2Worker@LocalWorkflow@U2@@ABE?AVQString@@XZ$4 100148b4 f   Metaphlan2Worker.obj
 0001:000138bd       __unwindfunclet$?getDefaultOutputDir@Metaphlan2Worker@LocalWorkflow@U2@@ABE?AVQString@@XZ$5 100148bd f   Metaphlan2Worker.obj
 0001:000138c5       __unwindfunclet$?getDefaultOutputDir@Metaphlan2Worker@LocalWorkflow@U2@@ABE?AVQString@@XZ$6 100148c5 f   Metaphlan2Worker.obj
 0001:000138df       __ehhandler$?getDefaultOutputDir@Metaphlan2Worker@LocalWorkflow@U2@@ABE?AVQString@@XZ 100148df f   Metaphlan2Worker.obj
 0001:00013900       __unwindfunclet$?getSettings@Metaphlan2Worker@LocalWorkflow@U2@@AAE?AUMetaphlan2TaskSettings@3@AAVU2OpStatus@3@@Z$0 10014900 f   Metaphlan2Worker.obj
 0001:00013908       __unwindfunclet$?getSettings@Metaphlan2Worker@LocalWorkflow@U2@@AAE?AUMetaphlan2TaskSettings@3@AAVU2OpStatus@3@@Z$1 10014908 f   Metaphlan2Worker.obj
 0001:00013911       __unwindfunclet$?getSettings@Metaphlan2Worker@LocalWorkflow@U2@@AAE?AUMetaphlan2TaskSettings@3@AAVU2OpStatus@3@@Z$2 10014911 f   Metaphlan2Worker.obj
 0001:0001391d       __unwindfunclet$?getSettings@Metaphlan2Worker@LocalWorkflow@U2@@AAE?AUMetaphlan2TaskSettings@3@AAVU2OpStatus@3@@Z$3 1001491d f   Metaphlan2Worker.obj
 0001:00013929       __unwindfunclet$?getSettings@Metaphlan2Worker@LocalWorkflow@U2@@AAE?AUMetaphlan2TaskSettings@3@AAVU2OpStatus@3@@Z$4 10014929 f   Metaphlan2Worker.obj
 0001:00013931       __unwindfunclet$?getSettings@Metaphlan2Worker@LocalWorkflow@U2@@AAE?AUMetaphlan2TaskSettings@3@AAVU2OpStatus@3@@Z$5 10014931 f   Metaphlan2Worker.obj
 0001:0001393a       __unwindfunclet$?getSettings@Metaphlan2Worker@LocalWorkflow@U2@@AAE?AUMetaphlan2TaskSettings@3@AAVU2OpStatus@3@@Z$6 1001493a f   Metaphlan2Worker.obj
 0001:00013946       __unwindfunclet$?getSettings@Metaphlan2Worker@LocalWorkflow@U2@@AAE?AUMetaphlan2TaskSettings@3@AAVU2OpStatus@3@@Z$7 10014946 f   Metaphlan2Worker.obj
 0001:0001394e       __unwindfunclet$?getSettings@Metaphlan2Worker@LocalWorkflow@U2@@AAE?AUMetaphlan2TaskSettings@3@AAVU2OpStatus@3@@Z$8 1001494e f   Metaphlan2Worker.obj
 0001:00013957       __unwindfunclet$?getSettings@Metaphlan2Worker@LocalWorkflow@U2@@AAE?AUMetaphlan2TaskSettings@3@AAVU2OpStatus@3@@Z$9 10014957 f   Metaphlan2Worker.obj
 0001:00013960       __unwindfunclet$?getSettings@Metaphlan2Worker@LocalWorkflow@U2@@AAE?AUMetaphlan2TaskSettings@3@AAVU2OpStatus@3@@Z$10 10014960 f   Metaphlan2Worker.obj
 0001:00013969       __unwindfunclet$?getSettings@Metaphlan2Worker@LocalWorkflow@U2@@AAE?AUMetaphlan2TaskSettings@3@AAVU2OpStatus@3@@Z$11 10014969 f   Metaphlan2Worker.obj
 0001:00013972       __unwindfunclet$?getSettings@Metaphlan2Worker@LocalWorkflow@U2@@AAE?AUMetaphlan2TaskSettings@3@AAVU2OpStatus@3@@Z$12 10014972 f   Metaphlan2Worker.obj
 0001:0001397b       __unwindfunclet$?getSettings@Metaphlan2Worker@LocalWorkflow@U2@@AAE?AUMetaphlan2TaskSettings@3@AAVU2OpStatus@3@@Z$13 1001497b f   Metaphlan2Worker.obj
 0001:00013984       __unwindfunclet$?getSettings@Metaphlan2Worker@LocalWorkflow@U2@@AAE?AUMetaphlan2TaskSettings@3@AAVU2OpStatus@3@@Z$14 10014984 f   Metaphlan2Worker.obj
 0001:0001398d       __unwindfunclet$?getSettings@Metaphlan2Worker@LocalWorkflow@U2@@AAE?AUMetaphlan2TaskSettings@3@AAVU2OpStatus@3@@Z$15 1001498d f   Metaphlan2Worker.obj
 0001:00013996       __unwindfunclet$?getSettings@Metaphlan2Worker@LocalWorkflow@U2@@AAE?AUMetaphlan2TaskSettings@3@AAVU2OpStatus@3@@Z$16 10014996 f   Metaphlan2Worker.obj
 0001:0001399f       __unwindfunclet$?getSettings@Metaphlan2Worker@LocalWorkflow@U2@@AAE?AUMetaphlan2TaskSettings@3@AAVU2OpStatus@3@@Z$17 1001499f f   Metaphlan2Worker.obj
 0001:000139a8       __unwindfunclet$?getSettings@Metaphlan2Worker@LocalWorkflow@U2@@AAE?AUMetaphlan2TaskSettings@3@AAVU2OpStatus@3@@Z$18 100149a8 f   Metaphlan2Worker.obj
 0001:000139b1       __unwindfunclet$?getSettings@Metaphlan2Worker@LocalWorkflow@U2@@AAE?AUMetaphlan2TaskSettings@3@AAVU2OpStatus@3@@Z$19 100149b1 f   Metaphlan2Worker.obj
 0001:000139ba       __unwindfunclet$?getSettings@Metaphlan2Worker@LocalWorkflow@U2@@AAE?AUMetaphlan2TaskSettings@3@AAVU2OpStatus@3@@Z$20 100149ba f   Metaphlan2Worker.obj
 0001:000139c3       __unwindfunclet$?getSettings@Metaphlan2Worker@LocalWorkflow@U2@@AAE?AUMetaphlan2TaskSettings@3@AAVU2OpStatus@3@@Z$21 100149c3 f   Metaphlan2Worker.obj
 0001:000139cc       __unwindfunclet$?getSettings@Metaphlan2Worker@LocalWorkflow@U2@@AAE?AUMetaphlan2TaskSettings@3@AAVU2OpStatus@3@@Z$22 100149cc f   Metaphlan2Worker.obj
 0001:000139d5       __unwindfunclet$?getSettings@Metaphlan2Worker@LocalWorkflow@U2@@AAE?AUMetaphlan2TaskSettings@3@AAVU2OpStatus@3@@Z$23 100149d5 f   Metaphlan2Worker.obj
 0001:000139ee       __unwindfunclet$?getSettings@Metaphlan2Worker@LocalWorkflow@U2@@AAE?AUMetaphlan2TaskSettings@3@AAVU2OpStatus@3@@Z$24 100149ee f   Metaphlan2Worker.obj
 0001:000139f7       __unwindfunclet$?getSettings@Metaphlan2Worker@LocalWorkflow@U2@@AAE?AUMetaphlan2TaskSettings@3@AAVU2OpStatus@3@@Z$25 100149f7 f   Metaphlan2Worker.obj
 0001:000139ff       __unwindfunclet$?getSettings@Metaphlan2Worker@LocalWorkflow@U2@@AAE?AUMetaphlan2TaskSettings@3@AAVU2OpStatus@3@@Z$26 100149ff f   Metaphlan2Worker.obj
 0001:00013a08       __unwindfunclet$?getSettings@Metaphlan2Worker@LocalWorkflow@U2@@AAE?AUMetaphlan2TaskSettings@3@AAVU2OpStatus@3@@Z$27 10014a08 f   Metaphlan2Worker.obj
 0001:00013a11       __unwindfunclet$?getSettings@Metaphlan2Worker@LocalWorkflow@U2@@AAE?AUMetaphlan2TaskSettings@3@AAVU2OpStatus@3@@Z$28 10014a11 f   Metaphlan2Worker.obj
 0001:00013a1a       __unwindfunclet$?getSettings@Metaphlan2Worker@LocalWorkflow@U2@@AAE?AUMetaphlan2TaskSettings@3@AAVU2OpStatus@3@@Z$29 10014a1a f   Metaphlan2Worker.obj
 0001:00013a23       __unwindfunclet$?getSettings@Metaphlan2Worker@LocalWorkflow@U2@@AAE?AUMetaphlan2TaskSettings@3@AAVU2OpStatus@3@@Z$30 10014a23 f   Metaphlan2Worker.obj
 0001:00013a2c       __unwindfunclet$?getSettings@Metaphlan2Worker@LocalWorkflow@U2@@AAE?AUMetaphlan2TaskSettings@3@AAVU2OpStatus@3@@Z$31 10014a2c f   Metaphlan2Worker.obj
 0001:00013a35       __unwindfunclet$?getSettings@Metaphlan2Worker@LocalWorkflow@U2@@AAE?AUMetaphlan2TaskSettings@3@AAVU2OpStatus@3@@Z$32 10014a35 f   Metaphlan2Worker.obj
 0001:00013a3e       __unwindfunclet$?getSettings@Metaphlan2Worker@LocalWorkflow@U2@@AAE?AUMetaphlan2TaskSettings@3@AAVU2OpStatus@3@@Z$33 10014a3e f   Metaphlan2Worker.obj
 0001:00013a47       __unwindfunclet$?getSettings@Metaphlan2Worker@LocalWorkflow@U2@@AAE?AUMetaphlan2TaskSettings@3@AAVU2OpStatus@3@@Z$34 10014a47 f   Metaphlan2Worker.obj
 0001:00013a50       __unwindfunclet$?getSettings@Metaphlan2Worker@LocalWorkflow@U2@@AAE?AUMetaphlan2TaskSettings@3@AAVU2OpStatus@3@@Z$35 10014a50 f   Metaphlan2Worker.obj
 0001:00013a59       __unwindfunclet$?getSettings@Metaphlan2Worker@LocalWorkflow@U2@@AAE?AUMetaphlan2TaskSettings@3@AAVU2OpStatus@3@@Z$36 10014a59 f   Metaphlan2Worker.obj
 0001:00013a62       __unwindfunclet$?getSettings@Metaphlan2Worker@LocalWorkflow@U2@@AAE?AUMetaphlan2TaskSettings@3@AAVU2OpStatus@3@@Z$37 10014a62 f   Metaphlan2Worker.obj
 0001:00013a6a       __unwindfunclet$?getSettings@Metaphlan2Worker@LocalWorkflow@U2@@AAE?AUMetaphlan2TaskSettings@3@AAVU2OpStatus@3@@Z$38 10014a6a f   Metaphlan2Worker.obj
 0001:00013a73       __unwindfunclet$?getSettings@Metaphlan2Worker@LocalWorkflow@U2@@AAE?AUMetaphlan2TaskSettings@3@AAVU2OpStatus@3@@Z$39 10014a73 f   Metaphlan2Worker.obj
 0001:00013a7c       __unwindfunclet$?getSettings@Metaphlan2Worker@LocalWorkflow@U2@@AAE?AUMetaphlan2TaskSettings@3@AAVU2OpStatus@3@@Z$40 10014a7c f   Metaphlan2Worker.obj
 0001:00013a85       __unwindfunclet$?getSettings@Metaphlan2Worker@LocalWorkflow@U2@@AAE?AUMetaphlan2TaskSettings@3@AAVU2OpStatus@3@@Z$41 10014a85 f   Metaphlan2Worker.obj
 0001:00013a8e       __unwindfunclet$?getSettings@Metaphlan2Worker@LocalWorkflow@U2@@AAE?AUMetaphlan2TaskSettings@3@AAVU2OpStatus@3@@Z$42 10014a8e f   Metaphlan2Worker.obj
 0001:00013a97       __unwindfunclet$?getSettings@Metaphlan2Worker@LocalWorkflow@U2@@AAE?AUMetaphlan2TaskSettings@3@AAVU2OpStatus@3@@Z$43 10014a97 f   Metaphlan2Worker.obj
 0001:00013aa0       __unwindfunclet$?getSettings@Metaphlan2Worker@LocalWorkflow@U2@@AAE?AUMetaphlan2TaskSettings@3@AAVU2OpStatus@3@@Z$44 10014aa0 f   Metaphlan2Worker.obj
 0001:00013aa9       __unwindfunclet$?getSettings@Metaphlan2Worker@LocalWorkflow@U2@@AAE?AUMetaphlan2TaskSettings@3@AAVU2OpStatus@3@@Z$45 10014aa9 f   Metaphlan2Worker.obj
 0001:00013ab2       __unwindfunclet$?getSettings@Metaphlan2Worker@LocalWorkflow@U2@@AAE?AUMetaphlan2TaskSettings@3@AAVU2OpStatus@3@@Z$46 10014ab2 f   Metaphlan2Worker.obj
 0001:00013abb       __unwindfunclet$?getSettings@Metaphlan2Worker@LocalWorkflow@U2@@AAE?AUMetaphlan2TaskSettings@3@AAVU2OpStatus@3@@Z$47 10014abb f   Metaphlan2Worker.obj
 0001:00013ac4       __unwindfunclet$?getSettings@Metaphlan2Worker@LocalWorkflow@U2@@AAE?AUMetaphlan2TaskSettings@3@AAVU2OpStatus@3@@Z$48 10014ac4 f   Metaphlan2Worker.obj
 0001:00013acd       __unwindfunclet$?getSettings@Metaphlan2Worker@LocalWorkflow@U2@@AAE?AUMetaphlan2TaskSettings@3@AAVU2OpStatus@3@@Z$49 10014acd f   Metaphlan2Worker.obj
 0001:00013ad6       __ehhandler$?getSettings@Metaphlan2Worker@LocalWorkflow@U2@@AAE?AUMetaphlan2TaskSettings@3@AAVU2OpStatus@3@@Z 10014ad6 f   Metaphlan2Worker.obj
 0001:00013b00       __unwindfunclet$?init@Metaphlan2Worker@LocalWorkflow@U2@@UAEXXZ$0 10014b00 f   Metaphlan2Worker.obj
 0001:00013b09       __unwindfunclet$?init@Metaphlan2Worker@LocalWorkflow@U2@@UAEXXZ$1 10014b09 f   Metaphlan2Worker.obj
 0001:00013b12       __unwindfunclet$?init@Metaphlan2Worker@LocalWorkflow@U2@@UAEXXZ$2 10014b12 f   Metaphlan2Worker.obj
 0001:00013b1b       __unwindfunclet$?init@Metaphlan2Worker@LocalWorkflow@U2@@UAEXXZ$3 10014b1b f   Metaphlan2Worker.obj
 0001:00013b24       __unwindfunclet$?init@Metaphlan2Worker@LocalWorkflow@U2@@UAEXXZ$4 10014b24 f   Metaphlan2Worker.obj
 0001:00013b2d       __unwindfunclet$?init@Metaphlan2Worker@LocalWorkflow@U2@@UAEXXZ$5 10014b2d f   Metaphlan2Worker.obj
 0001:00013b36       __unwindfunclet$?init@Metaphlan2Worker@LocalWorkflow@U2@@UAEXXZ$6 10014b36 f   Metaphlan2Worker.obj
 0001:00013b3f       __ehhandler$?init@Metaphlan2Worker@LocalWorkflow@U2@@UAEXXZ 10014b3f f   Metaphlan2Worker.obj
 0001:00013b60       __unwindfunclet$?node_construct@?$QList@VDescriptor@U2@@@@AAEXPAUNode@1@ABVDescriptor@U2@@@Z$0 10014b60 f   Metaphlan2Worker.obj
 0001:00013b6b       __ehhandler$?node_construct@?$QList@VDescriptor@U2@@@@AAEXPAUNode@1@ABVDescriptor@U2@@@Z 10014b6b f   Metaphlan2Worker.obj
 0001:00013b90       __unwindfunclet$?node_copy@?$QList@VDescriptor@U2@@@@AAEXPAUNode@1@00@Z$4 10014b90 f   Metaphlan2Worker.obj
 0001:00013b9b       __ehhandler$?node_copy@?$QList@VDescriptor@U2@@@@AAEXPAUNode@1@00@Z 10014b9b f   Metaphlan2Worker.obj
 0001:00013bc0       __unwindfunclet$?sl_taskFinished@Metaphlan2Worker@LocalWorkflow@U2@@AAEXPAVTask@3@@Z$0 10014bc0 f   Metaphlan2Worker.obj
 0001:00013bc9       __unwindfunclet$?sl_taskFinished@Metaphlan2Worker@LocalWorkflow@U2@@AAEXPAVTask@3@@Z$1 10014bc9 f   Metaphlan2Worker.obj
 0001:00013bd2       __ehhandler$?sl_taskFinished@Metaphlan2Worker@LocalWorkflow@U2@@AAEXPAVTask@3@@Z 10014bd2 f   Metaphlan2Worker.obj
 0001:00013bf0       __unwindfunclet$?tick@Metaphlan2Worker@LocalWorkflow@U2@@UAEPAVTask@3@XZ$0 10014bf0 f   Metaphlan2Worker.obj
 0001:00013bf9       __unwindfunclet$?tick@Metaphlan2Worker@LocalWorkflow@U2@@UAEPAVTask@3@XZ$1 10014bf9 f   Metaphlan2Worker.obj
 0001:00013c01       __unwindfunclet$?tick@Metaphlan2Worker@LocalWorkflow@U2@@UAEPAVTask@3@XZ$2 10014c01 f   Metaphlan2Worker.obj
 0001:00013c0c       __unwindfunclet$?tick@Metaphlan2Worker@LocalWorkflow@U2@@UAEPAVTask@3@XZ$3 10014c0c f   Metaphlan2Worker.obj
 0001:00013c26       __unwindfunclet$?tick@Metaphlan2Worker@LocalWorkflow@U2@@UAEPAVTask@3@XZ$4 10014c26 f   Metaphlan2Worker.obj
 0001:00013c31       __unwindfunclet$?tick@Metaphlan2Worker@LocalWorkflow@U2@@UAEPAVTask@3@XZ$5 10014c31 f   Metaphlan2Worker.obj
 0001:00013c39       __unwindfunclet$?tick@Metaphlan2Worker@LocalWorkflow@U2@@UAEPAVTask@3@XZ$6 10014c39 f   Metaphlan2Worker.obj
 0001:00013c44       __ehhandler$?tick@Metaphlan2Worker@LocalWorkflow@U2@@UAEPAVTask@3@XZ 10014c44 f   Metaphlan2Worker.obj
 0001:00013c60       __unwindfunclet$?uniqueKeys@?$QMap@VDescriptor@U2@@VQVariant@@@@QBE?AV?$QList@VDescriptor@U2@@@@XZ$1 10014c60 f   Metaphlan2Worker.obj
 0001:00013c79       __ehhandler$?uniqueKeys@?$QMap@VDescriptor@U2@@VQVariant@@@@QBE?AV?$QList@VDescriptor@U2@@@@XZ 10014c79 f   Metaphlan2Worker.obj
 0001:00013ca0       __unwindfunclet$??0?$QPair@VQString@@V1@@@QAE@ABU0@@Z$0 10014ca0 f   Metaphlan2WorkerFactory.obj
 0001:00013ca9       __ehhandler$??0?$QPair@VQString@@V1@@@QAE@ABU0@@Z 10014ca9 f   Metaphlan2WorkerFactory.obj
 0001:00013cd0       __unwindfunclet$??0?$QPair@VQString@@V1@@@QAE@ABVQString@@0@Z$0 10014cd0 f   Metaphlan2WorkerFactory.obj
 0001:00013cd9       __ehhandler$??0?$QPair@VQString@@V1@@@QAE@ABVQString@@0@Z 10014cd9 f   Metaphlan2WorkerFactory.obj
 0001:00013d00       __unwindfunclet$??1?$QPair@VQString@@V1@@@QAE@XZ$0 10014d00 f   Metaphlan2WorkerFactory.obj
 0001:00013d09       __ehhandler$??1?$QPair@VQString@@V1@@@QAE@XZ 10014d09 f   Metaphlan2WorkerFactory.obj
 0001:00013d30       __unwindfunclet$??A?$QMap@VDescriptor@U2@@V?$QExplicitlySharedDataPointer@VDataType@U2@@@@@@QAEAAV?$QExplicitlySharedDataPointer@VDataType@U2@@@@ABVDescriptor@U2@@@Z$0 10014d30 f   Metaphlan2WorkerFactory.obj
 0001:00013d38       __ehhandler$??A?$QMap@VDescriptor@U2@@V?$QExplicitlySharedDataPointer@VDataType@U2@@@@@@QAEAAV?$QExplicitlySharedDataPointer@VDataType@U2@@@@ABVDescriptor@U2@@@Z 10014d38 f   Metaphlan2WorkerFactory.obj
 0001:00013d60       __unwindfunclet$??H@YA?BVQString@@ABV0@PBD@Z$0 10014d60 f   Metaphlan2WorkerFactory.obj
 0001:00013d7a       __unwindfunclet$??H@YA?BVQString@@ABV0@PBD@Z$1 10014d7a f   Metaphlan2WorkerFactory.obj
 0001:00013d83       __ehhandler$??H@YA?BVQString@@ABV0@PBD@Z 10014d83 f   Metaphlan2WorkerFactory.obj
 0001:00013da0       __unwindfunclet$??_G?$QPair@VQString@@V1@@@QAEPAXI@Z$0 10014da0 f   Metaphlan2WorkerFactory.obj
 0001:00013da9       __ehhandler$??_G?$QPair@VQString@@V1@@@QAEPAXI@Z 10014da9 f   Metaphlan2WorkerFactory.obj
 0001:00013dd0       __unwindfunclet$??__EalgoLog@U2@@YAXXZ$0 10014dd0 f   Metaphlan2WorkerFactory.obj
 0001:00013dd9       __ehhandler$??__EalgoLog@U2@@YAXXZ 10014dd9 f   Metaphlan2WorkerFactory.obj
 0001:00013e00       __unwindfunclet$??__EcmdLog@U2@@YAXXZ$0 10014e00 f   Metaphlan2WorkerFactory.obj
 0001:00013e09       __ehhandler$??__EcmdLog@U2@@YAXXZ 10014e09 f   Metaphlan2WorkerFactory.obj
 0001:00013e30       __unwindfunclet$??__EcoreLog@U2@@YAXXZ$0 10014e30 f   Metaphlan2WorkerFactory.obj
 0001:00013e39       __ehhandler$??__EcoreLog@U2@@YAXXZ 10014e39 f   Metaphlan2WorkerFactory.obj
 0001:00013e60       __unwindfunclet$??__EioLog@U2@@YAXXZ$0 10014e60 f   Metaphlan2WorkerFactory.obj
 0001:00013e69       __ehhandler$??__EioLog@U2@@YAXXZ 10014e69 f   Metaphlan2WorkerFactory.obj
 0001:00013e90       __unwindfunclet$??__EperfLog@U2@@YAXXZ$0 10014e90 f   Metaphlan2WorkerFactory.obj
 0001:00013e99       __ehhandler$??__EperfLog@U2@@YAXXZ 10014e99 f   Metaphlan2WorkerFactory.obj
 0001:00013ec0       __unwindfunclet$??__EscriptLog@U2@@YAXXZ$0 10014ec0 f   Metaphlan2WorkerFactory.obj
 0001:00013ec9       __ehhandler$??__EscriptLog@U2@@YAXXZ 10014ec9 f   Metaphlan2WorkerFactory.obj
 0001:00013ef0       __unwindfunclet$??__EtaskLog@U2@@YAXXZ$0 10014ef0 f   Metaphlan2WorkerFactory.obj
 0001:00013ef9       __ehhandler$??__EtaskLog@U2@@YAXXZ 10014ef9 f   Metaphlan2WorkerFactory.obj
 0001:00013f20       __unwindfunclet$??__EuiLog@U2@@YAXXZ$0 10014f20 f   Metaphlan2WorkerFactory.obj
 0001:00013f29       __ehhandler$??__EuiLog@U2@@YAXXZ 10014f29 f   Metaphlan2WorkerFactory.obj
 0001:00013f50       __unwindfunclet$??__EuserActLog@U2@@YAXXZ$0 10014f50 f   Metaphlan2WorkerFactory.obj
 0001:00013f59       __ehhandler$??__EuserActLog@U2@@YAXXZ 10014f59 f   Metaphlan2WorkerFactory.obj
 0001:00013f80       __ehhandler$?append@?$QList@PAVAttribute@U2@@@@QAEXABQAVAttribute@U2@@@Z 10014f80 f   Metaphlan2WorkerFactory.obj
 0001:00013fa0       __ehhandler$?append@?$QList@PAVPortDescriptor@Workflow@U2@@@@QAEXABQAVPortDescriptor@Workflow@U2@@@Z 10014fa0 f   Metaphlan2WorkerFactory.obj
 0001:00013fc0       __ehhandler$?append@?$QList@U?$QPair@VQString@@V1@@@@@QAEXABU?$QPair@VQString@@V1@@@@Z 10014fc0 f   Metaphlan2WorkerFactory.obj
 0001:00013ff0       __unwindfunclet$?append@?$QList@VQVariant@@@@QAEXABVQVariant@@@Z$6 10014ff0 f   Metaphlan2WorkerFactory.obj
 0001:00013ffb       __ehhandler$?append@?$QList@VQVariant@@@@QAEXABVQVariant@@@Z 10014ffb f   Metaphlan2WorkerFactory.obj
 0001:00014020       __unwindfunclet$?createNode@?$QMapData@VDescriptor@U2@@V?$QExplicitlySharedDataPointer@VDataType@U2@@@@@@QAEPAU?$QMapNode@VDescriptor@U2@@V?$QExplicitlySharedDataPointer@VDataType@U2@@@@@@ABVDescriptor@U2@@ABV?$QExplicitlySharedDataPointer@VDataType@U2@@@@PAU2@_N@Z$4 10015020 f   Metaphlan2WorkerFactory.obj
 0001:00014034       __ehhandler$?createNode@?$QMapData@VDescriptor@U2@@V?$QExplicitlySharedDataPointer@VDataType@U2@@@@@@QAEPAU?$QMapNode@VDescriptor@U2@@V?$QExplicitlySharedDataPointer@VDataType@U2@@@@@@ABVDescriptor@U2@@ABV?$QExplicitlySharedDataPointer@VDataType@U2@@@@PAU2@_N@Z 10015034 f   Metaphlan2WorkerFactory.obj
 0001:00014050       __unwindfunclet$?createNode@?$QMapData@VQString@@PAVPropertyDelegate@U2@@@@QAEPAU?$QMapNode@VQString@@PAVPropertyDelegate@U2@@@@ABVQString@@ABQAVPropertyDelegate@U2@@PAU2@_N@Z$4 10015050 f   Metaphlan2WorkerFactory.obj
 0001:00014064       __ehhandler$?createNode@?$QMapData@VQString@@PAVPropertyDelegate@U2@@@@QAEPAU?$QMapNode@VQString@@PAVPropertyDelegate@U2@@@@ABVQString@@ABQAVPropertyDelegate@U2@@PAU2@_N@Z 10015064 f   Metaphlan2WorkerFactory.obj
 0001:00014080       __unwindfunclet$?createWorker@Metaphlan2WorkerFactory@LocalWorkflow@U2@@UAEPAVWorker@Workflow@3@PAVActor@53@@Z$0 10015080 f   Metaphlan2WorkerFactory.obj
 0001:0001408b       __ehhandler$?createWorker@Metaphlan2WorkerFactory@LocalWorkflow@U2@@UAEPAVWorker@Workflow@3@PAVActor@53@@Z 1001508b f   Metaphlan2WorkerFactory.obj
 0001:000140b0       __ehhandler$?detach_helper_grow@?$QList@PAVAttribute@U2@@@@AAEPAUNode@1@HH@Z 100150b0 f   Metaphlan2WorkerFactory.obj
 0001:000140d0       __ehhandler$?detach_helper_grow@?$QList@PAVPortDescriptor@Workflow@U2@@@@AAEPAUNode@1@HH@Z 100150d0 f   Metaphlan2WorkerFactory.obj
 0001:000140f0       __ehhandler$?detach_helper_grow@?$QList@U?$QPair@VQString@@V1@@@@@AAEPAUNode@1@HH@Z 100150f0 f   Metaphlan2WorkerFactory.obj
 0001:00014110       __ehhandler$?detach_helper_grow@?$QList@VQVariant@@@@AAEPAUNode@1@HH@Z 10015110 f   Metaphlan2WorkerFactory.obj
 0001:00014130       __unwindfunclet$?init@Metaphlan2WorkerFactory@LocalWorkflow@U2@@SAXXZ$0 10015130 f   Metaphlan2WorkerFactory.obj
 0001:00014138       __unwindfunclet$?init@Metaphlan2WorkerFactory@LocalWorkflow@U2@@SAXXZ$1 10015138 f   Metaphlan2WorkerFactory.obj
 0001:00014141       __unwindfunclet$?init@Metaphlan2WorkerFactory@LocalWorkflow@U2@@SAXXZ$2 10015141 f   Metaphlan2WorkerFactory.obj
 0001:0001414a       __unwindfunclet$?init@Metaphlan2WorkerFactory@LocalWorkflow@U2@@SAXXZ$3 1001514a f   Metaphlan2WorkerFactory.obj
 0001:00014153       __unwindfunclet$?init@Metaphlan2WorkerFactory@LocalWorkflow@U2@@SAXXZ$4 10015153 f   Metaphlan2WorkerFactory.obj
 0001:0001415c       __unwindfunclet$?init@Metaphlan2WorkerFactory@LocalWorkflow@U2@@SAXXZ$5 1001515c f   Metaphlan2WorkerFactory.obj
 0001:00014165       __unwindfunclet$?init@Metaphlan2WorkerFactory@LocalWorkflow@U2@@SAXXZ$6 10015165 f   Metaphlan2WorkerFactory.obj
 0001:00014171       __unwindfunclet$?init@Metaphlan2WorkerFactory@LocalWorkflow@U2@@SAXXZ$7 10015171 f   Metaphlan2WorkerFactory.obj
 0001:0001417a       __unwindfunclet$?init@Metaphlan2WorkerFactory@LocalWorkflow@U2@@SAXXZ$8 1001517a f   Metaphlan2WorkerFactory.obj
 0001:00014183       __unwindfunclet$?init@Metaphlan2WorkerFactory@LocalWorkflow@U2@@SAXXZ$9 10015183 f   Metaphlan2WorkerFactory.obj
 0001:0001418f       __unwindfunclet$?init@Metaphlan2WorkerFactory@LocalWorkflow@U2@@SAXXZ$10 1001518f f   Metaphlan2WorkerFactory.obj
 0001:00014197       __unwindfunclet$?init@Metaphlan2WorkerFactory@LocalWorkflow@U2@@SAXXZ$11 10015197 f   Metaphlan2WorkerFactory.obj
 0001:0001419f       __unwindfunclet$?init@Metaphlan2WorkerFactory@LocalWorkflow@U2@@SAXXZ$12 1001519f f   Metaphlan2WorkerFactory.obj
 0001:000141a7       __unwindfunclet$?init@Metaphlan2WorkerFactory@LocalWorkflow@U2@@SAXXZ$13 100151a7 f   Metaphlan2WorkerFactory.obj
 0001:000141b2       __unwindfunclet$?init@Metaphlan2WorkerFactory@LocalWorkflow@U2@@SAXXZ$14 100151b2 f   Metaphlan2WorkerFactory.obj
 0001:000141bd       __unwindfunclet$?init@Metaphlan2WorkerFactory@LocalWorkflow@U2@@SAXXZ$15 100151bd f   Metaphlan2WorkerFactory.obj
 0001:000141d7       __unwindfunclet$?init@Metaphlan2WorkerFactory@LocalWorkflow@U2@@SAXXZ$16 100151d7 f   Metaphlan2WorkerFactory.obj
 0001:000141f4       __unwindfunclet$?init@Metaphlan2WorkerFactory@LocalWorkflow@U2@@SAXXZ$18 100151f4 f   Metaphlan2WorkerFactory.obj
 0001:000141fc       __unwindfunclet$?init@Metaphlan2WorkerFactory@LocalWorkflow@U2@@SAXXZ$19 100151fc f   Metaphlan2WorkerFactory.obj
 0001:00014205       __unwindfunclet$?init@Metaphlan2WorkerFactory@LocalWorkflow@U2@@SAXXZ$20 10015205 f   Metaphlan2WorkerFactory.obj
 0001:0001420e       __unwindfunclet$?init@Metaphlan2WorkerFactory@LocalWorkflow@U2@@SAXXZ$21 1001520e f   Metaphlan2WorkerFactory.obj
 0001:00014217       __unwindfunclet$?init@Metaphlan2WorkerFactory@LocalWorkflow@U2@@SAXXZ$22 10015217 f   Metaphlan2WorkerFactory.obj
 0001:00014223       __unwindfunclet$?init@Metaphlan2WorkerFactory@LocalWorkflow@U2@@SAXXZ$23 10015223 f   Metaphlan2WorkerFactory.obj
 0001:0001422c       __unwindfunclet$?init@Metaphlan2WorkerFactory@LocalWorkflow@U2@@SAXXZ$24 1001522c f   Metaphlan2WorkerFactory.obj
 0001:00014235       __unwindfunclet$?init@Metaphlan2WorkerFactory@LocalWorkflow@U2@@SAXXZ$25 10015235 f   Metaphlan2WorkerFactory.obj
 0001:00014241       __unwindfunclet$?init@Metaphlan2WorkerFactory@LocalWorkflow@U2@@SAXXZ$26 10015241 f   Metaphlan2WorkerFactory.obj
 0001:0001424d       __unwindfunclet$?init@Metaphlan2WorkerFactory@LocalWorkflow@U2@@SAXXZ$27 1001524d f   Metaphlan2WorkerFactory.obj
 0001:00014259       __unwindfunclet$?init@Metaphlan2WorkerFactory@LocalWorkflow@U2@@SAXXZ$28 10015259 f   Metaphlan2WorkerFactory.obj
 0001:00014265       __unwindfunclet$?init@Metaphlan2WorkerFactory@LocalWorkflow@U2@@SAXXZ$29 10015265 f   Metaphlan2WorkerFactory.obj
 0001:00014271       __unwindfunclet$?init@Metaphlan2WorkerFactory@LocalWorkflow@U2@@SAXXZ$30 10015271 f   Metaphlan2WorkerFactory.obj
 0001:0001427d       __unwindfunclet$?init@Metaphlan2WorkerFactory@LocalWorkflow@U2@@SAXXZ$31 1001527d f   Metaphlan2WorkerFactory.obj
 0001:00014289       __unwindfunclet$?init@Metaphlan2WorkerFactory@LocalWorkflow@U2@@SAXXZ$32 10015289 f   Metaphlan2WorkerFactory.obj
 0001:00014295       __unwindfunclet$?init@Metaphlan2WorkerFactory@LocalWorkflow@U2@@SAXXZ$33 10015295 f   Metaphlan2WorkerFactory.obj
 0001:000142a1       __unwindfunclet$?init@Metaphlan2WorkerFactory@LocalWorkflow@U2@@SAXXZ$34 100152a1 f   Metaphlan2WorkerFactory.obj
 0001:000142ad       __unwindfunclet$?init@Metaphlan2WorkerFactory@LocalWorkflow@U2@@SAXXZ$35 100152ad f   Metaphlan2WorkerFactory.obj
 0001:000142b9       __unwindfunclet$?init@Metaphlan2WorkerFactory@LocalWorkflow@U2@@SAXXZ$36 100152b9 f   Metaphlan2WorkerFactory.obj
 0001:000142c5       __unwindfunclet$?init@Metaphlan2WorkerFactory@LocalWorkflow@U2@@SAXXZ$37 100152c5 f   Metaphlan2WorkerFactory.obj
 0001:000142d1       __unwindfunclet$?init@Metaphlan2WorkerFactory@LocalWorkflow@U2@@SAXXZ$38 100152d1 f   Metaphlan2WorkerFactory.obj
 0001:000142dd       __unwindfunclet$?init@Metaphlan2WorkerFactory@LocalWorkflow@U2@@SAXXZ$39 100152dd f   Metaphlan2WorkerFactory.obj
 0001:000142e9       __unwindfunclet$?init@Metaphlan2WorkerFactory@LocalWorkflow@U2@@SAXXZ$40 100152e9 f   Metaphlan2WorkerFactory.obj
 0001:000142f5       __unwindfunclet$?init@Metaphlan2WorkerFactory@LocalWorkflow@U2@@SAXXZ$41 100152f5 f   Metaphlan2WorkerFactory.obj
 0001:00014301       __unwindfunclet$?init@Metaphlan2WorkerFactory@LocalWorkflow@U2@@SAXXZ$42 10015301 f   Metaphlan2WorkerFactory.obj
 0001:0001430d       __unwindfunclet$?init@Metaphlan2WorkerFactory@LocalWorkflow@U2@@SAXXZ$43 1001530d f   Metaphlan2WorkerFactory.obj
 0001:00014319       __unwindfunclet$?init@Metaphlan2WorkerFactory@LocalWorkflow@U2@@SAXXZ$44 10015319 f   Metaphlan2WorkerFactory.obj
 0001:00014325       __unwindfunclet$?init@Metaphlan2WorkerFactory@LocalWorkflow@U2@@SAXXZ$45 10015325 f   Metaphlan2WorkerFactory.obj
 0001:00014331       __unwindfunclet$?init@Metaphlan2WorkerFactory@LocalWorkflow@U2@@SAXXZ$46 10015331 f   Metaphlan2WorkerFactory.obj
 0001:0001433c       __unwindfunclet$?init@Metaphlan2WorkerFactory@LocalWorkflow@U2@@SAXXZ$47 1001533c f   Metaphlan2WorkerFactory.obj
 0001:00014356       __unwindfunclet$?init@Metaphlan2WorkerFactory@LocalWorkflow@U2@@SAXXZ$49 10015356 f   Metaphlan2WorkerFactory.obj
 0001:00014361       __unwindfunclet$?init@Metaphlan2WorkerFactory@LocalWorkflow@U2@@SAXXZ$50 10015361 f   Metaphlan2WorkerFactory.obj
 0001:0001437b       __unwindfunclet$?init@Metaphlan2WorkerFactory@LocalWorkflow@U2@@SAXXZ$51 1001537b f   Metaphlan2WorkerFactory.obj
 0001:00014394       __unwindfunclet$?init@Metaphlan2WorkerFactory@LocalWorkflow@U2@@SAXXZ$52 10015394 f   Metaphlan2WorkerFactory.obj
 0001:0001439d       __unwindfunclet$?init@Metaphlan2WorkerFactory@LocalWorkflow@U2@@SAXXZ$53 1001539d f   Metaphlan2WorkerFactory.obj
 0001:000143a6       __unwindfunclet$?init@Metaphlan2WorkerFactory@LocalWorkflow@U2@@SAXXZ$54 100153a6 f   Metaphlan2WorkerFactory.obj
 0001:000143b1       __unwindfunclet$?init@Metaphlan2WorkerFactory@LocalWorkflow@U2@@SAXXZ$55 100153b1 f   Metaphlan2WorkerFactory.obj
 0001:000143cb       __unwindfunclet$?init@Metaphlan2WorkerFactory@LocalWorkflow@U2@@SAXXZ$57 100153cb f   Metaphlan2WorkerFactory.obj
 0001:000143d6       __unwindfunclet$?init@Metaphlan2WorkerFactory@LocalWorkflow@U2@@SAXXZ$58 100153d6 f   Metaphlan2WorkerFactory.obj
 0001:000143f0       __unwindfunclet$?init@Metaphlan2WorkerFactory@LocalWorkflow@U2@@SAXXZ$60 100153f0 f   Metaphlan2WorkerFactory.obj
 0001:000143fb       __unwindfunclet$?init@Metaphlan2WorkerFactory@LocalWorkflow@U2@@SAXXZ$61 100153fb f   Metaphlan2WorkerFactory.obj
 0001:0001441a       __unwindfunclet$?init@Metaphlan2WorkerFactory@LocalWorkflow@U2@@SAXXZ$63 1001541a f   Metaphlan2WorkerFactory.obj
 0001:00014425       __unwindfunclet$?init@Metaphlan2WorkerFactory@LocalWorkflow@U2@@SAXXZ$64 10015425 f   Metaphlan2WorkerFactory.obj
 0001:00014444       __unwindfunclet$?init@Metaphlan2WorkerFactory@LocalWorkflow@U2@@SAXXZ$66 10015444 f   Metaphlan2WorkerFactory.obj
 0001:0001444f       __unwindfunclet$?init@Metaphlan2WorkerFactory@LocalWorkflow@U2@@SAXXZ$67 1001544f f   Metaphlan2WorkerFactory.obj
 0001:0001446e       __unwindfunclet$?init@Metaphlan2WorkerFactory@LocalWorkflow@U2@@SAXXZ$69 1001546e f   Metaphlan2WorkerFactory.obj
 0001:00014479       __unwindfunclet$?init@Metaphlan2WorkerFactory@LocalWorkflow@U2@@SAXXZ$70 10015479 f   Metaphlan2WorkerFactory.obj
 0001:00014498       __unwindfunclet$?init@Metaphlan2WorkerFactory@LocalWorkflow@U2@@SAXXZ$72 10015498 f   Metaphlan2WorkerFactory.obj
 0001:000144a3       __unwindfunclet$?init@Metaphlan2WorkerFactory@LocalWorkflow@U2@@SAXXZ$73 100154a3 f   Metaphlan2WorkerFactory.obj
 0001:000144c2       __unwindfunclet$?init@Metaphlan2WorkerFactory@LocalWorkflow@U2@@SAXXZ$75 100154c2 f   Metaphlan2WorkerFactory.obj
 0001:000144cd       __unwindfunclet$?init@Metaphlan2WorkerFactory@LocalWorkflow@U2@@SAXXZ$76 100154cd f   Metaphlan2WorkerFactory.obj
 0001:000144ec       __unwindfunclet$?init@Metaphlan2WorkerFactory@LocalWorkflow@U2@@SAXXZ$78 100154ec f   Metaphlan2WorkerFactory.obj
 0001:000144f7       __unwindfunclet$?init@Metaphlan2WorkerFactory@LocalWorkflow@U2@@SAXXZ$79 100154f7 f   Metaphlan2WorkerFactory.obj
 0001:00014519       __unwindfunclet$?init@Metaphlan2WorkerFactory@LocalWorkflow@U2@@SAXXZ$80 10015519 f   Metaphlan2WorkerFactory.obj
 0001:00014538       __unwindfunclet$?init@Metaphlan2WorkerFactory@LocalWorkflow@U2@@SAXXZ$81 10015538 f   Metaphlan2WorkerFactory.obj
 0001:00014556       __unwindfunclet$?init@Metaphlan2WorkerFactory@LocalWorkflow@U2@@SAXXZ$82 10015556 f   Metaphlan2WorkerFactory.obj
 0001:00014561       __unwindfunclet$?init@Metaphlan2WorkerFactory@LocalWorkflow@U2@@SAXXZ$83 10015561 f   Metaphlan2WorkerFactory.obj
 0001:00014580       __unwindfunclet$?init@Metaphlan2WorkerFactory@LocalWorkflow@U2@@SAXXZ$84 10015580 f   Metaphlan2WorkerFactory.obj
 0001:0001459e       __unwindfunclet$?init@Metaphlan2WorkerFactory@LocalWorkflow@U2@@SAXXZ$85 1001559e f   Metaphlan2WorkerFactory.obj
 0001:000145a9       __unwindfunclet$?init@Metaphlan2WorkerFactory@LocalWorkflow@U2@@SAXXZ$86 100155a9 f   Metaphlan2WorkerFactory.obj
 0001:000145c8       __unwindfunclet$?init@Metaphlan2WorkerFactory@LocalWorkflow@U2@@SAXXZ$87 100155c8 f   Metaphlan2WorkerFactory.obj
 0001:000145e6       __unwindfunclet$?init@Metaphlan2WorkerFactory@LocalWorkflow@U2@@SAXXZ$88 100155e6 f   Metaphlan2WorkerFactory.obj
 0001:000145ee       __unwindfunclet$?init@Metaphlan2WorkerFactory@LocalWorkflow@U2@@SAXXZ$89 100155ee f   Metaphlan2WorkerFactory.obj
 0001:000145f6       __unwindfunclet$?init@Metaphlan2WorkerFactory@LocalWorkflow@U2@@SAXXZ$90 100155f6 f   Metaphlan2WorkerFactory.obj
 0001:000145ff       __unwindfunclet$?init@Metaphlan2WorkerFactory@LocalWorkflow@U2@@SAXXZ$91 100155ff f   Metaphlan2WorkerFactory.obj
 0001:0001460b       __unwindfunclet$?init@Metaphlan2WorkerFactory@LocalWorkflow@U2@@SAXXZ$92 1001560b f   Metaphlan2WorkerFactory.obj
 0001:00014616       __unwindfunclet$?init@Metaphlan2WorkerFactory@LocalWorkflow@U2@@SAXXZ$93 10015616 f   Metaphlan2WorkerFactory.obj
 0001:0001461e       __unwindfunclet$?init@Metaphlan2WorkerFactory@LocalWorkflow@U2@@SAXXZ$165 1001561e f   Metaphlan2WorkerFactory.obj
 0001:00014627       __unwindfunclet$?init@Metaphlan2WorkerFactory@LocalWorkflow@U2@@SAXXZ$94 10015627 f   Metaphlan2WorkerFactory.obj
 0001:0001462f       __unwindfunclet$?init@Metaphlan2WorkerFactory@LocalWorkflow@U2@@SAXXZ$167 1001562f f   Metaphlan2WorkerFactory.obj
 0001:00014638       __unwindfunclet$?init@Metaphlan2WorkerFactory@LocalWorkflow@U2@@SAXXZ$95 10015638 f   Metaphlan2WorkerFactory.obj
 0001:00014643       __unwindfunclet$?init@Metaphlan2WorkerFactory@LocalWorkflow@U2@@SAXXZ$96 10015643 f   Metaphlan2WorkerFactory.obj
 0001:00014662       __unwindfunclet$?init@Metaphlan2WorkerFactory@LocalWorkflow@U2@@SAXXZ$97 10015662 f   Metaphlan2WorkerFactory.obj
 0001:0001466a       __unwindfunclet$?init@Metaphlan2WorkerFactory@LocalWorkflow@U2@@SAXXZ$98 1001566a f   Metaphlan2WorkerFactory.obj
 0001:00014673       __unwindfunclet$?init@Metaphlan2WorkerFactory@LocalWorkflow@U2@@SAXXZ$99 10015673 f   Metaphlan2WorkerFactory.obj
 0001:0001467c       __unwindfunclet$?init@Metaphlan2WorkerFactory@LocalWorkflow@U2@@SAXXZ$100 1001567c f   Metaphlan2WorkerFactory.obj
 0001:00014685       __unwindfunclet$?init@Metaphlan2WorkerFactory@LocalWorkflow@U2@@SAXXZ$101 10015685 f   Metaphlan2WorkerFactory.obj
 0001:0001468e       __unwindfunclet$?init@Metaphlan2WorkerFactory@LocalWorkflow@U2@@SAXXZ$102 1001568e f   Metaphlan2WorkerFactory.obj
 0001:00014699       __unwindfunclet$?init@Metaphlan2WorkerFactory@LocalWorkflow@U2@@SAXXZ$103 10015699 f   Metaphlan2WorkerFactory.obj
 0001:000146a1       __unwindfunclet$?init@Metaphlan2WorkerFactory@LocalWorkflow@U2@@SAXXZ$104 100156a1 f   Metaphlan2WorkerFactory.obj
 0001:000146aa       __unwindfunclet$?init@Metaphlan2WorkerFactory@LocalWorkflow@U2@@SAXXZ$105 100156aa f   Metaphlan2WorkerFactory.obj
 0001:000146b3       __unwindfunclet$?init@Metaphlan2WorkerFactory@LocalWorkflow@U2@@SAXXZ$106 100156b3 f   Metaphlan2WorkerFactory.obj
 0001:000146bf       __unwindfunclet$?init@Metaphlan2WorkerFactory@LocalWorkflow@U2@@SAXXZ$107 100156bf f   Metaphlan2WorkerFactory.obj
 0001:000146cb       __unwindfunclet$?init@Metaphlan2WorkerFactory@LocalWorkflow@U2@@SAXXZ$108 100156cb f   Metaphlan2WorkerFactory.obj
 0001:000146d7       __unwindfunclet$?init@Metaphlan2WorkerFactory@LocalWorkflow@U2@@SAXXZ$109 100156d7 f   Metaphlan2WorkerFactory.obj
 0001:000146e3       __unwindfunclet$?init@Metaphlan2WorkerFactory@LocalWorkflow@U2@@SAXXZ$110 100156e3 f   Metaphlan2WorkerFactory.obj
 0001:000146ee       __unwindfunclet$?init@Metaphlan2WorkerFactory@LocalWorkflow@U2@@SAXXZ$111 100156ee f   Metaphlan2WorkerFactory.obj
 0001:000146f6       __unwindfunclet$?init@Metaphlan2WorkerFactory@LocalWorkflow@U2@@SAXXZ$112 100156f6 f   Metaphlan2WorkerFactory.obj
 0001:000146ff       __unwindfunclet$?init@Metaphlan2WorkerFactory@LocalWorkflow@U2@@SAXXZ$113 100156ff f   Metaphlan2WorkerFactory.obj
 0001:00014708       __unwindfunclet$?init@Metaphlan2WorkerFactory@LocalWorkflow@U2@@SAXXZ$114 10015708 f   Metaphlan2WorkerFactory.obj
 0001:00014714       __unwindfunclet$?init@Metaphlan2WorkerFactory@LocalWorkflow@U2@@SAXXZ$115 10015714 f   Metaphlan2WorkerFactory.obj
 0001:00014720       __unwindfunclet$?init@Metaphlan2WorkerFactory@LocalWorkflow@U2@@SAXXZ$116 10015720 f   Metaphlan2WorkerFactory.obj
 0001:0001472c       __unwindfunclet$?init@Metaphlan2WorkerFactory@LocalWorkflow@U2@@SAXXZ$117 1001572c f   Metaphlan2WorkerFactory.obj
 0001:00014738       __unwindfunclet$?init@Metaphlan2WorkerFactory@LocalWorkflow@U2@@SAXXZ$118 10015738 f   Metaphlan2WorkerFactory.obj
 0001:00014744       __unwindfunclet$?init@Metaphlan2WorkerFactory@LocalWorkflow@U2@@SAXXZ$119 10015744 f   Metaphlan2WorkerFactory.obj
 0001:0001474d       __unwindfunclet$?init@Metaphlan2WorkerFactory@LocalWorkflow@U2@@SAXXZ$120 1001574d f   Metaphlan2WorkerFactory.obj
 0001:00014758       __unwindfunclet$?init@Metaphlan2WorkerFactory@LocalWorkflow@U2@@SAXXZ$121 10015758 f   Metaphlan2WorkerFactory.obj
 0001:00014760       __unwindfunclet$?init@Metaphlan2WorkerFactory@LocalWorkflow@U2@@SAXXZ$122 10015760 f   Metaphlan2WorkerFactory.obj
 0001:00014769       __unwindfunclet$?init@Metaphlan2WorkerFactory@LocalWorkflow@U2@@SAXXZ$123 10015769 f   Metaphlan2WorkerFactory.obj
 0001:00014772       __unwindfunclet$?init@Metaphlan2WorkerFactory@LocalWorkflow@U2@@SAXXZ$124 10015772 f   Metaphlan2WorkerFactory.obj
 0001:0001477b       __unwindfunclet$?init@Metaphlan2WorkerFactory@LocalWorkflow@U2@@SAXXZ$125 1001577b f   Metaphlan2WorkerFactory.obj
 0001:00014784       __unwindfunclet$?init@Metaphlan2WorkerFactory@LocalWorkflow@U2@@SAXXZ$126 10015784 f   Metaphlan2WorkerFactory.obj
 0001:0001478f       __unwindfunclet$?init@Metaphlan2WorkerFactory@LocalWorkflow@U2@@SAXXZ$127 1001578f f   Metaphlan2WorkerFactory.obj
 0001:00014797       __unwindfunclet$?init@Metaphlan2WorkerFactory@LocalWorkflow@U2@@SAXXZ$128 10015797 f   Metaphlan2WorkerFactory.obj
 0001:000147a0       __unwindfunclet$?init@Metaphlan2WorkerFactory@LocalWorkflow@U2@@SAXXZ$129 100157a0 f   Metaphlan2WorkerFactory.obj
 0001:000147a9       __unwindfunclet$?init@Metaphlan2WorkerFactory@LocalWorkflow@U2@@SAXXZ$130 100157a9 f   Metaphlan2WorkerFactory.obj
 0001:000147b2       __unwindfunclet$?init@Metaphlan2WorkerFactory@LocalWorkflow@U2@@SAXXZ$131 100157b2 f   Metaphlan2WorkerFactory.obj
 0001:000147bb       __unwindfunclet$?init@Metaphlan2WorkerFactory@LocalWorkflow@U2@@SAXXZ$132 100157bb f   Metaphlan2WorkerFactory.obj
 0001:000147c6       __unwindfunclet$?init@Metaphlan2WorkerFactory@LocalWorkflow@U2@@SAXXZ$133 100157c6 f   Metaphlan2WorkerFactory.obj
 0001:000147d2       __unwindfunclet$?init@Metaphlan2WorkerFactory@LocalWorkflow@U2@@SAXXZ$134 100157d2 f   Metaphlan2WorkerFactory.obj
 0001:000147db       __unwindfunclet$?init@Metaphlan2WorkerFactory@LocalWorkflow@U2@@SAXXZ$135 100157db f   Metaphlan2WorkerFactory.obj
 0001:000147e4       __unwindfunclet$?init@Metaphlan2WorkerFactory@LocalWorkflow@U2@@SAXXZ$136 100157e4 f   Metaphlan2WorkerFactory.obj
 0001:000147ec       __unwindfunclet$?init@Metaphlan2WorkerFactory@LocalWorkflow@U2@@SAXXZ$137 100157ec f   Metaphlan2WorkerFactory.obj
 0001:000147f5       __unwindfunclet$?init@Metaphlan2WorkerFactory@LocalWorkflow@U2@@SAXXZ$138 100157f5 f   Metaphlan2WorkerFactory.obj
 0001:000147fe       __unwindfunclet$?init@Metaphlan2WorkerFactory@LocalWorkflow@U2@@SAXXZ$139 100157fe f   Metaphlan2WorkerFactory.obj
 0001:00014807       __unwindfunclet$?init@Metaphlan2WorkerFactory@LocalWorkflow@U2@@SAXXZ$140 10015807 f   Metaphlan2WorkerFactory.obj
 0001:00014812       __unwindfunclet$?init@Metaphlan2WorkerFactory@LocalWorkflow@U2@@SAXXZ$141 10015812 f   Metaphlan2WorkerFactory.obj
 0001:00014831       __unwindfunclet$?init@Metaphlan2WorkerFactory@LocalWorkflow@U2@@SAXXZ$142 10015831 f   Metaphlan2WorkerFactory.obj
 0001:0001483d       __unwindfunclet$?init@Metaphlan2WorkerFactory@LocalWorkflow@U2@@SAXXZ$143 1001583d f   Metaphlan2WorkerFactory.obj
 0001:00014846       __unwindfunclet$?init@Metaphlan2WorkerFactory@LocalWorkflow@U2@@SAXXZ$144 10015846 f   Metaphlan2WorkerFactory.obj
 0001:0001484f       __unwindfunclet$?init@Metaphlan2WorkerFactory@LocalWorkflow@U2@@SAXXZ$145 1001584f f   Metaphlan2WorkerFactory.obj
 0001:00014857       __unwindfunclet$?init@Metaphlan2WorkerFactory@LocalWorkflow@U2@@SAXXZ$146 10015857 f   Metaphlan2WorkerFactory.obj
 0001:00014860       __unwindfunclet$?init@Metaphlan2WorkerFactory@LocalWorkflow@U2@@SAXXZ$147 10015860 f   Metaphlan2WorkerFactory.obj
 0001:00014869       __unwindfunclet$?init@Metaphlan2WorkerFactory@LocalWorkflow@U2@@SAXXZ$148 10015869 f   Metaphlan2WorkerFactory.obj
 0001:00014872       __unwindfunclet$?init@Metaphlan2WorkerFactory@LocalWorkflow@U2@@SAXXZ$149 10015872 f   Metaphlan2WorkerFactory.obj
 0001:0001487d       __unwindfunclet$?init@Metaphlan2WorkerFactory@LocalWorkflow@U2@@SAXXZ$150 1001587d f   Metaphlan2WorkerFactory.obj
 0001:0001489c       __unwindfunclet$?init@Metaphlan2WorkerFactory@LocalWorkflow@U2@@SAXXZ$151 1001589c f   Metaphlan2WorkerFactory.obj
 0001:000148a5       __unwindfunclet$?init@Metaphlan2WorkerFactory@LocalWorkflow@U2@@SAXXZ$152 100158a5 f   Metaphlan2WorkerFactory.obj
 0001:000148ae       __unwindfunclet$?init@Metaphlan2WorkerFactory@LocalWorkflow@U2@@SAXXZ$153 100158ae f   Metaphlan2WorkerFactory.obj
 0001:000148ba       __unwindfunclet$?init@Metaphlan2WorkerFactory@LocalWorkflow@U2@@SAXXZ$154 100158ba f   Metaphlan2WorkerFactory.obj
 0001:000148c5       __unwindfunclet$?init@Metaphlan2WorkerFactory@LocalWorkflow@U2@@SAXXZ$155 100158c5 f   Metaphlan2WorkerFactory.obj
 0001:000148d0       __unwindfunclet$?init@Metaphlan2WorkerFactory@LocalWorkflow@U2@@SAXXZ$156 100158d0 f   Metaphlan2WorkerFactory.obj
 0001:000148db       __unwindfunclet$?init@Metaphlan2WorkerFactory@LocalWorkflow@U2@@SAXXZ$157 100158db f   Metaphlan2WorkerFactory.obj
 0001:000148e4       __unwindfunclet$?init@Metaphlan2WorkerFactory@LocalWorkflow@U2@@SAXXZ$158 100158e4 f   Metaphlan2WorkerFactory.obj
 0001:000148ed       __unwindfunclet$?init@Metaphlan2WorkerFactory@LocalWorkflow@U2@@SAXXZ$159 100158ed f   Metaphlan2WorkerFactory.obj
 0001:000148f6       __unwindfunclet$?init@Metaphlan2WorkerFactory@LocalWorkflow@U2@@SAXXZ$160 100158f6 f   Metaphlan2WorkerFactory.obj
 0001:000148ff       __unwindfunclet$?init@Metaphlan2WorkerFactory@LocalWorkflow@U2@@SAXXZ$161 100158ff f   Metaphlan2WorkerFactory.obj
 0001:00014908       __unwindfunclet$?init@Metaphlan2WorkerFactory@LocalWorkflow@U2@@SAXXZ$162 10015908 f   Metaphlan2WorkerFactory.obj
 0001:00014913       __unwindfunclet$?init@Metaphlan2WorkerFactory@LocalWorkflow@U2@@SAXXZ$163 10015913 f   Metaphlan2WorkerFactory.obj
 0001:0001491c       __unwindfunclet$?init@Metaphlan2WorkerFactory@LocalWorkflow@U2@@SAXXZ$164 1001591c f   Metaphlan2WorkerFactory.obj
 0001:00014927       __ehhandler$?init@Metaphlan2WorkerFactory@LocalWorkflow@U2@@SAXXZ 10015927 f   Metaphlan2WorkerFactory.obj
 0001:00014950       __unwindfunclet$?node_construct@?$QList@U?$QPair@VQString@@V1@@@@@AAEXPAUNode@1@ABU?$QPair@VQString@@V1@@@@Z$0 10015950 f   Metaphlan2WorkerFactory.obj
 0001:0001495b       __unwindfunclet$?node_construct@?$QList@U?$QPair@VQString@@V1@@@@@AAEXPAUNode@1@ABU?$QPair@VQString@@V1@@@@Z$2 1001595b f   Metaphlan2WorkerFactory.obj
 0001:00014964       __ehhandler$?node_construct@?$QList@U?$QPair@VQString@@V1@@@@@AAEXPAUNode@1@ABU?$QPair@VQString@@V1@@@@Z 10015964 f   Metaphlan2WorkerFactory.obj
 0001:00014980       __unwindfunclet$?node_construct@?$QList@VQVariant@@@@AAEXPAUNode@1@ABVQVariant@@@Z$0 10015980 f   Metaphlan2WorkerFactory.obj
 0001:0001498b       __ehhandler$?node_construct@?$QList@VQVariant@@@@AAEXPAUNode@1@ABVQVariant@@@Z 1001598b f   Metaphlan2WorkerFactory.obj
 0001:000149b0       __unwindfunclet$?node_copy@?$QList@U?$QPair@VQString@@V1@@@@@AAEXPAUNode@1@00@Z$4 100159b0 f   Metaphlan2WorkerFactory.obj
 0001:000149bb       __unwindfunclet$?node_copy@?$QList@U?$QPair@VQString@@V1@@@@@AAEXPAUNode@1@00@Z$6 100159bb f   Metaphlan2WorkerFactory.obj
 0001:000149c4       __unwindfunclet$?node_copy@?$QList@U?$QPair@VQString@@V1@@@@@AAEXPAUNode@1@00@Z$8 100159c4 f   Metaphlan2WorkerFactory.obj
 0001:000149cd       __ehhandler$?node_copy@?$QList@U?$QPair@VQString@@V1@@@@@AAEXPAUNode@1@00@Z 100159cd f   Metaphlan2WorkerFactory.obj
 0001:000149f0       __unwindfunclet$?node_copy@?$QList@VQVariant@@@@AAEXPAUNode@1@00@Z$4 100159f0 f   Metaphlan2WorkerFactory.obj
 0001:000149fb       __ehhandler$?node_copy@?$QList@VQVariant@@@@AAEXPAUNode@1@00@Z 100159fb f   Metaphlan2WorkerFactory.obj
 0001:00014a20       __unwindfunclet$?node_destruct@?$QList@U?$QPair@VQString@@V1@@@@@AAEXPAUNode@1@0@Z$0 10015a20 f   Metaphlan2WorkerFactory.obj
 0001:00014a29       __ehhandler$?node_destruct@?$QList@U?$QPair@VQString@@V1@@@@@AAEXPAUNode@1@0@Z 10015a29 f   Metaphlan2WorkerFactory.obj
 0001:00014a50       __unwindfunclet$?node_destruct@?$QList@U?$QPair@VQString@@V1@@@@@AAEXPAUNode@1@@Z$0 10015a50 f   Metaphlan2WorkerFactory.obj
 0001:00014a59       __ehhandler$?node_destruct@?$QList@U?$QPair@VQString@@V1@@@@@AAEXPAUNode@1@@Z 10015a59 f   Metaphlan2WorkerFactory.obj
 0001:00014a80       __unwindfunclet$??__EalgoLog@U2@@YAXXZ$0 10015a80 f   moc_Metaphlan2Prompter.obj
 0001:00014a89       __ehhandler$??__EalgoLog@U2@@YAXXZ 10015a89 f   moc_Metaphlan2Prompter.obj
 0001:00014ab0       __unwindfunclet$??__EcmdLog@U2@@YAXXZ$0 10015ab0 f   moc_Metaphlan2Prompter.obj
 0001:00014ab9       __ehhandler$??__EcmdLog@U2@@YAXXZ 10015ab9 f   moc_Metaphlan2Prompter.obj
 0001:00014ae0       __unwindfunclet$??__EcoreLog@U2@@YAXXZ$0 10015ae0 f   moc_Metaphlan2Prompter.obj
 0001:00014ae9       __ehhandler$??__EcoreLog@U2@@YAXXZ 10015ae9 f   moc_Metaphlan2Prompter.obj
 0001:00014b10       __unwindfunclet$??__EioLog@U2@@YAXXZ$0 10015b10 f   moc_Metaphlan2Prompter.obj
 0001:00014b19       __ehhandler$??__EioLog@U2@@YAXXZ 10015b19 f   moc_Metaphlan2Prompter.obj
 0001:00014b40       __unwindfunclet$??__EperfLog@U2@@YAXXZ$0 10015b40 f   moc_Metaphlan2Prompter.obj
 0001:00014b49       __ehhandler$??__EperfLog@U2@@YAXXZ 10015b49 f   moc_Metaphlan2Prompter.obj
 0001:00014b70       __unwindfunclet$??__EscriptLog@U2@@YAXXZ$0 10015b70 f   moc_Metaphlan2Prompter.obj
 0001:00014b79       __ehhandler$??__EscriptLog@U2@@YAXXZ 10015b79 f   moc_Metaphlan2Prompter.obj
 0001:00014ba0       __unwindfunclet$??__EtaskLog@U2@@YAXXZ$0 10015ba0 f   moc_Metaphlan2Prompter.obj
 0001:00014ba9       __ehhandler$??__EtaskLog@U2@@YAXXZ 10015ba9 f   moc_Metaphlan2Prompter.obj
 0001:00014bd0       __unwindfunclet$??__EuiLog@U2@@YAXXZ$0 10015bd0 f   moc_Metaphlan2Prompter.obj
 0001:00014bd9       __ehhandler$??__EuiLog@U2@@YAXXZ 10015bd9 f   moc_Metaphlan2Prompter.obj
 0001:00014c00       __unwindfunclet$??__EuserActLog@U2@@YAXXZ$0 10015c00 f   moc_Metaphlan2Prompter.obj
 0001:00014c09       __ehhandler$??__EuserActLog@U2@@YAXXZ 10015c09 f   moc_Metaphlan2Prompter.obj
 0001:00014c30       __unwindfunclet$??__EalgoLog@U2@@YAXXZ$0 10015c30 f   moc_Metaphlan2Task.obj
 0001:00014c39       __ehhandler$??__EalgoLog@U2@@YAXXZ 10015c39 f   moc_Metaphlan2Task.obj
 0001:00014c60       __unwindfunclet$??__EcmdLog@U2@@YAXXZ$0 10015c60 f   moc_Metaphlan2Task.obj
 0001:00014c69       __ehhandler$??__EcmdLog@U2@@YAXXZ 10015c69 f   moc_Metaphlan2Task.obj
 0001:00014c90       __unwindfunclet$??__EcoreLog@U2@@YAXXZ$0 10015c90 f   moc_Metaphlan2Task.obj
 0001:00014c99       __ehhandler$??__EcoreLog@U2@@YAXXZ 10015c99 f   moc_Metaphlan2Task.obj
 0001:00014cc0       __unwindfunclet$??__EioLog@U2@@YAXXZ$0 10015cc0 f   moc_Metaphlan2Task.obj
 0001:00014cc9       __ehhandler$??__EioLog@U2@@YAXXZ 10015cc9 f   moc_Metaphlan2Task.obj
 0001:00014cf0       __unwindfunclet$??__EperfLog@U2@@YAXXZ$0 10015cf0 f   moc_Metaphlan2Task.obj
 0001:00014cf9       __ehhandler$??__EperfLog@U2@@YAXXZ 10015cf9 f   moc_Metaphlan2Task.obj
 0001:00014d20       __unwindfunclet$??__EscriptLog@U2@@YAXXZ$0 10015d20 f   moc_Metaphlan2Task.obj
 0001:00014d29       __ehhandler$??__EscriptLog@U2@@YAXXZ 10015d29 f   moc_Metaphlan2Task.obj
 0001:00014d50       __unwindfunclet$??__EtaskLog@U2@@YAXXZ$0 10015d50 f   moc_Metaphlan2Task.obj
 0001:00014d59       __ehhandler$??__EtaskLog@U2@@YAXXZ 10015d59 f   moc_Metaphlan2Task.obj
 0001:00014d80       __unwindfunclet$??__EuiLog@U2@@YAXXZ$0 10015d80 f   moc_Metaphlan2Task.obj
 0001:00014d89       __ehhandler$??__EuiLog@U2@@YAXXZ 10015d89 f   moc_Metaphlan2Task.obj
 0001:00014db0       __unwindfunclet$??__EuserActLog@U2@@YAXXZ$0 10015db0 f   moc_Metaphlan2Task.obj
 0001:00014db9       __ehhandler$??__EuserActLog@U2@@YAXXZ 10015db9 f   moc_Metaphlan2Task.obj
 0001:00014de0       __unwindfunclet$??__EalgoLog@U2@@YAXXZ$0 10015de0 f   moc_Metaphlan2Worker.obj
 0001:00014de9       __ehhandler$??__EalgoLog@U2@@YAXXZ 10015de9 f   moc_Metaphlan2Worker.obj
 0001:00014e10       __unwindfunclet$??__EcmdLog@U2@@YAXXZ$0 10015e10 f   moc_Metaphlan2Worker.obj
 0001:00014e19       __ehhandler$??__EcmdLog@U2@@YAXXZ 10015e19 f   moc_Metaphlan2Worker.obj
 0001:00014e40       __unwindfunclet$??__EcoreLog@U2@@YAXXZ$0 10015e40 f   moc_Metaphlan2Worker.obj
 0001:00014e49       __ehhandler$??__EcoreLog@U2@@YAXXZ 10015e49 f   moc_Metaphlan2Worker.obj
 0001:00014e70       __unwindfunclet$??__EioLog@U2@@YAXXZ$0 10015e70 f   moc_Metaphlan2Worker.obj
 0001:00014e79       __ehhandler$??__EioLog@U2@@YAXXZ 10015e79 f   moc_Metaphlan2Worker.obj
 0001:00014ea0       __unwindfunclet$??__EperfLog@U2@@YAXXZ$0 10015ea0 f   moc_Metaphlan2Worker.obj
 0001:00014ea9       __ehhandler$??__EperfLog@U2@@YAXXZ 10015ea9 f   moc_Metaphlan2Worker.obj
 0001:00014ed0       __unwindfunclet$??__EscriptLog@U2@@YAXXZ$0 10015ed0 f   moc_Metaphlan2Worker.obj
 0001:00014ed9       __ehhandler$??__EscriptLog@U2@@YAXXZ 10015ed9 f   moc_Metaphlan2Worker.obj
 0001:00014f00       __unwindfunclet$??__EtaskLog@U2@@YAXXZ$0 10015f00 f   moc_Metaphlan2Worker.obj
 0001:00014f09       __ehhandler$??__EtaskLog@U2@@YAXXZ 10015f09 f   moc_Metaphlan2Worker.obj
 0001:00014f30       __unwindfunclet$??__EuiLog@U2@@YAXXZ$0 10015f30 f   moc_Metaphlan2Worker.obj
 0001:00014f39       __ehhandler$??__EuiLog@U2@@YAXXZ 10015f39 f   moc_Metaphlan2Worker.obj
 0001:00014f60       __unwindfunclet$??__EuserActLog@U2@@YAXXZ$0 10015f60 f   moc_Metaphlan2Worker.obj
 0001:00014f69       __ehhandler$??__EuserActLog@U2@@YAXXZ 10015f69 f   moc_Metaphlan2Worker.obj
 0001:00014f90       __unwindfunclet$?qt_metatype_id@?$QMetaTypeIdQObject@PAVTask@U2@@$00@@SAHXZ$0 10015f90 f   moc_Metaphlan2Worker.obj
 0001:00014f99       __ehhandler$?qt_metatype_id@?$QMetaTypeIdQObject@PAVTask@U2@@$00@@SAHXZ 10015f99 f   moc_Metaphlan2Worker.obj
 0001:00014fc0       ??__F?_Generic_object@?$_Error_objects@H@std@@2V_Generic_error_category@2@A@@YAXXZ 10015fc0 f   Metaphlan2LogParser.obj
 0001:00014fd0       ??__F?_Iostream_object@?$_Error_objects@H@std@@2V_Iostream_error_category@2@A@@YAXXZ 10015fd0 f   Metaphlan2LogParser.obj
 0001:00014fe0       ??__F?_System_object@?$_Error_objects@H@std@@2V_System_error_category@2@A@@YAXXZ 10015fe0 f   Metaphlan2LogParser.obj
 0001:00014ff0       ??__F?wellKnownErrors@Metaphlan2LogParser@U2@@0VQStringList@@B@@YAXXZ 10015ff0 f   Metaphlan2LogParser.obj
 0001:00015000       ??__FalgoLog@U2@@YAXXZ     10016000 f   Metaphlan2LogParser.obj
 0001:00015010       ??__FcmdLog@U2@@YAXXZ      10016010 f   Metaphlan2LogParser.obj
 0001:00015020       ??__FcoreLog@U2@@YAXXZ     10016020 f   Metaphlan2LogParser.obj
 0001:00015030       ??__FioLog@U2@@YAXXZ       10016030 f   Metaphlan2LogParser.obj
 0001:00015040       ??__FperfLog@U2@@YAXXZ     10016040 f   Metaphlan2LogParser.obj
 0001:00015050       ??__FscriptLog@U2@@YAXXZ   10016050 f   Metaphlan2LogParser.obj
 0001:00015060       ??__FtaskLog@U2@@YAXXZ     10016060 f   Metaphlan2LogParser.obj
 0001:00015070       ??__FuiLog@U2@@YAXXZ       10016070 f   Metaphlan2LogParser.obj
 0001:00015080       ??__FuserActLog@U2@@YAXXZ  10016080 f   Metaphlan2LogParser.obj
 0001:00015090       ??__F?_Generic_object@?$_Error_objects@H@std@@2V_Generic_error_category@2@A@@YAXXZ 10016090 f   Metaphlan2Prompter.obj
 0001:000150a0       ??__F?_Iostream_object@?$_Error_objects@H@std@@2V_Iostream_error_category@2@A@@YAXXZ 100160a0 f   Metaphlan2Prompter.obj
 0001:000150b0       ??__F?_System_object@?$_Error_objects@H@std@@2V_System_error_category@2@A@@YAXXZ 100160b0 f   Metaphlan2Prompter.obj
 0001:000150c0       ??__FalgoLog@U2@@YAXXZ     100160c0 f   Metaphlan2Prompter.obj
 0001:000150d0       ??__FcmdLog@U2@@YAXXZ      100160d0 f   Metaphlan2Prompter.obj
 0001:000150e0       ??__FcoreLog@U2@@YAXXZ     100160e0 f   Metaphlan2Prompter.obj
 0001:000150f0       ??__FioLog@U2@@YAXXZ       100160f0 f   Metaphlan2Prompter.obj
 0001:00015100       ??__FperfLog@U2@@YAXXZ     10016100 f   Metaphlan2Prompter.obj
 0001:00015110       ??__FscriptLog@U2@@YAXXZ   10016110 f   Metaphlan2Prompter.obj
 0001:00015120       ??__FtaskLog@U2@@YAXXZ     10016120 f   Metaphlan2Prompter.obj
 0001:00015130       ??__FuiLog@U2@@YAXXZ       10016130 f   Metaphlan2Prompter.obj
 0001:00015140       ??__FuserActLog@U2@@YAXXZ  10016140 f   Metaphlan2Prompter.obj
 0001:00015150       ??__F?ET_BOWTIE_2_ALIGNER@Metaphlan2Support@U2@@2VQString@@B@@YAXXZ 10016150 f   Metaphlan2Support.obj
 0001:00015160       ??__F?ET_PYTHON@Metaphlan2Support@U2@@2VQString@@B@@YAXXZ 10016160 f   Metaphlan2Support.obj
 0001:00015170       ??__F?ET_PYTHON_BIO@Metaphlan2Support@U2@@2VQString@@B@@YAXXZ 10016170 f   Metaphlan2Support.obj
 0001:00015180       ??__F?ET_PYTHON_NUMPY@Metaphlan2Support@U2@@2VQString@@B@@YAXXZ 10016180 f   Metaphlan2Support.obj
 0001:00015190       ??__F?TOOL_NAME@Metaphlan2Support@U2@@2VQString@@B@@YAXXZ 10016190 f   Metaphlan2Support.obj
 0001:000151a0       ??__F?UTIL_SCRIPT@Metaphlan2Support@U2@@2VQString@@B@@YAXXZ 100161a0 f   Metaphlan2Support.obj
 0001:000151b0       ??__F?_Generic_object@?$_Error_objects@H@std@@2V_Generic_error_category@2@A@@YAXXZ 100161b0 f   Metaphlan2Support.obj
 0001:000151c0       ??__F?_Iostream_object@?$_Error_objects@H@std@@2V_Iostream_error_category@2@A@@YAXXZ 100161c0 f   Metaphlan2Support.obj
 0001:000151d0       ??__F?_System_object@?$_Error_objects@H@std@@2V_System_error_category@2@A@@YAXXZ 100161d0 f   Metaphlan2Support.obj
 0001:000151e0       ??__FalgoLog@U2@@YAXXZ     100161e0 f   Metaphlan2Support.obj
 0001:000151f0       ??__FcmdLog@U2@@YAXXZ      100161f0 f   Metaphlan2Support.obj
 0001:00015200       ??__FcoreLog@U2@@YAXXZ     10016200 f   Metaphlan2Support.obj
 0001:00015210       ??__FioLog@U2@@YAXXZ       10016210 f   Metaphlan2Support.obj
 0001:00015220       ??__FperfLog@U2@@YAXXZ     10016220 f   Metaphlan2Support.obj
 0001:00015230       ??__FscriptLog@U2@@YAXXZ   10016230 f   Metaphlan2Support.obj
 0001:00015240       ??__FtaskLog@U2@@YAXXZ     10016240 f   Metaphlan2Support.obj
 0001:00015250       ??__FuiLog@U2@@YAXXZ       10016250 f   Metaphlan2Support.obj
 0001:00015260       ??__FuserActLog@U2@@YAXXZ  10016260 f   Metaphlan2Support.obj
 0001:00015270       ??__F?PLUGIN_DESCRIPRION@MetaphlanSupportPlugin@U2@@2VQString@@B@@YAXXZ 10016270 f   Metaphlan2SupportPlugin.obj
 0001:00015280       ??__F?PLUGIN_NAME@MetaphlanSupportPlugin@U2@@2VQString@@B@@YAXXZ 10016280 f   Metaphlan2SupportPlugin.obj
 0001:00015290       ??__F?_Generic_object@?$_Error_objects@H@std@@2V_Generic_error_category@2@A@@YAXXZ 10016290 f   Metaphlan2SupportPlugin.obj
 0001:000152a0       ??__F?_Iostream_object@?$_Error_objects@H@std@@2V_Iostream_error_category@2@A@@YAXXZ 100162a0 f   Metaphlan2SupportPlugin.obj
 0001:000152b0       ??__F?_System_object@?$_Error_objects@H@std@@2V_System_error_category@2@A@@YAXXZ 100162b0 f   Metaphlan2SupportPlugin.obj
 0001:000152c0       ??__FalgoLog@U2@@YAXXZ     100162c0 f   Metaphlan2SupportPlugin.obj
 0001:000152d0       ??__FcmdLog@U2@@YAXXZ      100162d0 f   Metaphlan2SupportPlugin.obj
 0001:000152e0       ??__FcoreLog@U2@@YAXXZ     100162e0 f   Metaphlan2SupportPlugin.obj
 0001:000152f0       ??__FioLog@U2@@YAXXZ       100162f0 f   Metaphlan2SupportPlugin.obj
 0001:00015300       ??__FperfLog@U2@@YAXXZ     10016300 f   Metaphlan2SupportPlugin.obj
 0001:00015310       ??__FscriptLog@U2@@YAXXZ   10016310 f   Metaphlan2SupportPlugin.obj
 0001:00015320       ??__FtaskLog@U2@@YAXXZ     10016320 f   Metaphlan2SupportPlugin.obj
 0001:00015330       ??__FuiLog@U2@@YAXXZ       10016330 f   Metaphlan2SupportPlugin.obj
 0001:00015340       ??__FuserActLog@U2@@YAXXZ  10016340 f   Metaphlan2SupportPlugin.obj
 0001:00015350       ??__F?_Generic_object@?$_Error_objects@H@std@@2V_Generic_error_category@2@A@@YAXXZ 10016350 f   Metaphlan2Task.obj
 0001:00015360       ??__F?_Iostream_object@?$_Error_objects@H@std@@2V_Iostream_error_category@2@A@@YAXXZ 10016360 f   Metaphlan2Task.obj
 0001:00015370       ??__F?_System_object@?$_Error_objects@H@std@@2V_System_error_category@2@A@@YAXXZ 10016370 f   Metaphlan2Task.obj
 0001:00015380       ??__FalgoLog@U2@@YAXXZ     10016380 f   Metaphlan2Task.obj
 0001:00015390       ??__FcmdLog@U2@@YAXXZ      10016390 f   Metaphlan2Task.obj
 0001:000153a0       ??__FcoreLog@U2@@YAXXZ     100163a0 f   Metaphlan2Task.obj
 0001:000153b0       ??__Fcvar@?1???0Metaphlan2ClassifyTask@U2@@QAE@ABUMetaphlan2TaskSettings@1@@Z@YAXXZ 100163b0 f   Metaphlan2Task.obj
 0001:000153c0       ??__FioLog@U2@@YAXXZ       100163c0 f   Metaphlan2Task.obj
 0001:000153d0       ??__FperfLog@U2@@YAXXZ     100163d0 f   Metaphlan2Task.obj
 0001:000153e0       ??__FscriptLog@U2@@YAXXZ   100163e0 f   Metaphlan2Task.obj
 0001:000153f0       ??__FtaskLog@U2@@YAXXZ     100163f0 f   Metaphlan2Task.obj
 0001:00015400       ??__FuiLog@U2@@YAXXZ       10016400 f   Metaphlan2Task.obj
 0001:00015410       ??__FuserActLog@U2@@YAXXZ  10016410 f   Metaphlan2Task.obj
 0001:00015420       ??__F?_Generic_object@?$_Error_objects@H@std@@2V_Generic_error_category@2@A@@YAXXZ 10016420 f   Metaphlan2Validator.obj
 0001:00015430       ??__F?_Iostream_object@?$_Error_objects@H@std@@2V_Iostream_error_category@2@A@@YAXXZ 10016430 f   Metaphlan2Validator.obj
 0001:00015440       ??__F?_System_object@?$_Error_objects@H@std@@2V_System_error_category@2@A@@YAXXZ 10016440 f   Metaphlan2Validator.obj
 0001:00015450       ??__FalgoLog@U2@@YAXXZ     10016450 f   Metaphlan2Validator.obj
 0001:00015460       ??__FcmdLog@U2@@YAXXZ      10016460 f   Metaphlan2Validator.obj
 0001:00015470       ??__FcoreLog@U2@@YAXXZ     10016470 f   Metaphlan2Validator.obj
 0001:00015480       ??__FioLog@U2@@YAXXZ       10016480 f   Metaphlan2Validator.obj
 0001:00015490       ??__FperfLog@U2@@YAXXZ     10016490 f   Metaphlan2Validator.obj
 0001:000154a0       ??__FscriptLog@U2@@YAXXZ   100164a0 f   Metaphlan2Validator.obj
 0001:000154b0       ??__FtaskLog@U2@@YAXXZ     100164b0 f   Metaphlan2Validator.obj
 0001:000154c0       ??__FuiLog@U2@@YAXXZ       100164c0 f   Metaphlan2Validator.obj
 0001:000154d0       ??__FuserActLog@U2@@YAXXZ  100164d0 f   Metaphlan2Validator.obj
 0001:000154e0       ??__F?BOWTIE2OUT_DIR@Metaphlan2Worker@LocalWorkflow@U2@@0VQString@@B@@YAXXZ 100164e0 f   Metaphlan2Worker.obj
 0001:000154f0       ??__F?BOWTIE2OUT_SUFFIX@Metaphlan2Worker@LocalWorkflow@U2@@0VQString@@B@@YAXXZ 100164f0 f   Metaphlan2Worker.obj
 0001:00015500       ??__F?METAPHLAN2_ROOT_DIR@Metaphlan2Worker@LocalWorkflow@U2@@0VQString@@B@@YAXXZ 10016500 f   Metaphlan2Worker.obj
 0001:00015510       ??__F?PROFILE_DIR@Metaphlan2Worker@LocalWorkflow@U2@@0VQString@@B@@YAXXZ 10016510 f   Metaphlan2Worker.obj
 0001:00015520       ??__F?PROFILE_SUFFIX@Metaphlan2Worker@LocalWorkflow@U2@@0VQString@@B@@YAXXZ 10016520 f   Metaphlan2Worker.obj
 0001:00015530       ??__F?_Generic_object@?$_Error_objects@H@std@@2V_Generic_error_category@2@A@@YAXXZ 10016530 f   Metaphlan2Worker.obj
 0001:00015540       ??__F?_Iostream_object@?$_Error_objects@H@std@@2V_Iostream_error_category@2@A@@YAXXZ 10016540 f   Metaphlan2Worker.obj
 0001:00015550       ??__F?_System_object@?$_Error_objects@H@std@@2V_System_error_category@2@A@@YAXXZ 10016550 f   Metaphlan2Worker.obj
 0001:00015560       ??__FalgoLog@U2@@YAXXZ     10016560 f   Metaphlan2Worker.obj
 0001:00015570       ??__FcmdLog@U2@@YAXXZ      10016570 f   Metaphlan2Worker.obj
 0001:00015580       ??__FcoreLog@U2@@YAXXZ     10016580 f   Metaphlan2Worker.obj
 0001:00015590       ??__FioLog@U2@@YAXXZ       10016590 f   Metaphlan2Worker.obj
 0001:000155a0       ??__FperfLog@U2@@YAXXZ     100165a0 f   Metaphlan2Worker.obj
 0001:000155b0       ??__FscriptLog@U2@@YAXXZ   100165b0 f   Metaphlan2Worker.obj
 0001:000155c0       ??__FtaskLog@U2@@YAXXZ     100165c0 f   Metaphlan2Worker.obj
 0001:000155d0       ??__FuiLog@U2@@YAXXZ       100165d0 f   Metaphlan2Worker.obj
 0001:000155e0       ??__FuserActLog@U2@@YAXXZ  100165e0 f   Metaphlan2Worker.obj
 0001:000155f0       ??__F?ACTOR_ID@Metaphlan2WorkerFactory@LocalWorkflow@U2@@2VQString@@B@@YAXXZ 100165f0 f   Metaphlan2WorkerFactory.obj
 0001:00015600       ??__F?ANALYSIS_TYPE@Metaphlan2WorkerFactory@LocalWorkflow@U2@@2VQString@@B@@YAXXZ 10016600 f   Metaphlan2WorkerFactory.obj
 0001:00015610       ??__F?ANALYSIS_TYPE_CLADE_PROFILES_TEXT@Metaphlan2WorkerFactory@LocalWorkflow@U2@@2VQString@@B@@YAXXZ 10016610 f   Metaphlan2WorkerFactory.obj
 0001:00015620       ??__F?ANALYSIS_TYPE_CLADE_PROFILES_VALUE@Metaphlan2WorkerFactory@LocalWorkflow@U2@@2VQString@@B@@YAXXZ 10016620 f   Metaphlan2WorkerFactory.obj
 0001:00015630       ??__F?ANALYSIS_TYPE_MARKER_AB_TABLE_TEXT@Metaphlan2WorkerFactory@LocalWorkflow@U2@@2VQString@@B@@YAXXZ 10016630 f   Metaphlan2WorkerFactory.obj
 0001:00015640       ??__F?ANALYSIS_TYPE_MARKER_AB_TABLE_VALUE@Metaphlan2WorkerFactory@LocalWorkflow@U2@@2VQString@@B@@YAXXZ 10016640 f   Metaphlan2WorkerFactory.obj
 0001:00015650       ??__F?ANALYSIS_TYPE_MARKER_PRES_TABLE_TEXT@Metaphlan2WorkerFactory@LocalWorkflow@U2@@2VQString@@B@@YAXXZ 10016650 f   Metaphlan2WorkerFactory.obj
 0001:00015660       ??__F?ANALYSIS_TYPE_MARKER_PRES_TABLE_VALUE@Metaphlan2WorkerFactory@LocalWorkflow@U2@@2VQString@@B@@YAXXZ 10016660 f   Metaphlan2WorkerFactory.obj
 0001:00015670       ??__F?ANALYSIS_TYPE_READS_MAP_TEXT@Metaphlan2WorkerFactory@LocalWorkflow@U2@@2VQString@@B@@YAXXZ 10016670 f   Metaphlan2WorkerFactory.obj
 0001:00015680       ??__F?ANALYSIS_TYPE_READS_MAP_VALUE@Metaphlan2WorkerFactory@LocalWorkflow@U2@@2VQString@@B@@YAXXZ 10016680 f   Metaphlan2WorkerFactory.obj
 0001:00015690       ??__F?ANALYSIS_TYPE_REL_AB_TEXT@Metaphlan2WorkerFactory@LocalWorkflow@U2@@2VQString@@B@@YAXXZ 10016690 f   Metaphlan2WorkerFactory.obj
 0001:000156a0       ??__F?ANALYSIS_TYPE_REL_AB_VALUE@Metaphlan2WorkerFactory@LocalWorkflow@U2@@2VQString@@B@@YAXXZ 100166a0 f   Metaphlan2WorkerFactory.obj
 0001:000156b0       ??__F?ANALYSIS_TYPE_REL_AB_W_READ_STATS_TEXT@Metaphlan2WorkerFactory@LocalWorkflow@U2@@2VQString@@B@@YAXXZ 100166b0 f   Metaphlan2WorkerFactory.obj
 0001:000156c0       ??__F?ANALYSIS_TYPE_REL_AB_W_READ_STATS_VALUE@Metaphlan2WorkerFactory@LocalWorkflow@U2@@2VQString@@B@@YAXXZ 100166c0 f   Metaphlan2WorkerFactory.obj
 0001:000156d0       ??__F?BOWTIE2_OUTPUT_URL@Metaphlan2WorkerFactory@LocalWorkflow@U2@@2VQString@@B@@YAXXZ 100166d0 f   Metaphlan2WorkerFactory.obj
 0001:000156e0       ??__F?DB_URL@Metaphlan2WorkerFactory@LocalWorkflow@U2@@2VQString@@B@@YAXXZ 100166e0 f   Metaphlan2WorkerFactory.obj
 0001:000156f0       ??__F?INPUT_PORT_ID@Metaphlan2WorkerFactory@LocalWorkflow@U2@@2VQString@@B@@YAXXZ 100166f0 f   Metaphlan2WorkerFactory.obj
 0001:00015700       ??__F?INPUT_SLOT@Metaphlan2WorkerFactory@LocalWorkflow@U2@@2VQString@@B@@YAXXZ 10016700 f   Metaphlan2WorkerFactory.obj
 0001:00015710       ??__F?NORMALIZE@Metaphlan2WorkerFactory@LocalWorkflow@U2@@2VQString@@B@@YAXXZ 10016710 f   Metaphlan2WorkerFactory.obj
 0001:00015720       ??__F?NOT_SKIP_NORMILIZE_BY_SIZE@Metaphlan2WorkerFactory@LocalWorkflow@U2@@2VQString@@B@@YAXXZ 10016720 f   Metaphlan2WorkerFactory.obj
 0001:00015730       ??__F?NUM_THREADS@Metaphlan2WorkerFactory@LocalWorkflow@U2@@2VQString@@B@@YAXXZ 10016730 f   Metaphlan2WorkerFactory.obj
 0001:00015740       ??__F?OUTPUT_URL@Metaphlan2WorkerFactory@LocalWorkflow@U2@@2VQString@@B@@YAXXZ 10016740 f   Metaphlan2WorkerFactory.obj
 0001:00015750       ??__F?PAIRED_END@Metaphlan2WorkerFactory@LocalWorkflow@U2@@2VQString@@B@@YAXXZ 10016750 f   Metaphlan2WorkerFactory.obj
 0001:00015760       ??__F?PAIRED_END_TEXT@Metaphlan2WorkerFactory@LocalWorkflow@U2@@2VQString@@B@@YAXXZ 10016760 f   Metaphlan2WorkerFactory.obj
 0001:00015770       ??__F?PAIRED_INPUT_SLOT@Metaphlan2WorkerFactory@LocalWorkflow@U2@@2VQString@@B@@YAXXZ 10016770 f   Metaphlan2WorkerFactory.obj
 0001:00015780       ??__F?PRESENCE_THRESHOLD@Metaphlan2WorkerFactory@LocalWorkflow@U2@@2VQString@@B@@YAXXZ 10016780 f   Metaphlan2WorkerFactory.obj
 0001:00015790       ??__F?SEQUENCING_READS@Metaphlan2WorkerFactory@LocalWorkflow@U2@@2VQString@@B@@YAXXZ 10016790 f   Metaphlan2WorkerFactory.obj
 0001:000157a0       ??__F?SINGLE_END@Metaphlan2WorkerFactory@LocalWorkflow@U2@@2VQString@@B@@YAXXZ 100167a0 f   Metaphlan2WorkerFactory.obj
 0001:000157b0       ??__F?SINGLE_END_TEXT@Metaphlan2WorkerFactory@LocalWorkflow@U2@@2VQString@@B@@YAXXZ 100167b0 f   Metaphlan2WorkerFactory.obj
 0001:000157c0       ??__F?SKIP_NORMILIZE_BY_SIZE@Metaphlan2WorkerFactory@LocalWorkflow@U2@@2VQString@@B@@YAXXZ 100167c0 f   Metaphlan2WorkerFactory.obj
 0001:000157d0       ??__F?TAX_LEVEL@Metaphlan2WorkerFactory@LocalWorkflow@U2@@2VQString@@B@@YAXXZ 100167d0 f   Metaphlan2WorkerFactory.obj
 0001:000157e0       ??__F?TAX_LEVEL_ALL_TEXT@Metaphlan2WorkerFactory@LocalWorkflow@U2@@2VQString@@B@@YAXXZ 100167e0 f   Metaphlan2WorkerFactory.obj
 0001:000157f0       ??__F?TAX_LEVEL_ALL_VALUE@Metaphlan2WorkerFactory@LocalWorkflow@U2@@2VQString@@B@@YAXXZ 100167f0 f   Metaphlan2WorkerFactory.obj
 0001:00015800       ??__F?TAX_LEVEL_CLASSES_TEXT@Metaphlan2WorkerFactory@LocalWorkflow@U2@@2VQString@@B@@YAXXZ 10016800 f   Metaphlan2WorkerFactory.obj
 0001:00015810       ??__F?TAX_LEVEL_CLASSES_VALUE@Metaphlan2WorkerFactory@LocalWorkflow@U2@@2VQString@@B@@YAXXZ 10016810 f   Metaphlan2WorkerFactory.obj
 0001:00015820       ??__F?TAX_LEVEL_FAMILIES_TEXT@Metaphlan2WorkerFactory@LocalWorkflow@U2@@2VQString@@B@@YAXXZ 10016820 f   Metaphlan2WorkerFactory.obj
 0001:00015830       ??__F?TAX_LEVEL_FAMILIES_VALUE@Metaphlan2WorkerFactory@LocalWorkflow@U2@@2VQString@@B@@YAXXZ 10016830 f   Metaphlan2WorkerFactory.obj
 0001:00015840       ??__F?TAX_LEVEL_GENERA_TEXT@Metaphlan2WorkerFactory@LocalWorkflow@U2@@2VQString@@B@@YAXXZ 10016840 f   Metaphlan2WorkerFactory.obj
 0001:00015850       ??__F?TAX_LEVEL_GENERA_VALUE@Metaphlan2WorkerFactory@LocalWorkflow@U2@@2VQString@@B@@YAXXZ 10016850 f   Metaphlan2WorkerFactory.obj
 0001:00015860       ??__F?TAX_LEVEL_KINGDOMS_TEXT@Metaphlan2WorkerFactory@LocalWorkflow@U2@@2VQString@@B@@YAXXZ 10016860 f   Metaphlan2WorkerFactory.obj
 0001:00015870       ??__F?TAX_LEVEL_KINGDOMS_VALUE@Metaphlan2WorkerFactory@LocalWorkflow@U2@@2VQString@@B@@YAXXZ 10016870 f   Metaphlan2WorkerFactory.obj
 0001:00015880       ??__F?TAX_LEVEL_ORDERS_TEXT@Metaphlan2WorkerFactory@LocalWorkflow@U2@@2VQString@@B@@YAXXZ 10016880 f   Metaphlan2WorkerFactory.obj
 0001:00015890       ??__F?TAX_LEVEL_ORDERS_VALUE@Metaphlan2WorkerFactory@LocalWorkflow@U2@@2VQString@@B@@YAXXZ 10016890 f   Metaphlan2WorkerFactory.obj
 0001:000158a0       ??__F?TAX_LEVEL_PHYLA_TEXT@Metaphlan2WorkerFactory@LocalWorkflow@U2@@2VQString@@B@@YAXXZ 100168a0 f   Metaphlan2WorkerFactory.obj
 0001:000158b0       ??__F?TAX_LEVEL_PHYLA_VALUE@Metaphlan2WorkerFactory@LocalWorkflow@U2@@2VQString@@B@@YAXXZ 100168b0 f   Metaphlan2WorkerFactory.obj
 0001:000158c0       ??__F?TAX_LEVEL_SPECIES_TEXT@Metaphlan2WorkerFactory@LocalWorkflow@U2@@2VQString@@B@@YAXXZ 100168c0 f   Metaphlan2WorkerFactory.obj
 0001:000158d0       ??__F?TAX_LEVEL_SPECIES_VALUE@Metaphlan2WorkerFactory@LocalWorkflow@U2@@2VQString@@B@@YAXXZ 100168d0 f   Metaphlan2WorkerFactory.obj
 0001:000158e0       ??__F?_Generic_object@?$_Error_objects@H@std@@2V_Generic_error_category@2@A@@YAXXZ 100168e0 f   Metaphlan2WorkerFactory.obj
 0001:000158f0       ??__F?_Iostream_object@?$_Error_objects@H@std@@2V_Iostream_error_category@2@A@@YAXXZ 100168f0 f   Metaphlan2WorkerFactory.obj
 0001:00015900       ??__F?_System_object@?$_Error_objects@H@std@@2V_System_error_category@2@A@@YAXXZ 10016900 f   Metaphlan2WorkerFactory.obj
 0001:00015910       ??__FalgoLog@U2@@YAXXZ     10016910 f   Metaphlan2WorkerFactory.obj
 0001:00015920       ??__FcmdLog@U2@@YAXXZ      10016920 f   Metaphlan2WorkerFactory.obj
 0001:00015930       ??__FcoreLog@U2@@YAXXZ     10016930 f   Metaphlan2WorkerFactory.obj
 0001:00015940       ??__FioLog@U2@@YAXXZ       10016940 f   Metaphlan2WorkerFactory.obj
 0001:00015950       ??__FperfLog@U2@@YAXXZ     10016950 f   Metaphlan2WorkerFactory.obj
 0001:00015960       ??__FscriptLog@U2@@YAXXZ   10016960 f   Metaphlan2WorkerFactory.obj
 0001:00015970       ??__FtaskLog@U2@@YAXXZ     10016970 f   Metaphlan2WorkerFactory.obj
 0001:00015980       ??__FuiLog@U2@@YAXXZ       10016980 f   Metaphlan2WorkerFactory.obj
 0001:00015990       ??__FuserActLog@U2@@YAXXZ  10016990 f   Metaphlan2WorkerFactory.obj
 0001:000159a0       ??__F?_Generic_object@?$_Error_objects@H@std@@2V_Generic_error_category@2@A@@YAXXZ 100169a0 f   moc_Metaphlan2Prompter.obj
 0001:000159b0       ??__F?_Iostream_object@?$_Error_objects@H@std@@2V_Iostream_error_category@2@A@@YAXXZ 100169b0 f   moc_Metaphlan2Prompter.obj
 0001:000159c0       ??__F?_System_object@?$_Error_objects@H@std@@2V_System_error_category@2@A@@YAXXZ 100169c0 f   moc_Metaphlan2Prompter.obj
 0001:000159d0       ??__FalgoLog@U2@@YAXXZ     100169d0 f   moc_Metaphlan2Prompter.obj
 0001:000159e0       ??__FcmdLog@U2@@YAXXZ      100169e0 f   moc_Metaphlan2Prompter.obj
 0001:000159f0       ??__FcoreLog@U2@@YAXXZ     100169f0 f   moc_Metaphlan2Prompter.obj
 0001:00015a00       ??__FioLog@U2@@YAXXZ       10016a00 f   moc_Metaphlan2Prompter.obj
 0001:00015a10       ??__FperfLog@U2@@YAXXZ     10016a10 f   moc_Metaphlan2Prompter.obj
 0001:00015a20       ??__FscriptLog@U2@@YAXXZ   10016a20 f   moc_Metaphlan2Prompter.obj
 0001:00015a30       ??__FtaskLog@U2@@YAXXZ     10016a30 f   moc_Metaphlan2Prompter.obj
 0001:00015a40       ??__FuiLog@U2@@YAXXZ       10016a40 f   moc_Metaphlan2Prompter.obj
 0001:00015a50       ??__FuserActLog@U2@@YAXXZ  10016a50 f   moc_Metaphlan2Prompter.obj
 0001:00015a60       ??__F?_Generic_object@?$_Error_objects@H@std@@2V_Generic_error_category@2@A@@YAXXZ 10016a60 f   moc_Metaphlan2Support.obj
 0001:00015a70       ??__F?_Iostream_object@?$_Error_objects@H@std@@2V_Iostream_error_category@2@A@@YAXXZ 10016a70 f   moc_Metaphlan2Support.obj
 0001:00015a80       ??__F?_System_object@?$_Error_objects@H@std@@2V_System_error_category@2@A@@YAXXZ 10016a80 f   moc_Metaphlan2Support.obj
 0001:00015a90       ??__F?_Generic_object@?$_Error_objects@H@std@@2V_Generic_error_category@2@A@@YAXXZ 10016a90 f   moc_Metaphlan2SupportPlugin.obj
 0001:00015aa0       ??__F?_Iostream_object@?$_Error_objects@H@std@@2V_Iostream_error_category@2@A@@YAXXZ 10016aa0 f   moc_Metaphlan2SupportPlugin.obj
 0001:00015ab0       ??__F?_System_object@?$_Error_objects@H@std@@2V_System_error_category@2@A@@YAXXZ 10016ab0 f   moc_Metaphlan2SupportPlugin.obj
 0001:00015ac0       ??__F?_Generic_object@?$_Error_objects@H@std@@2V_Generic_error_category@2@A@@YAXXZ 10016ac0 f   moc_Metaphlan2Task.obj
 0001:00015ad0       ??__F?_Iostream_object@?$_Error_objects@H@std@@2V_Iostream_error_category@2@A@@YAXXZ 10016ad0 f   moc_Metaphlan2Task.obj
 0001:00015ae0       ??__F?_System_object@?$_Error_objects@H@std@@2V_System_error_category@2@A@@YAXXZ 10016ae0 f   moc_Metaphlan2Task.obj
 0001:00015af0       ??__FalgoLog@U2@@YAXXZ     10016af0 f   moc_Metaphlan2Task.obj
 0001:00015b00       ??__FcmdLog@U2@@YAXXZ      10016b00 f   moc_Metaphlan2Task.obj
 0001:00015b10       ??__FcoreLog@U2@@YAXXZ     10016b10 f   moc_Metaphlan2Task.obj
 0001:00015b20       ??__FioLog@U2@@YAXXZ       10016b20 f   moc_Metaphlan2Task.obj
 0001:00015b30       ??__FperfLog@U2@@YAXXZ     10016b30 f   moc_Metaphlan2Task.obj
 0001:00015b40       ??__FscriptLog@U2@@YAXXZ   10016b40 f   moc_Metaphlan2Task.obj
 0001:00015b50       ??__FtaskLog@U2@@YAXXZ     10016b50 f   moc_Metaphlan2Task.obj
 0001:00015b60       ??__FuiLog@U2@@YAXXZ       10016b60 f   moc_Metaphlan2Task.obj
 0001:00015b70       ??__FuserActLog@U2@@YAXXZ  10016b70 f   moc_Metaphlan2Task.obj
 0001:00015b80       ??__F?_Generic_object@?$_Error_objects@H@std@@2V_Generic_error_category@2@A@@YAXXZ 10016b80 f   moc_Metaphlan2Worker.obj
 0001:00015b90       ??__F?_Iostream_object@?$_Error_objects@H@std@@2V_Iostream_error_category@2@A@@YAXXZ 10016b90 f   moc_Metaphlan2Worker.obj
 0001:00015ba0       ??__F?_System_object@?$_Error_objects@H@std@@2V_System_error_category@2@A@@YAXXZ 10016ba0 f   moc_Metaphlan2Worker.obj
 0001:00015bb0       ??__FalgoLog@U2@@YAXXZ     10016bb0 f   moc_Metaphlan2Worker.obj
 0001:00015bc0       ??__FcmdLog@U2@@YAXXZ      10016bc0 f   moc_Metaphlan2Worker.obj
 0001:00015bd0       ??__FcoreLog@U2@@YAXXZ     10016bd0 f   moc_Metaphlan2Worker.obj
 0001:00015be0       ??__FioLog@U2@@YAXXZ       10016be0 f   moc_Metaphlan2Worker.obj
 0001:00015bf0       ??__FperfLog@U2@@YAXXZ     10016bf0 f   moc_Metaphlan2Worker.obj
 0001:00015c00       ??__FscriptLog@U2@@YAXXZ   10016c00 f   moc_Metaphlan2Worker.obj
 0001:00015c10       ??__FtaskLog@U2@@YAXXZ     10016c10 f   moc_Metaphlan2Worker.obj
 0001:00015c20       ??__FuiLog@U2@@YAXXZ       10016c20 f   moc_Metaphlan2Worker.obj
 0001:00015c30       ??__FuserActLog@U2@@YAXXZ  10016c30 f   moc_Metaphlan2Worker.obj
 0002:00000748       _algoLog$initializer$      10017748     Metaphlan2LogParser.obj
 0002:0000074c       _cmdLog$initializer$       1001774c     Metaphlan2LogParser.obj
 0002:00000750       _coreLog$initializer$      10017750     Metaphlan2LogParser.obj
 0002:00000754       _ioLog$initializer$        10017754     Metaphlan2LogParser.obj
 0002:00000758       _perfLog$initializer$      10017758     Metaphlan2LogParser.obj
 0002:0000075c       _scriptLog$initializer$    1001775c     Metaphlan2LogParser.obj
 0002:00000760       _taskLog$initializer$      10017760     Metaphlan2LogParser.obj
 0002:00000764       _uiLog$initializer$        10017764     Metaphlan2LogParser.obj
 0002:00000768       _userActLog$initializer$   10017768     Metaphlan2LogParser.obj
 0002:0000076c       ?wellKnownErrors$initializer$@Metaphlan2LogParser@U2@@0P6AXXZA 1001776c     Metaphlan2LogParser.obj
 0002:00000770       ?_Generic_object$initializer$@?$_Error_objects@H@std@@2P6AXXZA 10017770     Metaphlan2LogParser.obj
 0002:00000774       ?_Iostream_object$initializer$@?$_Error_objects@H@std@@2P6AXXZA 10017774     Metaphlan2LogParser.obj
 0002:00000778       ?_System_object$initializer$@?$_Error_objects@H@std@@2P6AXXZA 10017778     Metaphlan2LogParser.obj
 0002:0000077c       _algoLog$initializer$      1001777c     Metaphlan2Prompter.obj
 0002:00000780       _cmdLog$initializer$       10017780     Metaphlan2Prompter.obj
 0002:00000784       _coreLog$initializer$      10017784     Metaphlan2Prompter.obj
 0002:00000788       _ioLog$initializer$        10017788     Metaphlan2Prompter.obj
 0002:0000078c       _perfLog$initializer$      1001778c     Metaphlan2Prompter.obj
 0002:00000790       _scriptLog$initializer$    10017790     Metaphlan2Prompter.obj
 0002:00000794       _taskLog$initializer$      10017794     Metaphlan2Prompter.obj
 0002:00000798       _uiLog$initializer$        10017798     Metaphlan2Prompter.obj
 0002:0000079c       _userActLog$initializer$   1001779c     Metaphlan2Prompter.obj
 0002:000007a0       _algoLog$initializer$      100177a0     Metaphlan2Support.obj
 0002:000007a4       _cmdLog$initializer$       100177a4     Metaphlan2Support.obj
 0002:000007a8       _coreLog$initializer$      100177a8     Metaphlan2Support.obj
 0002:000007ac       _ioLog$initializer$        100177ac     Metaphlan2Support.obj
 0002:000007b0       _perfLog$initializer$      100177b0     Metaphlan2Support.obj
 0002:000007b4       _scriptLog$initializer$    100177b4     Metaphlan2Support.obj
 0002:000007b8       _taskLog$initializer$      100177b8     Metaphlan2Support.obj
 0002:000007bc       _uiLog$initializer$        100177bc     Metaphlan2Support.obj
 0002:000007c0       _userActLog$initializer$   100177c0     Metaphlan2Support.obj
 0002:000007c4       ?TOOL_NAME$initializer$@Metaphlan2Support@U2@@2P6AXXZA 100177c4     Metaphlan2Support.obj
 0002:000007c8       ?UTIL_SCRIPT$initializer$@Metaphlan2Support@U2@@2P6AXXZA 100177c8     Metaphlan2Support.obj
 0002:000007cc       ?ET_BOWTIE_2_ALIGNER$initializer$@Metaphlan2Support@U2@@2P6AXXZA 100177cc     Metaphlan2Support.obj
 0002:000007d0       ?ET_PYTHON$initializer$@Metaphlan2Support@U2@@2P6AXXZA 100177d0     Metaphlan2Support.obj
 0002:000007d4       ?ET_PYTHON_BIO$initializer$@Metaphlan2Support@U2@@2P6AXXZA 100177d4     Metaphlan2Support.obj
 0002:000007d8       ?ET_PYTHON_NUMPY$initializer$@Metaphlan2Support@U2@@2P6AXXZA 100177d8     Metaphlan2Support.obj
 0002:000007dc       _algoLog$initializer$      100177dc     Metaphlan2SupportPlugin.obj
 0002:000007e0       _cmdLog$initializer$       100177e0     Metaphlan2SupportPlugin.obj
 0002:000007e4       _coreLog$initializer$      100177e4     Metaphlan2SupportPlugin.obj
 0002:000007e8       _ioLog$initializer$        100177e8     Metaphlan2SupportPlugin.obj
 0002:000007ec       _perfLog$initializer$      100177ec     Metaphlan2SupportPlugin.obj
 0002:000007f0       _scriptLog$initializer$    100177f0     Metaphlan2SupportPlugin.obj
 0002:000007f4       _taskLog$initializer$      100177f4     Metaphlan2SupportPlugin.obj
 0002:000007f8       _uiLog$initializer$        100177f8     Metaphlan2SupportPlugin.obj
 0002:000007fc       _userActLog$initializer$   100177fc     Metaphlan2SupportPlugin.obj
 0002:00000800       ?PLUGIN_NAME$initializer$@MetaphlanSupportPlugin@U2@@2P6AXXZA 10017800     Metaphlan2SupportPlugin.obj
 0002:00000804       ?PLUGIN_DESCRIPRION$initializer$@MetaphlanSupportPlugin@U2@@2P6AXXZA 10017804     Metaphlan2SupportPlugin.obj
 0002:00000808       _algoLog$initializer$      10017808     Metaphlan2Task.obj
 0002:0000080c       _cmdLog$initializer$       1001780c     Metaphlan2Task.obj
 0002:00000810       _coreLog$initializer$      10017810     Metaphlan2Task.obj
 0002:00000814       _ioLog$initializer$        10017814     Metaphlan2Task.obj
 0002:00000818       _perfLog$initializer$      10017818     Metaphlan2Task.obj
 0002:0000081c       _scriptLog$initializer$    1001781c     Metaphlan2Task.obj
 0002:00000820       _taskLog$initializer$      10017820     Metaphlan2Task.obj
 0002:00000824       _uiLog$initializer$        10017824     Metaphlan2Task.obj
 0002:00000828       _userActLog$initializer$   10017828     Metaphlan2Task.obj
 0002:0000082c       _algoLog$initializer$      1001782c     Metaphlan2Validator.obj
 0002:00000830       _cmdLog$initializer$       10017830     Metaphlan2Validator.obj
 0002:00000834       _coreLog$initializer$      10017834     Metaphlan2Validator.obj
 0002:00000838       _ioLog$initializer$        10017838     Metaphlan2Validator.obj
 0002:0000083c       _perfLog$initializer$      1001783c     Metaphlan2Validator.obj
 0002:00000840       _scriptLog$initializer$    10017840     Metaphlan2Validator.obj
 0002:00000844       _taskLog$initializer$      10017844     Metaphlan2Validator.obj
 0002:00000848       _uiLog$initializer$        10017848     Metaphlan2Validator.obj
 0002:0000084c       _userActLog$initializer$   1001784c     Metaphlan2Validator.obj
 0002:00000850       _algoLog$initializer$      10017850     Metaphlan2Worker.obj
 0002:00000854       _cmdLog$initializer$       10017854     Metaphlan2Worker.obj
 0002:00000858       _coreLog$initializer$      10017858     Metaphlan2Worker.obj
 0002:0000085c       _ioLog$initializer$        1001785c     Metaphlan2Worker.obj
 0002:00000860       _perfLog$initializer$      10017860     Metaphlan2Worker.obj
 0002:00000864       _scriptLog$initializer$    10017864     Metaphlan2Worker.obj
 0002:00000868       _taskLog$initializer$      10017868     Metaphlan2Worker.obj
 0002:0000086c       _uiLog$initializer$        1001786c     Metaphlan2Worker.obj
 0002:00000870       _userActLog$initializer$   10017870     Metaphlan2Worker.obj
 0002:00000874       ?METAPHLAN2_ROOT_DIR$initializer$@Metaphlan2Worker@LocalWorkflow@U2@@0P6AXXZA 10017874     Metaphlan2Worker.obj
 0002:00000878       ?BOWTIE2OUT_DIR$initializer$@Metaphlan2Worker@LocalWorkflow@U2@@0P6AXXZA 10017878     Metaphlan2Worker.obj
 0002:0000087c       ?BOWTIE2OUT_SUFFIX$initializer$@Metaphlan2Worker@LocalWorkflow@U2@@0P6AXXZA 1001787c     Metaphlan2Worker.obj
 0002:00000880       ?PROFILE_DIR$initializer$@Metaphlan2Worker@LocalWorkflow@U2@@0P6AXXZA 10017880     Metaphlan2Worker.obj
 0002:00000884       ?PROFILE_SUFFIX$initializer$@Metaphlan2Worker@LocalWorkflow@U2@@0P6AXXZA 10017884     Metaphlan2Worker.obj
 0002:00000888       _algoLog$initializer$      10017888     Metaphlan2WorkerFactory.obj
 0002:0000088c       _cmdLog$initializer$       1001788c     Metaphlan2WorkerFactory.obj
 0002:00000890       _coreLog$initializer$      10017890     Metaphlan2WorkerFactory.obj
 0002:00000894       _ioLog$initializer$        10017894     Metaphlan2WorkerFactory.obj
 0002:00000898       _perfLog$initializer$      10017898     Metaphlan2WorkerFactory.obj
 0002:0000089c       _scriptLog$initializer$    1001789c     Metaphlan2WorkerFactory.obj
 0002:000008a0       _taskLog$initializer$      100178a0     Metaphlan2WorkerFactory.obj
 0002:000008a4       _uiLog$initializer$        100178a4     Metaphlan2WorkerFactory.obj
 0002:000008a8       _userActLog$initializer$   100178a8     Metaphlan2WorkerFactory.obj
 0002:000008ac       ?ACTOR_ID$initializer$@Metaphlan2WorkerFactory@LocalWorkflow@U2@@2P6AXXZA 100178ac     Metaphlan2WorkerFactory.obj
 0002:000008b0       ?INPUT_PORT_ID$initializer$@Metaphlan2WorkerFactory@LocalWorkflow@U2@@2P6AXXZA 100178b0     Metaphlan2WorkerFactory.obj
 0002:000008b4       ?INPUT_SLOT$initializer$@Metaphlan2WorkerFactory@LocalWorkflow@U2@@2P6AXXZA 100178b4     Metaphlan2WorkerFactory.obj
 0002:000008b8       ?PAIRED_INPUT_SLOT$initializer$@Metaphlan2WorkerFactory@LocalWorkflow@U2@@2P6AXXZA 100178b8     Metaphlan2WorkerFactory.obj
 0002:000008bc       ?SEQUENCING_READS$initializer$@Metaphlan2WorkerFactory@LocalWorkflow@U2@@2P6AXXZA 100178bc     Metaphlan2WorkerFactory.obj
 0002:000008c0       ?DB_URL$initializer$@Metaphlan2WorkerFactory@LocalWorkflow@U2@@2P6AXXZA 100178c0     Metaphlan2WorkerFactory.obj
 0002:000008c4       ?NUM_THREADS$initializer$@Metaphlan2WorkerFactory@LocalWorkflow@U2@@2P6AXXZA 100178c4     Metaphlan2WorkerFactory.obj
 0002:000008c8       ?ANALYSIS_TYPE$initializer$@Metaphlan2WorkerFactory@LocalWorkflow@U2@@2P6AXXZA 100178c8     Metaphlan2WorkerFactory.obj
 0002:000008cc       ?TAX_LEVEL$initializer$@Metaphlan2WorkerFactory@LocalWorkflow@U2@@2P6AXXZA 100178cc     Metaphlan2WorkerFactory.obj
 0002:000008d0       ?NORMALIZE$initializer$@Metaphlan2WorkerFactory@LocalWorkflow@U2@@2P6AXXZA 100178d0     Metaphlan2WorkerFactory.obj
 0002:000008d4       ?PRESENCE_THRESHOLD$initializer$@Metaphlan2WorkerFactory@LocalWorkflow@U2@@2P6AXXZA 100178d4     Metaphlan2WorkerFactory.obj
 0002:000008d8       ?BOWTIE2_OUTPUT_URL$initializer$@Metaphlan2WorkerFactory@LocalWorkflow@U2@@2P6AXXZA 100178d8     Metaphlan2WorkerFactory.obj
 0002:000008dc       ?OUTPUT_URL$initializer$@Metaphlan2WorkerFactory@LocalWorkflow@U2@@2P6AXXZA 100178dc     Metaphlan2WorkerFactory.obj
 0002:000008e0       ?SINGLE_END_TEXT$initializer$@Metaphlan2WorkerFactory@LocalWorkflow@U2@@2P6AXXZA 100178e0     Metaphlan2WorkerFactory.obj
 0002:000008e4       ?PAIRED_END_TEXT$initializer$@Metaphlan2WorkerFactory@LocalWorkflow@U2@@2P6AXXZA 100178e4     Metaphlan2WorkerFactory.obj
 0002:000008e8       ?ANALYSIS_TYPE_REL_AB_TEXT$initializer$@Metaphlan2WorkerFactory@LocalWorkflow@U2@@2P6AXXZA 100178e8     Metaphlan2WorkerFactory.obj
 0002:000008ec       ?ANALYSIS_TYPE_REL_AB_W_READ_STATS_TEXT$initializer$@Metaphlan2WorkerFactory@LocalWorkflow@U2@@2P6AXXZA 100178ec     Metaphlan2WorkerFactory.obj
 0002:000008f0       ?ANALYSIS_TYPE_READS_MAP_TEXT$initializer$@Metaphlan2WorkerFactory@LocalWorkflow@U2@@2P6AXXZA 100178f0     Metaphlan2WorkerFactory.obj
 0002:000008f4       ?ANALYSIS_TYPE_CLADE_PROFILES_TEXT$initializer$@Metaphlan2WorkerFactory@LocalWorkflow@U2@@2P6AXXZA 100178f4     Metaphlan2WorkerFactory.obj
 0002:000008f8       ?ANALYSIS_TYPE_MARKER_AB_TABLE_TEXT$initializer$@Metaphlan2WorkerFactory@LocalWorkflow@U2@@2P6AXXZA 100178f8     Metaphlan2WorkerFactory.obj
 0002:000008fc       ?ANALYSIS_TYPE_MARKER_PRES_TABLE_TEXT$initializer$@Metaphlan2WorkerFactory@LocalWorkflow@U2@@2P6AXXZA 100178fc     Metaphlan2WorkerFactory.obj
 0002:00000900       ?ANALYSIS_TYPE_REL_AB_VALUE$initializer$@Metaphlan2WorkerFactory@LocalWorkflow@U2@@2P6AXXZA 10017900     Metaphlan2WorkerFactory.obj
 0002:00000904       ?ANALYSIS_TYPE_REL_AB_W_READ_STATS_VALUE$initializer$@Metaphlan2WorkerFactory@LocalWorkflow@U2@@2P6AXXZA 10017904     Metaphlan2WorkerFactory.obj
 0002:00000908       ?ANALYSIS_TYPE_READS_MAP_VALUE$initializer$@Metaphlan2WorkerFactory@LocalWorkflow@U2@@2P6AXXZA 10017908     Metaphlan2WorkerFactory.obj
 0002:0000090c       ?ANALYSIS_TYPE_CLADE_PROFILES_VALUE$initializer$@Metaphlan2WorkerFactory@LocalWorkflow@U2@@2P6AXXZA 1001790c     Metaphlan2WorkerFactory.obj
 0002:00000910       ?ANALYSIS_TYPE_MARKER_AB_TABLE_VALUE$initializer$@Metaphlan2WorkerFactory@LocalWorkflow@U2@@2P6AXXZA 10017910     Metaphlan2WorkerFactory.obj
 0002:00000914       ?ANALYSIS_TYPE_MARKER_PRES_TABLE_VALUE$initializer$@Metaphlan2WorkerFactory@LocalWorkflow@U2@@2P6AXXZA 10017914     Metaphlan2WorkerFactory.obj
 0002:00000918       ?TAX_LEVEL_ALL_TEXT$initializer$@Metaphlan2WorkerFactory@LocalWorkflow@U2@@2P6AXXZA 10017918     Metaphlan2WorkerFactory.obj
 0002:0000091c       ?TAX_LEVEL_KINGDOMS_TEXT$initializer$@Metaphlan2WorkerFactory@LocalWorkflow@U2@@2P6AXXZA 1001791c     Metaphlan2WorkerFactory.obj
 0002:00000920       ?TAX_LEVEL_PHYLA_TEXT$initializer$@Metaphlan2WorkerFactory@LocalWorkflow@U2@@2P6AXXZA 10017920     Metaphlan2WorkerFactory.obj
 0002:00000924       ?TAX_LEVEL_CLASSES_TEXT$initializer$@Metaphlan2WorkerFactory@LocalWorkflow@U2@@2P6AXXZA 10017924     Metaphlan2WorkerFactory.obj
 0002:00000928       ?TAX_LEVEL_ORDERS_TEXT$initializer$@Metaphlan2WorkerFactory@LocalWorkflow@U2@@2P6AXXZA 10017928     Metaphlan2WorkerFactory.obj
 0002:0000092c       ?TAX_LEVEL_FAMILIES_TEXT$initializer$@Metaphlan2WorkerFactory@LocalWorkflow@U2@@2P6AXXZA 1001792c     Metaphlan2WorkerFactory.obj
 0002:00000930       ?TAX_LEVEL_GENERA_TEXT$initializer$@Metaphlan2WorkerFactory@LocalWorkflow@U2@@2P6AXXZA 10017930     Metaphlan2WorkerFactory.obj
 0002:00000934       ?TAX_LEVEL_SPECIES_TEXT$initializer$@Metaphlan2WorkerFactory@LocalWorkflow@U2@@2P6AXXZA 10017934     Metaphlan2WorkerFactory.obj
 0002:00000938       ?TAX_LEVEL_ALL_VALUE$initializer$@Metaphlan2WorkerFactory@LocalWorkflow@U2@@2P6AXXZA 10017938     Metaphlan2WorkerFactory.obj
 0002:0000093c       ?TAX_LEVEL_KINGDOMS_VALUE$initializer$@Metaphlan2WorkerFactory@LocalWorkflow@U2@@2P6AXXZA 1001793c     Metaphlan2WorkerFactory.obj
 0002:00000940       ?TAX_LEVEL_PHYLA_VALUE$initializer$@Metaphlan2WorkerFactory@LocalWorkflow@U2@@2P6AXXZA 10017940     Metaphlan2WorkerFactory.obj
 0002:00000944       ?TAX_LEVEL_CLASSES_VALUE$initializer$@Metaphlan2WorkerFactory@LocalWorkflow@U2@@2P6AXXZA 10017944     Metaphlan2WorkerFactory.obj
 0002:00000948       ?TAX_LEVEL_ORDERS_VALUE$initializer$@Metaphlan2WorkerFactory@LocalWorkflow@U2@@2P6AXXZA 10017948     Metaphlan2WorkerFactory.obj
 0002:0000094c       ?TAX_LEVEL_FAMILIES_VALUE$initializer$@Metaphlan2WorkerFactory@LocalWorkflow@U2@@2P6AXXZA 1001794c     Metaphlan2WorkerFactory.obj
 0002:00000950       ?TAX_LEVEL_GENERA_VALUE$initializer$@Metaphlan2WorkerFactory@LocalWorkflow@U2@@2P6AXXZA 10017950     Metaphlan2WorkerFactory.obj
 0002:00000954       ?TAX_LEVEL_SPECIES_VALUE$initializer$@Metaphlan2WorkerFactory@LocalWorkflow@U2@@2P6AXXZA 10017954     Metaphlan2WorkerFactory.obj
 0002:00000958       ?SKIP_NORMILIZE_BY_SIZE$initializer$@Metaphlan2WorkerFactory@LocalWorkflow@U2@@2P6AXXZA 10017958     Metaphlan2WorkerFactory.obj
 0002:0000095c       ?NOT_SKIP_NORMILIZE_BY_SIZE$initializer$@Metaphlan2WorkerFactory@LocalWorkflow@U2@@2P6AXXZA 1001795c     Metaphlan2WorkerFactory.obj
 0002:00000960       ?SINGLE_END$initializer$@Metaphlan2WorkerFactory@LocalWorkflow@U2@@2P6AXXZA 10017960     Metaphlan2WorkerFactory.obj
 0002:00000964       ?PAIRED_END$initializer$@Metaphlan2WorkerFactory@LocalWorkflow@U2@@2P6AXXZA 10017964     Metaphlan2WorkerFactory.obj
 0002:00000968       _algoLog$initializer$      10017968     moc_Metaphlan2Prompter.obj
 0002:0000096c       _cmdLog$initializer$       1001796c     moc_Metaphlan2Prompter.obj
 0002:00000970       _coreLog$initializer$      10017970     moc_Metaphlan2Prompter.obj
 0002:00000974       _ioLog$initializer$        10017974     moc_Metaphlan2Prompter.obj
 0002:00000978       _perfLog$initializer$      10017978     moc_Metaphlan2Prompter.obj
 0002:0000097c       _scriptLog$initializer$    1001797c     moc_Metaphlan2Prompter.obj
 0002:00000980       _taskLog$initializer$      10017980     moc_Metaphlan2Prompter.obj
 0002:00000984       _uiLog$initializer$        10017984     moc_Metaphlan2Prompter.obj
 0002:00000988       _userActLog$initializer$   10017988     moc_Metaphlan2Prompter.obj
 0002:0000098c       ?staticMetaObject$initializer$@Metaphlan2Prompter@LocalWorkflow@U2@@2P6AXXZA 1001798c     moc_Metaphlan2Prompter.obj
 0002:00000990       ?staticMetaObject$initializer$@Metaphlan2Support@U2@@2P6AXXZA 10017990     moc_Metaphlan2Support.obj
 0002:00000994       ?staticMetaObject$initializer$@MetaphlanSupportPlugin@U2@@2P6AXXZA 10017994     moc_Metaphlan2SupportPlugin.obj
 0002:00000998       _algoLog$initializer$      10017998     moc_Metaphlan2Task.obj
 0002:0000099c       _cmdLog$initializer$       1001799c     moc_Metaphlan2Task.obj
 0002:000009a0       _coreLog$initializer$      100179a0     moc_Metaphlan2Task.obj
 0002:000009a4       _ioLog$initializer$        100179a4     moc_Metaphlan2Task.obj
 0002:000009a8       _perfLog$initializer$      100179a8     moc_Metaphlan2Task.obj
 0002:000009ac       _scriptLog$initializer$    100179ac     moc_Metaphlan2Task.obj
 0002:000009b0       _taskLog$initializer$      100179b0     moc_Metaphlan2Task.obj
 0002:000009b4       _uiLog$initializer$        100179b4     moc_Metaphlan2Task.obj
 0002:000009b8       _userActLog$initializer$   100179b8     moc_Metaphlan2Task.obj
 0002:000009bc       ?staticMetaObject$initializer$@Metaphlan2ClassifyTask@U2@@2P6AXXZA 100179bc     moc_Metaphlan2Task.obj
 0002:000009c0       _algoLog$initializer$      100179c0     moc_Metaphlan2Worker.obj
 0002:000009c4       _cmdLog$initializer$       100179c4     moc_Metaphlan2Worker.obj
 0002:000009c8       _coreLog$initializer$      100179c8     moc_Metaphlan2Worker.obj
 0002:000009cc       _ioLog$initializer$        100179cc     moc_Metaphlan2Worker.obj
 0002:000009d0       _perfLog$initializer$      100179d0     moc_Metaphlan2Worker.obj
 0002:000009d4       _scriptLog$initializer$    100179d4     moc_Metaphlan2Worker.obj
 0002:000009d8       _taskLog$initializer$      100179d8     moc_Metaphlan2Worker.obj
 0002:000009dc       _uiLog$initializer$        100179dc     moc_Metaphlan2Worker.obj
 0002:000009e0       _userActLog$initializer$   100179e0     moc_Metaphlan2Worker.obj
 0002:000009e4       ?staticMetaObject$initializer$@Metaphlan2Worker@LocalWorkflow@U2@@2P6AXXZA 100179e4     moc_Metaphlan2Worker.obj
 0002:000009f0       _pcinit                    100179f0     MSVCRT:crtdll.obj
 0002:000009f4       _pinit                     100179f4     MSVCRT:atonexit.obj
 0002:00002b3c       _qt_meta_stringdata_U2__LocalWorkflow__Metaphlan2Prompter 10019b3c     moc_Metaphlan2Prompter.obj
 0002:00002b74       _qt_meta_data_U2__LocalWorkflow__Metaphlan2Prompter 10019b74     moc_Metaphlan2Prompter.obj
 0002:00002bb0       _qt_meta_stringdata_U2__Metaphlan2Support 10019bb0     moc_Metaphlan2Support.obj
 0002:00002bd8       _qt_meta_data_U2__Metaphlan2Support 10019bd8     moc_Metaphlan2Support.obj
 0002:00002c14       _qt_meta_stringdata_U2__MetaphlanSupportPlugin 10019c14     moc_Metaphlan2SupportPlugin.obj
 0002:00002c40       _qt_meta_data_U2__MetaphlanSupportPlugin 10019c40     moc_Metaphlan2SupportPlugin.obj
 0002:00002c7c       _qt_meta_stringdata_U2__Metaphlan2ClassifyTask 10019c7c     moc_Metaphlan2Task.obj
 0002:00002ca8       _qt_meta_data_U2__Metaphlan2ClassifyTask 10019ca8     moc_Metaphlan2Task.obj
 0002:00002ce8       _qt_meta_stringdata_U2__LocalWorkflow__Metaphlan2Worker 10019ce8     moc_Metaphlan2Worker.obj
 0002:00002d78       _qt_meta_data_U2__LocalWorkflow__Metaphlan2Worker 10019d78     moc_Metaphlan2Worker.obj
 0002:00002de4       _GS_ExceptionPointers      10019de4     MSVCRT:gs_report.obj
 0002:00004270       __catchsym$?_Copy@?$basic_string@DU?$char_traits@D@std@@V?$allocator@D@2@@std@@QAEXII@Z$5 1001b270     Metaphlan2LogParser.obj
 0002:00004280       __catchsym$?_Copy@?$basic_string@DU?$char_traits@D@std@@V?$allocator@D@2@@std@@QAEXII@Z$4 1001b280     Metaphlan2LogParser.obj
 0002:00004290       __unwindtable$?_Copy@?$basic_string@DU?$char_traits@D@std@@V?$allocator@D@2@@std@@QAEXII@Z 1001b290     Metaphlan2LogParser.obj
 0002:000042b0       __ehfuncinfo$?_Copy@?$basic_string@DU?$char_traits@D@std@@V?$allocator@D@2@@std@@QAEXII@Z 1001b2b0     Metaphlan2LogParser.obj
 0002:000042d4       __tryblocktable$?_Copy@?$basic_string@DU?$char_traits@D@std@@V?$allocator@D@2@@std@@QAEXII@Z 1001b2d4     Metaphlan2LogParser.obj
 0002:000042fc       __catchsym$??0?$QList@VQString@@@@QAE@ABV0@@Z$2 1001b2fc     Metaphlan2LogParser.obj
 0002:0000430c       __unwindtable$??0?$QList@VQString@@@@QAE@ABV0@@Z 1001b30c     Metaphlan2LogParser.obj
 0002:0000431c       __tryblocktable$??0?$QList@VQString@@@@QAE@ABV0@@Z 1001b31c     Metaphlan2LogParser.obj
 0002:00004330       __ehfuncinfo$??0?$QList@VQString@@@@QAE@ABV0@@Z 1001b330     Metaphlan2LogParser.obj
 0002:00004354       __catchsym$?append@?$QList@VQString@@@@QAEXABVQString@@@Z$13 1001b354     Metaphlan2LogParser.obj
 0002:00004364       __catchsym$?append@?$QList@VQString@@@@QAEXABVQString@@@Z$12 1001b364     Metaphlan2LogParser.obj
 0002:00004374       __ehfuncinfo$?append@?$QList@VQString@@@@QAEXABVQString@@@Z 1001b374     Metaphlan2LogParser.obj
 0002:00004398       __tryblocktable$?append@?$QList@VQString@@@@QAEXABVQString@@@Z 1001b398     Metaphlan2LogParser.obj
 0002:000043c0       __unwindtable$?append@?$QList@VQString@@@@QAEXABVQString@@@Z 1001b3c0     Metaphlan2LogParser.obj
 0002:00004420       __catchsym$?detach_helper_grow@?$QList@VQString@@@@AAEPAUNode@1@HH@Z$5 1001b420     Metaphlan2LogParser.obj
 0002:00004430       __catchsym$?detach_helper_grow@?$QList@VQString@@@@AAEPAUNode@1@HH@Z$4 1001b430     Metaphlan2LogParser.obj
 0002:00004440       __unwindtable$?detach_helper_grow@?$QList@VQString@@@@AAEPAUNode@1@HH@Z 1001b440     Metaphlan2LogParser.obj
 0002:00004460       __ehfuncinfo$?detach_helper_grow@?$QList@VQString@@@@AAEPAUNode@1@HH@Z 1001b460     Metaphlan2LogParser.obj
 0002:00004484       __tryblocktable$?detach_helper_grow@?$QList@VQString@@@@AAEPAUNode@1@HH@Z 1001b484     Metaphlan2LogParser.obj
 0002:000044ac       __unwindtable$?node_construct@?$QList@VQString@@@@AAEXPAUNode@1@ABVQString@@@Z 1001b4ac     Metaphlan2LogParser.obj
 0002:000044bc       __ehfuncinfo$?node_construct@?$QList@VQString@@@@AAEXPAUNode@1@ABVQString@@@Z 1001b4bc     Metaphlan2LogParser.obj
 0002:000044e0       __catchsym$?node_copy@?$QList@VQString@@@@AAEXPAUNode@1@00@Z$6 1001b4e0     Metaphlan2LogParser.obj
 0002:000044f0       __tryblocktable$?node_copy@?$QList@VQString@@@@AAEXPAUNode@1@00@Z 1001b4f0     Metaphlan2LogParser.obj
 0002:00004504       __ehfuncinfo$?node_copy@?$QList@VQString@@@@AAEXPAUNode@1@00@Z 1001b504     Metaphlan2LogParser.obj
 0002:00004528       __unwindtable$?node_copy@?$QList@VQString@@@@AAEXPAUNode@1@00@Z 1001b528     Metaphlan2LogParser.obj
 0002:00004558       __unwindtable$??__EalgoLog@U2@@YAXXZ 1001b558     Metaphlan2LogParser.obj
 0002:00004560       __ehfuncinfo$??__EalgoLog@U2@@YAXXZ 1001b560     Metaphlan2LogParser.obj
 0002:00004584       __unwindtable$??__EcmdLog@U2@@YAXXZ 1001b584     Metaphlan2LogParser.obj
 0002:0000458c       __ehfuncinfo$??__EcmdLog@U2@@YAXXZ 1001b58c     Metaphlan2LogParser.obj
 0002:000045b0       __unwindtable$??__EcoreLog@U2@@YAXXZ 1001b5b0     Metaphlan2LogParser.obj
 0002:000045b8       __ehfuncinfo$??__EcoreLog@U2@@YAXXZ 1001b5b8     Metaphlan2LogParser.obj
 0002:000045dc       __unwindtable$??__EioLog@U2@@YAXXZ 1001b5dc     Metaphlan2LogParser.obj
 0002:000045e4       __ehfuncinfo$??__EioLog@U2@@YAXXZ 1001b5e4     Metaphlan2LogParser.obj
 0002:00004608       __unwindtable$??__EperfLog@U2@@YAXXZ 1001b608     Metaphlan2LogParser.obj
 0002:00004610       __ehfuncinfo$??__EperfLog@U2@@YAXXZ 1001b610     Metaphlan2LogParser.obj
 0002:00004634       __unwindtable$??__EscriptLog@U2@@YAXXZ 1001b634     Metaphlan2LogParser.obj
 0002:0000463c       __ehfuncinfo$??__EscriptLog@U2@@YAXXZ 1001b63c     Metaphlan2LogParser.obj
 0002:00004660       __unwindtable$??__EtaskLog@U2@@YAXXZ 1001b660     Metaphlan2LogParser.obj
 0002:00004668       __ehfuncinfo$??__EtaskLog@U2@@YAXXZ 1001b668     Metaphlan2LogParser.obj
 0002:0000468c       __unwindtable$??__EuiLog@U2@@YAXXZ 1001b68c     Metaphlan2LogParser.obj
 0002:00004694       __ehfuncinfo$??__EuiLog@U2@@YAXXZ 1001b694     Metaphlan2LogParser.obj
 0002:000046b8       __unwindtable$??__EuserActLog@U2@@YAXXZ 1001b6b8     Metaphlan2LogParser.obj
 0002:000046c0       __ehfuncinfo$??__EuserActLog@U2@@YAXXZ 1001b6c0     Metaphlan2LogParser.obj
 0002:000046e4       __unwindtable$?isError@Metaphlan2LogParser@U2@@EBE_NABVQString@@@Z 1001b6e4     Metaphlan2LogParser.obj
 0002:000046ec       __ehfuncinfo$?isError@Metaphlan2LogParser@U2@@EBE_NABVQString@@@Z 1001b6ec     Metaphlan2LogParser.obj
 0002:00004710       __unwindtable$?initWellKnownErrors@Metaphlan2LogParser@U2@@CA?AVQStringList@@XZ 1001b710     Metaphlan2LogParser.obj
 0002:00004720       __ehfuncinfo$?initWellKnownErrors@Metaphlan2LogParser@U2@@CA?AVQStringList@@XZ 1001b720     Metaphlan2LogParser.obj
 0002:00004744       __unwindtable$??__EalgoLog@U2@@YAXXZ 1001b744     Metaphlan2Prompter.obj
 0002:0000474c       __ehfuncinfo$??__EalgoLog@U2@@YAXXZ 1001b74c     Metaphlan2Prompter.obj
 0002:00004770       __unwindtable$??__EcmdLog@U2@@YAXXZ 1001b770     Metaphlan2Prompter.obj
 0002:00004778       __ehfuncinfo$??__EcmdLog@U2@@YAXXZ 1001b778     Metaphlan2Prompter.obj
 0002:0000479c       __unwindtable$??__EcoreLog@U2@@YAXXZ 1001b79c     Metaphlan2Prompter.obj
 0002:000047a4       __ehfuncinfo$??__EcoreLog@U2@@YAXXZ 1001b7a4     Metaphlan2Prompter.obj
 0002:000047c8       __unwindtable$??__EioLog@U2@@YAXXZ 1001b7c8     Metaphlan2Prompter.obj
 0002:000047d0       __ehfuncinfo$??__EioLog@U2@@YAXXZ 1001b7d0     Metaphlan2Prompter.obj
 0002:000047f4       __unwindtable$??__EperfLog@U2@@YAXXZ 1001b7f4     Metaphlan2Prompter.obj
 0002:000047fc       __ehfuncinfo$??__EperfLog@U2@@YAXXZ 1001b7fc     Metaphlan2Prompter.obj
 0002:00004820       __unwindtable$??__EscriptLog@U2@@YAXXZ 1001b820     Metaphlan2Prompter.obj
 0002:00004828       __ehfuncinfo$??__EscriptLog@U2@@YAXXZ 1001b828     Metaphlan2Prompter.obj
 0002:0000484c       __unwindtable$??__EtaskLog@U2@@YAXXZ 1001b84c     Metaphlan2Prompter.obj
 0002:00004854       __ehfuncinfo$??__EtaskLog@U2@@YAXXZ 1001b854     Metaphlan2Prompter.obj
 0002:00004878       __unwindtable$??__EuiLog@U2@@YAXXZ 1001b878     Metaphlan2Prompter.obj
 0002:00004880       __ehfuncinfo$??__EuiLog@U2@@YAXXZ 1001b880     Metaphlan2Prompter.obj
 0002:000048a4       __unwindtable$??__EuserActLog@U2@@YAXXZ 1001b8a4     Metaphlan2Prompter.obj
 0002:000048ac       __ehfuncinfo$??__EuserActLog@U2@@YAXXZ 1001b8ac     Metaphlan2Prompter.obj
 0002:000048d0       __ehfuncinfo$?createDescription@?$PrompterBase@VMetaphlan2Prompter@LocalWorkflow@U2@@@U2@@UAEPAVActorDocument@Workflow@2@PAVActor@42@@Z 1001b8d0     Metaphlan2Prompter.obj
 0002:000048f4       __unwindtable$?createDescription@?$PrompterBase@VMetaphlan2Prompter@LocalWorkflow@U2@@@U2@@UAEPAVActorDocument@Workflow@2@PAVActor@42@@Z 1001b8f4     Metaphlan2Prompter.obj
 0002:0000492c       __ehfuncinfo$?composeRichDoc@Metaphlan2Prompter@LocalWorkflow@U2@@EAE?AVQString@@XZ 1001b92c     Metaphlan2Prompter.obj
 0002:00004950       __unwindtable$?composeRichDoc@Metaphlan2Prompter@LocalWorkflow@U2@@EAE?AVQString@@XZ 1001b950     Metaphlan2Prompter.obj
 0002:000049a8       __catchsym$??0?$QList@PAVPort@Workflow@U2@@@@QAE@ABV0@@Z$2 1001b9a8     Metaphlan2Prompter.obj
 0002:000049b8       __unwindtable$??0?$QList@PAVPort@Workflow@U2@@@@QAE@ABV0@@Z 1001b9b8     Metaphlan2Prompter.obj
 0002:000049c8       __tryblocktable$??0?$QList@PAVPort@Workflow@U2@@@@QAE@ABV0@@Z 1001b9c8     Metaphlan2Prompter.obj
 0002:000049dc       __ehfuncinfo$??0?$QList@PAVPort@Workflow@U2@@@@QAE@ABV0@@Z 1001b9dc     Metaphlan2Prompter.obj
 0002:00004a00       __ehfuncinfo$??0Metaphlan2Support@U2@@QAE@ABVQString@@0@Z 1001ba00     Metaphlan2Support.obj
 0002:00004a24       __unwindtable$??0Metaphlan2Support@U2@@QAE@ABVQString@@0@Z 1001ba24     Metaphlan2Support.obj
 0002:00004a54       __ehfuncinfo$?performAdditionalChecks@Metaphlan2Support@U2@@UAEXABVQString@@@Z 1001ba54     Metaphlan2Support.obj
 0002:00004a78       __unwindtable$?performAdditionalChecks@Metaphlan2Support@U2@@UAEXABVQString@@@Z 1001ba78     Metaphlan2Support.obj
 0002:00004ad0       __unwindtable$??__EalgoLog@U2@@YAXXZ 1001bad0     Metaphlan2Support.obj
 0002:00004ad8       __ehfuncinfo$??__EalgoLog@U2@@YAXXZ 1001bad8     Metaphlan2Support.obj
 0002:00004afc       __unwindtable$??__EcmdLog@U2@@YAXXZ 1001bafc     Metaphlan2Support.obj
 0002:00004b04       __ehfuncinfo$??__EcmdLog@U2@@YAXXZ 1001bb04     Metaphlan2Support.obj
 0002:00004b28       __unwindtable$??__EcoreLog@U2@@YAXXZ 1001bb28     Metaphlan2Support.obj
 0002:00004b30       __ehfuncinfo$??__EcoreLog@U2@@YAXXZ 1001bb30     Metaphlan2Support.obj
 0002:00004b54       __unwindtable$??__EioLog@U2@@YAXXZ 1001bb54     Metaphlan2Support.obj
 0002:00004b5c       __ehfuncinfo$??__EioLog@U2@@YAXXZ 1001bb5c     Metaphlan2Support.obj
 0002:00004b80       __unwindtable$??__EperfLog@U2@@YAXXZ 1001bb80     Metaphlan2Support.obj
 0002:00004b88       __ehfuncinfo$??__EperfLog@U2@@YAXXZ 1001bb88     Metaphlan2Support.obj
 0002:00004bac       __unwindtable$??__EscriptLog@U2@@YAXXZ 1001bbac     Metaphlan2Support.obj
 0002:00004bb4       __ehfuncinfo$??__EscriptLog@U2@@YAXXZ 1001bbb4     Metaphlan2Support.obj
 0002:00004bd8       __unwindtable$??__EtaskLog@U2@@YAXXZ 1001bbd8     Metaphlan2Support.obj
 0002:00004be0       __ehfuncinfo$??__EtaskLog@U2@@YAXXZ 1001bbe0     Metaphlan2Support.obj
 0002:00004c04       __unwindtable$??__EuiLog@U2@@YAXXZ 1001bc04     Metaphlan2Support.obj
 0002:00004c0c       __ehfuncinfo$??__EuiLog@U2@@YAXXZ 1001bc0c     Metaphlan2Support.obj
 0002:00004c30       __unwindtable$??__EuserActLog@U2@@YAXXZ 1001bc30     Metaphlan2Support.obj
 0002:00004c38       __ehfuncinfo$??__EuserActLog@U2@@YAXXZ 1001bc38     Metaphlan2Support.obj
 0002:00004c5c       __unwindtable$??__EalgoLog@U2@@YAXXZ 1001bc5c     Metaphlan2SupportPlugin.obj
 0002:00004c64       __ehfuncinfo$??__EalgoLog@U2@@YAXXZ 1001bc64     Metaphlan2SupportPlugin.obj
 0002:00004c88       __unwindtable$??__EcmdLog@U2@@YAXXZ 1001bc88     Metaphlan2SupportPlugin.obj
 0002:00004c90       __ehfuncinfo$??__EcmdLog@U2@@YAXXZ 1001bc90     Metaphlan2SupportPlugin.obj
 0002:00004cb4       __unwindtable$??__EcoreLog@U2@@YAXXZ 1001bcb4     Metaphlan2SupportPlugin.obj
 0002:00004cbc       __ehfuncinfo$??__EcoreLog@U2@@YAXXZ 1001bcbc     Metaphlan2SupportPlugin.obj
 0002:00004ce0       __unwindtable$??__EioLog@U2@@YAXXZ 1001bce0     Metaphlan2SupportPlugin.obj
 0002:00004ce8       __ehfuncinfo$??__EioLog@U2@@YAXXZ 1001bce8     Metaphlan2SupportPlugin.obj
 0002:00004d0c       __unwindtable$??__EperfLog@U2@@YAXXZ 1001bd0c     Metaphlan2SupportPlugin.obj
 0002:00004d14       __ehfuncinfo$??__EperfLog@U2@@YAXXZ 1001bd14     Metaphlan2SupportPlugin.obj
 0002:00004d38       __unwindtable$??__EscriptLog@U2@@YAXXZ 1001bd38     Metaphlan2SupportPlugin.obj
 0002:00004d40       __ehfuncinfo$??__EscriptLog@U2@@YAXXZ 1001bd40     Metaphlan2SupportPlugin.obj
 0002:00004d64       __unwindtable$??__EtaskLog@U2@@YAXXZ 1001bd64     Metaphlan2SupportPlugin.obj
 0002:00004d6c       __ehfuncinfo$??__EtaskLog@U2@@YAXXZ 1001bd6c     Metaphlan2SupportPlugin.obj
 0002:00004d90       __unwindtable$??__EuiLog@U2@@YAXXZ 1001bd90     Metaphlan2SupportPlugin.obj
 0002:00004d98       __ehfuncinfo$??__EuiLog@U2@@YAXXZ 1001bd98     Metaphlan2SupportPlugin.obj
 0002:00004dbc       __unwindtable$??__EuserActLog@U2@@YAXXZ 1001bdbc     Metaphlan2SupportPlugin.obj
 0002:00004dc4       __ehfuncinfo$??__EuserActLog@U2@@YAXXZ 1001bdc4     Metaphlan2SupportPlugin.obj
 0002:00004de8       __unwindtable$??0MetaphlanSupportPlugin@U2@@QAE@XZ 1001bde8     Metaphlan2SupportPlugin.obj
 0002:00004e08       __ehfuncinfo$??0MetaphlanSupportPlugin@U2@@QAE@XZ 1001be08     Metaphlan2SupportPlugin.obj
 0002:00004e2c       __unwindtable$??1MetaphlanSupportPlugin@U2@@UAE@XZ 1001be2c     Metaphlan2SupportPlugin.obj
 0002:00004e34       __ehfuncinfo$??1MetaphlanSupportPlugin@U2@@UAE@XZ 1001be34     Metaphlan2SupportPlugin.obj
 0002:00004e58       __unwindtable$??_GMetaphlanSupportPlugin@U2@@UAEPAXI@Z 1001be58     Metaphlan2SupportPlugin.obj
 0002:00004e60       __ehfuncinfo$??_GMetaphlanSupportPlugin@U2@@UAEPAXI@Z 1001be60     Metaphlan2SupportPlugin.obj
 0002:00004e84       __catchsym$?detach_helper@?$QList@VQString@@@@AAEXH@Z$2 1001be84     Metaphlan2Task.obj
 0002:00004e94       __unwindtable$?detach_helper@?$QList@VQString@@@@AAEXH@Z 1001be94     Metaphlan2Task.obj
 0002:00004ea4       __tryblocktable$?detach_helper@?$QList@VQString@@@@AAEXH@Z 1001bea4     Metaphlan2Task.obj
 0002:00004eb8       __ehfuncinfo$?detach_helper@?$QList@VQString@@@@AAEXH@Z 1001beb8     Metaphlan2Task.obj
 0002:00004edc       __unwindtable$??__EalgoLog@U2@@YAXXZ 1001bedc     Metaphlan2Task.obj
 0002:00004ee4       __ehfuncinfo$??__EalgoLog@U2@@YAXXZ 1001bee4     Metaphlan2Task.obj
 0002:00004f08       __unwindtable$??__EcmdLog@U2@@YAXXZ 1001bf08     Metaphlan2Task.obj
 0002:00004f10       __ehfuncinfo$??__EcmdLog@U2@@YAXXZ 1001bf10     Metaphlan2Task.obj
 0002:00004f34       __unwindtable$??__EcoreLog@U2@@YAXXZ 1001bf34     Metaphlan2Task.obj
 0002:00004f3c       __ehfuncinfo$??__EcoreLog@U2@@YAXXZ 1001bf3c     Metaphlan2Task.obj
 0002:00004f60       __unwindtable$??__EioLog@U2@@YAXXZ 1001bf60     Metaphlan2Task.obj
 0002:00004f68       __ehfuncinfo$??__EioLog@U2@@YAXXZ 1001bf68     Metaphlan2Task.obj
 0002:00004f8c       __unwindtable$??__EperfLog@U2@@YAXXZ 1001bf8c     Metaphlan2Task.obj
 0002:00004f94       __ehfuncinfo$??__EperfLog@U2@@YAXXZ 1001bf94     Metaphlan2Task.obj
 0002:00004fb8       __unwindtable$??__EscriptLog@U2@@YAXXZ 1001bfb8     Metaphlan2Task.obj
 0002:00004fc0       __ehfuncinfo$??__EscriptLog@U2@@YAXXZ 1001bfc0     Metaphlan2Task.obj
 0002:00004fe4       __unwindtable$??__EtaskLog@U2@@YAXXZ 1001bfe4     Metaphlan2Task.obj
 0002:00004fec       __ehfuncinfo$??__EtaskLog@U2@@YAXXZ 1001bfec     Metaphlan2Task.obj
 0002:00005010       __unwindtable$??__EuiLog@U2@@YAXXZ 1001c010     Metaphlan2Task.obj
 0002:00005018       __ehfuncinfo$??__EuiLog@U2@@YAXXZ 1001c018     Metaphlan2Task.obj
 0002:0000503c       __unwindtable$??__EuserActLog@U2@@YAXXZ 1001c03c     Metaphlan2Task.obj
 0002:00005044       __ehfuncinfo$??__EuserActLog@U2@@YAXXZ 1001c044     Metaphlan2Task.obj
 0002:00005068       __catchsym$?append@?$QList@PAVTask@U2@@@@QAEXABQAVTask@U2@@@Z$6 1001c068     Metaphlan2Task.obj
 0002:00005078       __tryblocktable$?append@?$QList@PAVTask@U2@@@@QAEXABQAVTask@U2@@@Z 1001c078     Metaphlan2Task.obj
 0002:0000508c       __ehfuncinfo$?append@?$QList@PAVTask@U2@@@@QAEXABQAVTask@U2@@@Z 1001c08c     Metaphlan2Task.obj
 0002:000050b0       __unwindtable$?append@?$QList@PAVTask@U2@@@@QAEXABQAVTask@U2@@@Z 1001c0b0     Metaphlan2Task.obj
 0002:000050e0       __catchsym$?detach_helper_grow@?$QList@PAVTask@U2@@@@AAEPAUNode@1@HH@Z$5 1001c0e0     Metaphlan2Task.obj
 0002:000050f0       __catchsym$?detach_helper_grow@?$QList@PAVTask@U2@@@@AAEPAUNode@1@HH@Z$4 1001c0f0     Metaphlan2Task.obj
 0002:00005100       __unwindtable$?detach_helper_grow@?$QList@PAVTask@U2@@@@AAEPAUNode@1@HH@Z 1001c100     Metaphlan2Task.obj
 0002:00005120       __ehfuncinfo$?detach_helper_grow@?$QList@PAVTask@U2@@@@AAEPAUNode@1@HH@Z 1001c120     Metaphlan2Task.obj
 0002:00005144       __tryblocktable$?detach_helper_grow@?$QList@PAVTask@U2@@@@AAEPAUNode@1@HH@Z 1001c144     Metaphlan2Task.obj
 0002:0000516c       __ehfuncinfo$??0Metaphlan2TaskSettings@U2@@QAE@XZ 1001c16c     Metaphlan2Task.obj
 0002:00005190       __unwindtable$??0Metaphlan2TaskSettings@U2@@QAE@XZ 1001c190     Metaphlan2Task.obj
 0002:000051d8       __ehfuncinfo$??1Metaphlan2TaskSettings@U2@@QAE@XZ 1001c1d8     Metaphlan2Task.obj
 0002:000051fc       __unwindtable$??1Metaphlan2TaskSettings@U2@@QAE@XZ 1001c1fc     Metaphlan2Task.obj
 0002:00005244       __ehfuncinfo$??0Metaphlan2TaskSettings@U2@@QAE@ABU01@@Z 1001c244     Metaphlan2Task.obj
 0002:00005268       __unwindtable$??0Metaphlan2TaskSettings@U2@@QAE@ABU01@@Z 1001c268     Metaphlan2Task.obj
 0002:000052b0       __ehfuncinfo$??0Metaphlan2ClassifyTask@U2@@QAE@ABUMetaphlan2TaskSettings@1@@Z 1001c2b0     Metaphlan2Task.obj
 0002:000052d4       __unwindtable$??0Metaphlan2ClassifyTask@U2@@QAE@ABUMetaphlan2TaskSettings@1@@Z 1001c2d4     Metaphlan2Task.obj
 0002:00005344       __unwindtable$?prepare@Metaphlan2ClassifyTask@U2@@EAEXXZ 1001c344     Metaphlan2Task.obj
 0002:0000534c       __ehfuncinfo$?prepare@Metaphlan2ClassifyTask@U2@@EAEXXZ 1001c34c     Metaphlan2Task.obj
 0002:00005370       __unwindtable$?onSubTaskFinished@Metaphlan2ClassifyTask@U2@@EAE?AV?$QList@PAVTask@U2@@@@PAVTask@2@@Z 1001c370     Metaphlan2Task.obj
 0002:00005380       __ehfuncinfo$?onSubTaskFinished@Metaphlan2ClassifyTask@U2@@EAE?AV?$QList@PAVTask@U2@@@@PAVTask@2@@Z 1001c380     Metaphlan2Task.obj
 0002:000053a4       __ehfuncinfo$?getArguments@Metaphlan2ClassifyTask@U2@@AAE?AVQStringList@@XZ 1001c3a4     Metaphlan2Task.obj
 0002:000053c8       __unwindtable$?getArguments@Metaphlan2ClassifyTask@U2@@AAE?AVQStringList@@XZ 1001c3c8     Metaphlan2Task.obj
 0002:00005538       __ehfuncinfo$?prepareClassifyTask@Metaphlan2ClassifyTask@U2@@AAEXXZ 1001c538     Metaphlan2Task.obj
 0002:0000555c       __unwindtable$?prepareClassifyTask@Metaphlan2ClassifyTask@U2@@AAEXXZ 1001c55c     Metaphlan2Task.obj
 0002:000055ac       __ehfuncinfo$?detectInputFormats@Metaphlan2ClassifyTask@U2@@AAE?AVQString@@XZ 1001c5ac     Metaphlan2Task.obj
 0002:000055d0       __unwindtable$?detectInputFormats@Metaphlan2ClassifyTask@U2@@AAE?AVQString@@XZ 1001c5d0     Metaphlan2Task.obj
 0002:00005610       __unwindtable$?detectFormat@Metaphlan2ClassifyTask@U2@@AAE?AVQString@@ABVGUrl@2@@Z 1001c610     Metaphlan2Task.obj
 0002:00005630       __ehfuncinfo$?detectFormat@Metaphlan2ClassifyTask@U2@@AAE?AVQString@@ABVGUrl@2@@Z 1001c630     Metaphlan2Task.obj
 0002:00005654       __unwindtable$??1Metaphlan2ClassifyTask@U2@@UAE@XZ 1001c654     Metaphlan2Task.obj
 0002:0000565c       __ehfuncinfo$??1Metaphlan2ClassifyTask@U2@@UAE@XZ 1001c65c     Metaphlan2Task.obj
 0002:00005680       __unwindtable$??_GMetaphlan2ClassifyTask@U2@@UAEPAXI@Z 1001c680     Metaphlan2Task.obj
 0002:00005688       __ehfuncinfo$??_GMetaphlan2ClassifyTask@U2@@UAEPAXI@Z 1001c688     Metaphlan2Task.obj
 0002:000056ac       __unwindtable$??__EalgoLog@U2@@YAXXZ 1001c6ac     Metaphlan2Validator.obj
 0002:000056b4       __ehfuncinfo$??__EalgoLog@U2@@YAXXZ 1001c6b4     Metaphlan2Validator.obj
 0002:000056d8       __unwindtable$??__EcmdLog@U2@@YAXXZ 1001c6d8     Metaphlan2Validator.obj
 0002:000056e0       __ehfuncinfo$??__EcmdLog@U2@@YAXXZ 1001c6e0     Metaphlan2Validator.obj
 0002:00005704       __unwindtable$??__EcoreLog@U2@@YAXXZ 1001c704     Metaphlan2Validator.obj
 0002:0000570c       __ehfuncinfo$??__EcoreLog@U2@@YAXXZ 1001c70c     Metaphlan2Validator.obj
 0002:00005730       __unwindtable$??__EioLog@U2@@YAXXZ 1001c730     Metaphlan2Validator.obj
 0002:00005738       __ehfuncinfo$??__EioLog@U2@@YAXXZ 1001c738     Metaphlan2Validator.obj
 0002:0000575c       __unwindtable$??__EperfLog@U2@@YAXXZ 1001c75c     Metaphlan2Validator.obj
 0002:00005764       __ehfuncinfo$??__EperfLog@U2@@YAXXZ 1001c764     Metaphlan2Validator.obj
 0002:00005788       __unwindtable$??__EscriptLog@U2@@YAXXZ 1001c788     Metaphlan2Validator.obj
 0002:00005790       __ehfuncinfo$??__EscriptLog@U2@@YAXXZ 1001c790     Metaphlan2Validator.obj
 0002:000057b4       __unwindtable$??__EtaskLog@U2@@YAXXZ 1001c7b4     Metaphlan2Validator.obj
 0002:000057bc       __ehfuncinfo$??__EtaskLog@U2@@YAXXZ 1001c7bc     Metaphlan2Validator.obj
 0002:000057e0       __unwindtable$??__EuiLog@U2@@YAXXZ 1001c7e0     Metaphlan2Validator.obj
 0002:000057e8       __ehfuncinfo$??__EuiLog@U2@@YAXXZ 1001c7e8     Metaphlan2Validator.obj
 0002:0000580c       __unwindtable$??__EuserActLog@U2@@YAXXZ 1001c80c     Metaphlan2Validator.obj
 0002:00005814       __ehfuncinfo$??__EuserActLog@U2@@YAXXZ 1001c814     Metaphlan2Validator.obj
 0002:00005838       __ehfuncinfo$?validateDatabase@Metaphlan2Validator@Workflow@U2@@ABE_NPBVActor@23@AAV?$QList@VWorkflowNotification@U2@@@@@Z 1001c838     Metaphlan2Validator.obj
 0002:0000585c       __unwindtable$?validateDatabase@Metaphlan2Validator@Workflow@U2@@ABE_NPBVActor@23@AAV?$QList@VWorkflowNotification@U2@@@@@Z 1001c85c     Metaphlan2Validator.obj
 0002:000058fc       __catchsym$?append@?$QList@VWorkflowNotification@U2@@@@QAEXABVWorkflowNotification@U2@@@Z$11 1001c8fc     Metaphlan2Validator.obj
 0002:0000590c       __catchsym$?append@?$QList@VWorkflowNotification@U2@@@@QAEXABVWorkflowNotification@U2@@@Z$10 1001c90c     Metaphlan2Validator.obj
 0002:0000591c       __ehfuncinfo$?append@?$QList@VWorkflowNotification@U2@@@@QAEXABVWorkflowNotification@U2@@@Z 1001c91c     Metaphlan2Validator.obj
 0002:00005940       __tryblocktable$?append@?$QList@VWorkflowNotification@U2@@@@QAEXABVWorkflowNotification@U2@@@Z 1001c940     Metaphlan2Validator.obj
 0002:00005968       __unwindtable$?append@?$QList@VWorkflowNotification@U2@@@@QAEXABVWorkflowNotification@U2@@@Z 1001c968     Metaphlan2Validator.obj
 0002:000059b8       __catchsym$?detach_helper_grow@?$QList@VWorkflowNotification@U2@@@@AAEPAUNode@1@HH@Z$5 1001c9b8     Metaphlan2Validator.obj
 0002:000059c8       __catchsym$?detach_helper_grow@?$QList@VWorkflowNotification@U2@@@@AAEPAUNode@1@HH@Z$4 1001c9c8     Metaphlan2Validator.obj
 0002:000059d8       __unwindtable$?detach_helper_grow@?$QList@VWorkflowNotification@U2@@@@AAEPAUNode@1@HH@Z 1001c9d8     Metaphlan2Validator.obj
 0002:000059f8       __ehfuncinfo$?detach_helper_grow@?$QList@VWorkflowNotification@U2@@@@AAEPAUNode@1@HH@Z 1001c9f8     Metaphlan2Validator.obj
 0002:00005a1c       __tryblocktable$?detach_helper_grow@?$QList@VWorkflowNotification@U2@@@@AAEPAUNode@1@HH@Z 1001ca1c     Metaphlan2Validator.obj
 0002:00005a44       __unwindtable$?node_construct@?$QList@VWorkflowNotification@U2@@@@AAEXPAUNode@1@ABVWorkflowNotification@U2@@@Z 1001ca44     Metaphlan2Validator.obj
 0002:00005a54       __ehfuncinfo$?node_construct@?$QList@VWorkflowNotification@U2@@@@AAEXPAUNode@1@ABVWorkflowNotification@U2@@@Z 1001ca54     Metaphlan2Validator.obj
 0002:00005a78       __catchsym$?node_copy@?$QList@VWorkflowNotification@U2@@@@AAEXPAUNode@1@00@Z$6 1001ca78     Metaphlan2Validator.obj
 0002:00005a88       __tryblocktable$?node_copy@?$QList@VWorkflowNotification@U2@@@@AAEXPAUNode@1@00@Z 1001ca88     Metaphlan2Validator.obj
 0002:00005a9c       __ehfuncinfo$?node_copy@?$QList@VWorkflowNotification@U2@@@@AAEXPAUNode@1@00@Z 1001ca9c     Metaphlan2Validator.obj
 0002:00005ac0       __unwindtable$?node_copy@?$QList@VWorkflowNotification@U2@@@@AAEXPAUNode@1@00@Z 1001cac0     Metaphlan2Validator.obj
 0002:00005af0       __unwindtable$?metaType@?$QVariantValueHelper@VQString@@@QtPrivate@@SA?AVQString@@ABVQVariant@@@Z 1001caf0     Metaphlan2Validator.obj
 0002:00005b00       __ehfuncinfo$?metaType@?$QVariantValueHelper@VQString@@@QtPrivate@@SA?AVQString@@ABVQVariant@@@Z 1001cb00     Metaphlan2Validator.obj
 0002:00005b24       __unwindtable$??A?$QMap@VQString@@VQVariant@@@@QAEAAVQVariant@@ABVQString@@@Z 1001cb24     Metaphlan2Worker.obj
 0002:00005b2c       __ehfuncinfo$??A?$QMap@VQString@@VQVariant@@@@QAEAAVQVariant@@ABVQString@@@Z 1001cb2c     Metaphlan2Worker.obj
 0002:00005b50       __unwindtable$??__EalgoLog@U2@@YAXXZ 1001cb50     Metaphlan2Worker.obj
 0002:00005b58       __ehfuncinfo$??__EalgoLog@U2@@YAXXZ 1001cb58     Metaphlan2Worker.obj
 0002:00005b7c       __unwindtable$??__EcmdLog@U2@@YAXXZ 1001cb7c     Metaphlan2Worker.obj
 0002:00005b84       __ehfuncinfo$??__EcmdLog@U2@@YAXXZ 1001cb84     Metaphlan2Worker.obj
 0002:00005ba8       __unwindtable$??__EcoreLog@U2@@YAXXZ 1001cba8     Metaphlan2Worker.obj
 0002:00005bb0       __ehfuncinfo$??__EcoreLog@U2@@YAXXZ 1001cbb0     Metaphlan2Worker.obj
 0002:00005bd4       __unwindtable$??__EioLog@U2@@YAXXZ 1001cbd4     Metaphlan2Worker.obj
 0002:00005bdc       __ehfuncinfo$??__EioLog@U2@@YAXXZ 1001cbdc     Metaphlan2Worker.obj
 0002:00005c00       __unwindtable$??__EperfLog@U2@@YAXXZ 1001cc00     Metaphlan2Worker.obj
 0002:00005c08       __ehfuncinfo$??__EperfLog@U2@@YAXXZ 1001cc08     Metaphlan2Worker.obj
 0002:00005c2c       __unwindtable$??__EscriptLog@U2@@YAXXZ 1001cc2c     Metaphlan2Worker.obj
 0002:00005c34       __ehfuncinfo$??__EscriptLog@U2@@YAXXZ 1001cc34     Metaphlan2Worker.obj
 0002:00005c58       __unwindtable$??__EtaskLog@U2@@YAXXZ 1001cc58     Metaphlan2Worker.obj
 0002:00005c60       __ehfuncinfo$??__EtaskLog@U2@@YAXXZ 1001cc60     Metaphlan2Worker.obj
 0002:00005c84       __unwindtable$??__EuiLog@U2@@YAXXZ 1001cc84     Metaphlan2Worker.obj
 0002:00005c8c       __ehfuncinfo$??__EuiLog@U2@@YAXXZ 1001cc8c     Metaphlan2Worker.obj
 0002:00005cb0       __unwindtable$??__EuserActLog@U2@@YAXXZ 1001ccb0     Metaphlan2Worker.obj
 0002:00005cb8       __ehfuncinfo$??__EuserActLog@U2@@YAXXZ 1001ccb8     Metaphlan2Worker.obj
 0002:00005cdc       __catchsym$??0?$QList@VDescriptor@U2@@@@QAE@ABV0@@Z$2 1001ccdc     Metaphlan2Worker.obj
 0002:00005cec       __unwindtable$??0?$QList@VDescriptor@U2@@@@QAE@ABV0@@Z 1001ccec     Metaphlan2Worker.obj
 0002:00005cfc       __tryblocktable$??0?$QList@VDescriptor@U2@@@@QAE@ABV0@@Z 1001ccfc     Metaphlan2Worker.obj
 0002:00005d10       __ehfuncinfo$??0?$QList@VDescriptor@U2@@@@QAE@ABV0@@Z 1001cd10     Metaphlan2Worker.obj
 0002:00005d34       __catchsym$?append@?$QList@VDescriptor@U2@@@@QAEXABVDescriptor@U2@@@Z$9 1001cd34     Metaphlan2Worker.obj
 0002:00005d44       __catchsym$?append@?$QList@VDescriptor@U2@@@@QAEXABVDescriptor@U2@@@Z$8 1001cd44     Metaphlan2Worker.obj
 0002:00005d54       __ehfuncinfo$?append@?$QList@VDescriptor@U2@@@@QAEXABVDescriptor@U2@@@Z 1001cd54     Metaphlan2Worker.obj
 0002:00005d78       __tryblocktable$?append@?$QList@VDescriptor@U2@@@@QAEXABVDescriptor@U2@@@Z 1001cd78     Metaphlan2Worker.obj
 0002:00005da0       __unwindtable$?append@?$QList@VDescriptor@U2@@@@QAEXABVDescriptor@U2@@@Z 1001cda0     Metaphlan2Worker.obj
 0002:00005de0       __catchsym$?detach_helper_grow@?$QList@VDescriptor@U2@@@@AAEPAUNode@1@HH@Z$5 1001cde0     Metaphlan2Worker.obj
 0002:00005df0       __catchsym$?detach_helper_grow@?$QList@VDescriptor@U2@@@@AAEPAUNode@1@HH@Z$4 1001cdf0     Metaphlan2Worker.obj
 0002:00005e00       __unwindtable$?detach_helper_grow@?$QList@VDescriptor@U2@@@@AAEPAUNode@1@HH@Z 1001ce00     Metaphlan2Worker.obj
 0002:00005e20       __ehfuncinfo$?detach_helper_grow@?$QList@VDescriptor@U2@@@@AAEPAUNode@1@HH@Z 1001ce20     Metaphlan2Worker.obj
 0002:00005e44       __tryblocktable$?detach_helper_grow@?$QList@VDescriptor@U2@@@@AAEPAUNode@1@HH@Z 1001ce44     Metaphlan2Worker.obj
 0002:00005e6c       __catchsym$?detach_helper@?$QList@VDescriptor@U2@@@@AAEXH@Z$2 1001ce6c     Metaphlan2Worker.obj
 0002:00005e7c       __unwindtable$?detach_helper@?$QList@VDescriptor@U2@@@@AAEXH@Z 1001ce7c     Metaphlan2Worker.obj
 0002:00005e8c       __tryblocktable$?detach_helper@?$QList@VDescriptor@U2@@@@AAEXH@Z 1001ce8c     Metaphlan2Worker.obj
 0002:00005ea0       __ehfuncinfo$?detach_helper@?$QList@VDescriptor@U2@@@@AAEXH@Z 1001cea0     Metaphlan2Worker.obj
 0002:00005ec4       __unwindtable$?node_construct@?$QList@VDescriptor@U2@@@@AAEXPAUNode@1@ABVDescriptor@U2@@@Z 1001cec4     Metaphlan2Worker.obj
 0002:00005ed4       __ehfuncinfo$?node_construct@?$QList@VDescriptor@U2@@@@AAEXPAUNode@1@ABVDescriptor@U2@@@Z 1001ced4     Metaphlan2Worker.obj
 0002:00005ef8       __catchsym$?node_copy@?$QList@VDescriptor@U2@@@@AAEXPAUNode@1@00@Z$6 1001cef8     Metaphlan2Worker.obj
 0002:00005f08       __tryblocktable$?node_copy@?$QList@VDescriptor@U2@@@@AAEXPAUNode@1@00@Z 1001cf08     Metaphlan2Worker.obj
 0002:00005f1c       __ehfuncinfo$?node_copy@?$QList@VDescriptor@U2@@@@AAEXPAUNode@1@00@Z 1001cf1c     Metaphlan2Worker.obj
 0002:00005f40       __unwindtable$?node_copy@?$QList@VDescriptor@U2@@@@AAEXPAUNode@1@00@Z 1001cf40     Metaphlan2Worker.obj
 0002:00005f70       __unwindtable$??A?$QMap@VQString@@VQScriptValue@@@@QAEAAVQScriptValue@@ABVQString@@@Z 1001cf70     Metaphlan2Worker.obj
 0002:00005f78       __ehfuncinfo$??A?$QMap@VQString@@VQScriptValue@@@@QAEAAVQScriptValue@@ABVQString@@@Z 1001cf78     Metaphlan2Worker.obj
 0002:00005f9c       __unwindtable$?uniqueKeys@?$QMap@VDescriptor@U2@@VQVariant@@@@QBE?AV?$QList@VDescriptor@U2@@@@XZ 1001cf9c     Metaphlan2Worker.obj
 0002:00005fa4       __ehfuncinfo$?uniqueKeys@?$QMap@VDescriptor@U2@@VQVariant@@@@QBE?AV?$QList@VDescriptor@U2@@@@XZ 1001cfa4     Metaphlan2Worker.obj
 0002:00005fc8       __ehfuncinfo$??$getAttributeValue@VQString@@@Attribute@U2@@QBE?AVQString@@PAVWorkflowContext@Workflow@1@@Z 1001cfc8     Metaphlan2Worker.obj
 0002:00005fec       __unwindtable$??$getAttributeValue@VQString@@@Attribute@U2@@QBE?AVQString@@PAVWorkflowContext@Workflow@1@@Z 1001cfec     Metaphlan2Worker.obj
 0002:0000605c       __ehfuncinfo$??$getAttributeValue@H@Attribute@U2@@QBEHPAVWorkflowContext@Workflow@1@@Z 1001d05c     Metaphlan2Worker.obj
 0002:00006080       __unwindtable$??$getAttributeValue@H@Attribute@U2@@QBEHPAVWorkflowContext@Workflow@1@@Z 1001d080     Metaphlan2Worker.obj
 0002:000060e8       __unwindtable$??$getValue@VQString@@@BaseWorker@LocalWorkflow@U2@@IBE?AVQString@@ABV3@@Z 1001d0e8     Metaphlan2Worker.obj
 0002:000060f8       __ehfuncinfo$??$getValue@VQString@@@BaseWorker@LocalWorkflow@U2@@IBE?AVQString@@ABV3@@Z 1001d0f8     Metaphlan2Worker.obj
 0002:0000611c       __ehfuncinfo$?init@Metaphlan2Worker@LocalWorkflow@U2@@UAEXXZ 1001d11c     Metaphlan2Worker.obj
 0002:00006140       __unwindtable$?init@Metaphlan2Worker@LocalWorkflow@U2@@UAEXXZ 1001d140     Metaphlan2Worker.obj
 0002:00006178       __ehfuncinfo$?tick@Metaphlan2Worker@LocalWorkflow@U2@@UAEPAVTask@3@XZ 1001d178     Metaphlan2Worker.obj
 0002:0000619c       __unwindtable$?tick@Metaphlan2Worker@LocalWorkflow@U2@@UAEPAVTask@3@XZ 1001d19c     Metaphlan2Worker.obj
 0002:000061dc       __unwindtable$?sl_taskFinished@Metaphlan2Worker@LocalWorkflow@U2@@AAEXPAVTask@3@@Z 1001d1dc     Metaphlan2Worker.obj
 0002:000061ec       __ehfuncinfo$?sl_taskFinished@Metaphlan2Worker@LocalWorkflow@U2@@AAEXPAVTask@3@@Z 1001d1ec     Metaphlan2Worker.obj
 0002:00006210       __ehfuncinfo$?getSettings@Metaphlan2Worker@LocalWorkflow@U2@@AAE?AUMetaphlan2TaskSettings@3@AAVU2OpStatus@3@@Z 1001d210     Metaphlan2Worker.obj
 0002:00006234       __unwindtable$?getSettings@Metaphlan2Worker@LocalWorkflow@U2@@AAE?AUMetaphlan2TaskSettings@3@AAVU2OpStatus@3@@Z 1001d234     Metaphlan2Worker.obj
 0002:000063c4       __ehfuncinfo$?getDefaultOutputDir@Metaphlan2Worker@LocalWorkflow@U2@@ABE?AVQString@@XZ 1001d3c4     Metaphlan2Worker.obj
 0002:000063e8       __unwindtable$?getDefaultOutputDir@Metaphlan2Worker@LocalWorkflow@U2@@ABE?AVQString@@XZ 1001d3e8     Metaphlan2Worker.obj
 0002:00006438       __ehfuncinfo$?createOutputToolDirectory@Metaphlan2Worker@LocalWorkflow@U2@@ABE?AVQString@@ABV4@ABVMessage@Workflow@3@_NW4Output@123@@Z 1001d438     Metaphlan2Worker.obj
 0002:0000645c       __unwindtable$?createOutputToolDirectory@Metaphlan2Worker@LocalWorkflow@U2@@ABE?AVQString@@ABV4@ABVMessage@Workflow@3@_NW4Output@123@@Z 1001d45c     Metaphlan2Worker.obj
 0002:000064c4       __unwindtable$?createDirectory@Metaphlan2Worker@LocalWorkflow@U2@@ABEXAAVQString@@@Z 1001d4c4     Metaphlan2Worker.obj
 0002:000064e4       __ehfuncinfo$?createDirectory@Metaphlan2Worker@LocalWorkflow@U2@@ABEXAAVQString@@@Z 1001d4e4     Metaphlan2Worker.obj
 0002:00006508       __unwindtable$?addOutputToDashboard@Metaphlan2Worker@LocalWorkflow@U2@@ABEXABVQString@@0@Z 1001d508     Metaphlan2Worker.obj
 0002:00006520       __ehfuncinfo$?addOutputToDashboard@Metaphlan2Worker@LocalWorkflow@U2@@ABEXABVQString@@0@Z 1001d520     Metaphlan2Worker.obj
 0002:00006544       __catchsym$?createNode@?$QMapData@VQString@@VQVariant@@@@QAEPAU?$QMapNode@VQString@@VQVariant@@@@ABVQString@@ABVQVariant@@PAU2@_N@Z$7 1001d544     Metaphlan2Worker.obj
 0002:00006554       __catchsym$?createNode@?$QMapData@VQString@@VQVariant@@@@QAEPAU?$QMapNode@VQString@@VQVariant@@@@ABVQString@@ABVQVariant@@PAU2@_N@Z$6 1001d554     Metaphlan2Worker.obj
 0002:00006564       __ehfuncinfo$?createNode@?$QMapData@VQString@@VQVariant@@@@QAEPAU?$QMapNode@VQString@@VQVariant@@@@ABVQString@@ABVQVariant@@PAU2@_N@Z 1001d564     Metaphlan2Worker.obj
 0002:00006588       __tryblocktable$?createNode@?$QMapData@VQString@@VQVariant@@@@QAEPAU?$QMapNode@VQString@@VQVariant@@@@ABVQString@@ABVQVariant@@PAU2@_N@Z 1001d588     Metaphlan2Worker.obj
 0002:000065b0       __unwindtable$?createNode@?$QMapData@VQString@@VQVariant@@@@QAEPAU?$QMapNode@VQString@@VQVariant@@@@ABVQString@@ABVQVariant@@PAU2@_N@Z 1001d5b0     Metaphlan2Worker.obj
 0002:000065e0       __catchsym$?createNode@?$QMapData@VQString@@VQScriptValue@@@@QAEPAU?$QMapNode@VQString@@VQScriptValue@@@@ABVQString@@ABVQScriptValue@@PAU2@_N@Z$7 1001d5e0     Metaphlan2Worker.obj
 0002:000065f0       __catchsym$?createNode@?$QMapData@VQString@@VQScriptValue@@@@QAEPAU?$QMapNode@VQString@@VQScriptValue@@@@ABVQString@@ABVQScriptValue@@PAU2@_N@Z$6 1001d5f0     Metaphlan2Worker.obj
 0002:00006600       __ehfuncinfo$?createNode@?$QMapData@VQString@@VQScriptValue@@@@QAEPAU?$QMapNode@VQString@@VQScriptValue@@@@ABVQString@@ABVQScriptValue@@PAU2@_N@Z 1001d600     Metaphlan2Worker.obj
 0002:00006624       __tryblocktable$?createNode@?$QMapData@VQString@@VQScriptValue@@@@QAEPAU?$QMapNode@VQString@@VQScriptValue@@@@ABVQString@@ABVQScriptValue@@PAU2@_N@Z 1001d624     Metaphlan2Worker.obj
 0002:0000664c       __unwindtable$?createNode@?$QMapData@VQString@@VQScriptValue@@@@QAEPAU?$QMapNode@VQString@@VQScriptValue@@@@ABVQString@@ABVQScriptValue@@PAU2@_N@Z 1001d64c     Metaphlan2Worker.obj
 0002:0000667c       __unwindtable$??H@YA?BVQString@@ABV0@PBD@Z 1001d67c     Metaphlan2WorkerFactory.obj
 0002:0000668c       __ehfuncinfo$??H@YA?BVQString@@ABV0@PBD@Z 1001d68c     Metaphlan2WorkerFactory.obj
 0002:000066b0       __catchsym$?append@?$QList@VQVariant@@@@QAEXABVQVariant@@@Z$11 1001d6b0     Metaphlan2WorkerFactory.obj
 0002:000066c0       __catchsym$?append@?$QList@VQVariant@@@@QAEXABVQVariant@@@Z$10 1001d6c0     Metaphlan2WorkerFactory.obj
 0002:000066d0       __ehfuncinfo$?append@?$QList@VQVariant@@@@QAEXABVQVariant@@@Z 1001d6d0     Metaphlan2WorkerFactory.obj
 0002:000066f4       __tryblocktable$?append@?$QList@VQVariant@@@@QAEXABVQVariant@@@Z 1001d6f4     Metaphlan2WorkerFactory.obj
 0002:0000671c       __unwindtable$?append@?$QList@VQVariant@@@@QAEXABVQVariant@@@Z 1001d71c     Metaphlan2WorkerFactory.obj
 0002:0000676c       __catchsym$?detach_helper_grow@?$QList@VQVariant@@@@AAEPAUNode@1@HH@Z$5 1001d76c     Metaphlan2WorkerFactory.obj
 0002:0000677c       __catchsym$?detach_helper_grow@?$QList@VQVariant@@@@AAEPAUNode@1@HH@Z$4 1001d77c     Metaphlan2WorkerFactory.obj
 0002:0000678c       __unwindtable$?detach_helper_grow@?$QList@VQVariant@@@@AAEPAUNode@1@HH@Z 1001d78c     Metaphlan2WorkerFactory.obj
 0002:000067ac       __ehfuncinfo$?detach_helper_grow@?$QList@VQVariant@@@@AAEPAUNode@1@HH@Z 1001d7ac     Metaphlan2WorkerFactory.obj
 0002:000067d0       __tryblocktable$?detach_helper_grow@?$QList@VQVariant@@@@AAEPAUNode@1@HH@Z 1001d7d0     Metaphlan2WorkerFactory.obj
 0002:000067f8       __unwindtable$?node_construct@?$QList@VQVariant@@@@AAEXPAUNode@1@ABVQVariant@@@Z 1001d7f8     Metaphlan2WorkerFactory.obj
 0002:00006808       __ehfuncinfo$?node_construct@?$QList@VQVariant@@@@AAEXPAUNode@1@ABVQVariant@@@Z 1001d808     Metaphlan2WorkerFactory.obj
 0002:0000682c       __catchsym$?node_copy@?$QList@VQVariant@@@@AAEXPAUNode@1@00@Z$6 1001d82c     Metaphlan2WorkerFactory.obj
 0002:0000683c       __tryblocktable$?node_copy@?$QList@VQVariant@@@@AAEXPAUNode@1@00@Z 1001d83c     Metaphlan2WorkerFactory.obj
 0002:00006850       __ehfuncinfo$?node_copy@?$QList@VQVariant@@@@AAEXPAUNode@1@00@Z 1001d850     Metaphlan2WorkerFactory.obj
 0002:00006874       __unwindtable$?node_copy@?$QList@VQVariant@@@@AAEXPAUNode@1@00@Z 1001d874     Metaphlan2WorkerFactory.obj
 0002:000068a4       __unwindtable$??__EalgoLog@U2@@YAXXZ 1001d8a4     Metaphlan2WorkerFactory.obj
 0002:000068ac       __ehfuncinfo$??__EalgoLog@U2@@YAXXZ 1001d8ac     Metaphlan2WorkerFactory.obj
 0002:000068d0       __unwindtable$??__EcmdLog@U2@@YAXXZ 1001d8d0     Metaphlan2WorkerFactory.obj
 0002:000068d8       __ehfuncinfo$??__EcmdLog@U2@@YAXXZ 1001d8d8     Metaphlan2WorkerFactory.obj
 0002:000068fc       __unwindtable$??__EcoreLog@U2@@YAXXZ 1001d8fc     Metaphlan2WorkerFactory.obj
 0002:00006904       __ehfuncinfo$??__EcoreLog@U2@@YAXXZ 1001d904     Metaphlan2WorkerFactory.obj
 0002:00006928       __unwindtable$??__EioLog@U2@@YAXXZ 1001d928     Metaphlan2WorkerFactory.obj
 0002:00006930       __ehfuncinfo$??__EioLog@U2@@YAXXZ 1001d930     Metaphlan2WorkerFactory.obj
 0002:00006954       __unwindtable$??__EperfLog@U2@@YAXXZ 1001d954     Metaphlan2WorkerFactory.obj
 0002:0000695c       __ehfuncinfo$??__EperfLog@U2@@YAXXZ 1001d95c     Metaphlan2WorkerFactory.obj
 0002:00006980       __unwindtable$??__EscriptLog@U2@@YAXXZ 1001d980     Metaphlan2WorkerFactory.obj
 0002:00006988       __ehfuncinfo$??__EscriptLog@U2@@YAXXZ 1001d988     Metaphlan2WorkerFactory.obj
 0002:000069ac       __unwindtable$??__EtaskLog@U2@@YAXXZ 1001d9ac     Metaphlan2WorkerFactory.obj
 0002:000069b4       __ehfuncinfo$??__EtaskLog@U2@@YAXXZ 1001d9b4     Metaphlan2WorkerFactory.obj
 0002:000069d8       __unwindtable$??__EuiLog@U2@@YAXXZ 1001d9d8     Metaphlan2WorkerFactory.obj
 0002:000069e0       __ehfuncinfo$??__EuiLog@U2@@YAXXZ 1001d9e0     Metaphlan2WorkerFactory.obj
 0002:00006a04       __unwindtable$??__EuserActLog@U2@@YAXXZ 1001da04     Metaphlan2WorkerFactory.obj
 0002:00006a0c       __ehfuncinfo$??__EuserActLog@U2@@YAXXZ 1001da0c     Metaphlan2WorkerFactory.obj
 0002:00006a30       __unwindtable$??A?$QMap@VDescriptor@U2@@V?$QExplicitlySharedDataPointer@VDataType@U2@@@@@@QAEAAV?$QExplicitlySharedDataPointer@VDataType@U2@@@@ABVDescriptor@U2@@@Z 1001da30     Metaphlan2WorkerFactory.obj
 0002:00006a38       __ehfuncinfo$??A?$QMap@VDescriptor@U2@@V?$QExplicitlySharedDataPointer@VDataType@U2@@@@@@QAEAAV?$QExplicitlySharedDataPointer@VDataType@U2@@@@ABVDescriptor@U2@@@Z 1001da38     Metaphlan2WorkerFactory.obj
 0002:00006a5c       __catchsym$?append@?$QList@PAVAttribute@U2@@@@QAEXABQAVAttribute@U2@@@Z$6 1001da5c     Metaphlan2WorkerFactory.obj
 0002:00006a6c       __tryblocktable$?append@?$QList@PAVAttribute@U2@@@@QAEXABQAVAttribute@U2@@@Z 1001da6c     Metaphlan2WorkerFactory.obj
 0002:00006a80       __ehfuncinfo$?append@?$QList@PAVAttribute@U2@@@@QAEXABQAVAttribute@U2@@@Z 1001da80     Metaphlan2WorkerFactory.obj
 0002:00006aa4       __unwindtable$?append@?$QList@PAVAttribute@U2@@@@QAEXABQAVAttribute@U2@@@Z 1001daa4     Metaphlan2WorkerFactory.obj
 0002:00006ad4       __catchsym$?detach_helper_grow@?$QList@PAVAttribute@U2@@@@AAEPAUNode@1@HH@Z$5 1001dad4     Metaphlan2WorkerFactory.obj
 0002:00006ae4       __catchsym$?detach_helper_grow@?$QList@PAVAttribute@U2@@@@AAEPAUNode@1@HH@Z$4 1001dae4     Metaphlan2WorkerFactory.obj
 0002:00006af4       __unwindtable$?detach_helper_grow@?$QList@PAVAttribute@U2@@@@AAEPAUNode@1@HH@Z 1001daf4     Metaphlan2WorkerFactory.obj
 0002:00006b14       __ehfuncinfo$?detach_helper_grow@?$QList@PAVAttribute@U2@@@@AAEPAUNode@1@HH@Z 1001db14     Metaphlan2WorkerFactory.obj
 0002:00006b38       __tryblocktable$?detach_helper_grow@?$QList@PAVAttribute@U2@@@@AAEPAUNode@1@HH@Z 1001db38     Metaphlan2WorkerFactory.obj
 0002:00006b60       __catchsym$?append@?$QList@PAVPortDescriptor@Workflow@U2@@@@QAEXABQAVPortDescriptor@Workflow@U2@@@Z$6 1001db60     Metaphlan2WorkerFactory.obj
 0002:00006b70       __tryblocktable$?append@?$QList@PAVPortDescriptor@Workflow@U2@@@@QAEXABQAVPortDescriptor@Workflow@U2@@@Z 1001db70     Metaphlan2WorkerFactory.obj
 0002:00006b84       __ehfuncinfo$?append@?$QList@PAVPortDescriptor@Workflow@U2@@@@QAEXABQAVPortDescriptor@Workflow@U2@@@Z 1001db84     Metaphlan2WorkerFactory.obj
 0002:00006ba8       __unwindtable$?append@?$QList@PAVPortDescriptor@Workflow@U2@@@@QAEXABQAVPortDescriptor@Workflow@U2@@@Z 1001dba8     Metaphlan2WorkerFactory.obj
 0002:00006bd8       __catchsym$?detach_helper_grow@?$QList@PAVPortDescriptor@Workflow@U2@@@@AAEPAUNode@1@HH@Z$5 1001dbd8     Metaphlan2WorkerFactory.obj
 0002:00006be8       __catchsym$?detach_helper_grow@?$QList@PAVPortDescriptor@Workflow@U2@@@@AAEPAUNode@1@HH@Z$4 1001dbe8     Metaphlan2WorkerFactory.obj
 0002:00006bf8       __unwindtable$?detach_helper_grow@?$QList@PAVPortDescriptor@Workflow@U2@@@@AAEPAUNode@1@HH@Z 1001dbf8     Metaphlan2WorkerFactory.obj
 0002:00006c18       __ehfuncinfo$?detach_helper_grow@?$QList@PAVPortDescriptor@Workflow@U2@@@@AAEPAUNode@1@HH@Z 1001dc18     Metaphlan2WorkerFactory.obj
 0002:00006c3c       __tryblocktable$?detach_helper_grow@?$QList@PAVPortDescriptor@Workflow@U2@@@@AAEPAUNode@1@HH@Z 1001dc3c     Metaphlan2WorkerFactory.obj
 0002:00006c64       __unwindtable$??0?$QPair@VQString@@V1@@@QAE@ABVQString@@0@Z 1001dc64     Metaphlan2WorkerFactory.obj
 0002:00006c6c       __ehfuncinfo$??0?$QPair@VQString@@V1@@@QAE@ABVQString@@0@Z 1001dc6c     Metaphlan2WorkerFactory.obj
 0002:00006c90       __unwindtable$??1?$QPair@VQString@@V1@@@QAE@XZ 1001dc90     Metaphlan2WorkerFactory.obj
 0002:00006c98       __ehfuncinfo$??1?$QPair@VQString@@V1@@@QAE@XZ 1001dc98     Metaphlan2WorkerFactory.obj
 0002:00006cbc       __unwindtable$??0?$QPair@VQString@@V1@@@QAE@ABU0@@Z 1001dcbc     Metaphlan2WorkerFactory.obj
 0002:00006cc4       __ehfuncinfo$??0?$QPair@VQString@@V1@@@QAE@ABU0@@Z 1001dcc4     Metaphlan2WorkerFactory.obj
 0002:00006ce8       __unwindtable$??_G?$QPair@VQString@@V1@@@QAEPAXI@Z 1001dce8     Metaphlan2WorkerFactory.obj
 0002:00006cf0       __ehfuncinfo$??_G?$QPair@VQString@@V1@@@QAEPAXI@Z 1001dcf0     Metaphlan2WorkerFactory.obj
 0002:00006d14       __unwindtable$?createWorker@Metaphlan2WorkerFactory@LocalWorkflow@U2@@UAEPAVWorker@Workflow@3@PAVActor@53@@Z 1001dd14     Metaphlan2WorkerFactory.obj
 0002:00006d1c       __ehfuncinfo$?createWorker@Metaphlan2WorkerFactory@LocalWorkflow@U2@@UAEPAVWorker@Workflow@3@PAVActor@53@@Z 1001dd1c     Metaphlan2WorkerFactory.obj
 0002:00006d40       __ehfuncinfo$?init@Metaphlan2WorkerFactory@LocalWorkflow@U2@@SAXXZ 1001dd40     Metaphlan2WorkerFactory.obj
 0002:00006d64       __unwindtable$?init@Metaphlan2WorkerFactory@LocalWorkflow@U2@@SAXXZ 1001dd64     Metaphlan2WorkerFactory.obj
 0002:000073e4       __catchsym$?append@?$QList@U?$QPair@VQString@@V1@@@@@QAEXABU?$QPair@VQString@@V1@@@@Z$7 1001e3e4     Metaphlan2WorkerFactory.obj
 0002:000073f4       __catchsym$?append@?$QList@U?$QPair@VQString@@V1@@@@@QAEXABU?$QPair@VQString@@V1@@@@Z$6 1001e3f4     Metaphlan2WorkerFactory.obj
 0002:00007404       __ehfuncinfo$?append@?$QList@U?$QPair@VQString@@V1@@@@@QAEXABU?$QPair@VQString@@V1@@@@Z 1001e404     Metaphlan2WorkerFactory.obj
 0002:00007428       __tryblocktable$?append@?$QList@U?$QPair@VQString@@V1@@@@@QAEXABU?$QPair@VQString@@V1@@@@Z 1001e428     Metaphlan2WorkerFactory.obj
 0002:00007450       __unwindtable$?append@?$QList@U?$QPair@VQString@@V1@@@@@QAEXABU?$QPair@VQString@@V1@@@@Z 1001e450     Metaphlan2WorkerFactory.obj
 0002:00007480       __catchsym$?detach_helper_grow@?$QList@U?$QPair@VQString@@V1@@@@@AAEPAUNode@1@HH@Z$5 1001e480     Metaphlan2WorkerFactory.obj
 0002:00007490       __catchsym$?detach_helper_grow@?$QList@U?$QPair@VQString@@V1@@@@@AAEPAUNode@1@HH@Z$4 1001e490     Metaphlan2WorkerFactory.obj
 0002:000074a0       __unwindtable$?detach_helper_grow@?$QList@U?$QPair@VQString@@V1@@@@@AAEPAUNode@1@HH@Z 1001e4a0     Metaphlan2WorkerFactory.obj
 0002:000074c0       __ehfuncinfo$?detach_helper_grow@?$QList@U?$QPair@VQString@@V1@@@@@AAEPAUNode@1@HH@Z 1001e4c0     Metaphlan2WorkerFactory.obj
 0002:000074e4       __tryblocktable$?detach_helper_grow@?$QList@U?$QPair@VQString@@V1@@@@@AAEPAUNode@1@HH@Z 1001e4e4     Metaphlan2WorkerFactory.obj
 0002:0000750c       __unwindtable$?node_construct@?$QList@U?$QPair@VQString@@V1@@@@@AAEXPAUNode@1@ABU?$QPair@VQString@@V1@@@@Z 1001e50c     Metaphlan2WorkerFactory.obj
 0002:0000752c       __ehfuncinfo$?node_construct@?$QList@U?$QPair@VQString@@V1@@@@@AAEXPAUNode@1@ABU?$QPair@VQString@@V1@@@@Z 1001e52c     Metaphlan2WorkerFactory.obj
 0002:00007550       __unwindtable$?node_destruct@?$QList@U?$QPair@VQString@@V1@@@@@AAEXPAUNode@1@@Z 1001e550     Metaphlan2WorkerFactory.obj
 0002:00007560       __ehfuncinfo$?node_destruct@?$QList@U?$QPair@VQString@@V1@@@@@AAEXPAUNode@1@@Z 1001e560     Metaphlan2WorkerFactory.obj
 0002:00007584       __catchsym$?node_copy@?$QList@U?$QPair@VQString@@V1@@@@@AAEXPAUNode@1@00@Z$14 1001e584     Metaphlan2WorkerFactory.obj
 0002:00007594       __tryblocktable$?node_copy@?$QList@U?$QPair@VQString@@V1@@@@@AAEXPAUNode@1@00@Z 1001e594     Metaphlan2WorkerFactory.obj
 0002:000075a8       __ehfuncinfo$?node_copy@?$QList@U?$QPair@VQString@@V1@@@@@AAEXPAUNode@1@00@Z 1001e5a8     Metaphlan2WorkerFactory.obj
 0002:000075cc       __unwindtable$?node_copy@?$QList@U?$QPair@VQString@@V1@@@@@AAEXPAUNode@1@00@Z 1001e5cc     Metaphlan2WorkerFactory.obj
 0002:0000761c       __unwindtable$?node_destruct@?$QList@U?$QPair@VQString@@V1@@@@@AAEXPAUNode@1@0@Z 1001e61c     Metaphlan2WorkerFactory.obj
 0002:0000762c       __ehfuncinfo$?node_destruct@?$QList@U?$QPair@VQString@@V1@@@@@AAEXPAUNode@1@0@Z 1001e62c     Metaphlan2WorkerFactory.obj
 0002:00007650       __catchsym$?createNode@?$QMapData@VDescriptor@U2@@V?$QExplicitlySharedDataPointer@VDataType@U2@@@@@@QAEPAU?$QMapNode@VDescriptor@U2@@V?$QExplicitlySharedDataPointer@VDataType@U2@@@@@@ABVDescriptor@U2@@ABV?$QExplicitlySharedDataPointer@VDataType@U2@@@@PAU2@_N@Z$6 1001e650     Metaphlan2WorkerFactory.obj
 0002:00007660       __tryblocktable$?createNode@?$QMapData@VDescriptor@U2@@V?$QExplicitlySharedDataPointer@VDataType@U2@@@@@@QAEPAU?$QMapNode@VDescriptor@U2@@V?$QExplicitlySharedDataPointer@VDataType@U2@@@@@@ABVDescriptor@U2@@ABV?$QExplicitlySharedDataPointer@VDataType@U2@@@@PAU2@_N@Z 1001e660     Metaphlan2WorkerFactory.obj
 0002:00007674       __ehfuncinfo$?createNode@?$QMapData@VDescriptor@U2@@V?$QExplicitlySharedDataPointer@VDataType@U2@@@@@@QAEPAU?$QMapNode@VDescriptor@U2@@V?$QExplicitlySharedDataPointer@VDataType@U2@@@@@@ABVDescriptor@U2@@ABV?$QExplicitlySharedDataPointer@VDataType@U2@@@@PAU2@_N@Z 1001e674     Metaphlan2WorkerFactory.obj
 0002:00007698       __unwindtable$?createNode@?$QMapData@VDescriptor@U2@@V?$QExplicitlySharedDataPointer@VDataType@U2@@@@@@QAEPAU?$QMapNode@VDescriptor@U2@@V?$QExplicitlySharedDataPointer@VDataType@U2@@@@@@ABVDescriptor@U2@@ABV?$QExplicitlySharedDataPointer@VDataType@U2@@@@PAU2@_N@Z 1001e698     Metaphlan2WorkerFactory.obj
 0002:000076c0       __catchsym$?createNode@?$QMapData@VQString@@PAVPropertyDelegate@U2@@@@QAEPAU?$QMapNode@VQString@@PAVPropertyDelegate@U2@@@@ABVQString@@ABQAVPropertyDelegate@U2@@PAU2@_N@Z$5 1001e6c0     Metaphlan2WorkerFactory.obj
 0002:000076d0       __tryblocktable$?createNode@?$QMapData@VQString@@PAVPropertyDelegate@U2@@@@QAEPAU?$QMapNode@VQString@@PAVPropertyDelegate@U2@@@@ABVQString@@ABQAVPropertyDelegate@U2@@PAU2@_N@Z 1001e6d0     Metaphlan2WorkerFactory.obj
 0002:000076e4       __ehfuncinfo$?createNode@?$QMapData@VQString@@PAVPropertyDelegate@U2@@@@QAEPAU?$QMapNode@VQString@@PAVPropertyDelegate@U2@@@@ABVQString@@ABQAVPropertyDelegate@U2@@PAU2@_N@Z 1001e6e4     Metaphlan2WorkerFactory.obj
 0002:00007708       __unwindtable$?createNode@?$QMapData@VQString@@PAVPropertyDelegate@U2@@@@QAEPAU?$QMapNode@VQString@@PAVPropertyDelegate@U2@@@@ABVQString@@ABQAVPropertyDelegate@U2@@PAU2@_N@Z 1001e708     Metaphlan2WorkerFactory.obj
 0002:00007730       __unwindtable$??__EalgoLog@U2@@YAXXZ 1001e730     moc_Metaphlan2Prompter.obj
 0002:00007738       __ehfuncinfo$??__EalgoLog@U2@@YAXXZ 1001e738     moc_Metaphlan2Prompter.obj
 0002:0000775c       __unwindtable$??__EcmdLog@U2@@YAXXZ 1001e75c     moc_Metaphlan2Prompter.obj
 0002:00007764       __ehfuncinfo$??__EcmdLog@U2@@YAXXZ 1001e764     moc_Metaphlan2Prompter.obj
 0002:00007788       __unwindtable$??__EcoreLog@U2@@YAXXZ 1001e788     moc_Metaphlan2Prompter.obj
 0002:00007790       __ehfuncinfo$??__EcoreLog@U2@@YAXXZ 1001e790     moc_Metaphlan2Prompter.obj
 0002:000077b4       __unwindtable$??__EioLog@U2@@YAXXZ 1001e7b4     moc_Metaphlan2Prompter.obj
 0002:000077bc       __ehfuncinfo$??__EioLog@U2@@YAXXZ 1001e7bc     moc_Metaphlan2Prompter.obj
 0002:000077e0       __unwindtable$??__EperfLog@U2@@YAXXZ 1001e7e0     moc_Metaphlan2Prompter.obj
 0002:000077e8       __ehfuncinfo$??__EperfLog@U2@@YAXXZ 1001e7e8     moc_Metaphlan2Prompter.obj
 0002:0000780c       __unwindtable$??__EscriptLog@U2@@YAXXZ 1001e80c     moc_Metaphlan2Prompter.obj
 0002:00007814       __ehfuncinfo$??__EscriptLog@U2@@YAXXZ 1001e814     moc_Metaphlan2Prompter.obj
 0002:00007838       __unwindtable$??__EtaskLog@U2@@YAXXZ 1001e838     moc_Metaphlan2Prompter.obj
 0002:00007840       __ehfuncinfo$??__EtaskLog@U2@@YAXXZ 1001e840     moc_Metaphlan2Prompter.obj
 0002:00007864       __unwindtable$??__EuiLog@U2@@YAXXZ 1001e864     moc_Metaphlan2Prompter.obj
 0002:0000786c       __ehfuncinfo$??__EuiLog@U2@@YAXXZ 1001e86c     moc_Metaphlan2Prompter.obj
 0002:00007890       __unwindtable$??__EuserActLog@U2@@YAXXZ 1001e890     moc_Metaphlan2Prompter.obj
 0002:00007898       __ehfuncinfo$??__EuserActLog@U2@@YAXXZ 1001e898     moc_Metaphlan2Prompter.obj
 0002:000078bc       __unwindtable$??__EalgoLog@U2@@YAXXZ 1001e8bc     moc_Metaphlan2Task.obj
 0002:000078c4       __ehfuncinfo$??__EalgoLog@U2@@YAXXZ 1001e8c4     moc_Metaphlan2Task.obj
 0002:000078e8       __unwindtable$??__EcmdLog@U2@@YAXXZ 1001e8e8     moc_Metaphlan2Task.obj
 0002:000078f0       __ehfuncinfo$??__EcmdLog@U2@@YAXXZ 1001e8f0     moc_Metaphlan2Task.obj
 0002:00007914       __unwindtable$??__EcoreLog@U2@@YAXXZ 1001e914     moc_Metaphlan2Task.obj
 0002:0000791c       __ehfuncinfo$??__EcoreLog@U2@@YAXXZ 1001e91c     moc_Metaphlan2Task.obj
 0002:00007940       __unwindtable$??__EioLog@U2@@YAXXZ 1001e940     moc_Metaphlan2Task.obj
 0002:00007948       __ehfuncinfo$??__EioLog@U2@@YAXXZ 1001e948     moc_Metaphlan2Task.obj
 0002:0000796c       __unwindtable$??__EperfLog@U2@@YAXXZ 1001e96c     moc_Metaphlan2Task.obj
 0002:00007974       __ehfuncinfo$??__EperfLog@U2@@YAXXZ 1001e974     moc_Metaphlan2Task.obj
 0002:00007998       __unwindtable$??__EscriptLog@U2@@YAXXZ 1001e998     moc_Metaphlan2Task.obj
 0002:000079a0       __ehfuncinfo$??__EscriptLog@U2@@YAXXZ 1001e9a0     moc_Metaphlan2Task.obj
 0002:000079c4       __unwindtable$??__EtaskLog@U2@@YAXXZ 1001e9c4     moc_Metaphlan2Task.obj
 0002:000079cc       __ehfuncinfo$??__EtaskLog@U2@@YAXXZ 1001e9cc     moc_Metaphlan2Task.obj
 0002:000079f0       __unwindtable$??__EuiLog@U2@@YAXXZ 1001e9f0     moc_Metaphlan2Task.obj
 0002:000079f8       __ehfuncinfo$??__EuiLog@U2@@YAXXZ 1001e9f8     moc_Metaphlan2Task.obj
 0002:00007a1c       __unwindtable$??__EuserActLog@U2@@YAXXZ 1001ea1c     moc_Metaphlan2Task.obj
 0002:00007a24       __ehfuncinfo$??__EuserActLog@U2@@YAXXZ 1001ea24     moc_Metaphlan2Task.obj
 0002:00007a48       __unwindtable$??__EalgoLog@U2@@YAXXZ 1001ea48     moc_Metaphlan2Worker.obj
 0002:00007a50       __ehfuncinfo$??__EalgoLog@U2@@YAXXZ 1001ea50     moc_Metaphlan2Worker.obj
 0002:00007a74       __unwindtable$??__EcmdLog@U2@@YAXXZ 1001ea74     moc_Metaphlan2Worker.obj
 0002:00007a7c       __ehfuncinfo$??__EcmdLog@U2@@YAXXZ 1001ea7c     moc_Metaphlan2Worker.obj
 0002:00007aa0       __unwindtable$??__EcoreLog@U2@@YAXXZ 1001eaa0     moc_Metaphlan2Worker.obj
 0002:00007aa8       __ehfuncinfo$??__EcoreLog@U2@@YAXXZ 1001eaa8     moc_Metaphlan2Worker.obj
 0002:00007acc       __unwindtable$??__EioLog@U2@@YAXXZ 1001eacc     moc_Metaphlan2Worker.obj
 0002:00007ad4       __ehfuncinfo$??__EioLog@U2@@YAXXZ 1001ead4     moc_Metaphlan2Worker.obj
 0002:00007af8       __unwindtable$??__EperfLog@U2@@YAXXZ 1001eaf8     moc_Metaphlan2Worker.obj
 0002:00007b00       __ehfuncinfo$??__EperfLog@U2@@YAXXZ 1001eb00     moc_Metaphlan2Worker.obj
 0002:00007b24       __unwindtable$??__EscriptLog@U2@@YAXXZ 1001eb24     moc_Metaphlan2Worker.obj
 0002:00007b2c       __ehfuncinfo$??__EscriptLog@U2@@YAXXZ 1001eb2c     moc_Metaphlan2Worker.obj
 0002:00007b50       __unwindtable$??__EtaskLog@U2@@YAXXZ 1001eb50     moc_Metaphlan2Worker.obj
 0002:00007b58       __ehfuncinfo$??__EtaskLog@U2@@YAXXZ 1001eb58     moc_Metaphlan2Worker.obj
 0002:00007b7c       __unwindtable$??__EuiLog@U2@@YAXXZ 1001eb7c     moc_Metaphlan2Worker.obj
 0002:00007b84       __ehfuncinfo$??__EuiLog@U2@@YAXXZ 1001eb84     moc_Metaphlan2Worker.obj
 0002:00007ba8       __unwindtable$??__EuserActLog@U2@@YAXXZ 1001eba8     moc_Metaphlan2Worker.obj
 0002:00007bb0       __ehfuncinfo$??__EuserActLog@U2@@YAXXZ 1001ebb0     moc_Metaphlan2Worker.obj
 0002:00007bd4       __unwindtable$?qt_metatype_id@?$QMetaTypeIdQObject@PAVTask@U2@@$00@@SAHXZ 1001ebd4     moc_Metaphlan2Worker.obj
 0002:00007bdc       __ehfuncinfo$?qt_metatype_id@?$QMetaTypeIdQObject@PAVTask@U2@@$00@@SAHXZ 1001ebdc     moc_Metaphlan2Worker.obj
 0002:00007c00       __sehtable$__onexit        1001ec00     MSVCRT:atonexit.obj
 0002:00007c20       __sehtable$___DllMainCRTStartup 1001ec20     MSVCRT:crtdll.obj
 0002:00007c48       __sehtable$??_M@YGXPAXIHP6EX0@Z@Z 1001ec48     MSVCRT:ehvecdtr.obj
 0002:00007c68       __sehtable$?__ArrayUnwind@@YGXPAXIHP6EX0@Z@Z 1001ec68     MSVCRT:ehvecdtr.obj
 0002:00007c88       __sehtable$__IsNonwritableInCurrentImage 1001ec88     MSVCRT:pesect.obj
 0002:00007cb0       .edata                     1001ecb0     metaphlan2_support.exp
 0002:00007cd8       rgpv                       1001ecd8     metaphlan2_support.exp
 0002:00007cdc       rgszName                   1001ecdc     metaphlan2_support.exp
 0002:00007ce0       rgwOrd                     1001ece0     metaphlan2_support.exp
 0002:00007ce2       szName                     1001ece2     metaphlan2_support.exp
 0002:00007cf9       $N00001                    1001ecf9     metaphlan2_support.exp
 0002:0000877e       .idata$6                   1001f77e     ngs_reads_classification:ngs_reads_classification.dll
 0002:00009ccc       .idata$6                   10020ccc     U2Core:U2Core.dll
 0002:00009dae       .idata$6                   10020dae     U2Formats:U2Formats.dll
 0002:00009e12       .idata$6                   10020e12     U2Gui:U2Gui.dll
 0002:0000c152       .idata$6                   10023152     U2Lang:U2Lang.dll
 0002:0000cdca       .idata$6                   10023dca     U2Designer:U2Designer.dll
 0002:0000d21a       .idata$6                   1002421a     Qt5Widgets:Qt5Widgets.dll
 0002:0000d2cc       .idata$6                   100242cc     Qt5Gui:Qt5Gui.dll
 0002:0000d43e       .idata$6                   1002443e     Qt5Script:Qt5Script.dll
 0002:0000e194       .idata$6                   10025194     Qt5Core:Qt5Core.dll
 0002:0000e23a       .idata$6                   1002523a     msvcprt:MSVCP120.dll
 0002:0000e2be       .idata$6                   100252be     MSVCRT:MSVCR120.dll
 0002:0000e4d2       .idata$6                   100254d2     kernel32:KERNEL32.dll
 0003:00000978       __Tuple_alloc              10026978     Metaphlan2LogParser.obj
 0003:00000979       _ignore                    10026979     Metaphlan2LogParser.obj
 0003:0000097a       _allocator_arg             1002697a     Metaphlan2LogParser.obj
 0003:0000097b       _piecewise_construct       1002697b     Metaphlan2LogParser.obj
 0003:0000097c       _taskLog                   1002697c     Metaphlan2LogParser.obj
 0003:00000984       _algoLog                   10026984     Metaphlan2LogParser.obj
 0003:00000990       _userActLog                10026990     Metaphlan2LogParser.obj
 0003:00000998       _ioLog                     10026998     Metaphlan2LogParser.obj
 0003:000009a0       _coreLog                   100269a0     Metaphlan2LogParser.obj
 0003:000009a8       _uiLog                     100269a8     Metaphlan2LogParser.obj
 0003:000009b0       _scriptLog                 100269b0     Metaphlan2LogParser.obj
 0003:000009b8       _perfLog                   100269b8     Metaphlan2LogParser.obj
 0003:000009c0       _cmdLog                    100269c0     Metaphlan2LogParser.obj
 0003:000009d0       __Tuple_alloc              100269d0     Metaphlan2Prompter.obj
 0003:000009d1       _ignore                    100269d1     Metaphlan2Prompter.obj
 0003:000009d2       _allocator_arg             100269d2     Metaphlan2Prompter.obj
 0003:000009d3       _piecewise_construct       100269d3     Metaphlan2Prompter.obj
 0003:000009d4       _taskLog                   100269d4     Metaphlan2Prompter.obj
 0003:000009dc       _algoLog                   100269dc     Metaphlan2Prompter.obj
 0003:000009e4       _userActLog                100269e4     Metaphlan2Prompter.obj
 0003:000009ec       _ioLog                     100269ec     Metaphlan2Prompter.obj
 0003:000009f4       _coreLog                   100269f4     Metaphlan2Prompter.obj
 0003:000009fc       _uiLog                     100269fc     Metaphlan2Prompter.obj
 0003:00000a04       _scriptLog                 10026a04     Metaphlan2Prompter.obj
 0003:00000a0c       _perfLog                   10026a0c     Metaphlan2Prompter.obj
 0003:00000a14       _cmdLog                    10026a14     Metaphlan2Prompter.obj
 0003:00000a1c       __Tuple_alloc              10026a1c     Metaphlan2Support.obj
 0003:00000a1d       _ignore                    10026a1d     Metaphlan2Support.obj
 0003:00000a1e       _allocator_arg             10026a1e     Metaphlan2Support.obj
 0003:00000a1f       _piecewise_construct       10026a1f     Metaphlan2Support.obj
 0003:00000a20       _taskLog                   10026a20     Metaphlan2Support.obj
 0003:00000a28       _algoLog                   10026a28     Metaphlan2Support.obj
 0003:00000a30       _userActLog                10026a30     Metaphlan2Support.obj
 0003:00000a38       _ioLog                     10026a38     Metaphlan2Support.obj
 0003:00000a40       _coreLog                   10026a40     Metaphlan2Support.obj
 0003:00000a48       _uiLog                     10026a48     Metaphlan2Support.obj
 0003:00000a50       _scriptLog                 10026a50     Metaphlan2Support.obj
 0003:00000a5c       _perfLog                   10026a5c     Metaphlan2Support.obj
 0003:00000a70       _cmdLog                    10026a70     Metaphlan2Support.obj
 0003:00000a80       __Tuple_alloc              10026a80     Metaphlan2SupportPlugin.obj
 0003:00000a81       _ignore                    10026a81     Metaphlan2SupportPlugin.obj
 0003:00000a82       _allocator_arg             10026a82     Metaphlan2SupportPlugin.obj
 0003:00000a83       _piecewise_construct       10026a83     Metaphlan2SupportPlugin.obj
 0003:00000a88       _taskLog                   10026a88     Metaphlan2SupportPlugin.obj
 0003:00000a90       _algoLog                   10026a90     Metaphlan2SupportPlugin.obj
 0003:00000a98       _userActLog                10026a98     Metaphlan2SupportPlugin.obj
 0003:00000aa0       _ioLog                     10026aa0     Metaphlan2SupportPlugin.obj
 0003:00000aa8       _coreLog                   10026aa8     Metaphlan2SupportPlugin.obj
 0003:00000ab0       _uiLog                     10026ab0     Metaphlan2SupportPlugin.obj
 0003:00000ab8       _scriptLog                 10026ab8     Metaphlan2SupportPlugin.obj
 0003:00000ac0       _perfLog                   10026ac0     Metaphlan2SupportPlugin.obj
 0003:00000ac8       _cmdLog                    10026ac8     Metaphlan2SupportPlugin.obj
 0003:00000ad4       __Tuple_alloc              10026ad4     Metaphlan2Task.obj
 0003:00000ad5       _ignore                    10026ad5     Metaphlan2Task.obj
 0003:00000ad6       _allocator_arg             10026ad6     Metaphlan2Task.obj
 0003:00000ad7       _piecewise_construct       10026ad7     Metaphlan2Task.obj
 0003:00000ad8       _taskLog                   10026ad8     Metaphlan2Task.obj
 0003:00000ae0       _algoLog                   10026ae0     Metaphlan2Task.obj
 0003:00000ae8       _userActLog                10026ae8     Metaphlan2Task.obj
 0003:00000af0       _ioLog                     10026af0     Metaphlan2Task.obj
 0003:00000af8       _coreLog                   10026af8     Metaphlan2Task.obj
 0003:00000b00       _uiLog                     10026b00     Metaphlan2Task.obj
 0003:00000b08       _scriptLog                 10026b08     Metaphlan2Task.obj
 0003:00000b10       _perfLog                   10026b10     Metaphlan2Task.obj
 0003:00000b18       _cmdLog                    10026b18     Metaphlan2Task.obj
 0003:00000b20       ?cvar@?1???0Metaphlan2ClassifyTask@U2@@QAE@ABUMetaphlan2TaskSettings@2@@Z@4VGReportableCounter@2@A 10026b20     Metaphlan2Task.obj
 0003:00000b48       ?$S1@?1???0Metaphlan2ClassifyTask@U2@@QAE@ABUMetaphlan2TaskSettings@2@@Z@4IA 10026b48     Metaphlan2Task.obj
 0003:00000b4c       __Tuple_alloc              10026b4c     Metaphlan2Validator.obj
 0003:00000b4d       _ignore                    10026b4d     Metaphlan2Validator.obj
 0003:00000b4e       _allocator_arg             10026b4e     Metaphlan2Validator.obj
 0003:00000b4f       _piecewise_construct       10026b4f     Metaphlan2Validator.obj
 0003:00000b50       _taskLog                   10026b50     Metaphlan2Validator.obj
 0003:00000b58       _algoLog                   10026b58     Metaphlan2Validator.obj
 0003:00000b60       _userActLog                10026b60     Metaphlan2Validator.obj
 0003:00000b68       _ioLog                     10026b68     Metaphlan2Validator.obj
 0003:00000b70       _coreLog                   10026b70     Metaphlan2Validator.obj
 0003:00000b78       _uiLog                     10026b78     Metaphlan2Validator.obj
 0003:00000b80       _scriptLog                 10026b80     Metaphlan2Validator.obj
 0003:00000b88       _perfLog                   10026b88     Metaphlan2Validator.obj
 0003:00000b90       _cmdLog                    10026b90     Metaphlan2Validator.obj
 0003:00000b98       __Tuple_alloc              10026b98     Metaphlan2Worker.obj
 0003:00000b99       _ignore                    10026b99     Metaphlan2Worker.obj
 0003:00000b9a       _allocator_arg             10026b9a     Metaphlan2Worker.obj
 0003:00000b9b       _piecewise_construct       10026b9b     Metaphlan2Worker.obj
 0003:00000ba8       _taskLog                   10026ba8     Metaphlan2Worker.obj
 0003:00000bb0       _algoLog                   10026bb0     Metaphlan2Worker.obj
 0003:00000bb8       _userActLog                10026bb8     Metaphlan2Worker.obj
 0003:00000bc0       _ioLog                     10026bc0     Metaphlan2Worker.obj
 0003:00000bc8       _coreLog                   10026bc8     Metaphlan2Worker.obj
 0003:00000bd0       _uiLog                     10026bd0     Metaphlan2Worker.obj
 0003:00000bd8       _scriptLog                 10026bd8     Metaphlan2Worker.obj
 0003:00000be8       _perfLog                   10026be8     Metaphlan2Worker.obj
 0003:00000bf0       _cmdLog                    10026bf0     Metaphlan2Worker.obj
 0003:00000bf8       __Tuple_alloc              10026bf8     Metaphlan2WorkerFactory.obj
 0003:00000bf9       _ignore                    10026bf9     Metaphlan2WorkerFactory.obj
 0003:00000bfa       _allocator_arg             10026bfa     Metaphlan2WorkerFactory.obj
 0003:00000bfb       _piecewise_construct       10026bfb     Metaphlan2WorkerFactory.obj
 0003:00000c18       _taskLog                   10026c18     Metaphlan2WorkerFactory.obj
 0003:00000c20       _algoLog                   10026c20     Metaphlan2WorkerFactory.obj
 0003:00000c28       _userActLog                10026c28     Metaphlan2WorkerFactory.obj
 0003:00000c30       _ioLog                     10026c30     Metaphlan2WorkerFactory.obj
 0003:00000c38       _coreLog                   10026c38     Metaphlan2WorkerFactory.obj
 0003:00000c64       _uiLog                     10026c64     Metaphlan2WorkerFactory.obj
 0003:00000c6c       _scriptLog                 10026c6c     Metaphlan2WorkerFactory.obj
 0003:00000c8c       _perfLog                   10026c8c     Metaphlan2WorkerFactory.obj
 0003:00000ca4       _cmdLog                    10026ca4     Metaphlan2WorkerFactory.obj
 0003:00000d00       __Tuple_alloc              10026d00     moc_Metaphlan2Prompter.obj
 0003:00000d01       _ignore                    10026d01     moc_Metaphlan2Prompter.obj
 0003:00000d02       _allocator_arg             10026d02     moc_Metaphlan2Prompter.obj
 0003:00000d03       _piecewise_construct       10026d03     moc_Metaphlan2Prompter.obj
 0003:00000d04       _taskLog                   10026d04     moc_Metaphlan2Prompter.obj
 0003:00000d0c       _algoLog                   10026d0c     moc_Metaphlan2Prompter.obj
 0003:00000d14       _userActLog                10026d14     moc_Metaphlan2Prompter.obj
 0003:00000d1c       _ioLog                     10026d1c     moc_Metaphlan2Prompter.obj
 0003:00000d24       _coreLog                   10026d24     moc_Metaphlan2Prompter.obj
 0003:00000d2c       _uiLog                     10026d2c     moc_Metaphlan2Prompter.obj
 0003:00000d34       _scriptLog                 10026d34     moc_Metaphlan2Prompter.obj
 0003:00000d3c       _perfLog                   10026d3c     moc_Metaphlan2Prompter.obj
 0003:00000d44       _cmdLog                    10026d44     moc_Metaphlan2Prompter.obj
 0003:00000d4c       __Tuple_alloc              10026d4c     moc_Metaphlan2Support.obj
 0003:00000d4d       _ignore                    10026d4d     moc_Metaphlan2Support.obj
 0003:00000d4e       _allocator_arg             10026d4e     moc_Metaphlan2Support.obj
 0003:00000d4f       _piecewise_construct       10026d4f     moc_Metaphlan2Support.obj
 0003:00000d50       __Tuple_alloc              10026d50     moc_Metaphlan2SupportPlugin.obj
 0003:00000d51       _ignore                    10026d51     moc_Metaphlan2SupportPlugin.obj
 0003:00000d52       _allocator_arg             10026d52     moc_Metaphlan2SupportPlugin.obj
 0003:00000d53       _piecewise_construct       10026d53     moc_Metaphlan2SupportPlugin.obj
 0003:00000d54       __Tuple_alloc              10026d54     moc_Metaphlan2Task.obj
 0003:00000d55       _ignore                    10026d55     moc_Metaphlan2Task.obj
 0003:00000d56       _allocator_arg             10026d56     moc_Metaphlan2Task.obj
 0003:00000d57       _piecewise_construct       10026d57     moc_Metaphlan2Task.obj
 0003:00000d58       _taskLog                   10026d58     moc_Metaphlan2Task.obj
 0003:00000d60       _algoLog                   10026d60     moc_Metaphlan2Task.obj
 0003:00000d68       _userActLog                10026d68     moc_Metaphlan2Task.obj
 0003:00000d70       _ioLog                     10026d70     moc_Metaphlan2Task.obj
 0003:00000d78       _coreLog                   10026d78     moc_Metaphlan2Task.obj
 0003:00000d80       _uiLog                     10026d80     moc_Metaphlan2Task.obj
 0003:00000d88       _scriptLog                 10026d88     moc_Metaphlan2Task.obj
 0003:00000d90       _perfLog                   10026d90     moc_Metaphlan2Task.obj
 0003:00000d98       _cmdLog                    10026d98     moc_Metaphlan2Task.obj
 0003:00000da0       __Tuple_alloc              10026da0     moc_Metaphlan2Worker.obj
 0003:00000da1       _ignore                    10026da1     moc_Metaphlan2Worker.obj
 0003:00000da2       _allocator_arg             10026da2     moc_Metaphlan2Worker.obj
 0003:00000da3       _piecewise_construct       10026da3     moc_Metaphlan2Worker.obj
 0003:00000da4       _taskLog                   10026da4     moc_Metaphlan2Worker.obj
 0003:00000dac       _algoLog                   10026dac     moc_Metaphlan2Worker.obj
 0003:00000db4       _userActLog                10026db4     moc_Metaphlan2Worker.obj
 0003:00000dbc       _ioLog                     10026dbc     moc_Metaphlan2Worker.obj
 0003:00000dc4       _coreLog                   10026dc4     moc_Metaphlan2Worker.obj
 0003:00000dcc       _uiLog                     10026dcc     moc_Metaphlan2Worker.obj
 0003:00000dd4       _scriptLog                 10026dd4     moc_Metaphlan2Worker.obj
 0003:00000ddc       _perfLog                   10026ddc     moc_Metaphlan2Worker.obj
 0003:00000de4       _cmdLog                    10026de4     moc_Metaphlan2Worker.obj
 0003:00000df0       ___proc_attached           10026df0     MSVCRT:crtdll.obj
 0003:00000df8       _GS_ExceptionRecord        10026df8     MSVCRT:gs_report.obj
 0003:00000e48       _GS_ContextRecord          10026e48     MSVCRT:gs_report.obj
 0003:00001114       _DebuggerWasPresent        10027114     MSVCRT:gs_report.obj
 0004:00000060       $R000000                   10028060     * linker generated manifest res *

 Exports

  ordinal    name

        1    _ugene_plugin_init
               exported name: ugene_plugin_init
